 RakSAMPClient

 Timestamp is 4fd5e5b7 (Mon Jun 11 16:33:59 2012)

 Preferred load address is 00400000

 Start         Length     Name                   Class
 0001:00000000 00061848H .text                   CODE
 0001:00061850 00001850H .text$x                 CODE
 0001:000630a0 000000fcH .text$yc                CODE
 0001:000631a0 00000058H .text$yd                CODE
 0002:00000000 0000030cH .idata$5                DATA
 0002:0000030c 00000004H .CRT$XCA                DATA
 0002:00000310 00000004H .CRT$XCC                DATA
 0002:00000314 0000002cH .CRT$XCU                DATA
 0002:00000340 00000004H .CRT$XCZ                DATA
 0002:00000344 00000004H .CRT$XIA                DATA
 0002:00000348 00000014H .CRT$XIC                DATA
 0002:0000035c 00000004H .CRT$XIY                DATA
 0002:00000360 00000004H .CRT$XIZ                DATA
 0002:00000364 00000004H .CRT$XPA                DATA
 0002:00000368 00000004H .CRT$XPX                DATA
 0002:0000036c 00000004H .CRT$XPXA               DATA
 0002:00000370 00000004H .CRT$XPZ                DATA
 0002:00000374 00000004H .CRT$XTA                DATA
 0002:00000378 00000004H .CRT$XTZ                DATA
 0002:00000380 00008878H .rdata                  DATA
 0002:00008bf8 00000059H .rdata$debug            DATA
 0002:00008c54 0000083cH .rdata$r                DATA
 0002:00009490 00000294H .rdata$sxdata           DATA
 0002:00009724 00000004H .rtc$IAA                DATA
 0002:00009728 00000004H .rtc$IZZ                DATA
 0002:0000972c 00000004H .rtc$TAA                DATA
 0002:00009730 00000004H .rtc$TZZ                DATA
 0002:00009738 00002bb4H .xdata$x                DATA
 0002:0000c2ec 00000078H .idata$2                DATA
 0002:0000c364 00000014H .idata$3                DATA
 0002:0000c378 0000030cH .idata$4                DATA
 0002:0000c684 00000c0eH .idata$6                DATA
 0002:0000d292 00000000H .edata                  DATA
 0003:00000000 00006911H .data                   DATA
 0003:00006920 000e50e4H .bss                    DATA
 0004:00000000 000000a0H .rsrc$01                DATA
 0004:000000a0 00001640H .rsrc$02                DATA

  Address         Publics by Value              Rva+Base       Lib:Object

 0000:00000000       __except_list              00000000     <absolute>
 0000:000000a5       ___safe_se_handler_count   000000a5     <absolute>
 0000:00000000       ___ImageBase               00400000     <linker-defined>
 0001:00000000       ?GetWriteOffset@BitStream@RakNet@@QBEHXZ 00401000 f i BitStream.obj
 0001:00000010       ??$Read@_N@BitStream@RakNet@@QAE_NAA_N@Z 00401010 f i BitStream.obj
 0001:00000070       ??0BitStream@RakNet@@QAE@XZ 00401070 f   BitStream.obj
 0001:000000a0       ??0BitStream@RakNet@@QAE@H@Z 004010a0 f   BitStream.obj
 0001:00000100       ??0BitStream@RakNet@@QAE@PAEI_N@Z 00401100 f   BitStream.obj
 0001:00000180       ?SetNumberOfBitsAllocated@BitStream@RakNet@@QAEXI@Z 00401180 f   BitStream.obj
 0001:00000190       ??1BitStream@RakNet@@QAE@XZ 00401190 f   BitStream.obj
 0001:000001b0       ?Reset@BitStream@RakNet@@QAEXXZ 004011b0 f   BitStream.obj
 0001:000001c0       ?ResetReadPointer@BitStream@RakNet@@QAEXXZ 004011c0 f   BitStream.obj
 0001:000001d0       ?ResetWritePointer@BitStream@RakNet@@QAEXXZ 004011d0 f   BitStream.obj
 0001:000001e0       ?ReadBit@BitStream@RakNet@@QAE_NXZ 004011e0 f   BitStream.obj
 0001:00000210       ?AlignWriteToByteBoundary@BitStream@RakNet@@QAEXXZ 00401210 f   BitStream.obj
 0001:00000230       ?AlignReadToByteBoundary@BitStream@RakNet@@QAEXXZ 00401230 f   BitStream.obj
 0001:00000250       ?SetData@BitStream@RakNet@@QAEXPAE@Z 00401250 f   BitStream.obj
 0001:00000260       ?ReadBits@BitStream@RakNet@@QAE_NPAEH_N@Z 00401260 f   BitStream.obj
 0001:00000310       ?ReadCompressed@BitStream@RakNet@@AAE_NPAEH_N@Z 00401310 f   BitStream.obj
 0001:00000410       ?AddBitsAndReallocate@BitStream@RakNet@@QAEXH@Z 00401410 f   BitStream.obj
 0001:00000490       ?AssertStreamEmpty@BitStream@RakNet@@QAEXXZ 00401490 f   BitStream.obj
 0001:000004b0       ?PrintBits@BitStream@RakNet@@QBEXXZ 004014b0 f   BitStream.obj
 0001:00000550       ?CopyData@BitStream@RakNet@@QBEHPAPAE@Z 00401550 f   BitStream.obj
 0001:00000590       ?IgnoreBits@BitStream@RakNet@@QAEXH@Z 00401590 f   BitStream.obj
 0001:000005a0       ?SetWriteOffset@BitStream@RakNet@@QAEXH@Z 004015a0 f   BitStream.obj
 0001:000005b0       ?AssertCopyData@BitStream@RakNet@@QAEXXZ 004015b0 f   BitStream.obj
 0001:00000600       ?ReverseBytes@BitStream@RakNet@@AAEXPAE0H@Z 00401600 f   BitStream.obj
 0001:00000630       ?DoEndianSwap@BitStream@RakNet@@ABE_NXZ 00401630 f   BitStream.obj
 0001:00000640       ?GetNumberOfBitsUsed@BitStream@RakNet@@QBEHXZ 00401640 f i BitStream.obj
 0001:00000650       ?Write@BitStream@RakNet@@QAEXPAV12@H@Z 00401650 f   BitStream.obj
 0001:00000730       ?Read@BitStream@RakNet@@QAE_NPADH@Z 00401730 f   BitStream.obj
 0001:00000790       ?Write0@BitStream@RakNet@@QAEXXZ 00401790 f   BitStream.obj
 0001:000007b0       ?Write1@BitStream@RakNet@@QAEXXZ 004017b0 f   BitStream.obj
 0001:000007f0       ?ReadAlignedBytes@BitStream@RakNet@@QAE_NPAEH@Z 004017f0 f   BitStream.obj
 0001:00000850       ?WriteBits@BitStream@RakNet@@QAEXPBEH_N@Z 00401850 f   BitStream.obj
 0001:000008f0       ??$Write@_N@BitStream@RakNet@@QAEX_N@Z 004018f0 f i BitStream.obj
 0001:00000950       ?Write@BitStream@RakNet@@QAEXPBDH@Z 00401950 f   BitStream.obj
 0001:000009c0       ?Write@BitStream@RakNet@@QAEXPAV12@@Z 004019c0 f   BitStream.obj
 0001:000009d0       ?WriteAlignedBytes@BitStream@RakNet@@QAEXPBEH@Z 004019d0 f   BitStream.obj
 0001:000009f0       ?WriteCompressed@BitStream@RakNet@@AAEXPBEH_N@Z 004019f0 f   BitStream.obj
 0001:00000ba0       ?Add@CheckSum@@QAEXE@Z     00401ba0 f   CheckSum.obj
 0001:00000bd0       ?Add@CheckSum@@QAEXPAEI@Z  00401bd0 f   CheckSum.obj
 0001:00000c20       ?Add@CheckSum@@QAEXI@Z     00401c20 f   CheckSum.obj
 0001:00000cb0       ?Add@CheckSum@@QAEXG@Z     00401cb0 f   CheckSum.obj
 0001:00000d00       ?Clear@CheckSum@@QAEXXZ    00401d00 f i DataBlockEncryptor.obj
 0001:00000d30       ?Get@CheckSum@@QAEIXZ      00401d30 f i DataBlockEncryptor.obj
 0001:00000d40       ??0DataBlockEncryptor@@QAE@XZ 00401d40 f   DataBlockEncryptor.obj
 0001:00000d50       ??1DataBlockEncryptor@@QAE@XZ 00401d50 f   DataBlockEncryptor.obj
 0001:00000d60       ?IsKeySet@DataBlockEncryptor@@QBE_NXZ 00401d60 f   DataBlockEncryptor.obj
 0001:00000d70       ?SetKey@DataBlockEncryptor@@QAEXQBE@Z 00401d70 f   DataBlockEncryptor.obj
 0001:00000dc0       ?UnsetKey@DataBlockEncryptor@@QAEXXZ 00401dc0 f   DataBlockEncryptor.obj
 0001:00000dd0       ??0CheckSum@@QAE@XZ        00401dd0 f i DataBlockEncryptor.obj
 0001:00000e00       ?Encrypt@DataBlockEncryptor@@QAEXPAEH0PAH@Z 00401e00 f   DataBlockEncryptor.obj
 0001:00000f90       ?Decrypt@DataBlockEncryptor@@QAE_NPAEH0PAH@Z 00401f90 f   DataBlockEncryptor.obj
 0001:00001150       ??$Write@I@BitStream@RakNet@@QAEXI@Z 00402150 f i DataCompressor.obj
 0001:00001170       ??$Read@I@BitStream@RakNet@@QAE_NAAI@Z 00402170 f i DataCompressor.obj
 0001:00001190       ??$WriteCompressed@I@BitStream@RakNet@@QAEXI@Z 00402190 f i DataCompressor.obj
 0001:000011b0       ??$ReadCompressed@I@BitStream@RakNet@@QAE_NAAI@Z 004021b0 f i DataCompressor.obj
 0001:000011d0       ?Compress@DataCompressor@@SAXPAEIPAVBitStream@RakNet@@@Z 004021d0 f   DataCompressor.obj
 0001:00001350       ?DecompressAndAllocate@DataCompressor@@SAIPAVBitStream@RakNet@@PAPAE@Z 00402350 f   DataCompressor.obj
 0001:00001490       ??0ByteQueue@DataStructures@@QAE@XZ 00402490 f   DS_ByteQueue.obj
 0001:000014a0       ?Clear@ByteQueue@DataStructures@@QAEXXZ 004024a0 f   DS_ByteQueue.obj
 0001:000014e0       ?GetBytesWritten@ByteQueue@DataStructures@@QBEIXZ 004024e0 f   DS_ByteQueue.obj
 0001:00001500       ?IncrementReadOffset@ByteQueue@DataStructures@@QAEXI@Z 00402500 f   DS_ByteQueue.obj
 0001:00001520       ?Print@ByteQueue@DataStructures@@QAEXXZ 00402520 f   DS_ByteQueue.obj
 0001:00001560       ??1ByteQueue@DataStructures@@QAE@XZ 00402560 f   DS_ByteQueue.obj
 0001:000015a0       ?WriteBytes@ByteQueue@DataStructures@@QAEXPBDI@Z 004025a0 f   DS_ByteQueue.obj
 0001:000016b0       ?ReadBytes@ByteQueue@DataStructures@@QAE_NPADI_N@Z 004026b0 f   DS_ByteQueue.obj
 0001:00001750       ??0HuffmanEncodingTree@@QAE@XZ 00402750 f   DS_HuffmanEncodingTree.obj
 0001:00001760       ?DecodeArray@HuffmanEncodingTree@@QAEIPAVBitStream@RakNet@@IIPAE@Z 00402760 f   DS_HuffmanEncodingTree.obj
 0001:000017c0       ?DecodeArray@HuffmanEncodingTree@@QAEXPAEIPAVBitStream@RakNet@@@Z 004027c0 f   DS_HuffmanEncodingTree.obj
 0001:00001890       ??0?$Queue@PAUHuffmanEncodingTreeNode@@@DataStructures@@QAE@XZ 00402890 f i DS_HuffmanEncodingTree.obj
 0001:000018d0       ??1?$Queue@PAUHuffmanEncodingTreeNode@@@DataStructures@@QAE@XZ 004028d0 f i DS_HuffmanEncodingTree.obj
 0001:000018e0       ?Push@?$Queue@PAUHuffmanEncodingTreeNode@@@DataStructures@@QAEXABQAUHuffmanEncodingTreeNode@@@Z 004028e0 f i DS_HuffmanEncodingTree.obj
 0001:000019b0       ?Pop@?$Queue@PAUHuffmanEncodingTreeNode@@@DataStructures@@QAEPAUHuffmanEncodingTreeNode@@XZ 004029b0 f i DS_HuffmanEncodingTree.obj
 0001:000019e0       ?Size@?$Queue@PAUHuffmanEncodingTreeNode@@@DataStructures@@QBEIXZ 004029e0 f i DS_HuffmanEncodingTree.obj
 0001:00001a00       ??0?$CircularLinkedList@PAUHuffmanEncodingTreeNode@@@DataStructures@@QAE@XZ 00402a00 f i DS_HuffmanEncodingTree.obj
 0001:00001a10       ?Insert@?$CircularLinkedList@PAUHuffmanEncodingTreeNode@@@DataStructures@@QAEXABQAUHuffmanEncodingTreeNode@@@Z 00402a10 f i DS_HuffmanEncodingTree.obj
 0001:00001ae0       ?Add@?$CircularLinkedList@PAUHuffmanEncodingTreeNode@@@DataStructures@@QAEAAPAUHuffmanEncodingTreeNode@@ABQAU3@@Z 00402ae0 f i DS_HuffmanEncodingTree.obj
 0001:00001ba0       ?Size@?$CircularLinkedList@PAUHuffmanEncodingTreeNode@@@DataStructures@@QAEIXZ 00402ba0 f i DS_HuffmanEncodingTree.obj
 0001:00001bb0       ?Peek@?$CircularLinkedList@PAUHuffmanEncodingTreeNode@@@DataStructures@@QAEAAPAUHuffmanEncodingTreeNode@@XZ 00402bb0 f i DS_HuffmanEncodingTree.obj
 0001:00001bc0       ?Beginning@?$CircularLinkedList@PAUHuffmanEncodingTreeNode@@@DataStructures@@QAEXXZ 00402bc0 f i DS_HuffmanEncodingTree.obj
 0001:00001bd0       ?End@?$CircularLinkedList@PAUHuffmanEncodingTreeNode@@@DataStructures@@QAEXXZ 00402bd0 f i DS_HuffmanEncodingTree.obj
 0001:00001be0       ??E?$LinkedList@PAUHuffmanEncodingTreeNode@@@DataStructures@@QAEAAV01@XZ 00402be0 f i DS_HuffmanEncodingTree.obj
 0001:00001c00       ?Del@?$CircularLinkedList@PAUHuffmanEncodingTreeNode@@@DataStructures@@QAEXXZ 00402c00 f i DS_HuffmanEncodingTree.obj
 0001:00001c60       ?Clear@?$CircularLinkedList@PAUHuffmanEncodingTreeNode@@@DataStructures@@QAEXXZ 00402c60 f i DS_HuffmanEncodingTree.obj
 0001:00001cb0       ?FreeMemory@HuffmanEncodingTree@@QAEXXZ 00402cb0 f   DS_HuffmanEncodingTree.obj
 0001:00001e10       ?EncodeArray@HuffmanEncodingTree@@QAEXPAEIPAVBitStream@RakNet@@@Z 00402e10 f   DS_HuffmanEncodingTree.obj
 0001:00001eb0       ?InsertNodeIntoSortedList@HuffmanEncodingTree@@ABEXPAUHuffmanEncodingTreeNode@@PAV?$LinkedList@PAUHuffmanEncodingTreeNode@@@DataStructures@@@Z 00402eb0 f   DS_HuffmanEncodingTree.obj
 0001:00001f40       ??1?$CircularLinkedList@PAUHuffmanEncodingTreeNode@@@DataStructures@@QAE@XZ 00402f40 f i DS_HuffmanEncodingTree.obj
 0001:00001f50       ?Pop@?$CircularLinkedList@PAUHuffmanEncodingTreeNode@@@DataStructures@@QAEPAUHuffmanEncodingTreeNode@@XZ 00402f50 f i DS_HuffmanEncodingTree.obj
 0001:00001f60       ??1?$LinkedList@PAUHuffmanEncodingTreeNode@@@DataStructures@@QAE@XZ 00402f60 f i DS_HuffmanEncodingTree.obj
 0001:00001fb0       ??1HuffmanEncodingTree@@QAE@XZ 00402fb0 f   DS_HuffmanEncodingTree.obj
 0001:00001fc0       ??0?$LinkedList@PAUHuffmanEncodingTreeNode@@@DataStructures@@QAE@XZ 00402fc0 f i DS_HuffmanEncodingTree.obj
 0001:00001fd0       ?GenerateFromFrequencyTable@HuffmanEncodingTree@@QAEXQAI@Z 00402fd0 f   DS_HuffmanEncodingTree.obj
 0001:00002260       ??0Cell@Table@DataStructures@@QAE@XZ 00403260 f   DS_Table.obj
 0001:00002270       ??4Cell@Table@DataStructures@@QAEAAU012@ABU012@@Z 00403270 f   DS_Table.obj
 0001:000022c0       ??0Cell@Table@DataStructures@@QAE@ABU012@@Z 004032c0 f   DS_Table.obj
 0001:00002310       ?Set@Cell@Table@DataStructures@@QAEXH@Z 00403310 f   DS_Table.obj
 0001:00002350       ?Set@Cell@Table@DataStructures@@QAEXPAD@Z 00403350 f   DS_Table.obj
 0001:000023d0       ?Set@Cell@Table@DataStructures@@QAEXPADH@Z 004033d0 f   DS_Table.obj
 0001:00002430       ?Get@Cell@Table@DataStructures@@QAEXPAH@Z 00403430 f   DS_Table.obj
 0001:00002470       ?Get@Cell@Table@DataStructures@@QAEXPAD@Z 00403470 f   DS_Table.obj
 0001:000024b0       ?Get@Cell@Table@DataStructures@@QAEXPADPAH@Z 004034b0 f   DS_Table.obj
 0001:00002500       ??0Cell@Table@DataStructures@@QAE@HPADW4ColumnType@12@@Z 00403500 f   DS_Table.obj
 0001:00002570       ?Clear@Cell@Table@DataStructures@@QAEXXZ 00403570 f   DS_Table.obj
 0001:00002590       ??0ColumnDescriptor@Table@DataStructures@@QAE@XZ 00403590 f   DS_Table.obj
 0001:000025a0       ??1ColumnDescriptor@Table@DataStructures@@QAE@XZ 004035a0 f   DS_Table.obj
 0001:000025b0       ??0ColumnDescriptor@Table@DataStructures@@QAE@QADW4ColumnType@12@@Z 004035b0 f   DS_Table.obj
 0001:000025e0       ??0FilterQuery@Table@DataStructures@@QAE@XZ 004035e0 f   DS_Table.obj
 0001:000025f0       ??1FilterQuery@Table@DataStructures@@QAE@XZ 004035f0 f   DS_Table.obj
 0001:00002600       ??0FilterQuery@Table@DataStructures@@QAE@IPAUCell@12@W4FilterQueryType@12@@Z 00403600 f   DS_Table.obj
 0001:00002620       ?GetColumns@Table@DataStructures@@QAEAAV?$List@UColumnDescriptor@Table@DataStructures@@@2@XZ 00403620 f   DS_Table.obj
 0001:00002630       ?GetRows@Table@DataStructures@@QAEAAV?$BPlusTree@IPAURow@Table@DataStructures@@$0BA@@2@XZ 00403630 f   DS_Table.obj
 0001:00002640       ??0?$List@PAUCell@Table@DataStructures@@@DataStructures@@QAE@XZ 00403640 f i DS_Table.obj
 0001:00002650       ??1?$List@PAUCell@Table@DataStructures@@@DataStructures@@QAE@XZ 00403650 f i DS_Table.obj
 0001:00002660       ??A?$List@PAUCell@Table@DataStructures@@@DataStructures@@QBEAAPAUCell@Table@1@I@Z 00403660 f i DS_Table.obj
 0001:00002670       ?Insert@?$List@PAUCell@Table@DataStructures@@@DataStructures@@QAEXQAUCell@Table@2@@Z 00403670 f i DS_Table.obj
 0001:000026e0       ?Size@?$List@PAUCell@Table@DataStructures@@@DataStructures@@QBEIXZ 004036e0 f i DS_Table.obj
 0001:000026f0       ?GetListHead@?$BPlusTree@IPAURow@Table@DataStructures@@$0BA@@DataStructures@@QBEPAU?$Page@IPAURow@Table@DataStructures@@$0BA@@2@XZ 004036f0 f i DS_Table.obj
 0001:00002700       ?ForEachData@?$BPlusTree@IPAURow@Table@DataStructures@@$0BA@@DataStructures@@QAEXP6AXPAURow@Table@2@H@Z@Z 00403700 f i DS_Table.obj
 0001:00002750       ??0?$List@UColumnDescriptor@Table@DataStructures@@@DataStructures@@QAE@XZ 00403750 f i DS_Table.obj
 0001:00002760       ??A?$List@UColumnDescriptor@Table@DataStructures@@@DataStructures@@QBEAAUColumnDescriptor@Table@1@I@Z 00403760 f i DS_Table.obj
 0001:00002770       ?Size@?$List@UColumnDescriptor@Table@DataStructures@@@DataStructures@@QBEIXZ 00403770 f i DS_Table.obj
 0001:00002780       ??A?$List@UCell@Table@DataStructures@@@DataStructures@@QBEAAUCell@Table@1@I@Z 00403780 f i DS_Table.obj
 0001:00002790       ?Size@?$List@UCell@Table@DataStructures@@@DataStructures@@QBEIXZ 00403790 f i DS_Table.obj
 0001:000027a0       ??0?$List@I@DataStructures@@QAE@ABV01@@Z 004037a0 f i DS_Table.obj
 0001:00002800       ??0?$List@I@DataStructures@@QAE@XZ 00403800 f i DS_Table.obj
 0001:00002810       ??1?$List@I@DataStructures@@QAE@XZ 00403810 f i DS_Table.obj
 0001:00002820       ??A?$List@I@DataStructures@@QBEAAII@Z 00403820 f i DS_Table.obj
 0001:00002830       ?Insert@?$List@I@DataStructures@@QAEXI@Z 00403830 f i DS_Table.obj
 0001:000028a0       ?Size@?$List@I@DataStructures@@QBEIXZ 004038a0 f i DS_Table.obj
 0001:000028b0       ??_EColumnDescriptor@Table@DataStructures@@QAEPAXI@Z 004038b0 f i DS_Table.obj
 0001:00002900       ?Del@?$List@PAUCell@Table@DataStructures@@@DataStructures@@QAEXI@Z 00403900 f i DS_Table.obj
 0001:00002910       ?DeleteFromPageAtIndex@?$BPlusTree@IPAURow@Table@DataStructures@@$0BA@@DataStructures@@IAEXHPAU?$Page@IPAURow@Table@DataStructures@@$0BA@@2@@Z 00403910 f i DS_Table.obj
 0001:00002990       ?GetIndexOf@?$BPlusTree@IPAURow@Table@DataStructures@@$0BA@@DataStructures@@IBE_NIPAU?$Page@IPAURow@Table@DataStructures@@$0BA@@2@PAH@Z 00403990 f i DS_Table.obj
 0001:00002a10       ?GetLeafFromKey@?$BPlusTree@IPAURow@Table@DataStructures@@$0BA@@DataStructures@@IBEPAU?$Page@IPAURow@Table@DataStructures@@$0BA@@2@I@Z 00403a10 f i DS_Table.obj
 0001:00002a50       ?Del@?$List@UColumnDescriptor@Table@DataStructures@@@DataStructures@@QAEXI@Z 00403a50 f i DS_Table.obj
 0001:00002a60       ??0?$List@PAURow@Table@DataStructures@@@DataStructures@@QAE@XZ 00403a60 f i DS_Table.obj
 0001:00002a70       ??1?$List@PAURow@Table@DataStructures@@@DataStructures@@QAE@XZ 00403a70 f i DS_Table.obj
 0001:00002a80       ??A?$List@PAURow@Table@DataStructures@@@DataStructures@@QBEAAPAURow@Table@1@I@Z 00403a80 f i DS_Table.obj
 0001:00002a90       ?Insert@?$List@PAURow@Table@DataStructures@@@DataStructures@@QAEXQAURow@Table@2@@Z 00403a90 f i DS_Table.obj
 0001:00002b00       ?Insert@?$List@PAURow@Table@DataStructures@@@DataStructures@@QAEXQAURow@Table@2@I@Z 00403b00 f i DS_Table.obj
 0001:00002b90       ?Size@?$List@PAURow@Table@DataStructures@@@DataStructures@@QBEIXZ 00403b90 f i DS_Table.obj
 0001:00002ba0       ?CanRotateLeft@?$BPlusTree@IPAURow@Table@DataStructures@@$0BA@@DataStructures@@IAE_NPAU?$Page@IPAURow@Table@DataStructures@@$0BA@@2@H@Z 00403ba0 f i DS_Table.obj
 0001:00002bd0       ?CanRotateRight@?$BPlusTree@IPAURow@Table@DataStructures@@$0BA@@DataStructures@@IAE_NPAU?$Page@IPAURow@Table@DataStructures@@$0BA@@2@H@Z 00403bd0 f i DS_Table.obj
 0001:00002c00       ?RotateRight@?$BPlusTree@IPAURow@Table@DataStructures@@$0BA@@DataStructures@@IAEXPAU?$Page@IPAURow@Table@DataStructures@@$0BA@@2@HPAUReturnAction@12@@Z 00403c00 f i DS_Table.obj
 0001:00002c80       ?RotateLeft@?$BPlusTree@IPAURow@Table@DataStructures@@$0BA@@DataStructures@@IAEXPAU?$Page@IPAURow@Table@DataStructures@@$0BA@@2@HPAUReturnAction@12@@Z 00403c80 f i DS_Table.obj
 0001:00002d00       ??0?$Queue@PAU?$Page@IPAURow@Table@DataStructures@@$0BA@@DataStructures@@@DataStructures@@QAE@XZ 00403d00 f i DS_Table.obj
 0001:00002d40       ??1?$Queue@PAU?$Page@IPAURow@Table@DataStructures@@$0BA@@DataStructures@@@DataStructures@@QAE@XZ 00403d40 f i DS_Table.obj
 0001:00002d50       ?Push@?$Queue@PAU?$Page@IPAURow@Table@DataStructures@@$0BA@@DataStructures@@@DataStructures@@QAEXABQAU?$Page@IPAURow@Table@DataStructures@@$0BA@@2@@Z 00403d50 f i DS_Table.obj
 0001:00002e20       ?Pop@?$Queue@PAU?$Page@IPAURow@Table@DataStructures@@$0BA@@DataStructures@@@DataStructures@@QAEPAU?$Page@IPAURow@Table@DataStructures@@$0BA@@2@XZ 00403e20 f i DS_Table.obj
 0001:00002e50       ?Size@?$Queue@PAU?$Page@IPAURow@Table@DataStructures@@$0BA@@DataStructures@@@DataStructures@@QBEIXZ 00403e50 f i DS_Table.obj
 0001:00002e70       ??0?$List@PAU?$Page@IPAURow@Table@DataStructures@@$0BA@@DataStructures@@@DataStructures@@QAE@XZ 00403e70 f i DS_Table.obj
 0001:00002e80       ??1?$List@PAU?$Page@IPAURow@Table@DataStructures@@$0BA@@DataStructures@@@DataStructures@@QAE@XZ 00403e80 f i DS_Table.obj
 0001:00002e90       ??A?$List@PAU?$Page@IPAURow@Table@DataStructures@@$0BA@@DataStructures@@@DataStructures@@QBEAAPAU?$Page@IPAURow@Table@DataStructures@@$0BA@@1@I@Z 00403e90 f i DS_Table.obj
 0001:00002ea0       ?Insert@?$List@PAU?$Page@IPAURow@Table@DataStructures@@$0BA@@DataStructures@@@DataStructures@@QAEXQAU?$Page@IPAURow@Table@DataStructures@@$0BA@@2@@Z 00403ea0 f i DS_Table.obj
 0001:00002f10       ?Del@?$List@PAU?$Page@IPAURow@Table@DataStructures@@$0BA@@DataStructures@@@DataStructures@@QAEXI@Z 00403f10 f i DS_Table.obj
 0001:00002f20       ?Size@?$List@PAU?$Page@IPAURow@Table@DataStructures@@$0BA@@DataStructures@@@DataStructures@@QBEIXZ 00403f20 f i DS_Table.obj
 0001:00002f30       ?Clear@?$List@PAURow@Table@DataStructures@@@DataStructures@@QAEX_N@Z 00403f30 f i DS_Table.obj
 0001:00002f70       ?ShiftNodeLeft@?$BPlusTree@IPAURow@Table@DataStructures@@$0BA@@DataStructures@@IAEXPAU?$Page@IPAURow@Table@DataStructures@@$0BA@@2@@Z 00403f70 f i DS_Table.obj
 0001:00002fe0       ?ShiftNodeRight@?$BPlusTree@IPAURow@Table@DataStructures@@$0BA@@DataStructures@@IAEXPAU?$Page@IPAURow@Table@DataStructures@@$0BA@@2@@Z 00403fe0 f i DS_Table.obj
 0001:00003060       ?ExtendRows@@YAXPAURow@Table@DataStructures@@H@Z 00404060 f   DS_Table.obj
 0001:00003090       ??1Row@Table@DataStructures@@QAE@XZ 00404090 f i DS_Table.obj
 0001:000030a0       ??1Cell@Table@DataStructures@@QAE@XZ 004040a0 f   DS_Table.obj
 0001:000030c0       ?UpdateCell@Row@Table@DataStructures@@QAEXIH@Z 004040c0 f   DS_Table.obj
 0001:00003120       ?UpdateCell@Row@Table@DataStructures@@QAEXIPAD@Z 00404120 f   DS_Table.obj
 0001:00003160       ?UpdateCell@Row@Table@DataStructures@@QAEXIHPAD@Z 00404160 f   DS_Table.obj
 0001:000031a0       ?ColumnIndex@Table@DataStructures@@QAEIQAD@Z 004041a0 f   DS_Table.obj
 0001:00003200       ?ColumnName@Table@DataStructures@@QAEPADI@Z 00404200 f   DS_Table.obj
 0001:00003220       ?GetColumnType@Table@DataStructures@@QAE?AW4ColumnType@12@I@Z 00404220 f   DS_Table.obj
 0001:00003240       ?GetColumnCount@Table@DataStructures@@QBEIXZ 00404240 f   DS_Table.obj
 0001:00003250       ??0Row@Table@DataStructures@@QAE@XZ 00404250 f i DS_Table.obj
 0001:00003260       ?GetRowByIndex@Table@DataStructures@@QAEPAURow@12@I@Z 00404260 f   DS_Table.obj
 0001:000032a0       ?RowSort@@YAHABQAURow@Table@DataStructures@@0@Z 004042a0 f   DS_Table.obj
 0001:00003470       ?PrintRow@Table@DataStructures@@QAEXPADHD_NPAURow@12@@Z 00404470 f   DS_Table.obj
 0001:00003660       ?GetListHead@Table@DataStructures@@QAEPAU?$Page@IPAURow@Table@DataStructures@@$0BA@@2@XZ 00404660 f   DS_Table.obj
 0001:00003670       ?RemoveAtIndex@?$List@PAUCell@Table@DataStructures@@@DataStructures@@QAEXI@Z 00404670 f i DS_Table.obj
 0001:000036b0       ?Get@?$BPlusTree@IPAURow@Table@DataStructures@@$0BA@@DataStructures@@QBE_NIAAPAURow@Table@2@@Z 004046b0 f i DS_Table.obj
 0001:00003700       ?Size@?$BPlusTree@IPAURow@Table@DataStructures@@$0BA@@DataStructures@@QBEIXZ 00404700 f i DS_Table.obj
 0001:00003720       ??1?$List@UColumnDescriptor@Table@DataStructures@@@DataStructures@@QAE@XZ 00404720 f i DS_Table.obj
 0001:00003750       ?Insert@?$List@UColumnDescriptor@Table@DataStructures@@@DataStructures@@QAEXUColumnDescriptor@Table@2@@Z 00404750 f i DS_Table.obj
 0001:00003860       ?RemoveAtIndex@?$List@UColumnDescriptor@Table@DataStructures@@@DataStructures@@QAEXI@Z 00404860 f i DS_Table.obj
 0001:000038a0       ?Clear@?$List@UColumnDescriptor@Table@DataStructures@@@DataStructures@@QAEX_N@Z 004048a0 f i DS_Table.obj
 0001:00003900       ??0?$OrderedList@PAURow@Table@DataStructures@@PAU123@$1?RowSort@@YAHABQAU123@0@Z@DataStructures@@QAE@XZ 00404900 f i DS_Table.obj
 0001:00003910       ??A?$OrderedList@PAURow@Table@DataStructures@@PAU123@$1?RowSort@@YAHABQAU123@0@Z@DataStructures@@QBEAAPAURow@Table@1@I@Z 00404910 f i DS_Table.obj
 0001:00003920       ?Size@?$OrderedList@PAURow@Table@DataStructures@@PAU123@$1?RowSort@@YAHABQAU123@0@Z@DataStructures@@QBEIXZ 00404920 f i DS_Table.obj
 0001:00003930       ??0?$MemoryPool@U?$Page@IPAURow@Table@DataStructures@@$0BA@@DataStructures@@@DataStructures@@QAE@XZ 00404930 f i DS_Table.obj
 0001:00003940       ??1?$MemoryPool@U?$Page@IPAURow@Table@DataStructures@@$0BA@@DataStructures@@@DataStructures@@QAE@XZ 00404940 f i DS_Table.obj
 0001:000039b0       ?Allocate@?$MemoryPool@U?$Page@IPAURow@Table@DataStructures@@$0BA@@DataStructures@@@DataStructures@@QAEPAU?$Page@IPAURow@Table@DataStructures@@$0BA@@2@XZ 004049b0 f i DS_Table.obj
 0001:000039d0       ?Release@?$MemoryPool@U?$Page@IPAURow@Table@DataStructures@@$0BA@@DataStructures@@@DataStructures@@QAEXPAU?$Page@IPAURow@Table@DataStructures@@$0BA@@2@@Z 004049d0 f i DS_Table.obj
 0001:000039e0       ?GetIndexFromKey@?$OrderedList@PAURow@Table@DataStructures@@PAU123@$1?RowSort@@YAHABQAU123@0@Z@DataStructures@@QBEIABQAURow@Table@2@PA_N@Z 004049e0 f i DS_Table.obj
 0001:00003a70       ?Clear@?$OrderedList@PAURow@Table@DataStructures@@PAU123@$1?RowSort@@YAHABQAU123@0@Z@DataStructures@@QAEXXZ 00404a70 f i DS_Table.obj
 0001:00003ab0       ?InsertIntoNode@?$BPlusTree@IPAURow@Table@DataStructures@@$0BA@@DataStructures@@IAEPAU?$Page@IPAURow@Table@DataStructures@@$0BA@@2@IABQAURow@Table@2@HPAU32@1PAUReturnAction@12@@Z 00404ab0 f i DS_Table.obj
 0001:00003ed0       ?FixUnderflow@?$BPlusTree@IPAURow@Table@DataStructures@@$0BA@@DataStructures@@IAE_NHPAU?$Page@IPAURow@Table@DataStructures@@$0BA@@2@IPAUReturnAction@12@@Z 00404ed0 f i DS_Table.obj
 0001:00004140       ??_GCell@Table@DataStructures@@QAEPAXI@Z 00405140 f i DS_Table.obj
 0001:00004170       ??_GRow@Table@DataStructures@@QAEPAXI@Z 00405170 f i DS_Table.obj
 0001:000041a0       ?AddColumn@Table@DataStructures@@QAEIQADW4ColumnType@12@@Z 004051a0 f   DS_Table.obj
 0001:00004210       ?RemoveColumn@Table@DataStructures@@QAEXI@Z 00405210 f   DS_Table.obj
 0001:000042f0       ?GetRowCount@Table@DataStructures@@QBEIXZ 004052f0 f   DS_Table.obj
 0001:00004310       ?GetRowByID@Table@DataStructures@@QAEPAURow@12@I@Z 00405310 f   DS_Table.obj
 0001:00004350       ?DeleteRow@Table@DataStructures@@IAEXPAURow@12@@Z 00405350 f   DS_Table.obj
 0001:000043b0       ??0?$BPlusTree@IPAURow@Table@DataStructures@@$0BA@@DataStructures@@QAE@XZ 004053b0 f i DS_Table.obj
 0001:000043d0       ??1?$OrderedList@PAURow@Table@DataStructures@@PAU123@$1?RowSort@@YAHABQAU123@0@Z@DataStructures@@QAE@XZ 004053d0 f i DS_Table.obj
 0001:00004450       ?Insert@?$OrderedList@PAURow@Table@DataStructures@@PAU123@$1?RowSort@@YAHABQAU123@0@Z@DataStructures@@QAEIABQAURow@Table@2@0@Z 00405450 f i DS_Table.obj
 0001:000044b0       ?FreePages@?$BPlusTree@IPAURow@Table@DataStructures@@$0BA@@DataStructures@@IAEXXZ 004054b0 f i DS_Table.obj
 0001:00004630       ?InsertBranchDown@?$BPlusTree@IPAURow@Table@DataStructures@@$0BA@@DataStructures@@IAEPAU?$Page@IPAURow@Table@DataStructures@@$0BA@@2@IABQAURow@Table@2@PAU32@PAUReturnAction@12@PA_N@Z 00405630 f i DS_Table.obj
 0001:000048d0       ?FindDeleteRebalance@?$BPlusTree@IPAURow@Table@DataStructures@@$0BA@@DataStructures@@IAE_NIPAU?$Page@IPAURow@Table@DataStructures@@$0BA@@2@PA_NIPAUReturnAction@12@AAPAURow@Table@2@@Z 004058d0 f i DS_Table.obj
 0001:00004a40       ?FreeRow@@YAXPAURow@Table@DataStructures@@H@Z 00405a40 f   DS_Table.obj
 0001:00004aa0       ?UpdateCell@Table@DataStructures@@QAE_NIIH@Z 00405aa0 f   DS_Table.obj
 0001:00004b20       ?UpdateCell@Table@DataStructures@@QAE_NIIPAD@Z 00405b20 f   DS_Table.obj
 0001:00004bc0       ?UpdateCell@Table@DataStructures@@QAE_NIIHPAD@Z 00405bc0 f   DS_Table.obj
 0001:00004c60       ?SortTable@Table@DataStructures@@QAEXPAUSortQuery@12@IPAPAURow@12@@Z 00405c60 f   DS_Table.obj
 0001:00004f10       ?Delete@?$BPlusTree@IPAURow@Table@DataStructures@@$0BA@@DataStructures@@QAE_NIAAPAURow@Table@2@@Z 00405f10 f i DS_Table.obj
 0001:00004ff0       ?Delete@?$BPlusTree@IPAURow@Table@DataStructures@@$0BA@@DataStructures@@QAE_NI@Z 00405ff0 f i DS_Table.obj
 0001:00005010       ?Insert@?$BPlusTree@IPAURow@Table@DataStructures@@$0BA@@DataStructures@@QAE_NIABQAURow@Table@2@@Z 00406010 f i DS_Table.obj
 0001:00005150       ?Clear@?$BPlusTree@IPAURow@Table@DataStructures@@$0BA@@DataStructures@@QAEXXZ 00406150 f i DS_Table.obj
 0001:00005170       ?AddRow@Table@DataStructures@@QAEPAURow@12@I@Z 00406170 f   DS_Table.obj
 0001:00005220       ?AddRow@Table@DataStructures@@QAEPAURow@12@IAAV?$List@UCell@Table@DataStructures@@@2@@Z 00406220 f   DS_Table.obj
 0001:00005340       ?AddRowColumns@Table@DataStructures@@IAEPAURow@12@IPAU312@V?$List@I@2@@Z 00406340 f   DS_Table.obj
 0001:00005480       ?RemoveRow@Table@DataStructures@@QAEXI@Z 00406480 f   DS_Table.obj
 0001:000054b0       ?RemoveRows@Table@DataStructures@@QAEXPAV12@@Z 004064b0 f   DS_Table.obj
 0001:00005500       ?QueryRow@Table@DataStructures@@IAEXAAV?$List@I@2@0IPAURow@12@PAUFilterQuery@12@PAV12@@Z 00406500 f   DS_Table.obj
 0001:000058c0       ?Clear@Table@DataStructures@@QAEXXZ 004068c0 f   DS_Table.obj
 0001:00005900       ??1?$BPlusTree@IPAURow@Table@DataStructures@@$0BA@@DataStructures@@QAE@XZ 00406900 f i DS_Table.obj
 0001:00005960       ??0Table@DataStructures@@QAE@XZ 00406960 f   DS_Table.obj
 0001:00005980       ??1Table@DataStructures@@QAE@XZ 00406980 f   DS_Table.obj
 0001:00005a20       ?QueryTable@Table@DataStructures@@QAEXPAIIPAUFilterQuery@12@I0IPAV12@@Z 00406a20 f   DS_Table.obj
 0001:00005d20       ?GetTime@RakNet@@YAIXZ     00406d20 f   GetTime.obj
 0001:00005d80       ?GetTimeNS@RakNet@@YA_JXZ  00406d80 f   GetTime.obj
 0001:00005e20       ??0?$Queue@PAUInternalPacket@@@DataStructures@@QAE@XZ 00406e20 f i InternalPacketPool.obj
 0001:00005e60       ??1?$Queue@PAUInternalPacket@@@DataStructures@@QAE@XZ 00406e60 f i InternalPacketPool.obj
 0001:00005e70       ?Push@?$Queue@PAUInternalPacket@@@DataStructures@@QAEXABQAUInternalPacket@@@Z 00406e70 f i InternalPacketPool.obj
 0001:00005f40       ?Pop@?$Queue@PAUInternalPacket@@@DataStructures@@QAEPAUInternalPacket@@XZ 00406f40 f i InternalPacketPool.obj
 0001:00005f70       ?Size@?$Queue@PAUInternalPacket@@@DataStructures@@QBEIXZ 00406f70 f i InternalPacketPool.obj
 0001:00005f90       ?ClearAndForceAllocation@?$Queue@PAUInternalPacket@@@DataStructures@@QAEXH@Z 00406f90 f i InternalPacketPool.obj
 0001:00005fd0       ??0InternalPacketPool@@QAE@XZ 00406fd0 f   InternalPacketPool.obj
 0001:00006090       ?ClearPool@InternalPacketPool@@QAEXXZ 00407090 f   InternalPacketPool.obj
 0001:000060f0       ?ReleasePointer@InternalPacketPool@@QAEXPAUInternalPacket@@@Z 004070f0 f   InternalPacketPool.obj
 0001:00006110       ??1InternalPacketPool@@QAE@XZ 00407110 f   InternalPacketPool.obj
 0001:00006170       ??4PlayerID@@QAEAAU0@ABU0@@Z 00407170 f i NetworkIDGenerator.obj
 0001:00006190       ??8NetworkIDNode@@QBE_NABU0@@Z 00407190 f   NetworkIDGenerator.obj
 0001:000061b0       ??ONetworkIDNode@@QBE_NABU0@@Z 004071b0 f   NetworkIDGenerator.obj
 0001:000061d0       ??MNetworkIDNode@@QBE_NABU0@@Z 004071d0 f   NetworkIDGenerator.obj
 0001:000061f0       ??0NetworkIDNode@@QAE@XZ   004071f0 f   NetworkIDGenerator.obj
 0001:00006200       ??0NetworkIDNode@@QAE@UNetworkID@@PAVNetworkIDGenerator@@@Z 00407200 f   NetworkIDGenerator.obj
 0001:00006220       ??0NetworkIDGenerator@@QAE@XZ 00407220 f   NetworkIDGenerator.obj
 0001:00006250       ?GetStaticNetworkID@NetworkIDGenerator@@SAGXZ 00407250 f   NetworkIDGenerator.obj
 0001:00006260       ?SetStaticNetworkID@NetworkIDGenerator@@SAXG@Z 00407260 f   NetworkIDGenerator.obj
 0001:00006270       ?SetExternalPlayerID@NetworkIDGenerator@@SAXUPlayerID@@@Z 00407270 f   NetworkIDGenerator.obj
 0001:000062d0       ?GetExternalPlayerID@NetworkIDGenerator@@SA?AUPlayerID@@XZ 004072d0 f   NetworkIDGenerator.obj
 0001:000062f0       ?RequiresSetParent@NetworkIDGenerator@@UBE_NXZ 004072f0 f   NetworkIDGenerator.obj
 0001:00006300       ?SetParent@NetworkIDGenerator@@UAEXPAX@Z 00407300 f   NetworkIDGenerator.obj
 0001:00006310       ?GetParent@NetworkIDGenerator@@UBEPAXXZ 00407310 f   NetworkIDGenerator.obj
 0001:00006320       ??0?$BinarySearchTree@UNetworkIDNode@@@DataStructures@@QAE@XZ 00407320 f i NetworkIDGenerator.obj
 0001:00006340       ?Find@?$BinarySearchTree@UNetworkIDNode@@@DataStructures@@IAEAAPAUnode@12@ABUNetworkIDNode@@PAPAU312@@Z 00407340 f i NetworkIDGenerator.obj
 0001:00006440       ??4NetworkIDNode@@QAEAAU0@ABU0@@Z 00407440 f i NetworkIDGenerator.obj
 0001:00006460       ?FindParent@?$BinarySearchTree@UNetworkIDNode@@@DataStructures@@IAEAAPAUnode@12@ABUNetworkIDNode@@@Z 00407460 f i NetworkIDGenerator.obj
 0001:00006480       ?RotateRight@?$AVLBalancedBinarySearchTree@UNetworkIDNode@@@DataStructures@@AAEXPAUnode@?$BinarySearchTree@UNetworkIDNode@@@2@@Z 00407480 f i NetworkIDGenerator.obj
 0001:000064f0       ?RotateLeft@?$AVLBalancedBinarySearchTree@UNetworkIDNode@@@DataStructures@@AAEXPAUnode@?$BinarySearchTree@UNetworkIDNode@@@2@@Z 004074f0 f i NetworkIDGenerator.obj
 0001:00006560       ?DoubleRotateRight@?$AVLBalancedBinarySearchTree@UNetworkIDNode@@@DataStructures@@AAEXPAUnode@?$BinarySearchTree@UNetworkIDNode@@@2@@Z 00407560 f i NetworkIDGenerator.obj
 0001:00006590       ?DoubleRotateLeft@?$AVLBalancedBinarySearchTree@UNetworkIDNode@@@DataStructures@@AAEXPAUnode@?$BinarySearchTree@UNetworkIDNode@@@2@@Z 00407590 f i NetworkIDGenerator.obj
 0001:000065c0       ?HeightRecursive@?$BinarySearchTree@UNetworkIDNode@@@DataStructures@@IAEIPAUnode@12@@Z 004075c0 f i NetworkIDGenerator.obj
 0001:00006620       ?GetPointerToNode@?$BinarySearchTree@UNetworkIDNode@@@DataStructures@@QAEAAPAUNetworkIDNode@@ABU3@@Z 00407620 f i NetworkIDGenerator.obj
 0001:00006650       ?Clear@?$BinarySearchTree@UNetworkIDNode@@@DataStructures@@QAEXXZ 00407650 f i NetworkIDGenerator.obj
 0001:000066e0       ?Add@?$BinarySearchTree@UNetworkIDNode@@@DataStructures@@QAEPAUnode@12@ABUNetworkIDNode@@@Z 004076e0 f i NetworkIDGenerator.obj
 0001:00006810       ?Del@?$BinarySearchTree@UNetworkIDNode@@@DataStructures@@QAEPAUnode@12@ABUNetworkIDNode@@@Z 00407810 f i NetworkIDGenerator.obj
 0001:00006990       ?Height@?$BinarySearchTree@UNetworkIDNode@@@DataStructures@@QAEIPAUnode@12@@Z 00407990 f i NetworkIDGenerator.obj
 0001:000069b0       ?RightHigher@?$AVLBalancedBinarySearchTree@UNetworkIDNode@@@DataStructures@@AAE_NPAUnode@?$BinarySearchTree@UNetworkIDNode@@@2@@Z 004079b0 f i NetworkIDGenerator.obj
 0001:00006a10       ?LeftHigher@?$AVLBalancedBinarySearchTree@UNetworkIDNode@@@DataStructures@@AAE_NPAUnode@?$BinarySearchTree@UNetworkIDNode@@@2@@Z 00407a10 f i NetworkIDGenerator.obj
 0001:00006a70       ?GET_BASE_OBJECT_FROM_ID@NetworkIDGenerator@@SAPAXUNetworkID@@@Z 00407a70 f   NetworkIDGenerator.obj
 0001:00006af0       ?GET_OBJECT_FROM_ID@NetworkIDGenerator@@SAPAXUNetworkID@@@Z 00407af0 f   NetworkIDGenerator.obj
 0001:00006b40       ?GET_OBJECT_FROM_ID@@YAPAXUNetworkID@@@Z 00407b40 f   NetworkIDGenerator.obj
 0001:00006b90       ??1?$BinarySearchTree@UNetworkIDNode@@@DataStructures@@UAE@XZ 00407b90 f i NetworkIDGenerator.obj
 0001:00006ba0       ??1?$AVLBalancedBinarySearchTree@UNetworkIDNode@@@DataStructures@@UAE@XZ 00407ba0 f i NetworkIDGenerator.obj
 0001:00006c00       ??_G?$BinarySearchTree@UNetworkIDNode@@@DataStructures@@UAEPAXI@Z 00407c00 f i NetworkIDGenerator.obj
 0001:00006c00       ??_E?$BinarySearchTree@UNetworkIDNode@@@DataStructures@@UAEPAXI@Z 00407c00 f i NetworkIDGenerator.obj
 0001:00006c30       ?BalanceTree@?$AVLBalancedBinarySearchTree@UNetworkIDNode@@@DataStructures@@AAEXPAUnode@?$BinarySearchTree@UNetworkIDNode@@@2@_N@Z 00407c30 f i NetworkIDGenerator.obj
 0001:00006e10       ??0?$AVLBalancedBinarySearchTree@UNetworkIDNode@@@DataStructures@@QAE@XZ 00407e10 f i NetworkIDGenerator.obj
 0001:00006e30       ??_G?$AVLBalancedBinarySearchTree@UNetworkIDNode@@@DataStructures@@UAEPAXI@Z 00407e30 f i NetworkIDGenerator.obj
 0001:00006e30       ??_E?$AVLBalancedBinarySearchTree@UNetworkIDNode@@@DataStructures@@UAEPAXI@Z 00407e30 f i NetworkIDGenerator.obj
 0001:00006e50       ?Add@?$AVLBalancedBinarySearchTree@UNetworkIDNode@@@DataStructures@@QAEXABUNetworkIDNode@@@Z 00407e50 f i NetworkIDGenerator.obj
 0001:00006e70       ?Del@?$AVLBalancedBinarySearchTree@UNetworkIDNode@@@DataStructures@@QAEXABUNetworkIDNode@@@Z 00407e70 f i NetworkIDGenerator.obj
 0001:00006e90       ??1NetworkIDGenerator@@UAE@XZ 00407e90 f   NetworkIDGenerator.obj
 0001:00006f60       ?SetNetworkID@NetworkIDGenerator@@UAEXUNetworkID@@@Z 00407f60 f   NetworkIDGenerator.obj
 0001:00007120       ?GenerateID@NetworkIDGenerator@@IAEXXZ 00408120 f   NetworkIDGenerator.obj
 0001:00007250       ??_GNetworkIDGenerator@@UAEPAXI@Z 00408250 f i NetworkIDGenerator.obj
 0001:00007250       ??_ENetworkIDGenerator@@UAEPAXI@Z 00408250 f i NetworkIDGenerator.obj
 0001:00007270       ?GetNetworkID@NetworkIDGenerator@@UAE?AUNetworkID@@XZ 00408270 f   NetworkIDGenerator.obj
 0001:000072b0       ?my_itoa@@YAPADHPADH@Z     004082b0 f   NetworkTypes.obj
 0001:00007320       ??8PlayerID@@QBE_NABU0@@Z  00408320 f   NetworkTypes.obj
 0001:00007350       ??9PlayerID@@QBE_NABU0@@Z  00408350 f   NetworkTypes.obj
 0001:00007380       ??OPlayerID@@QBE_NABU0@@Z  00408380 f   NetworkTypes.obj
 0001:000073b0       ??MPlayerID@@QBE_NABU0@@Z  004083b0 f   NetworkTypes.obj
 0001:000073e0       ?ToString@PlayerID@@QBEPAD_N@Z 004083e0 f   NetworkTypes.obj
 0001:00007450       ?SetBinaryAddress@PlayerID@@QAEXPBD@Z 00408450 f   NetworkTypes.obj
 0001:00007470       ??4NetworkID@@QAEAAU0@ABU0@@Z 00408470 f   NetworkTypes.obj
 0001:00007490       ??8NetworkID@@QBE_NABU0@@Z 00408490 f   NetworkTypes.obj
 0001:000074e0       ??9NetworkID@@QBE_NABU0@@Z 004084e0 f   NetworkTypes.obj
 0001:00007530       ??ONetworkID@@QBE_NABU0@@Z 00408530 f   NetworkTypes.obj
 0001:00007590       ??MNetworkID@@QBE_NABU0@@Z 00408590 f   NetworkTypes.obj
 0001:000075f0       ?IsPeerToPeerMode@NetworkID@@SA_NXZ 004085f0 f   NetworkTypes.obj
 0001:00007600       ?SetPeerToPeerMode@NetworkID@@SAX_N@Z 00408600 f   NetworkTypes.obj
 0001:00007610       ?OnAttach@PluginInterface@@UAEXPAVRakPeerInterface@@@Z 00408610 f   PluginInterface.obj
 0001:00007620       ?OnDetach@PluginInterface@@UAEXPAVRakPeerInterface@@@Z 00408620 f   PluginInterface.obj
 0001:00007630       ?OnInitialize@PluginInterface@@UAEXPAVRakPeerInterface@@@Z 00408630 f   PluginInterface.obj
 0001:00007640       ?Update@PluginInterface@@UAEXPAVRakPeerInterface@@@Z 00408640 f   PluginInterface.obj
 0001:00007650       ?OnReceive@PluginInterface@@UAE?AW4PluginReceiveResult@@PAVRakPeerInterface@@PAUPacket@@@Z 00408650 f   PluginInterface.obj
 0001:00007660       ?OnDisconnect@PluginInterface@@UAEXPAVRakPeerInterface@@@Z 00408660 f   PluginInterface.obj
 0001:00007670       ?OnCloseConnection@PluginInterface@@UAEXPAVRakPeerInterface@@UPlayerID@@@Z 00408670 f   PluginInterface.obj
 0001:00007680       ?OnDirectSocketSend@PluginInterface@@UAEXPBDIUPlayerID@@@Z 00408680 f   PluginInterface.obj
 0001:00007690       ?OnDirectSocketReceive@PluginInterface@@UAEXPBDIUPlayerID@@@Z 00408690 f   PluginInterface.obj
 0001:000076a0       ?OnInternalPacket@PluginInterface@@UAEXPAUInternalPacket@@IUPlayerID@@I_N@Z 004086a0 f   PluginInterface.obj
 0001:000076b0       ?Instance@SocketLayer@@SAPAV1@XZ 004086b0 f i RakClient.obj
 0001:000076c0       ?GetNumberOfBytesUsed@BitStream@RakNet@@QBEHXZ 004086c0 f i RakClient.obj
 0001:000076d0       ?GetReadOffset@BitStream@RakNet@@QBEHXZ 004086d0 f i RakClient.obj
 0001:000076e0       ?GetData@BitStream@RakNet@@QBEPAEXZ 004086e0 f i RakClient.obj
 0001:000076f0       ??1RakClientInterface@@UAE@XZ 004086f0 f i RakClient.obj
 0001:00007700       ??_ERakClientInterface@@UAEPAXI@Z 00408700 f i RakClient.obj
 0001:00007700       ??_GRakClientInterface@@UAEPAXI@Z 00408700 f i RakClient.obj
 0001:00007720       ??0CVector@@QAE@MMM@Z      00408720 f i RakClient.obj
 0001:00007740       ??0RakClientInterface@@QAE@XZ 00408740 f i RakClient.obj
 0001:00007750       ??0OtherClientsStruct@RakClient@@QAE@XZ 00408750 f i RakClient.obj
 0001:00007760       ??1OtherClientsStruct@RakClient@@QAE@XZ 00408760 f i RakClient.obj
 0001:00007770       ??1RakClient@@UAE@XZ       00408770 f   RakClient.obj
 0001:00007800       ?Connect@RakClient@@UAE_NPBDGGIH@Z 00408800 f   RakClient.obj
 0001:000078c0       ?Disconnect@RakClient@@UAEXIE@Z 004088c0 f   RakClient.obj
 0001:000078d0       ?InitializeSecurity@RakClient@@UAEXPBD0@Z 004088d0 f   RakClient.obj
 0001:000078f0       ?SetPassword@RakClient@@UAEXPBD@Z 004088f0 f   RakClient.obj
 0001:00007940       ?HasPassword@RakClient@@UBE_NXZ 00408940 f   RakClient.obj
 0001:00007960       ?Send@RakClient@@UAE_NPBDHW4PacketPriority@@W4PacketReliability@@D@Z 00408960 f   RakClient.obj
 0001:000079a0       ?Send@RakClient@@UAE_NPAVBitStream@RakNet@@W4PacketPriority@@W4PacketReliability@@D@Z 004089a0 f   RakClient.obj
 0001:000079e0       ?DeallocatePacket@RakClient@@UAEXPAUPacket@@@Z 004089e0 f   RakClient.obj
 0001:000079f0       ?PingServer@RakClient@@UAEXXZ 004089f0 f   RakClient.obj
 0001:00007a10       ?PingServer@RakClient@@UAEXPBDGG_N@Z 00408a10 f   RakClient.obj
 0001:00007a50       ?GetAveragePing@RakClient@@UAEHXZ 00408a50 f   RakClient.obj
 0001:00007a80       ?GetLastPing@RakClient@@UBEHXZ 00408a80 f   RakClient.obj
 0001:00007ab0       ?GetLowestPing@RakClient@@UBEHXZ 00408ab0 f   RakClient.obj
 0001:00007ae0       ?GetPlayerPing@RakClient@@UAEHUPlayerID@@@Z 00408ae0 f   RakClient.obj
 0001:00007b30       ?StartOccasionalPing@RakClient@@UAEXXZ 00408b30 f   RakClient.obj
 0001:00007b40       ?StopOccasionalPing@RakClient@@UAEXXZ 00408b40 f   RakClient.obj
 0001:00007b50       ?IsConnected@RakClient@@UBE_NXZ 00408b50 f   RakClient.obj
 0001:00007b70       ?GetSynchronizedRandomInteger@RakClient@@UBEIXZ 00408b70 f   RakClient.obj
 0001:00007b90       ?GenerateCompressionLayer@RakClient@@UAE_NQAI_N@Z 00408b90 f   RakClient.obj
 0001:00007ba0       ?DeleteCompressionLayer@RakClient@@UAE_N_N@Z 00408ba0 f   RakClient.obj
 0001:00007bb0       ?RegisterAsRemoteProcedureCall@RakClient@@UAEXPAHP6AXPAURPCParameters@@@Z@Z 00408bb0 f   RakClient.obj
 0001:00007bc0       ?RegisterClassMemberRPC@RakClient@@UAEXPAHPAX@Z 00408bc0 f   RakClient.obj
 0001:00007bd0       ?UnregisterAsRemoteProcedureCall@RakClient@@UAEXPAH@Z 00408bd0 f   RakClient.obj
 0001:00007be0       ?RPC@RakClient@@UAE_NPAHPBDIW4PacketPriority@@W4PacketReliability@@D_NUNetworkID@@PAVBitStream@RakNet@@@Z 00408be0 f   RakClient.obj
 0001:00007c50       ?RPC@RakClient@@UAE_NPAHPAVBitStream@RakNet@@W4PacketPriority@@W4PacketReliability@@D_NUNetworkID@@1@Z 00408c50 f   RakClient.obj
 0001:00007cc0       ?SetTrackFrequencyTable@RakClient@@UAEX_N@Z 00408cc0 f   RakClient.obj
 0001:00007cd0       ?GetSendFrequencyTable@RakClient@@UAE_NQAI@Z 00408cd0 f   RakClient.obj
 0001:00007ce0       ?GetCompressionRatio@RakClient@@UBEMXZ 00408ce0 f   RakClient.obj
 0001:00007cf0       ?GetDecompressionRatio@RakClient@@UBEMXZ 00408cf0 f   RakClient.obj
 0001:00007d00       ?AttachPlugin@RakClient@@UAEXPAVPluginInterface@@@Z 00408d00 f   RakClient.obj
 0001:00007d10       ?DetachPlugin@RakClient@@UAEXPAVPluginInterface@@@Z 00408d10 f   RakClient.obj
 0001:00007d20       ?GetStaticServerData@RakClient@@UAEPAVBitStream@RakNet@@XZ 00408d20 f   RakClient.obj
 0001:00007d40       ?SetStaticServerData@RakClient@@UAEXPBDH@Z 00408d40 f   RakClient.obj
 0001:00007d70       ?SendStaticClientDataToServer@RakClient@@UAEXXZ 00408d70 f   RakClient.obj
 0001:00007d90       ?GetServerID@RakClient@@UBE?AUPlayerID@@XZ 00408d90 f   RakClient.obj
 0001:00007dc0       ?GetPlayerID@RakClient@@UBE?AUPlayerID@@XZ 00408dc0 f   RakClient.obj
 0001:00007e50       ?GetInternalID@RakClient@@UBE?AUPlayerID@@XZ 00408e50 f   RakClient.obj
 0001:00007e70       ?PlayerIDToDottedIP@RakClient@@UBEPBDUPlayerID@@@Z 00408e70 f   RakClient.obj
 0001:00007e90       ?PushBackPacket@RakClient@@UAEXPAUPacket@@_N@Z 00408e90 f   RakClient.obj
 0001:00007ea0       ?SetRouterInterface@RakClient@@UAEXPAVRouterInterface@@@Z 00408ea0 f   RakClient.obj
 0001:00007eb0       ?RemoveRouterInterface@RakClient@@UAEXPAVRouterInterface@@@Z 00408eb0 f   RakClient.obj
 0001:00007ec0       ?SetTimeoutTime@RakClient@@UAEXI@Z 00408ec0 f   RakClient.obj
 0001:00007f00       ?SetMTUSize@RakClient@@UAE_NH@Z 00408f00 f   RakClient.obj
 0001:00007f10       ?GetMTUSize@RakClient@@UBEHXZ 00408f10 f   RakClient.obj
 0001:00007f20       ?AllowConnectionResponseIPMigration@RakClient@@UAEX_N@Z 00408f20 f   RakClient.obj
 0001:00007f30       ?AdvertiseSystem@RakClient@@UAEXPBDG0H@Z 00408f30 f   RakClient.obj
 0001:00007f40       ?GetStatistics@RakClient@@UAEQAURakNetStatisticsStruct@@XZ 00408f40 f   RakClient.obj
 0001:00007f60       ?ApplyNetworkSimulator@RakClient@@UAEXNGG@Z 00408f60 f   RakClient.obj
 0001:00007f80       ?IsNetworkSimulatorActive@RakClient@@UAE_NXZ 00408f80 f   RakClient.obj
 0001:00007f90       ?GetOtherClientIndexByPlayerID@RakClient@@AAEHUPlayerID@@@Z 00408f90 f   RakClient.obj
 0001:00007fd0       ?GetFreeOtherClientIndex@RakClient@@AAEHXZ 00408fd0 f   RakClient.obj
 0001:00007ff0       ?GetPlayerIndex@RakClient@@UAEGXZ 00408ff0 f   RakClient.obj
 0001:00008000       ??$Read@G@BitStream@RakNet@@QAE_NAAG@Z 00409000 f i RakClient.obj
 0001:00008020       ??$Read@F@BitStream@RakNet@@QAE_NAAF@Z 00409020 f i RakClient.obj
 0001:00008040       ??$Read@E@BitStream@RakNet@@QAE_NAAE@Z 00409040 f i RakClient.obj
 0001:00008060       ?Disconnect@RakClient@@WKGI@AEXIE@Z 00409060 f i RakClient.obj
 0001:00008070       ?IsNetworkSimulatorActive@RakClient@@WKGI@AE_NXZ 00409070 f i RakClient.obj
 0001:00008080       ?GenerateCompressionLayer@RakClient@@WKGI@AE_NQAI_N@Z 00409080 f i RakClient.obj
 0001:00008090       ?DeallocatePacket@RakClient@@WKGI@AEXPAUPacket@@@Z 00409090 f i RakClient.obj
 0001:000080a0       ?SetRouterInterface@RakClient@@WKGI@AEXPAVRouterInterface@@@Z 004090a0 f i RakClient.obj
 0001:000080b0       ?GetInternalID@RakClient@@WKGI@BE?AUPlayerID@@XZ 004090b0 f i RakClient.obj
 0001:000080c0       ??_ERakClient@@WKGI@AEPAXI@Z 004090c0 f i RakClient.obj
 0001:000080d0       ?PlayerIDToDottedIP@RakClient@@WKGI@BEPBDUPlayerID@@@Z 004090d0 f i RakClient.obj
 0001:000080e0       ?UnregisterAsRemoteProcedureCall@RakClient@@WKGI@AEXPAH@Z 004090e0 f i RakClient.obj
 0001:000080f0       ?DetachPlugin@RakClient@@WKGI@AEXPAVPluginInterface@@@Z 004090f0 f i RakClient.obj
 0001:00008100       ?AttachPlugin@RakClient@@WKGI@AEXPAVPluginInterface@@@Z 00409100 f i RakClient.obj
 0001:00008110       ?RegisterAsRemoteProcedureCall@RakClient@@WKGI@AEXPAHP6AXPAURPCParameters@@@Z@Z 00409110 f i RakClient.obj
 0001:00008120       ?AllowConnectionResponseIPMigration@RakClient@@WKGI@AEX_N@Z 00409120 f i RakClient.obj
 0001:00008130       ?GetDecompressionRatio@RakClient@@WKGI@BEMXZ 00409130 f i RakClient.obj
 0001:00008140       ?SetMTUSize@RakClient@@WKGI@AE_NH@Z 00409140 f i RakClient.obj
 0001:00008150       ?GetMTUSize@RakClient@@WKGI@BEHXZ 00409150 f i RakClient.obj
 0001:00008160       ?PushBackPacket@RakClient@@WKGI@AEXPAUPacket@@_N@Z 00409160 f i RakClient.obj
 0001:00008170       ?AdvertiseSystem@RakClient@@WKGI@AEXPBDG0H@Z 00409170 f i RakClient.obj
 0001:00008180       ?RegisterClassMemberRPC@RakClient@@WKGI@AEXPAHPAX@Z 00409180 f i RakClient.obj
 0001:00008190       ?ApplyNetworkSimulator@RakClient@@WKGI@AEXNGG@Z 00409190 f i RakClient.obj
 0001:000081a0       ?RemoveRouterInterface@RakClient@@WKGI@AEXPAVRouterInterface@@@Z 004091a0 f i RakClient.obj
 0001:000081b0       ?GetCompressionRatio@RakClient@@WKGI@BEMXZ 004091b0 f i RakClient.obj
 0001:000081c0       ?DeleteCompressionLayer@RakClient@@WKGI@AE_N_N@Z 004091c0 f i RakClient.obj
 0001:000081d0       ??0RakClient@@QAE@XZ       004091d0 f   RakClient.obj
 0001:00008280       ??_GRakClient@@UAEPAXI@Z   00409280 f i RakClient.obj
 0001:00008280       ??_ERakClient@@UAEPAXI@Z   00409280 f i RakClient.obj
 0001:000082a0       ?Receive@RakClient@@UAEPAUPacket@@XZ 004092a0 f   RakClient.obj
 0001:00008710       ?GetStaticClientData@RakClient@@UAEPAVBitStream@RakNet@@UPlayerID@@@Z 00409710 f   RakClient.obj
 0001:00008760       ?SetStaticClientData@RakClient@@UAEXUPlayerID@@PBDH@Z 00409760 f   RakClient.obj
 0001:00008800       ?Receive@RakClient@@WKGI@AEPAUPacket@@XZ 00409800 f i RakClient.obj
 0001:00008810       ?StatisticsToString@@YAXPAURakNetStatisticsStruct@@PADH@Z 00409810 f   RakNetStatistics.obj
 0001:00008c20       ?GetRakClientInterface@RakNetworkFactory@@SAPAVRakClientInterface@@XZ 00409c20 f   RakNetworkFactory.obj
 0001:00008c90       ?GetRakServerInterface@RakNetworkFactory@@SAPAVRakServerInterface@@XZ 00409c90 f   RakNetworkFactory.obj
 0001:00008cf0       ?GetRakPeerInterface@RakNetworkFactory@@SAPAVRakPeerInterface@@XZ 00409cf0 f   RakNetworkFactory.obj
 0001:00008d50       ?DestroyRakClientInterface@RakNetworkFactory@@SAXPAVRakClientInterface@@@Z 00409d50 f   RakNetworkFactory.obj
 0001:00008d70       ?DestroyRakServerInterface@RakNetworkFactory@@SAXPAVRakServerInterface@@@Z 00409d70 f   RakNetworkFactory.obj
 0001:00008d90       ?DestroyRakPeerInterface@RakNetworkFactory@@SAXPAVRakPeerInterface@@@Z 00409d90 f   RakNetworkFactory.obj
 0001:00008db0       ??1RakPeerInterface@@UAE@XZ 00409db0 f i RakPeer.obj
 0001:00008dc0       ??_GRakPeerInterface@@UAEPAXI@Z 00409dc0 f i RakPeer.obj
 0001:00008dc0       ??_ERakPeerInterface@@UAEPAXI@Z 00409dc0 f i RakPeer.obj
 0001:00008de0       ?GetNumberOfUnreadBits@BitStream@RakNet@@QBEHXZ 00409de0 f i RakPeer.obj
 0001:00008df0       ??YRakNetStatisticsStruct@@QAE?AU0@ABU0@@Z 00409df0 f i RakPeer.obj
 0001:00008f70       ?PlayerIDAndIndexComp@@YAHABUPlayerID@@ABUPlayerIDAndIndex@@@Z 00409f70 f   RakPeer.obj
 0001:00008fa0       ?AllocPacket@@YAPAUPacket@@I@Z 00409fa0 f   RakPeer.obj
 0001:00008fc0       ?AllocPacket@@YAPAUPacket@@IPAE@Z 00409fc0 f   RakPeer.obj
 0001:00008fe0       ??0RakPeerInterface@@QAE@XZ 00409fe0 f i RakPeer.obj
 0001:00008ff0       ??0RemoteSystemStruct@RakPeer@@QAE@XZ 00409ff0 f i RakPeer.obj
 0001:00009050       ??1RemoteSystemStruct@RakPeer@@QAE@XZ 0040a050 f i RakPeer.obj
 0001:000090b0       ?DisableSecurity@RakPeer@@UAEXXZ 0040a0b0 f   RakPeer.obj
 0001:000090c0       ?SetMaximumIncomingConnections@RakPeer@@UAEXG@Z 0040a0c0 f   RakPeer.obj
 0001:000090d0       ?GetMaximumIncomingConnections@RakPeer@@UBEGXZ 0040a0d0 f   RakPeer.obj
 0001:000090e0       ?SetIncomingPassword@RakPeer@@UAEXPBDH@Z 0040a0e0 f   RakPeer.obj
 0001:00009130       ?GetIncomingPassword@RakPeer@@UAEXPADPAH@Z 0040a130 f   RakPeer.obj
 0001:00009170       ?GetConnectionList@RakPeer@@UBE_NPAUPlayerID@@PAG@Z 0040a170 f   RakPeer.obj
 0001:00009250       ?DeallocatePacket@RakPeer@@UAEXPAUPacket@@@Z 0040a250 f   RakPeer.obj
 0001:00009280       ?GetMaximumNumberOfPeers@RakPeer@@UBEGXZ 0040a280 f   RakPeer.obj
 0001:00009290       ?RegisterAsRemoteProcedureCall@RakPeer@@UAEXPAHP6AXPAURPCParameters@@@Z@Z 0040a290 f   RakPeer.obj
 0001:000092c0       ?RegisterClassMemberRPC@RakPeer@@UAEXPAHPAX@Z 0040a2c0 f   RakPeer.obj
 0001:000092f0       ?UnregisterAsRemoteProcedureCall@RakPeer@@UAEXPAH@Z 0040a2f0 f   RakPeer.obj
 0001:00009310       ?GetPlayerIDFromIndex@RakPeer@@UAE?AUPlayerID@@H@Z 0040a310 f   RakPeer.obj
 0001:00009370       ?SetOccasionalPing@RakPeer@@UAEX_N@Z 0040a370 f   RakPeer.obj
 0001:00009380       ?SetOfflinePingResponse@RakPeer@@UAEXPBDI@Z 0040a380 f   RakPeer.obj
 0001:000093f0       ?GetInternalID@RakPeer@@UBE?AUPlayerID@@XZ 0040a3f0 f   RakPeer.obj
 0001:00009410       ?GetExternalID@RakPeer@@UBE?AUPlayerID@@U2@@Z 0040a410 f   RakPeer.obj
 0001:000094d0       ?SetMTUSize@RakPeer@@UAE_NH@Z 0040a4d0 f   RakPeer.obj
 0001:00009520       ?GetMTUSize@RakPeer@@UBEHXZ 0040a520 f   RakPeer.obj
 0001:00009530       ?GetNumberOfAddresses@RakPeer@@UAEIXZ 0040a530 f   RakPeer.obj
 0001:00009580       ?PlayerIDToDottedIP@RakPeer@@UBEPBDUPlayerID@@@Z 0040a580 f   RakPeer.obj
 0001:00009590       ?GetLocalIP@RakPeer@@UAEPBDI@Z 0040a590 f   RakPeer.obj
 0001:000095d0       ?AllowConnectionResponseIPMigration@RakPeer@@UAEX_N@Z 0040a5d0 f   RakPeer.obj
 0001:000095e0       ?SetSplitMessageProgressInterval@RakPeer@@UAEXH@Z 0040a5e0 f   RakPeer.obj
 0001:00009630       ?SetUnreliableTimeout@RakPeer@@UAEXI@Z 0040a630 f   RakPeer.obj
 0001:00009680       ?SetCompileFrequencyTable@RakPeer@@UAEX_N@Z 0040a680 f   RakPeer.obj
 0001:00009690       ?GetOutgoingFrequencyTable@RakPeer@@UAE_NQAI@Z 0040a690 f   RakPeer.obj
 0001:000096d0       ?GenerateCompressionLayer@RakPeer@@UAE_NQAI_N@Z 0040a6d0 f   RakPeer.obj
 0001:000097b0       ??_GHuffmanEncodingTree@@QAEPAXI@Z 0040a7b0 f i RakPeer.obj
 0001:000097d0       ?GetCompressionRatio@RakPeer@@UBEMXZ 0040a7d0 f   RakPeer.obj
 0001:00009810       ?GetDecompressionRatio@RakPeer@@UBEMXZ 0040a810 f   RakPeer.obj
 0001:00009850       ?SetRouterInterface@RakPeer@@UAEXPAVRouterInterface@@@Z 0040a850 f   RakPeer.obj
 0001:00009860       ?RemoveRouterInterface@RakPeer@@UAEXPAVRouterInterface@@@Z 0040a860 f   RakPeer.obj
 0001:00009880       ?ApplyNetworkSimulator@RakPeer@@UAEXNGG@Z 0040a880 f   RakPeer.obj
 0001:00009900       ?IsNetworkSimulatorActive@RakPeer@@UAE_NXZ 0040a900 f   RakPeer.obj
 0001:00009930       ?IPToPlayerID@RakPeer@@UAEXPBDGPAUPlayerID@@@Z 0040a930 f   RakPeer.obj
 0001:00009960       ?GetNumberOfRemoteInitiatedConnections@RakPeer@@IBEGXZ 0040a960 f   RakPeer.obj
 0001:000099c0       ?HandleRPCReplyPacket@RakPeer@@IAEXPBDHUPlayerID@@@Z 0040a9c0 f   RakPeer.obj
 0001:00009a30       ?GenerateSYNCookieRandomNumber@RakPeer@@IAEXXZ 0040aa30 f   RakPeer.obj
 0001:00009aa0       ?AllowIncomingConnections@RakPeer@@IBE_NXZ 0040aaa0 f   RakPeer.obj
 0001:00009ac0       ?ValidSendTarget@RakPeer@@IAE_NUPlayerID@@_N@Z 0040aac0 f   RakPeer.obj
 0001:00009b50       ?ProcessPortUnreachable@@YGXIGPAVRakPeer@@@Z 0040ab50 f   RakPeer.obj
 0001:00009b60       ??$Write@G@BitStream@RakNet@@QAEXG@Z 0040ab60 f i RakPeer.obj
 0001:00009b80       ??0?$List@PAUBanStruct@RakPeer@@@DataStructures@@QAE@XZ 0040ab80 f i RakPeer.obj
 0001:00009b90       ??1?$List@PAUBanStruct@RakPeer@@@DataStructures@@QAE@XZ 0040ab90 f i RakPeer.obj
 0001:00009ba0       ??A?$List@PAUBanStruct@RakPeer@@@DataStructures@@QBEAAPAUBanStruct@RakPeer@@I@Z 0040aba0 f i RakPeer.obj
 0001:00009bb0       ?Insert@?$List@PAUBanStruct@RakPeer@@@DataStructures@@QAEXQAUBanStruct@RakPeer@@@Z 0040abb0 f i RakPeer.obj
 0001:00009c20       ?Size@?$List@PAUBanStruct@RakPeer@@@DataStructures@@QBEIXZ 0040ac20 f i RakPeer.obj
 0001:00009c30       ?Clear@?$List@PAUBanStruct@RakPeer@@@DataStructures@@QAEX_N@Z 0040ac30 f i RakPeer.obj
 0001:00009c70       ??0?$List@PAVPluginInterface@@@DataStructures@@QAE@XZ 0040ac70 f i RakPeer.obj
 0001:00009c80       ??1?$List@PAVPluginInterface@@@DataStructures@@QAE@XZ 0040ac80 f i RakPeer.obj
 0001:00009c90       ??A?$List@PAVPluginInterface@@@DataStructures@@QBEAAPAVPluginInterface@@I@Z 0040ac90 f i RakPeer.obj
 0001:00009ca0       ?Insert@?$List@PAVPluginInterface@@@DataStructures@@QAEXQAVPluginInterface@@@Z 0040aca0 f i RakPeer.obj
 0001:00009d10       ?Del@?$List@PAVPluginInterface@@@DataStructures@@QAEXI@Z 0040ad10 f i RakPeer.obj
 0001:00009d20       ?GetIndexOf@?$List@PAVPluginInterface@@@DataStructures@@QAEIQAVPluginInterface@@@Z 0040ad20 f i RakPeer.obj
 0001:00009d50       ?Size@?$List@PAVPluginInterface@@@DataStructures@@QBEIXZ 0040ad50 f i RakPeer.obj
 0001:00009d60       ??0?$SingleProducerConsumer@URequestedConnectionStruct@RakPeer@@@DataStructures@@QAE@XZ 0040ad60 f i RakPeer.obj
 0001:00009df0       ??1?$SingleProducerConsumer@URequestedConnectionStruct@RakPeer@@@DataStructures@@QAE@XZ 0040adf0 f i RakPeer.obj
 0001:00009e40       ?WriteLock@?$SingleProducerConsumer@URequestedConnectionStruct@RakPeer@@@DataStructures@@QAEPAURequestedConnectionStruct@RakPeer@@XZ 0040ae40 f i RakPeer.obj
 0001:00009ed0       ?WriteUnlock@?$SingleProducerConsumer@URequestedConnectionStruct@RakPeer@@@DataStructures@@QAEXXZ 0040aed0 f i RakPeer.obj
 0001:00009ef0       ?ReadLock@?$SingleProducerConsumer@URequestedConnectionStruct@RakPeer@@@DataStructures@@QAEPAURequestedConnectionStruct@RakPeer@@XZ 0040aef0 f i RakPeer.obj
 0001:00009f10       ?CancelReadLock@?$SingleProducerConsumer@URequestedConnectionStruct@RakPeer@@@DataStructures@@QAEXPAURequestedConnectionStruct@RakPeer@@@Z 0040af10 f i RakPeer.obj
 0001:00009f20       ?ReadUnlock@?$SingleProducerConsumer@URequestedConnectionStruct@RakPeer@@@DataStructures@@QAEXXZ 0040af20 f i RakPeer.obj
 0001:00009f40       ?Clear@?$SingleProducerConsumer@URequestedConnectionStruct@RakPeer@@@DataStructures@@QAEXXZ 0040af40 f i RakPeer.obj
 0001:00009fc0       ??0?$SingleProducerConsumer@UBufferedCommandStruct@RakPeer@@@DataStructures@@QAE@XZ 0040afc0 f i RakPeer.obj
 0001:0000a030       ??1?$SingleProducerConsumer@UBufferedCommandStruct@RakPeer@@@DataStructures@@QAE@XZ 0040b030 f i RakPeer.obj
 0001:0000a070       ?WriteLock@?$SingleProducerConsumer@UBufferedCommandStruct@RakPeer@@@DataStructures@@QAEPAUBufferedCommandStruct@RakPeer@@XZ 0040b070 f i RakPeer.obj
 0001:0000a0e0       ?WriteUnlock@?$SingleProducerConsumer@UBufferedCommandStruct@RakPeer@@@DataStructures@@QAEXXZ 0040b0e0 f i RakPeer.obj
 0001:0000a100       ?ReadLock@?$SingleProducerConsumer@UBufferedCommandStruct@RakPeer@@@DataStructures@@QAEPAUBufferedCommandStruct@RakPeer@@XZ 0040b100 f i RakPeer.obj
 0001:0000a120       ?ReadUnlock@?$SingleProducerConsumer@UBufferedCommandStruct@RakPeer@@@DataStructures@@QAEXXZ 0040b120 f i RakPeer.obj
 0001:0000a140       ?Clear@?$SingleProducerConsumer@UBufferedCommandStruct@RakPeer@@@DataStructures@@QAEXXZ 0040b140 f i RakPeer.obj
 0001:0000a1b0       ??0?$SingleProducerConsumer@PAUPacket@@@DataStructures@@QAE@XZ 0040b1b0 f i RakPeer.obj
 0001:0000a220       ??1?$SingleProducerConsumer@PAUPacket@@@DataStructures@@QAE@XZ 0040b220 f i RakPeer.obj
 0001:0000a260       ?WriteLock@?$SingleProducerConsumer@PAUPacket@@@DataStructures@@QAEPAPAUPacket@@XZ 0040b260 f i RakPeer.obj
 0001:0000a2d0       ?WriteUnlock@?$SingleProducerConsumer@PAUPacket@@@DataStructures@@QAEXXZ 0040b2d0 f i RakPeer.obj
 0001:0000a2f0       ?ReadLock@?$SingleProducerConsumer@PAUPacket@@@DataStructures@@QAEPAPAUPacket@@XZ 0040b2f0 f i RakPeer.obj
 0001:0000a310       ?ReadUnlock@?$SingleProducerConsumer@PAUPacket@@@DataStructures@@QAEXXZ 0040b310 f i RakPeer.obj
 0001:0000a330       ?Clear@?$SingleProducerConsumer@PAUPacket@@@DataStructures@@QAEXXZ 0040b330 f i RakPeer.obj
 0001:0000a3a0       ??0?$Queue@PAUPacket@@@DataStructures@@QAE@XZ 0040b3a0 f i RakPeer.obj
 0001:0000a3e0       ??1?$Queue@PAUPacket@@@DataStructures@@QAE@XZ 0040b3e0 f i RakPeer.obj
 0001:0000a3f0       ?Push@?$Queue@PAUPacket@@@DataStructures@@QAEXABQAUPacket@@@Z 0040b3f0 f i RakPeer.obj
 0001:0000a4c0       ?PushAtHead@?$Queue@PAUPacket@@@DataStructures@@QAEXABQAUPacket@@I@Z 0040b4c0 f i RakPeer.obj
 0001:0000a5b0       ??A?$Queue@PAUPacket@@@DataStructures@@QBEAAPAUPacket@@I@Z 0040b5b0 f i RakPeer.obj
 0001:0000a5e0       ?Pop@?$Queue@PAUPacket@@@DataStructures@@QAEPAUPacket@@XZ 0040b5e0 f i RakPeer.obj
 0001:0000a610       ?Size@?$Queue@PAUPacket@@@DataStructures@@QBEIXZ 0040b610 f i RakPeer.obj
 0001:0000a630       ?Clear@?$Queue@PAUPacket@@@DataStructures@@QAEXXZ 0040b630 f i RakPeer.obj
 0001:0000a670       ??$Write@E@BitStream@RakNet@@QAEXE@Z 0040b670 f i RakPeer.obj
 0001:0000a690       ??$WriteCompressed@E@BitStream@RakNet@@QAEXE@Z 0040b690 f i RakPeer.obj
 0001:0000a6b0       ??$ReadCompressed@E@BitStream@RakNet@@QAE_NAAE@Z 0040b6b0 f i RakPeer.obj
 0001:0000a6d0       ??$usetw@$$BY07I@big@@YAXAAY07II@Z 0040b6d0 f i RakPeer.obj
 0001:0000a700       ??$set@$$BY07I@big@@YAXAAY07I0@Z 0040b700 f i RakPeer.obj
 0001:0000a720       ??$zero@$$BY07I@big@@YAXAAY07I@Z 0040b720 f i RakPeer.obj
 0001:0000a740       ??$zero@$$BY03I@big@@YAXAAY03I@Z 0040b740 f i RakPeer.obj
 0001:0000a760       ??0?$List@UPlayerIDAndIndex@@@DataStructures@@QAE@XZ 0040b760 f i RakPeer.obj
 0001:0000a770       ??1?$List@UPlayerIDAndIndex@@@DataStructures@@QAE@XZ 0040b770 f i RakPeer.obj
 0001:0000a780       ??A?$List@UPlayerIDAndIndex@@@DataStructures@@QBEAAUPlayerIDAndIndex@@I@Z 0040b780 f i RakPeer.obj
 0001:0000a790       ?Size@?$List@UPlayerIDAndIndex@@@DataStructures@@QBEIXZ 0040b790 f i RakPeer.obj
 0001:0000a7a0       ?Clear@?$List@UPlayerIDAndIndex@@@DataStructures@@QAEX_N@Z 0040b7a0 f i RakPeer.obj
 0001:0000a7e0       ?Del@?$List@PAUBanStruct@RakPeer@@@DataStructures@@QAEXI@Z 0040b7e0 f i RakPeer.obj
 0001:0000a7f0       ??$ugreater@$$BY03I@big@@YA_NAAY03I0@Z 0040b7f0 f i RakPeer.obj
 0001:0000a830       ??$set@$$BY03I@big@@YAXAAY03I0@Z 0040b830 f i RakPeer.obj
 0001:0000a850       ??$decrement@$$BY03I@big@@YAXAAY03I@Z 0040b850 f i RakPeer.obj
 0001:0000a870       ??$sethigh@$$BY07I$$BY0BA@I@big@@YAXAAY0BA@IAAY07I@Z 0040b870 f i RakPeer.obj
 0001:0000a8a0       ??$decrement@$$BY0BA@I@big@@YAXAAY0BA@I@Z 0040b8a0 f i RakPeer.obj
 0001:0000a8f0       ??$usetlow@$$BY07I$$BY0BA@I@big@@YAXAAY0BA@IAAY07I@Z 0040b8f0 f i RakPeer.obj
 0001:0000a920       ??$takelow@$$BY07I$$BY0BA@I@big@@YAXAAY07IAAY0BA@I@Z 0040b920 f i RakPeer.obj
 0001:0000a940       ??$usetlow@$$BY03I$$BY07I@big@@YAXAAY07IAAY03I@Z 0040b940 f i RakPeer.obj
 0001:0000a970       ??$decrement@$$BY07I@big@@YAXAAY07I@Z 0040b970 f i RakPeer.obj
 0001:0000a990       ??$takelow@$$BY03I$$BY07I@big@@YAXAAY03IAAY07I@Z 0040b990 f i RakPeer.obj
 0001:0000a9b0       ??$subtract@$$BY03I@big@@YAXAAY03I0@Z 0040b9b0 f i RakPeer.obj
 0001:0000aa10       ??$add@$$BY03I@big@@YAXAAY03I0@Z 0040ba10 f i RakPeer.obj
 0001:0000aa70       ??$add@$$BY07I@big@@YAXAAY07I0@Z 0040ba70 f i RakPeer.obj
 0001:0000aad0       ??$usetw@$$BY0BA@I@big@@YAXAAY0BA@II@Z 0040bad0 f i RakPeer.obj
 0001:0000aaf0       ??4PlayerIDAndIndex@@QAEAAU0@ABU0@@Z 0040baf0 f i RakPeer.obj
 0001:0000ab10       ?Del@?$List@UPlayerIDAndIndex@@@DataStructures@@QAEXI@Z 0040bb10 f i RakPeer.obj
 0001:0000ab20       ??$shiftLeft@$$BY07I@big@@YAXAAY07II@Z 0040bb20 f i RakPeer.obj
 0001:0000ac00       ??$ugreater@$$BY07I@big@@YA_NAAY07I0@Z 0040bc00 f i RakPeer.obj
 0001:0000ac40       ??$equal@$$BY07I@big@@YA_NAAY07I0@Z 0040bc40 f i RakPeer.obj
 0001:0000acb0       ??$usetw@$$BY03I@big@@YAXAAY03II@Z 0040bcb0 f i RakPeer.obj
 0001:0000acd0       ??$isZero@$$BY03I@big@@YA_NAAY03I@Z 0040bcd0 f i RakPeer.obj
 0001:0000acf0       ??$sethigh@$$BY03I$$BY07I@big@@YAXAAY07IAAY03I@Z 0040bcf0 f i RakPeer.obj
 0001:0000ad20       ??$ushiftRight1@$$BY03I@big@@YAXAAY03I@Z 0040bd20 f i RakPeer.obj
 0001:0000ad60       ??$equal@$$BY03I@big@@YA_NAAY03I0@Z 0040bd60 f i RakPeer.obj
 0001:0000add0       ??$isZero@$$BY07I@big@@YA_NAAY07I@Z 0040bdd0 f i RakPeer.obj
 0001:0000adf0       ??$subtract@$$BY07I@big@@YAXAAY07I0@Z 0040bdf0 f i RakPeer.obj
 0001:0000ae50       ??$set@$$BY0BA@I@big@@YAXAAY0BA@I0@Z 0040be50 f i RakPeer.obj
 0001:0000ae70       ??$zero@$$BY0BA@I@big@@YAXAAY0BA@I@Z 0040be70 f i RakPeer.obj
 0001:0000ae90       ??$ugreater@$$BY0BA@I@big@@YA_NAAY0BA@I0@Z 0040be90 f i RakPeer.obj
 0001:0000aed0       ??$shiftLeft@$$BY0BA@I@big@@YAXAAY0BA@II@Z 0040bed0 f i RakPeer.obj
 0001:0000af60       ??$shiftLeft1@$$BY0BA@I@big@@YAXAAY0BA@I@Z 0040bf60 f i RakPeer.obj
 0001:0000af90       ??$ushiftRight1@$$BY0BA@I@big@@YAXAAY0BA@I@Z 0040bf90 f i RakPeer.obj
 0001:0000afc0       ??$subtract@$$BY0BA@I@big@@YAXAAY0BA@I0@Z 0040bfc0 f i RakPeer.obj
 0001:0000b020       ??$shiftLeft1@$$BY07I@big@@YAXAAY07I@Z 0040c020 f i RakPeer.obj
 0001:0000b090       ??$ushiftRight1@$$BY07I@big@@YAXAAY07I@Z 0040c090 f i RakPeer.obj
 0001:0000b110       ??$usquare@$$BY07I@big@@YAXAAY07I@Z 0040c110 f i RakPeer.obj
 0001:0000b220       ??$add@$$BY0BA@I@big@@YAXAAY0BA@I0@Z 0040c220 f i RakPeer.obj
 0001:0000b280       ??$usetlow@$$BY0BA@I$$BY0BA@I@big@@YAXAAY0BA@I0@Z 0040c280 f i RakPeer.obj
 0001:0000b2b0       ??$shiftLeft@$$BY03I@big@@YAXAAY03II@Z 0040c2b0 f i RakPeer.obj
 0001:0000b350       ??$shiftLeft1@$$BY03I@big@@YAXAAY03I@Z 0040c350 f i RakPeer.obj
 0001:0000b390       ??$umultiply@$$BY03I$$BY07I@big@@YAXAAY07IAAY03I@Z 0040c390 f i RakPeer.obj
 0001:0000b490       ??$umultiply@$$BY07I$$BY0BA@I@big@@YAXAAY0BA@IAAY07I@Z 0040c490 f i RakPeer.obj
 0001:0000b580       ??$usetlow@$$BY07I$$BY07I@big@@YAXAAY07I0@Z 0040c580 f i RakPeer.obj
 0001:0000b5b0       ??$Write@UPlayerID@@@BitStream@RakNet@@QAEXUPlayerID@@@Z 0040c5b0 f i RakPeer.obj
 0001:0000b5f0       ??$Write@UNetworkID@@@BitStream@RakNet@@QAEXUNetworkID@@@Z 0040c5f0 f i RakPeer.obj
 0001:0000b650       ??$Read@UPlayerID@@@BitStream@RakNet@@QAE_NAAUPlayerID@@@Z 0040c650 f i RakPeer.obj
 0001:0000b680       ??$Read@UNetworkID@@@BitStream@RakNet@@QAE_NAAUNetworkID@@@Z 0040c680 f i RakPeer.obj
 0001:0000b6c0       ??_ERemoteSystemStruct@RakPeer@@QAEPAXI@Z 0040c6c0 f i RakPeer.obj
 0001:0000b720       ?RPC@RakPeer@@UAE_NPAHPAVBitStream@RakNet@@W4PacketPriority@@W4PacketReliability@@DUPlayerID@@_N5UNetworkID@@1@Z 0040c720 f   RakPeer.obj
 0001:0000b7e0       ?AddToBanList@RakPeer@@UAEXPBDI@Z 0040c7e0 f   RakPeer.obj
 0001:0000b950       ?ClearBanList@RakPeer@@UAEXXZ 0040c950 f   RakPeer.obj
 0001:0000b9f0       ?Ping@RakPeer@@UAEXPBDG_N@Z 0040c9f0 f   RakPeer.obj
 0001:0000bb40       ?AdvertiseSystem@RakPeer@@UAEXPBDG0H@Z 0040cb40 f   RakPeer.obj
 0001:0000bce0       ?DeleteCompressionLayer@RakPeer@@UAE_N_N@Z 0040cce0 f   RakPeer.obj
 0001:0000bd60       ?AttachPlugin@RakPeer@@UAEXPAVPluginInterface@@@Z 0040cd60 f   RakPeer.obj
 0001:0000bdb0       ?DetachPlugin@RakPeer@@UAEXPAVPluginInterface@@@Z 0040cdb0 f   RakPeer.obj
 0001:0000be20       ?PushBackPacket@RakPeer@@UAEXPAUPacket@@_N@Z 0040ce20 f   RakPeer.obj
 0001:0000be80       ?SendBuffered@RakPeer@@IAEXPBDHW4PacketPriority@@W4PacketReliability@@DUPlayerID@@_NW4ConnectMode@RemoteSystemStruct@1@@Z 0040ce80 f   RakPeer.obj
 0001:0000bf30       ?ClearBufferedCommands@RakPeer@@IAEXXZ 0040cf30 f   RakPeer.obj
 0001:0000bfa0       ?ClearRequestedConnectionList@RakPeer@@IAEXXZ 0040cfa0 f   RakPeer.obj
 0001:0000c020       ?AddPacketToProducer@RakPeer@@IAEXPAUPacket@@@Z 0040d020 f i RakPeer.obj
 0001:0000c050       ?getPublicKey@?$RSACrypt@$$BY07I@big@@QAEXAAIAAY07I@Z 0040d050 f i RakPeer.obj
 0001:0000c070       ?reset@?$RSACrypt@$$BY07I@big@@QAEXXZ 0040d070 f i RakPeer.obj
 0001:0000c100       ??0?$OrderedList@UPlayerID@@UPlayerIDAndIndex@@$1?PlayerIDAndIndexComp@@YAHABU1@ABU2@@Z@DataStructures@@QAE@XZ 0040d100 f i RakPeer.obj
 0001:0000c110       ?GetIndexFromKey@?$OrderedList@UPlayerID@@UPlayerIDAndIndex@@$1?PlayerIDAndIndexComp@@YAHABU1@ABU2@@Z@DataStructures@@QBEIABUPlayerID@@PA_N@Z 0040d110 f i RakPeer.obj
 0001:0000c1b0       ??A?$OrderedList@UPlayerID@@UPlayerIDAndIndex@@$1?PlayerIDAndIndexComp@@YAHABU1@ABU2@@Z@DataStructures@@QBEAAUPlayerIDAndIndex@@I@Z 0040d1b0 f i RakPeer.obj
 0001:0000c1c0       ?Clear@?$OrderedList@UPlayerID@@UPlayerIDAndIndex@@$1?PlayerIDAndIndexComp@@YAHABU1@ABU2@@Z@DataStructures@@QAEXXZ 0040d1c0 f i RakPeer.obj
 0001:0000c200       ?RemoveAtIndex@?$List@PAUBanStruct@RakPeer@@@DataStructures@@QAEXI@Z 0040d200 f i RakPeer.obj
 0001:0000c240       ?Insert@?$List@UPlayerIDAndIndex@@@DataStructures@@QAEXUPlayerIDAndIndex@@@Z 0040d240 f i RakPeer.obj
 0001:0000c2d0       ?Insert@?$List@UPlayerIDAndIndex@@@DataStructures@@QAEXUPlayerIDAndIndex@@I@Z 0040d2d0 f i RakPeer.obj
 0001:0000c380       ?RemoveAtIndex@?$List@UPlayerIDAndIndex@@@DataStructures@@QAEXI@Z 0040d380 f i RakPeer.obj
 0001:0000c3c0       ??$umultiply@$$BY03I$$BY07I@big@@YAXAAY03I0AAY07I@Z 0040d3c0 f i RakPeer.obj
 0001:0000c4d0       ??$udivide@$$BY0BA@I@big@@YAXAAY0BA@I000@Z 0040d4d0 f i RakPeer.obj
 0001:0000c730       ??$umodulo@$$BY0BA@I@big@@YAXAAY0BA@I00@Z 0040d730 f i RakPeer.obj
 0001:0000c950       ??$umodulo@$$BY07I@big@@YAXAAY07I00@Z 0040d950 f i RakPeer.obj
 0001:0000cc90       ??$umultiply@$$BY07I$$BY07I@big@@YAXAAY07I0@Z 0040dc90 f i RakPeer.obj
 0001:0000cd90       ??$usquare@$$BY0BA@I@big@@YAXAAY0BA@I@Z 0040dd90 f i RakPeer.obj
 0001:0000cea0       ??$umultiply@$$BY0BA@I$$BY0BA@I@big@@YAXAAY0BA@I00@Z 0040dea0 f i RakPeer.obj
 0001:0000cfa0       ??$GCD@$$BY07I@big@@YAXAAY07I00@Z 0040dfa0 f i RakPeer.obj
 0001:0000d060       ??$udivide@$$BY03I@big@@YAXAAY03I000@Z 0040e060 f i RakPeer.obj
 0001:0000d330       ??$SubMulMod@$$BY03I@big@@YAXAAY03I0000@Z 0040e330 f i RakPeer.obj
 0001:0000d450       ??$udivide@$$BY07I@big@@YAXAAY07I000@Z 0040e450 f i RakPeer.obj
 0001:0000d810       ??$umodulo@$$BY03I@big@@YAXAAY03I00@Z 0040e810 f i RakPeer.obj
 0001:0000da70       ??$SubMulMod@$$BY07I@big@@YAXAAY07I0000@Z 0040ea70 f i RakPeer.obj
 0001:0000dbb0       ??$umultiply@$$BY07I$$BY07I@big@@YAXAAY07I00@Z 0040ebb0 f i RakPeer.obj
 0001:0000dcc0       ?Send@RakPeer@@UAE_NPBDHW4PacketPriority@@W4PacketReliability@@DUPlayerID@@_N@Z 0040ecc0 f   RakPeer.obj
 0001:0000ddb0       ?Send@RakPeer@@UAE_NPAVBitStream@RakNet@@W4PacketPriority@@W4PacketReliability@@DUPlayerID@@_N@Z 0040edb0 f   RakPeer.obj
 0001:0000de90       ?RemoveFromBanList@RakPeer@@UAEXPBD@Z 0040ee90 f   RakPeer.obj
 0001:0000dfb0       ?IsBanned@RakPeer@@UAE_NPBD@Z 0040efb0 f   RakPeer.obj
 0001:0000e100       ?GetIndexFromPlayerID@RakPeer@@IAEHUPlayerID@@_N@Z 0040f100 f   RakPeer.obj
 0001:0000e1f0       ?GetRemoteSystemFromPlayerID@RakPeer@@IBEPAURemoteSystemStruct@1@UPlayerID@@_N1@Z 0040f1f0 f   RakPeer.obj
 0001:0000e2e0       ?GetBestClockDifferential@RakPeer@@IBEIUPlayerID@@@Z 0040f2e0 f   RakPeer.obj
 0001:0000e340       ?HandleRPCPacket@RakPeer@@IAE_NPBDHUPlayerID@@@Z 0040f340 f   RakPeer.obj
 0001:0000e760       ?SendImmediate@RakPeer@@IAE_NPADHW4PacketPriority@@W4PacketReliability@@DUPlayerID@@_N4_J@Z 0040f760 f   RakPeer.obj
 0001:0000ea40       ??0?$RSACrypt@$$BY07I@big@@QAE@XZ 0040fa40 f i RakPeer.obj
 0001:0000ea50       ??1?$RSACrypt@$$BY07I@big@@QAE@XZ 0040fa50 f i RakPeer.obj
 0001:0000ea60       ??1?$OrderedList@UPlayerID@@UPlayerIDAndIndex@@$1?PlayerIDAndIndexComp@@YAHABU1@ABU2@@Z@DataStructures@@QAE@XZ 0040fa60 f i RakPeer.obj
 0001:0000eae0       ?Insert@?$OrderedList@UPlayerID@@UPlayerIDAndIndex@@$1?PlayerIDAndIndexComp@@YAHABU1@ABU2@@Z@DataStructures@@QAEIABUPlayerID@@ABUPlayerIDAndIndex@@@Z 0040fae0 f i RakPeer.obj
 0001:0000eb60       ?Remove@?$OrderedList@UPlayerID@@UPlayerIDAndIndex@@$1?PlayerIDAndIndexComp@@YAHABU1@ABU2@@Z@DataStructures@@QAEIABUPlayerID@@@Z 0040fb60 f i RakPeer.obj
 0001:0000ebe0       ??$rModn@$$BY07I@big@@YAXAAY07I0@Z 0040fbe0 f i RakPeer.obj
 0001:0000ecb0       ??$simpleModExp@$$BY07I@big@@YAXAAY07I000@Z 0040fcb0 f i RakPeer.obj
 0001:0000ee70       ??$computePublicExponent@$$BY07I@big@@YAXAAY07I0@Z 0040fe70 f i RakPeer.obj
 0001:0000efe0       ??$computeModularInverse@$$BY03I@big@@YAXAAY03I00@Z 0040ffe0 f i RakPeer.obj
 0001:0000f280       ??$rModn@$$BY03I@big@@YAXAAY03I0@Z 00410280 f i RakPeer.obj
 0001:0000f320       ??$computeRinverse@$$BY07I@big@@YAXAAY07I0@Z 00410320 f i RakPeer.obj
 0001:0000f620       ??$simpleModExp@$$BY03I@big@@YAXAAY03I000@Z 00410620 f i RakPeer.obj
 0001:0000f7c0       ??$computeModularInverse@$$BY07I@big@@YAXAAY07I00@Z 004107c0 f i RakPeer.obj
 0001:0000fa40       ??$computeRinverse@$$BY03I@big@@YAXAAY03I0@Z 00410a40 f i RakPeer.obj
 0001:0000fd10       ??0RakPeer@@QAE@XZ         00410d10 f   RakPeer.obj
 0001:0000ff50       ?IsActive@RakPeer@@UBE_NXZ 00410f50 f i RakPeer.obj
 0001:0000ff60       ?RPC@RakPeer@@UAE_NPAHPBDIW4PacketPriority@@W4PacketReliability@@DUPlayerID@@_N5UNetworkID@@PAVBitStream@RakNet@@@Z 00410f60 f   RakPeer.obj
 0001:00010420       ?GetIndexFromPlayerID@RakPeer@@UAEHUPlayerID@@@Z 00411420 f   RakPeer.obj
 0001:00010440       ?GetAveragePing@RakPeer@@UAEHUPlayerID@@@Z 00411440 f   RakPeer.obj
 0001:000104a0       ?GetLastPing@RakPeer@@UBEHUPlayerID@@@Z 004114a0 f   RakPeer.obj
 0001:000104e0       ?GetLowestPing@RakPeer@@UBEHUPlayerID@@@Z 004114e0 f   RakPeer.obj
 0001:00010510       ?GetRemoteStaticData@RakPeer@@UAEPAVBitStream@RakNet@@UPlayerID@@@Z 00411510 f   RakPeer.obj
 0001:00010560       ?SetRemoteStaticData@RakPeer@@UAEXUPlayerID@@PBDH@Z 00411560 f   RakPeer.obj
 0001:000105e0       ?SetTimeoutTime@RakPeer@@UAEXIUPlayerID@@@Z 004115e0 f   RakPeer.obj
 0001:00010610       ?GetRPCMap@RakPeer@@UAEPAURPCMap@@UPlayerID@@@Z 00411610 f   RakPeer.obj
 0001:00010660       ?GetStatistics@RakPeer@@UAEQAURakNetStatisticsStruct@@UPlayerID@@@Z 00411660 f   RakPeer.obj
 0001:00010710       ?SendConnectionRequest@RakPeer@@IAE_NPBDGPADH@Z 00411710 f   RakPeer.obj
 0001:00010810       ?OnConnectionRequest@RakPeer@@IAEXPAURemoteSystemStruct@1@PAE_N@Z 00411810 f   RakPeer.obj
 0001:00010970       ?NotifyAndFlagForDisconnect@RakPeer@@IAEXUPlayerID@@_NE@Z 00411970 f   RakPeer.obj
 0001:00010a90       ?AssignPlayerIDToRemoteSystemList@RakPeer@@IAEPAURemoteSystemStruct@1@UPlayerID@@W4ConnectMode@21@@Z 00411a90 f   RakPeer.obj
 0001:00010c30       ?ShiftIncomingTimestamp@RakPeer@@IBEXPAEUPlayerID@@@Z 00411c30 f   RakPeer.obj
 0001:00010cf0       ?SecuredConnectionResponse@RakPeer@@IAEXUPlayerID@@@Z 00411cf0 f   RakPeer.obj
 0001:00010e30       ?SendStaticDataInternal@RakPeer@@IAEXUPlayerID@@_N@Z 00411e30 f   RakPeer.obj
 0001:00010f80       ?PingInternal@RakPeer@@IAEXUPlayerID@@_N@Z 00411f80 f   RakPeer.obj
 0001:00011090       ?CloseConnectionInternal@RakPeer@@IAEXUPlayerID@@_N1E@Z 00412090 f   RakPeer.obj
 0001:00011200       ?ProcessNetworkPacket@@YGXIGPBDHPAVRakPeer@@@Z 00412200 f   RakPeer.obj
 0001:00011ee0       ??$computeNRinverse@$$BY07I@big@@YAXAAY07I0@Z 00412ee0 f i RakPeer.obj
 0001:00011fb0       ??$CRTModExp@$$BY03I$$BY07I@big@@YAXAAY07I00AAY03I111111@Z 00412fb0 f i RakPeer.obj
 0001:00012290       ??$computePrivateExponent@$$BY07I@big@@YAXAAY07I00@Z 00413290 f i RakPeer.obj
 0001:000122a0       ??$computeNRinverse@$$BY03I@big@@YAXAAY03I0@Z 004132a0 f i RakPeer.obj
 0001:00012360       ??$RabinMillerPrimalityTest@$$BY03I@big@@YA_NAAY03II@Z 00413360 f i RakPeer.obj
 0001:00012780       ?Connect@RakPeer@@UAE_NPBDGPADH@Z 00413780 f   RakPeer.obj
 0001:00012880       ?Disconnect@RakPeer@@UAEXIE@Z 00413880 f   RakPeer.obj
 0001:00012b90       ?ReceiveIgnoreRPC@RakPeer@@IAEPAUPacket@@XZ 00413b90 f   RakPeer.obj
 0001:00012df0       ?CloseConnection@RakPeer@@UAEXUPlayerID@@_NE@Z 00413df0 f   RakPeer.obj
 0001:00012e10       ?Ping@RakPeer@@UAEXUPlayerID@@@Z 00413e10 f   RakPeer.obj
 0001:00012e30       ?SendStaticData@RakPeer@@UAEXUPlayerID@@@Z 00413e30 f   RakPeer.obj
 0001:00012e50       ?ParseConnectionRequestPacket@RakPeer@@IAEXPAURemoteSystemStruct@1@UPlayerID@@PBDH@Z 00413e50 f   RakPeer.obj
 0001:00012f50       ?setPublicKey@?$RSACrypt@$$BY07I@big@@QAEXIAAY07I@Z 00413f50 f i RakPeer.obj
 0001:00012fb0       ?encrypt@?$RSACrypt@$$BY07I@big@@QAEXAAY07I0@Z 00413fb0 f i RakPeer.obj
 0001:00013020       ?decrypt@?$RSACrypt@$$BY07I@big@@QAEXAAY07I0@Z 00414020 f i RakPeer.obj
 0001:00013080       ??$setPrivateKey@$$BY03I@?$RSACrypt@$$BY07I@big@@QAEXAAY03I0@Z 00414080 f i RakPeer.obj
 0001:00013260       ??$generateStrongPseudoPrime@$$BY03I@big@@YAXAAY03I@Z 00414260 f i RakPeer.obj
 0001:000132a0       ??1RakPeer@@UAE@XZ         004142a0 f   RakPeer.obj
 0001:00013410       ?Receive@RakPeer@@UAEPAUPacket@@XZ 00414410 f   RakPeer.obj
 0001:00013470       ?SecuredConnectionConfirmation@RakPeer@@IAEXPAURemoteSystemStruct@1@PAD@Z 00414470 f   RakPeer.obj
 0001:000137f0       ?RunUpdateCycle@RakPeer@@IAE_NXZ 004147f0 f   RakPeer.obj
 0001:00014b50       ?UpdateNetworkLoop@@YGIPAX@Z 00415b50 f   RakPeer.obj
 0001:00014c20       ?generateKeys@?$RSACrypt@$$BY07I@big@@QAEXXZ 00415c20 f i RakPeer.obj
 0001:00014c60       ??_ERakPeer@@UAEPAXI@Z     00415c60 f i RakPeer.obj
 0001:00014c60       ??_GRakPeer@@UAEPAXI@Z     00415c60 f i RakPeer.obj
 0001:00014c80       ?Initialize@RakPeer@@UAE_NGGHPBD@Z 00415c80 f   RakPeer.obj
 0001:00014f90       ?InitializeSecurity@RakPeer@@UAEXPBD000@Z 00415f90 f   RakPeer.obj
 0001:000150d0       ??1RakServerInterface@@UAE@XZ 004160d0 f i rakserver.obj
 0001:000150e0       ??_ERakServerInterface@@UAEPAXI@Z 004160e0 f i rakserver.obj
 0001:000150e0       ??_GRakServerInterface@@UAEPAXI@Z 004160e0 f i rakserver.obj
 0001:00015100       ??0RakServerInterface@@QAE@XZ 00416100 f i rakserver.obj
 0001:00015110       ??1RakServer@@UAE@XZ       00416110 f   rakserver.obj
 0001:00015160       ?InitializeSecurity@RakServer@@UAEXPBD0@Z 00416160 f   rakserver.obj
 0001:00015180       ?DisableSecurity@RakServer@@UAEXXZ 00416180 f   rakserver.obj
 0001:00015190       ?Start@RakServer@@UAE_NGIHGPBD@Z 00416190 f   rakserver.obj
 0001:00015210       ?SetPassword@RakServer@@UAEXPBD@Z 00416210 f   rakserver.obj
 0001:00015250       ?HasPassword@RakServer@@UAE_NXZ 00416250 f   rakserver.obj
 0001:00015270       ?Disconnect@RakServer@@UAEXIE@Z 00416270 f   rakserver.obj
 0001:00015280       ?Send@RakServer@@UAE_NPBDHW4PacketPriority@@W4PacketReliability@@DUPlayerID@@_N@Z 00416280 f   rakserver.obj
 0001:000152c0       ?Send@RakServer@@UAE_NPAVBitStream@RakNet@@W4PacketPriority@@W4PacketReliability@@DUPlayerID@@_N@Z 004162c0 f   rakserver.obj
 0001:000152f0       ?Kick@RakServer@@UAEXUPlayerID@@@Z 004162f0 f   rakserver.obj
 0001:00015310       ?DeallocatePacket@RakServer@@UAEXPAUPacket@@@Z 00416310 f   rakserver.obj
 0001:00015320       ?SetAllowedPlayers@RakServer@@UAEXG@Z 00416320 f   rakserver.obj
 0001:00015330       ?GetAllowedPlayers@RakServer@@UBEGXZ 00416330 f   rakserver.obj
 0001:00015340       ?GetConnectedPlayers@RakServer@@UAEGXZ 00416340 f   rakserver.obj
 0001:00015360       ?GetPlayerIPFromID@RakServer@@UAEXUPlayerID@@QADPAG@Z 00416360 f   rakserver.obj
 0001:00015390       ?PingPlayer@RakServer@@UAEXUPlayerID@@@Z 00416390 f   rakserver.obj
 0001:000153b0       ?GetAveragePing@RakServer@@UAEHUPlayerID@@@Z 004163b0 f   rakserver.obj
 0001:000153d0       ?GetLastPing@RakServer@@UAEHUPlayerID@@@Z 004163d0 f   rakserver.obj
 0001:000153f0       ?GetLowestPing@RakServer@@UAEHUPlayerID@@@Z 004163f0 f   rakserver.obj
 0001:00015410       ?StartOccasionalPing@RakServer@@UAEXXZ 00416410 f   rakserver.obj
 0001:00015420       ?StopOccasionalPing@RakServer@@UAEXXZ 00416420 f   rakserver.obj
 0001:00015430       ?IsActive@RakServer@@UBE_NXZ 00416430 f   rakserver.obj
 0001:00015440       ?GetSynchronizedRandomInteger@RakServer@@UBEIXZ 00416440 f   rakserver.obj
 0001:00015450       ?StartSynchronizedRandomInteger@RakServer@@UAEXXZ 00416450 f   rakserver.obj
 0001:00015460       ?StopSynchronizedRandomInteger@RakServer@@UAEXXZ 00416460 f   rakserver.obj
 0001:00015470       ?GenerateCompressionLayer@RakServer@@UAE_NQAI_N@Z 00416470 f   rakserver.obj
 0001:00015480       ?DeleteCompressionLayer@RakServer@@UAE_N_N@Z 00416480 f   rakserver.obj
 0001:00015490       ?RegisterAsRemoteProcedureCall@RakServer@@UAEXPAHP6AXPAURPCParameters@@@Z@Z 00416490 f   rakserver.obj
 0001:000154a0       ?RegisterClassMemberRPC@RakServer@@UAEXPAHPAX@Z 004164a0 f   rakserver.obj
 0001:000154b0       ?UnregisterAsRemoteProcedureCall@RakServer@@UAEXPAH@Z 004164b0 f   rakserver.obj
 0001:000154c0       ?RPC@RakServer@@UAE_NPAHPBDIW4PacketPriority@@W4PacketReliability@@DUPlayerID@@_N5UNetworkID@@PAVBitStream@RakNet@@@Z 004164c0 f   rakserver.obj
 0001:00015520       ?RPC@RakServer@@UAE_NPAHPAVBitStream@RakNet@@W4PacketPriority@@W4PacketReliability@@DUPlayerID@@_N5UNetworkID@@1@Z 00416520 f   rakserver.obj
 0001:00015580       ?SetTrackFrequencyTable@RakServer@@UAEX_N@Z 00416580 f   rakserver.obj
 0001:00015590       ?GetSendFrequencyTable@RakServer@@UAE_NQAI@Z 00416590 f   rakserver.obj
 0001:000155a0       ?GetCompressionRatio@RakServer@@UBEMXZ 004165a0 f   rakserver.obj
 0001:000155b0       ?GetDecompressionRatio@RakServer@@UBEMXZ 004165b0 f   rakserver.obj
 0001:000155c0       ?AttachPlugin@RakServer@@UAEXPAVPluginInterface@@@Z 004165c0 f   rakserver.obj
 0001:000155d0       ?DetachPlugin@RakServer@@UAEXPAVPluginInterface@@@Z 004165d0 f   rakserver.obj
 0001:000155e0       ?GetStaticServerData@RakServer@@UAEPAVBitStream@RakNet@@XZ 004165e0 f   rakserver.obj
 0001:00015600       ?SetStaticServerData@RakServer@@UAEXPBDH@Z 00416600 f   rakserver.obj
 0001:00015630       ?SetRelayStaticClientData@RakServer@@UAEX_N@Z 00416630 f   rakserver.obj
 0001:00015640       ?SendStaticServerDataToClient@RakServer@@UAEXUPlayerID@@@Z 00416640 f   rakserver.obj
 0001:00015660       ?SetOfflinePingResponse@RakServer@@UAEXPBDI@Z 00416660 f   rakserver.obj
 0001:00015670       ?GetStaticClientData@RakServer@@UAEPAVBitStream@RakNet@@UPlayerID@@@Z 00416670 f   rakserver.obj
 0001:00015690       ?SetStaticClientData@RakServer@@UAEXUPlayerID@@PBDH@Z 00416690 f   rakserver.obj
 0001:000156b0       ?GetNumberOfAddresses@RakServer@@UAEIXZ 004166b0 f   rakserver.obj
 0001:000156c0       ?GetInternalID@RakServer@@UBE?AUPlayerID@@XZ 004166c0 f   rakserver.obj
 0001:000156e0       ?PushBackPacket@RakServer@@UAEXPAUPacket@@_N@Z 004166e0 f   rakserver.obj
 0001:000156f0       ?SetRouterInterface@RakServer@@UAEXPAVRouterInterface@@@Z 004166f0 f   rakserver.obj
 0001:00015700       ?RemoveRouterInterface@RakServer@@UAEXPAVRouterInterface@@@Z 00416700 f   rakserver.obj
 0001:00015710       ?GetLocalIP@RakServer@@UAEPBDI@Z 00416710 f   rakserver.obj
 0001:00015720       ?GetIndexFromPlayerID@RakServer@@UAEHUPlayerID@@@Z 00416720 f   rakserver.obj
 0001:00015740       ?GetPlayerIDFromIndex@RakServer@@UAE?AUPlayerID@@H@Z 00416740 f   rakserver.obj
 0001:00015760       ?AddToBanList@RakServer@@UAEXPBD@Z 00416760 f   rakserver.obj
 0001:00015780       ?RemoveFromBanList@RakServer@@UAEXPBD@Z 00416780 f   rakserver.obj
 0001:00015790       ?ClearBanList@RakServer@@UAEXXZ 00416790 f   rakserver.obj
 0001:000157a0       ?IsBanned@RakServer@@UAE_NPBD@Z 004167a0 f   rakserver.obj
 0001:000157b0       ?IsActivePlayerID@RakServer@@UAE_NUPlayerID@@@Z 004167b0 f   rakserver.obj
 0001:000157d0       ?SetTimeoutTime@RakServer@@UAEXIUPlayerID@@@Z 004167d0 f   rakserver.obj
 0001:000157f0       ?SetMTUSize@RakServer@@UAE_NH@Z 004167f0 f   rakserver.obj
 0001:00015800       ?GetMTUSize@RakServer@@UBEHXZ 00416800 f   rakserver.obj
 0001:00015810       ?AdvertiseSystem@RakServer@@UAEXPBDG0H@Z 00416810 f   rakserver.obj
 0001:00015820       ?GetStatistics@RakServer@@UAEQAURakNetStatisticsStruct@@UPlayerID@@@Z 00416820 f   rakserver.obj
 0001:00015840       ?ApplyNetworkSimulator@RakServer@@UAEXNGG@Z 00416840 f   rakserver.obj
 0001:00015860       ?IsNetworkSimulatorActive@RakServer@@UAE_NXZ 00416860 f   rakserver.obj
 0001:00015870       ?AdvertiseSystem@RakServer@@W7AEXPBDG0H@Z 00416870 f i rakserver.obj
 0001:00015880       ?SetOfflinePingResponse@RakServer@@W7AEXPBDI@Z 00416880 f i rakserver.obj
 0001:00015890       ?GetPlayerIDFromIndex@RakServer@@W7AE?AUPlayerID@@H@Z 00416890 f i rakserver.obj
 0001:000158a0       ?DeleteCompressionLayer@RakServer@@W7AE_N_N@Z 004168a0 f i rakserver.obj
 0001:000158b0       ?ClearBanList@RakServer@@W7AEXXZ 004168b0 f i rakserver.obj
 0001:000158c0       ?RegisterClassMemberRPC@RakServer@@W7AEXPAHPAX@Z 004168c0 f i rakserver.obj
 0001:000158d0       ?ApplyNetworkSimulator@RakServer@@W7AEXNGG@Z 004168d0 f i rakserver.obj
 0001:000158e0       ?GenerateCompressionLayer@RakServer@@W7AE_NQAI_N@Z 004168e0 f i rakserver.obj
 0001:000158f0       ?DeallocatePacket@RakServer@@W7AEXPAUPacket@@@Z 004168f0 f i rakserver.obj
 0001:00015900       ?RemoveRouterInterface@RakServer@@W7AEXPAVRouterInterface@@@Z 00416900 f i rakserver.obj
 0001:00015910       ?GetCompressionRatio@RakServer@@W7BEMXZ 00416910 f i rakserver.obj
 0001:00015920       ?SetRouterInterface@RakServer@@W7AEXPAVRouterInterface@@@Z 00416920 f i rakserver.obj
 0001:00015930       ?Disconnect@RakServer@@W7AEXIE@Z 00416930 f i rakserver.obj
 0001:00015940       ?RemoveFromBanList@RakServer@@W7AEXPBD@Z 00416940 f i rakserver.obj
 0001:00015950       ?Send@RakServer@@W7AE_NPBDHW4PacketPriority@@W4PacketReliability@@DUPlayerID@@_N@Z 00416950 f i rakserver.obj
 0001:00015960       ?Send@RakServer@@W7AE_NPAVBitStream@RakNet@@W4PacketPriority@@W4PacketReliability@@DUPlayerID@@_N@Z 00416960 f i rakserver.obj
 0001:00015970       ?IsNetworkSimulatorActive@RakServer@@W7AE_NXZ 00416970 f i rakserver.obj
 0001:00015980       ?SetTimeoutTime@RakServer@@W7AEXIUPlayerID@@@Z 00416980 f i rakserver.obj
 0001:00015990       ??_ERakServer@@W7AEPAXI@Z  00416990 f i rakserver.obj
 0001:000159a0       ?IsActive@RakServer@@W7BE_NXZ 004169a0 f i rakserver.obj
 0001:000159b0       ?GetLocalIP@RakServer@@W7AEPBDI@Z 004169b0 f i rakserver.obj
 0001:000159c0       ?GetInternalID@RakServer@@W7BE?AUPlayerID@@XZ 004169c0 f i rakserver.obj
 0001:000159d0       ?IsBanned@RakServer@@W7AE_NPBD@Z 004169d0 f i rakserver.obj
 0001:000159e0       ?UnregisterAsRemoteProcedureCall@RakServer@@W7AEXPAH@Z 004169e0 f i rakserver.obj
 0001:000159f0       ?GetStatistics@RakServer@@W7AEQAURakNetStatisticsStruct@@UPlayerID@@@Z 004169f0 f i rakserver.obj
 0001:00015a00       ?DetachPlugin@RakServer@@W7AEXPAVPluginInterface@@@Z 00416a00 f i rakserver.obj
 0001:00015a10       ?RPC@RakServer@@W7AE_NPAHPBDIW4PacketPriority@@W4PacketReliability@@DUPlayerID@@_N5UNetworkID@@PAVBitStream@RakNet@@@Z 00416a10 f i rakserver.obj
 0001:00015a20       ?RPC@RakServer@@W7AE_NPAHPAVBitStream@RakNet@@W4PacketPriority@@W4PacketReliability@@DUPlayerID@@_N5UNetworkID@@1@Z 00416a20 f i rakserver.obj
 0001:00015a30       ?GetNumberOfAddresses@RakServer@@W7AEIXZ 00416a30 f i rakserver.obj
 0001:00015a40       ?GetDecompressionRatio@RakServer@@W7BEMXZ 00416a40 f i rakserver.obj
 0001:00015a50       ?AttachPlugin@RakServer@@W7AEXPAVPluginInterface@@@Z 00416a50 f i rakserver.obj
 0001:00015a60       ?GetIndexFromPlayerID@RakServer@@W7AEHUPlayerID@@@Z 00416a60 f i rakserver.obj
 0001:00015a70       ?RegisterAsRemoteProcedureCall@RakServer@@W7AEXPAHP6AXPAURPCParameters@@@Z@Z 00416a70 f i rakserver.obj
 0001:00015a80       ?DisableSecurity@RakServer@@W7AEXXZ 00416a80 f i rakserver.obj
 0001:00015a90       ?GetAveragePing@RakServer@@W7AEHUPlayerID@@@Z 00416a90 f i rakserver.obj
 0001:00015aa0       ?SetMTUSize@RakServer@@W7AE_NH@Z 00416aa0 f i rakserver.obj
 0001:00015ab0       ?PushBackPacket@RakServer@@W7AEXPAUPacket@@_N@Z 00416ab0 f i rakserver.obj
 0001:00015ac0       ?GetMTUSize@RakServer@@W7BEHXZ 00416ac0 f i rakserver.obj
 0001:00015ad0       ??0RakServer@@QAE@XZ       00416ad0 f   rakserver.obj
 0001:00015b40       ??_ERakServer@@UAEPAXI@Z   00416b40 f i rakserver.obj
 0001:00015b40       ??_GRakServer@@UAEPAXI@Z   00416b40 f i rakserver.obj
 0001:00015b60       ?Receive@RakServer@@UAEPAUPacket@@XZ 00416b60 f   rakserver.obj
 0001:00016270       ?ChangeStaticClientData@RakServer@@UAEXUPlayerID@@U2@@Z 00417270 f   rakserver.obj
 0001:00016390       ?Receive@RakServer@@W7AEPAUPacket@@XZ 00417390 f i rakserver.obj
 0001:000163a0       ?RakSleep@@YAXI@Z          004173a0 f   RakSleep.obj
 0001:000163b0       ?seedMT@@YAXI@Z            004173b0 f   Rand.obj
 0001:000163f0       ?reloadMT@@YAIXZ           004173f0 f   Rand.obj
 0001:00016520       ?randomMT@@YAIXZ           00417520 f   Rand.obj
 0001:00016570       ?frandomMT@@YAMXZ          00417570 f   Rand.obj
 0001:000165e0       ?SplitPacketIndexComp@@YAHABIABQAUInternalPacket@@@Z 004175e0 f   ReliabilityLayer.obj
 0001:00016610       ?SetEncryptionKey@ReliabilityLayer@@QAEXPBE@Z 00417610 f   ReliabilityLayer.obj
 0001:00016630       ?SetSocket@ReliabilityLayer@@QAEXI@Z 00417630 f   ReliabilityLayer.obj
 0001:00016640       ?GetSocket@ReliabilityLayer@@QAEIXZ 00417640 f   ReliabilityLayer.obj
 0001:00016650       ?SetTimeoutTime@ReliabilityLayer@@QAEXI@Z 00417650 f   ReliabilityLayer.obj
 0001:00016660       ?GetTimeoutTime@ReliabilityLayer@@QAEIXZ 00417660 f   ReliabilityLayer.obj
 0001:00016670       ?FreeThreadedMemory@ReliabilityLayer@@AAEXXZ 00417670 f   ReliabilityLayer.obj
 0001:00016680       ?SendBitStream@ReliabilityLayer@@AAEXIUPlayerID@@PAVBitStream@RakNet@@@Z 00417680 f   ReliabilityLayer.obj
 0001:00016790       ?ApplyNetworkSimulator@ReliabilityLayer@@QAEXNII@Z 00417790 f   ReliabilityLayer.obj
 0001:000167d0       ?SetSplitMessageProgressInterval@ReliabilityLayer@@QAEXH@Z 004177d0 f   ReliabilityLayer.obj
 0001:000167e0       ?SetUnreliableTimeout@ReliabilityLayer@@QAEXI@Z 004177e0 f   ReliabilityLayer.obj
 0001:00016800       ?IsSendThrottled@ReliabilityLayer@@AAE_NH@Z 00417800 f   ReliabilityLayer.obj
 0001:00016810       ?UpdateWindowFromPacketloss@ReliabilityLayer@@AAEX_J@Z 00417810 f   ReliabilityLayer.obj
 0001:00016820       ?UpdateWindowFromAck@ReliabilityLayer@@AAEX_J@Z 00417820 f   ReliabilityLayer.obj
 0001:00016830       ?GetBitStreamHeaderLength@ReliabilityLayer@@AAEHQBUInternalPacket@@@Z 00417830 f   ReliabilityLayer.obj
 0001:00016860       ?GetSHA1@ReliabilityLayer@@AAEXQAEIQAD@Z 00417860 f   ReliabilityLayer.obj
 0001:00016910       ?CheckSHA1@ReliabilityLayer@@AAE_NQADQAEI@Z 00417910 f   ReliabilityLayer.obj
 0001:00016960       ?IsOlderOrderedPacket@ReliabilityLayer@@AAE_NGG@Z 00417960 f   ReliabilityLayer.obj
 0001:000169b0       ?IsCheater@ReliabilityLayer@@QBE_NXZ 004179b0 f   ReliabilityLayer.obj
 0001:000169c0       ?IsDeadConnection@ReliabilityLayer@@QBE_NXZ 004179c0 f   ReliabilityLayer.obj
 0001:000169d0       ?KillConnection@ReliabilityLayer@@QAEXXZ 004179d0 f   ReliabilityLayer.obj
 0001:000169e0       ?UpdateNextActionTime@ReliabilityLayer@@AAEXXZ 004179e0 f   ReliabilityLayer.obj
 0001:00016a20       ?UpdateThreadedMemory@ReliabilityLayer@@AAEXXZ 00417a20 f   ReliabilityLayer.obj
 0001:00016a40       ?PushAtHead@?$Queue@PAUInternalPacket@@@DataStructures@@QAEXABQAUInternalPacket@@I@Z 00417a40 f i ReliabilityLayer.obj
 0001:00016b30       ??A?$Queue@PAUInternalPacket@@@DataStructures@@QBEAAPAUInternalPacket@@I@Z 00417b30 f i ReliabilityLayer.obj
 0001:00016b60       ?Peek@?$Queue@PAUInternalPacket@@@DataStructures@@QBEPAUInternalPacket@@XZ 00417b60 f i ReliabilityLayer.obj
 0001:00016b70       ??A?$List@PAUInternalPacket@@@DataStructures@@QBEAAPAUInternalPacket@@I@Z 00417b70 f i ReliabilityLayer.obj
 0001:00016b80       ?Size@?$List@PAUInternalPacket@@@DataStructures@@QBEIXZ 00417b80 f i ReliabilityLayer.obj
 0001:00016b90       ??A?$OrderedList@IPAUInternalPacket@@$1?SplitPacketIndexComp@@YAHABIABQAU1@@Z@DataStructures@@QBEAAPAUInternalPacket@@I@Z 00417b90 f i ReliabilityLayer.obj
 0001:00016ba0       ?Size@?$OrderedList@IPAUInternalPacket@@$1?SplitPacketIndexComp@@YAHABIABQAU1@@Z@DataStructures@@QBEIXZ 00417ba0 f i ReliabilityLayer.obj
 0001:00016bb0       ??0?$List@PAV?$LinkedList@PAUInternalPacket@@@DataStructures@@@DataStructures@@QAE@XZ 00417bb0 f i ReliabilityLayer.obj
 0001:00016bc0       ??1?$List@PAV?$LinkedList@PAUInternalPacket@@@DataStructures@@@DataStructures@@QAE@XZ 00417bc0 f i ReliabilityLayer.obj
 0001:00016bd0       ??A?$List@PAV?$LinkedList@PAUInternalPacket@@@DataStructures@@@DataStructures@@QBEAAPAV?$LinkedList@PAUInternalPacket@@@1@I@Z 00417bd0 f i ReliabilityLayer.obj
 0001:00016be0       ?Replace@?$List@PAV?$LinkedList@PAUInternalPacket@@@DataStructures@@@DataStructures@@QAEXQAV?$LinkedList@PAUInternalPacket@@@2@0I@Z 00417be0 f i ReliabilityLayer.obj
 0001:00016c80       ?Size@?$List@PAV?$LinkedList@PAUInternalPacket@@@DataStructures@@@DataStructures@@QBEIXZ 00417c80 f i ReliabilityLayer.obj
 0001:00016c90       ?Clear@?$List@PAV?$LinkedList@PAUInternalPacket@@@DataStructures@@@DataStructures@@QAEX_N@Z 00417c90 f i ReliabilityLayer.obj
 0001:00016cd0       ??$RangeNodeComp@G@DataStructures@@YAHABGABU?$RangeNode@G@0@@Z 00417cd0 f i ReliabilityLayer.obj
 0001:00016d00       ?IsEmpty@?$BPlusTree@GPAUInternalPacket@@$0CA@@DataStructures@@QBE_NXZ 00417d00 f i ReliabilityLayer.obj
 0001:00016d10       ??0?$Queue@_J@DataStructures@@QAE@XZ 00417d10 f i ReliabilityLayer.obj
 0001:00016d50       ??1?$Queue@_J@DataStructures@@QAE@XZ 00417d50 f i ReliabilityLayer.obj
 0001:00016d60       ?Push@?$Queue@_J@DataStructures@@QAEXAB_J@Z 00417d60 f i ReliabilityLayer.obj
 0001:00016e40       ??A?$Queue@_J@DataStructures@@QBEAA_JI@Z 00417e40 f i ReliabilityLayer.obj
 0001:00016e70       ?Peek@?$Queue@_J@DataStructures@@QBE_JXZ 00417e70 f i ReliabilityLayer.obj
 0001:00016e80       ?Pop@?$Queue@_J@DataStructures@@QAE_JXZ 00417e80 f i ReliabilityLayer.obj
 0001:00016ec0       ?Size@?$Queue@_J@DataStructures@@QBEIXZ 00417ec0 f i ReliabilityLayer.obj
 0001:00016ee0       ?AllocationSize@?$Queue@_J@DataStructures@@QBEIXZ 00417ee0 f i ReliabilityLayer.obj
 0001:00016ef0       ?Compress@?$Queue@_J@DataStructures@@QAEXXZ 00417ef0 f i ReliabilityLayer.obj
 0001:00016fa0       ?ClearAndForceAllocation@?$Queue@_J@DataStructures@@QAEXH@Z 00417fa0 f i ReliabilityLayer.obj
 0001:00016fe0       ??0?$List@PAUDataAndTime@ReliabilityLayer@@@DataStructures@@QAE@XZ 00417fe0 f i ReliabilityLayer.obj
 0001:00016ff0       ??1?$List@PAUDataAndTime@ReliabilityLayer@@@DataStructures@@QAE@XZ 00417ff0 f i ReliabilityLayer.obj
 0001:00017000       ??A?$List@PAUDataAndTime@ReliabilityLayer@@@DataStructures@@QBEAAPAUDataAndTime@ReliabilityLayer@@I@Z 00418000 f i ReliabilityLayer.obj
 0001:00017010       ?Insert@?$List@PAUDataAndTime@ReliabilityLayer@@@DataStructures@@QAEXQAUDataAndTime@ReliabilityLayer@@@Z 00418010 f i ReliabilityLayer.obj
 0001:00017080       ?Del@?$List@PAUDataAndTime@ReliabilityLayer@@@DataStructures@@QAEXI@Z 00418080 f i ReliabilityLayer.obj
 0001:00017090       ?Size@?$List@PAUDataAndTime@ReliabilityLayer@@@DataStructures@@QBEIXZ 00418090 f i ReliabilityLayer.obj
 0001:000170a0       ?Clear@?$List@PAUDataAndTime@ReliabilityLayer@@@DataStructures@@QAEX_N@Z 004180a0 f i ReliabilityLayer.obj
 0001:000170e0       ??0?$CircularLinkedList@PAUInternalPacket@@@DataStructures@@QAE@XZ 004180e0 f i ReliabilityLayer.obj
 0001:000170f0       ?Add@?$CircularLinkedList@PAUInternalPacket@@@DataStructures@@QAEAAPAUInternalPacket@@ABQAU3@@Z 004180f0 f i ReliabilityLayer.obj
 0001:000171b0       ?Size@?$CircularLinkedList@PAUInternalPacket@@@DataStructures@@QAEIXZ 004181b0 f i ReliabilityLayer.obj
 0001:000171c0       ?Peek@?$CircularLinkedList@PAUInternalPacket@@@DataStructures@@QAEAAPAUInternalPacket@@XZ 004181c0 f i ReliabilityLayer.obj
 0001:000171d0       ?Beginning@?$CircularLinkedList@PAUInternalPacket@@@DataStructures@@QAEXXZ 004181d0 f i ReliabilityLayer.obj
 0001:000171e0       ?End@?$CircularLinkedList@PAUInternalPacket@@@DataStructures@@QAEXXZ 004181e0 f i ReliabilityLayer.obj
 0001:000171f0       ??$WriteCompressed@G@BitStream@RakNet@@QAEXG@Z 004181f0 f i ReliabilityLayer.obj
 0001:00017210       ??$ReadCompressed@G@BitStream@RakNet@@QAE_NAAG@Z 00418210 f i ReliabilityLayer.obj
 0001:00017230       ??0?$RangeNode@G@DataStructures@@QAE@XZ 00418230 f i ReliabilityLayer.obj
 0001:00017240       ??1?$RangeNode@G@DataStructures@@QAE@XZ 00418240 f i ReliabilityLayer.obj
 0001:00017250       ??0?$RangeNode@G@DataStructures@@QAE@GG@Z 00418250 f i ReliabilityLayer.obj
 0001:00017270       ??0?$List@PAUInternalPacket@@@DataStructures@@QAE@XZ 00418270 f i ReliabilityLayer.obj
 0001:00017280       ??1?$List@PAUInternalPacket@@@DataStructures@@QAE@XZ 00418280 f i ReliabilityLayer.obj
 0001:00017290       ?Insert@?$List@PAUInternalPacket@@@DataStructures@@QAEXQAUInternalPacket@@@Z 00418290 f i ReliabilityLayer.obj
 0001:00017300       ?Insert@?$List@PAUInternalPacket@@@DataStructures@@QAEXQAUInternalPacket@@I@Z 00418300 f i ReliabilityLayer.obj
 0001:00017390       ?Del@?$List@PAUInternalPacket@@@DataStructures@@QAEXI@Z 00418390 f i ReliabilityLayer.obj
 0001:000173a0       ?GetIndexFromKey@?$OrderedList@IPAUInternalPacket@@$1?SplitPacketIndexComp@@YAHABIABQAU1@@Z@DataStructures@@QBEIABIPA_N@Z 004183a0 f i ReliabilityLayer.obj
 0001:00017420       ??A?$List@U?$RangeNode@G@DataStructures@@@DataStructures@@QBEAAU?$RangeNode@G@1@I@Z 00418420 f i ReliabilityLayer.obj
 0001:00017430       ?Size@?$List@U?$RangeNode@G@DataStructures@@@DataStructures@@QBEIXZ 00418430 f i ReliabilityLayer.obj
 0001:00017440       ?GetListHead@?$BPlusTree@GPAUInternalPacket@@$0CA@@DataStructures@@QBEPAU?$Page@GPAUInternalPacket@@$0CA@@2@XZ 00418440 f i ReliabilityLayer.obj
 0001:00017450       ?DeleteFromPageAtIndex@?$BPlusTree@GPAUInternalPacket@@$0CA@@DataStructures@@IAEXHPAU?$Page@GPAUInternalPacket@@$0CA@@2@@Z 00418450 f i ReliabilityLayer.obj
 0001:000174d0       ?GetIndexOf@?$BPlusTree@GPAUInternalPacket@@$0CA@@DataStructures@@IBE_NGPAU?$Page@GPAUInternalPacket@@$0CA@@2@PAH@Z 004184d0 f i ReliabilityLayer.obj
 0001:00017560       ??0?$List@PAUSplitPacketChannel@@@DataStructures@@QAE@XZ 00418560 f i ReliabilityLayer.obj
 0001:00017570       ??1?$List@PAUSplitPacketChannel@@@DataStructures@@QAE@XZ 00418570 f i ReliabilityLayer.obj
 0001:00017580       ??A?$List@PAUSplitPacketChannel@@@DataStructures@@QBEAAPAUSplitPacketChannel@@I@Z 00418580 f i ReliabilityLayer.obj
 0001:00017590       ?Insert@?$List@PAUSplitPacketChannel@@@DataStructures@@QAEXQAUSplitPacketChannel@@@Z 00418590 f i ReliabilityLayer.obj
 0001:00017600       ?Insert@?$List@PAUSplitPacketChannel@@@DataStructures@@QAEXQAUSplitPacketChannel@@I@Z 00418600 f i ReliabilityLayer.obj
 0001:00017690       ?Size@?$List@PAUSplitPacketChannel@@@DataStructures@@QBEIXZ 00418690 f i ReliabilityLayer.obj
 0001:000176a0       ?Clear@?$List@PAUSplitPacketChannel@@@DataStructures@@QAEX_N@Z 004186a0 f i ReliabilityLayer.obj
 0001:000176e0       ?Del@?$CircularLinkedList@PAUInternalPacket@@@DataStructures@@QAEXXZ 004186e0 f i ReliabilityLayer.obj
 0001:00017740       ?Clear@?$CircularLinkedList@PAUInternalPacket@@@DataStructures@@QAEXXZ 00418740 f i ReliabilityLayer.obj
 0001:00017790       ??E?$LinkedList@PAUInternalPacket@@@DataStructures@@QAEAAV01@XZ 00418790 f i ReliabilityLayer.obj
 0001:000177b0       ?Clear@?$List@PAUInternalPacket@@@DataStructures@@QAEX_N@Z 004187b0 f i ReliabilityLayer.obj
 0001:000177f0       ??0?$List@U?$RangeNode@G@DataStructures@@@DataStructures@@QAE@XZ 004187f0 f i ReliabilityLayer.obj
 0001:00017800       ?Del@?$List@U?$RangeNode@G@DataStructures@@@DataStructures@@QAEXI@Z 00418800 f i ReliabilityLayer.obj
 0001:00017810       ?CanRotateLeft@?$BPlusTree@GPAUInternalPacket@@$0CA@@DataStructures@@IAE_NPAU?$Page@GPAUInternalPacket@@$0CA@@2@H@Z 00418810 f i ReliabilityLayer.obj
 0001:00017840       ?CanRotateRight@?$BPlusTree@GPAUInternalPacket@@$0CA@@DataStructures@@IAE_NPAU?$Page@GPAUInternalPacket@@$0CA@@2@H@Z 00418840 f i ReliabilityLayer.obj
 0001:00017870       ?RotateRight@?$BPlusTree@GPAUInternalPacket@@$0CA@@DataStructures@@IAEXPAU?$Page@GPAUInternalPacket@@$0CA@@2@HPAUReturnAction@12@@Z 00418870 f i ReliabilityLayer.obj
 0001:00017900       ?RotateLeft@?$BPlusTree@GPAUInternalPacket@@$0CA@@DataStructures@@IAEXPAU?$Page@GPAUInternalPacket@@$0CA@@2@HPAUReturnAction@12@@Z 00418900 f i ReliabilityLayer.obj
 0001:00017990       ??0?$Queue@PAU?$Page@GPAUInternalPacket@@$0CA@@DataStructures@@@DataStructures@@QAE@XZ 00418990 f i ReliabilityLayer.obj
 0001:000179d0       ??1?$Queue@PAU?$Page@GPAUInternalPacket@@$0CA@@DataStructures@@@DataStructures@@QAE@XZ 004189d0 f i ReliabilityLayer.obj
 0001:000179e0       ?Push@?$Queue@PAU?$Page@GPAUInternalPacket@@$0CA@@DataStructures@@@DataStructures@@QAEXABQAU?$Page@GPAUInternalPacket@@$0CA@@2@@Z 004189e0 f i ReliabilityLayer.obj
 0001:00017ab0       ?Pop@?$Queue@PAU?$Page@GPAUInternalPacket@@$0CA@@DataStructures@@@DataStructures@@QAEPAU?$Page@GPAUInternalPacket@@$0CA@@2@XZ 00418ab0 f i ReliabilityLayer.obj
 0001:00017ae0       ?Size@?$Queue@PAU?$Page@GPAUInternalPacket@@$0CA@@DataStructures@@@DataStructures@@QBEIXZ 00418ae0 f i ReliabilityLayer.obj
 0001:00017b00       ??0?$List@PAU?$Page@GPAUInternalPacket@@$0CA@@DataStructures@@@DataStructures@@QAE@XZ 00418b00 f i ReliabilityLayer.obj
 0001:00017b10       ??1?$List@PAU?$Page@GPAUInternalPacket@@$0CA@@DataStructures@@@DataStructures@@QAE@XZ 00418b10 f i ReliabilityLayer.obj
 0001:00017b20       ??A?$List@PAU?$Page@GPAUInternalPacket@@$0CA@@DataStructures@@@DataStructures@@QBEAAPAU?$Page@GPAUInternalPacket@@$0CA@@1@I@Z 00418b20 f i ReliabilityLayer.obj
 0001:00017b30       ?Insert@?$List@PAU?$Page@GPAUInternalPacket@@$0CA@@DataStructures@@@DataStructures@@QAEXQAU?$Page@GPAUInternalPacket@@$0CA@@2@@Z 00418b30 f i ReliabilityLayer.obj
 0001:00017ba0       ?Del@?$List@PAU?$Page@GPAUInternalPacket@@$0CA@@DataStructures@@@DataStructures@@QAEXI@Z 00418ba0 f i ReliabilityLayer.obj
 0001:00017bb0       ?Size@?$List@PAU?$Page@GPAUInternalPacket@@$0CA@@DataStructures@@@DataStructures@@QBEIXZ 00418bb0 f i ReliabilityLayer.obj
 0001:00017bc0       ?Del@?$List@PAUSplitPacketChannel@@@DataStructures@@QAEXI@Z 00418bc0 f i ReliabilityLayer.obj
 0001:00017bd0       ??_E?$RangeNode@G@DataStructures@@QAEPAXI@Z 00418bd0 f i ReliabilityLayer.obj
 0001:00017c20       ?ShiftNodeLeft@?$BPlusTree@GPAUInternalPacket@@$0CA@@DataStructures@@IAEXPAU?$Page@GPAUInternalPacket@@$0CA@@2@@Z 00418c20 f i ReliabilityLayer.obj
 0001:00017c90       ?ShiftNodeRight@?$BPlusTree@GPAUInternalPacket@@$0CA@@DataStructures@@IAEXPAU?$Page@GPAUInternalPacket@@$0CA@@2@@Z 00418c90 f i ReliabilityLayer.obj
 0001:00017d10       ?GetPointer@InternalPacketPool@@QAEPAUInternalPacket@@XZ 00418d10 f i ReliabilityLayer.obj
 0001:00017d70       ?SplitPacketChannelComp@@YAHABGABQAUSplitPacketChannel@@@Z 00418d70 f   ReliabilityLayer.obj
 0001:00017da0       ?Receive@ReliabilityLayer@@QAEHPAPAE@Z 00418da0 f   ReliabilityLayer.obj
 0001:00017e20       ?WriteToBitStreamFromInternalPacket@ReliabilityLayer@@AAEHPAVBitStream@RakNet@@QBUInternalPacket@@@Z 00418e20 f   ReliabilityLayer.obj
 0001:00017f30       ?CreateInternalPacketFromBitStream@ReliabilityLayer@@AAEPAUInternalPacket@@PAVBitStream@RakNet@@_J@Z 00418f30 f   ReliabilityLayer.obj
 0001:000180d0       ?SplitPacket@ReliabilityLayer@@AAEXPAUInternalPacket@@H@Z 004190d0 f   ReliabilityLayer.obj
 0001:00018380       ?CreateInternalPacketCopy@ReliabilityLayer@@AAEPAUInternalPacket@@PAU2@HH_J@Z 00419380 f   ReliabilityLayer.obj
 0001:00018410       ?GetOrderingListAtOrderingStream@ReliabilityLayer@@AAEPAV?$LinkedList@PAUInternalPacket@@@DataStructures@@E@Z 00419410 f   ReliabilityLayer.obj
 0001:00018430       ?InsertPacketIntoResendList@ReliabilityLayer@@AAEXPAUInternalPacket@@_J_N2@Z 00419430 f   ReliabilityLayer.obj
 0001:000184b0       ?SetPing@ReliabilityLayer@@QAEXI@Z 004194b0 f   ReliabilityLayer.obj
 0001:00018540       ?Del@?$Queue@PAUInternalPacket@@@DataStructures@@QAEXI@Z 00419540 f i ReliabilityLayer.obj
 0001:000185b0       ?RemoveAtIndex@?$List@PAUInternalPacket@@@DataStructures@@QAEXI@Z 004195b0 f i ReliabilityLayer.obj
 0001:000185f0       ??0?$OrderedList@IPAUInternalPacket@@$1?SplitPacketIndexComp@@YAHABIABQAU1@@Z@DataStructures@@QAE@XZ 004195f0 f i ReliabilityLayer.obj
 0001:00018600       ?Insert@?$OrderedList@IPAUInternalPacket@@$1?SplitPacketIndexComp@@YAHABIABQAU1@@Z@DataStructures@@QAEIABIABQAUInternalPacket@@@Z 00419600 f i ReliabilityLayer.obj
 0001:00018660       ??A?$OrderedList@GU?$RangeNode@G@DataStructures@@$1??$RangeNodeComp@G@2@YAHABGABU12@@Z@DataStructures@@QBEAAU?$RangeNode@G@1@I@Z 00419660 f i ReliabilityLayer.obj
 0001:00018670       ?Size@?$OrderedList@GU?$RangeNode@G@DataStructures@@$1??$RangeNodeComp@G@2@YAHABGABU12@@Z@DataStructures@@QBEIXZ 00419670 f i ReliabilityLayer.obj
 0001:00018680       ?Size@?$RangeList@G@DataStructures@@QAEIXZ 00419680 f i ReliabilityLayer.obj
 0001:00018690       ?Size@?$BPlusTree@GPAUInternalPacket@@$0CA@@DataStructures@@QBEIXZ 00419690 f i ReliabilityLayer.obj
 0001:000186b0       ??0?$OrderedList@GPAUSplitPacketChannel@@$1?SplitPacketChannelComp@@YAHABGABQAU1@@Z@DataStructures@@QAE@XZ 004196b0 f i ReliabilityLayer.obj
 0001:000186c0       ?GetIndexFromKey@?$OrderedList@GPAUSplitPacketChannel@@$1?SplitPacketChannelComp@@YAHABGABQAU1@@Z@DataStructures@@QBEIABGPA_N@Z 004196c0 f i ReliabilityLayer.obj
 0001:00018740       ?Insert@?$OrderedList@GPAUSplitPacketChannel@@$1?SplitPacketChannelComp@@YAHABGABQAU1@@Z@DataStructures@@QAEIABGABQAUSplitPacketChannel@@@Z 00419740 f i ReliabilityLayer.obj
 0001:000187a0       ??A?$OrderedList@GPAUSplitPacketChannel@@$1?SplitPacketChannelComp@@YAHABGABQAU1@@Z@DataStructures@@QBEAAPAUSplitPacketChannel@@I@Z 004197a0 f i ReliabilityLayer.obj
 0001:000187b0       ?Clear@?$OrderedList@GPAUSplitPacketChannel@@$1?SplitPacketChannelComp@@YAHABGABQAU1@@Z@DataStructures@@QAEXXZ 004197b0 f i ReliabilityLayer.obj
 0001:000187f0       ?Size@?$OrderedList@GPAUSplitPacketChannel@@$1?SplitPacketChannelComp@@YAHABGABQAU1@@Z@DataStructures@@QBEIXZ 004197f0 f i ReliabilityLayer.obj
 0001:00018800       ??1?$CircularLinkedList@PAUInternalPacket@@@DataStructures@@QAE@XZ 00419800 f i ReliabilityLayer.obj
 0001:00018810       ?Pop@?$CircularLinkedList@PAUInternalPacket@@@DataStructures@@QAEPAUInternalPacket@@XZ 00419810 f i ReliabilityLayer.obj
 0001:00018820       ??1?$LinkedList@PAUInternalPacket@@@DataStructures@@QAE@XZ 00419820 f i ReliabilityLayer.obj
 0001:00018870       ??E?$LinkedList@PAUInternalPacket@@@DataStructures@@QAEAAV01@H@Z 00419870 f i ReliabilityLayer.obj
 0001:00018890       ?Clear@?$OrderedList@IPAUInternalPacket@@$1?SplitPacketIndexComp@@YAHABIABQAU1@@Z@DataStructures@@QAEXXZ 00419890 f i ReliabilityLayer.obj
 0001:000188d0       ?GetIndexFromKey@?$OrderedList@GU?$RangeNode@G@DataStructures@@$1??$RangeNodeComp@G@2@YAHABGABU12@@Z@DataStructures@@QBEIABGPA_N@Z 004198d0 f i ReliabilityLayer.obj
 0001:00018950       ?Del@?$OrderedList@GU?$RangeNode@G@DataStructures@@$1??$RangeNodeComp@G@2@YAHABGABU12@@Z@DataStructures@@QAEXI@Z 00419950 f i ReliabilityLayer.obj
 0001:00018960       ??0?$MemoryPool@U?$Page@GPAUInternalPacket@@$0CA@@DataStructures@@@DataStructures@@QAE@XZ 00419960 f i ReliabilityLayer.obj
 0001:00018970       ??1?$MemoryPool@U?$Page@GPAUInternalPacket@@$0CA@@DataStructures@@@DataStructures@@QAE@XZ 00419970 f i ReliabilityLayer.obj
 0001:000189e0       ?Preallocate@?$MemoryPool@U?$Page@GPAUInternalPacket@@$0CA@@DataStructures@@@DataStructures@@QAEXI@Z 004199e0 f i ReliabilityLayer.obj
 0001:00018a20       ?Allocate@?$MemoryPool@U?$Page@GPAUInternalPacket@@$0CA@@DataStructures@@@DataStructures@@QAEPAU?$Page@GPAUInternalPacket@@$0CA@@2@XZ 00419a20 f i ReliabilityLayer.obj
 0001:00018a40       ?Release@?$MemoryPool@U?$Page@GPAUInternalPacket@@$0CA@@DataStructures@@@DataStructures@@QAEXPAU?$Page@GPAUInternalPacket@@$0CA@@2@@Z 00419a40 f i ReliabilityLayer.obj
 0001:00018a50       ?RemoveAtIndex@?$List@PAUSplitPacketChannel@@@DataStructures@@QAEXI@Z 00419a50 f i ReliabilityLayer.obj
 0001:00018a90       ??1?$List@U?$RangeNode@G@DataStructures@@@DataStructures@@QAE@XZ 00419a90 f i ReliabilityLayer.obj
 0001:00018ac0       ?Insert@?$List@U?$RangeNode@G@DataStructures@@@DataStructures@@QAEXU?$RangeNode@G@2@@Z 00419ac0 f i ReliabilityLayer.obj
 0001:00018bc0       ?Insert@?$List@U?$RangeNode@G@DataStructures@@@DataStructures@@QAEXU?$RangeNode@G@2@I@Z 00419bc0 f i ReliabilityLayer.obj
 0001:00018cd0       ?RemoveAtIndex@?$List@U?$RangeNode@G@DataStructures@@@DataStructures@@QAEXI@Z 00419cd0 f i ReliabilityLayer.obj
 0001:00018d10       ?Clear@?$List@U?$RangeNode@G@DataStructures@@@DataStructures@@QAEX_N@Z 00419d10 f i ReliabilityLayer.obj
 0001:00018d70       ?InsertIntoNode@?$BPlusTree@GPAUInternalPacket@@$0CA@@DataStructures@@IAEPAU?$Page@GPAUInternalPacket@@$0CA@@2@GABQAUInternalPacket@@HPAU32@1PAUReturnAction@12@@Z 00419d70 f i ReliabilityLayer.obj
 0001:000191a0       ?FixUnderflow@?$BPlusTree@GPAUInternalPacket@@$0CA@@DataStructures@@IAE_NHPAU?$Page@GPAUInternalPacket@@$0CA@@2@GPAUReturnAction@12@@Z 0041a1a0 f i ReliabilityLayer.obj
 0001:00019420       ??_G?$LinkedList@PAUInternalPacket@@@DataStructures@@QAEPAXI@Z 0041a420 f i ReliabilityLayer.obj
 0001:00019480       ?Send@ReliabilityLayer@@QAE_NPADHW4PacketPriority@@W4PacketReliability@@E_NH_J@Z 0041a480 f   ReliabilityLayer.obj
 0001:00019620       ?IsDataWaiting@ReliabilityLayer@@QAE_NXZ 0041a620 f   ReliabilityLayer.obj
 0001:000196a0       ?AreAcksWaiting@ReliabilityLayer@@QAE_NXZ 0041a6a0 f   ReliabilityLayer.obj
 0001:000196b0       ?DeleteSequencedPacketsInList@ReliabilityLayer@@AAEXEAAV?$List@PAUInternalPacket@@@DataStructures@@H@Z 0041a6b0 f   ReliabilityLayer.obj
 0001:00019740       ?DeleteSequencedPacketsInList@ReliabilityLayer@@AAEXEAAV?$Queue@PAUInternalPacket@@@DataStructures@@@Z 0041a740 f   ReliabilityLayer.obj
 0001:00019830       ?GetResendListDataSize@ReliabilityLayer@@ABEIXZ 0041a830 f   ReliabilityLayer.obj
 0001:00019850       ??0?$LinkedList@PAUInternalPacket@@@DataStructures@@QAE@XZ 0041a850 f i ReliabilityLayer.obj
 0001:00019860       ??1?$OrderedList@IPAUInternalPacket@@$1?SplitPacketIndexComp@@YAHABIABQAU1@@Z@DataStructures@@QAE@XZ 0041a860 f i ReliabilityLayer.obj
 0001:000198e0       ?Serialize@?$RangeList@G@DataStructures@@QAEIPAVBitStream@RakNet@@H_N@Z 0041a8e0 f i ReliabilityLayer.obj
 0001:00019a90       ??0?$BPlusTree@GPAUInternalPacket@@$0CA@@DataStructures@@QAE@XZ 0041aa90 f i ReliabilityLayer.obj
 0001:00019ab0       ?Preallocate@?$BPlusTree@GPAUInternalPacket@@$0CA@@DataStructures@@QAEXH@Z 0041aab0 f i ReliabilityLayer.obj
 0001:00019ac0       ??1?$OrderedList@GPAUSplitPacketChannel@@$1?SplitPacketChannelComp@@YAHABGABQAU1@@Z@DataStructures@@QAE@XZ 0041aac0 f i ReliabilityLayer.obj
 0001:00019b40       ?RemoveAtIndex@?$OrderedList@GPAUSplitPacketChannel@@$1?SplitPacketChannelComp@@YAHABGABQAU1@@Z@DataStructures@@QAEXI@Z 0041ab40 f i ReliabilityLayer.obj
 0001:00019b80       ??0?$OrderedList@GU?$RangeNode@G@DataStructures@@$1??$RangeNodeComp@G@2@YAHABGABU12@@Z@DataStructures@@QAE@XZ 0041ab80 f i ReliabilityLayer.obj
 0001:00019b90       ?Insert@?$OrderedList@GU?$RangeNode@G@DataStructures@@$1??$RangeNodeComp@G@2@YAHABGABU12@@Z@DataStructures@@QAEIABGABU?$RangeNode@G@2@@Z 0041ab90 f i ReliabilityLayer.obj
 0001:00019bf0       ?RemoveAtIndex@?$OrderedList@GU?$RangeNode@G@DataStructures@@$1??$RangeNodeComp@G@2@YAHABGABU12@@Z@DataStructures@@QAEXI@Z 0041abf0 f i ReliabilityLayer.obj
 0001:00019c30       ?InsertAtIndex@?$OrderedList@GU?$RangeNode@G@DataStructures@@$1??$RangeNodeComp@G@2@YAHABGABU12@@Z@DataStructures@@QAEXABU?$RangeNode@G@2@I@Z 0041ac30 f i ReliabilityLayer.obj
 0001:00019c40       ?InsertAtEnd@?$OrderedList@GU?$RangeNode@G@DataStructures@@$1??$RangeNodeComp@G@2@YAHABGABU12@@Z@DataStructures@@QAEXABU?$RangeNode@G@2@@Z 0041ac40 f i ReliabilityLayer.obj
 0001:00019c50       ?Clear@?$OrderedList@GU?$RangeNode@G@DataStructures@@$1??$RangeNodeComp@G@2@YAHABGABU12@@Z@DataStructures@@QAEXXZ 0041ac50 f i ReliabilityLayer.obj
 0001:00019ca0       ?FreePages@?$BPlusTree@GPAUInternalPacket@@$0CA@@DataStructures@@IAEXXZ 0041aca0 f i ReliabilityLayer.obj
 0001:00019e20       ?InsertBranchDown@?$BPlusTree@GPAUInternalPacket@@$0CA@@DataStructures@@IAEPAU?$Page@GPAUInternalPacket@@$0CA@@2@GABQAUInternalPacket@@PAU32@PAUReturnAction@12@PA_N@Z 0041ae20 f i ReliabilityLayer.obj
 0001:0001a0d0       ?FindDeleteRebalance@?$BPlusTree@GPAUInternalPacket@@$0CA@@DataStructures@@IAE_NGPAU?$Page@GPAUInternalPacket@@$0CA@@2@PA_NGPAUReturnAction@12@AAPAUInternalPacket@@@Z 0041b0d0 f i ReliabilityLayer.obj
 0001:0001a240       ?InitializeVariables@ReliabilityLayer@@AAEXXZ 0041b240 f   ReliabilityLayer.obj
 0001:0001a3a0       ??1SplitPacketChannel@@QAE@XZ 0041b3a0 f i ReliabilityLayer.obj
 0001:0001a3b0       ??0SplitPacketChannel@@QAE@XZ 0041b3b0 f i ReliabilityLayer.obj
 0001:0001a3c0       ?AddToOrderingList@ReliabilityLayer@@AAEXPAUInternalPacket@@@Z 0041b3c0 f   ReliabilityLayer.obj
 0001:0001a460       ?GetStatistics@ReliabilityLayer@@QAEQAURakNetStatisticsStruct@@XZ 0041b460 f   ReliabilityLayer.obj
 0001:0001a580       ?Insert@?$RangeList@G@DataStructures@@QAEXG@Z 0041b580 f i ReliabilityLayer.obj
 0001:0001a6e0       ?Clear@?$RangeList@G@DataStructures@@QAEXXZ 0041b6e0 f i ReliabilityLayer.obj
 0001:0001a730       ?Deserialize@?$RangeList@G@DataStructures@@QAE_NPAVBitStream@RakNet@@@Z 0041b730 f i ReliabilityLayer.obj
 0001:0001a860       ?Delete@?$BPlusTree@GPAUInternalPacket@@$0CA@@DataStructures@@QAE_NGAAPAUInternalPacket@@@Z 0041b860 f i ReliabilityLayer.obj
 0001:0001a940       ?Insert@?$BPlusTree@GPAUInternalPacket@@$0CA@@DataStructures@@QAE_NGABQAUInternalPacket@@@Z 0041b940 f i ReliabilityLayer.obj
 0001:0001aa80       ?Clear@?$BPlusTree@GPAUInternalPacket@@$0CA@@DataStructures@@QAEXXZ 0041ba80 f i ReliabilityLayer.obj
 0001:0001aaa0       ??1?$OrderedList@GU?$RangeNode@G@DataStructures@@$1??$RangeNodeComp@G@2@YAHABGABU12@@Z@DataStructures@@QAE@XZ 0041baa0 f i ReliabilityLayer.obj
 0001:0001ab50       ??_GSplitPacketChannel@@QAEPAXI@Z 0041bb50 f i ReliabilityLayer.obj
 0001:0001ab80       ?GenerateDatagram@ReliabilityLayer@@AAEIPAVBitStream@RakNet@@HPA_N_JUPlayerID@@AAV?$List@PAVPluginInterface@@@DataStructures@@@Z 0041bb80 f   ReliabilityLayer.obj
 0001:0001b130       ?RemovePacketFromResendListAndDeleteOlderReliableSequenced@ReliabilityLayer@@AAEIG_J@Z 0041c130 f   ReliabilityLayer.obj
 0001:0001b180       ?SendAcknowledgementPacket@ReliabilityLayer@@AAEXG_J@Z 0041c180 f   ReliabilityLayer.obj
 0001:0001b1a0       ?InsertIntoSplitPacketList@ReliabilityLayer@@AAEXPAUInternalPacket@@_J@Z 0041c1a0 f   ReliabilityLayer.obj
 0001:0001b320       ?BuildPacketFromSplitPacketList@ReliabilityLayer@@AAEPAUInternalPacket@@G_J@Z 0041c320 f   ReliabilityLayer.obj
 0001:0001b4e0       ?DeleteOldUnreliableSplitPackets@ReliabilityLayer@@AAEX_J@Z 0041c4e0 f   ReliabilityLayer.obj
 0001:0001b5e0       ??0?$RangeList@G@DataStructures@@QAE@XZ 0041c5e0 f i ReliabilityLayer.obj
 0001:0001b5f0       ??1?$RangeList@G@DataStructures@@QAE@XZ 0041c5f0 f i ReliabilityLayer.obj
 0001:0001b680       ??1?$BPlusTree@GPAUInternalPacket@@$0CA@@DataStructures@@QAE@XZ 0041c680 f i ReliabilityLayer.obj
 0001:0001b6e0       ??0ReliabilityLayer@@QAE@XZ 0041c6e0 f   ReliabilityLayer.obj
 0001:0001b880       ?FreeThreadSafeMemory@ReliabilityLayer@@AAEXXZ 0041c880 f   ReliabilityLayer.obj
 0001:0001bdc0       ?HandleSocketReceiveFromConnectedPlayer@ReliabilityLayer@@QAE_NPBDHUPlayerID@@AAV?$List@PAVPluginInterface@@@DataStructures@@H@Z 0041cdc0 f   ReliabilityLayer.obj
 0001:0001c5b0       ?Update@ReliabilityLayer@@QAEXIUPlayerID@@H_JAAV?$List@PAVPluginInterface@@@DataStructures@@@Z 0041d5b0 f   ReliabilityLayer.obj
 0001:0001cc80       ?FreeMemory@ReliabilityLayer@@AAEX_N@Z 0041dc80 f   ReliabilityLayer.obj
 0001:0001cca0       ??1ReliabilityLayer@@QAE@XZ 0041dca0 f   ReliabilityLayer.obj
 0001:0001cdd0       ?Reset@ReliabilityLayer@@QAEX_N@Z 0041ddd0 f   ReliabilityLayer.obj
 0001:0001cdf0       ?mul@@YAEEE@Z              0041ddf0 f   rijndael.obj
 0001:0001ce30       ?KeyAddition@@YAXQAY03E0E@Z 0041de30 f   rijndael.obj
 0001:0001ce80       ?ShiftRow@@YAXQAY03EEE@Z   0041de80 f   rijndael.obj
 0001:0001cef0       ?Substitution@@YAXQAY03EQAEE@Z 0041def0 f   rijndael.obj
 0001:0001cf40       ?MixColumn@@YAXQAY03EE@Z   0041df40 f   rijndael.obj
 0001:0001d090       ?InvMixColumn@@YAXQAY03EE@Z 0041e090 f   rijndael.obj
 0001:0001d0e0       ?rijndaelKeySched@@YAHQAY03EHQAY133E@Z 0041e0e0 f   rijndael.obj
 0001:0001d290       ?rijndaelKeyEnctoDec@@YAHHQAY133E@Z 0041e290 f   rijndael.obj
 0001:0001d2d0       ?rijndaelEncrypt@@YAHQAE0QAY133E@Z 0041e2d0 f   rijndael.obj
 0001:0001d6b0       ?rijndaelEncryptRound@@YAHQAY03EQAY133EH@Z 0041e6b0 f   rijndael.obj
 0001:0001d970       ?rijndaelDecrypt@@YAHQAE0QAY133E@Z 0041e970 f   rijndael.obj
 0001:0001dd10       ?rijndaelDecryptRound@@YAHQAY03EQAY133EH@Z 0041ed10 f   rijndael.obj
 0001:0001ddc0       ?makeKey@@YAHPAUkeyInstance@@EHPAD@Z 0041edc0 f   rijndael.obj
 0001:0001dee0       ?cipherInit@@YAHPAUcipherInstance@@EPAD@Z 0041eee0 f   rijndael.obj
 0001:0001df40       ?blockEncrypt@@YAHPAUcipherInstance@@PAUkeyInstance@@PAEH2@Z 0041ef40 f   rijndael.obj
 0001:0001e290       ?blockDecrypt@@YAHPAUcipherInstance@@PAUkeyInstance@@PAEH2@Z 0041f290 f   rijndael.obj
 0001:0001e5d0       ?cipherUpdateRounds@@YAHPAUcipherInstance@@PAUkeyInstance@@PAEH2H@Z 0041f5d0 f   rijndael.obj
 0001:0001e680       ??0?$List@PAURPCNode@@@DataStructures@@QAE@XZ 0041f680 f i RPCMap.obj
 0001:0001e690       ??1?$List@PAURPCNode@@@DataStructures@@QAE@XZ 0041f690 f i RPCMap.obj
 0001:0001e6a0       ??A?$List@PAURPCNode@@@DataStructures@@QBEAAPAURPCNode@@I@Z 0041f6a0 f i RPCMap.obj
 0001:0001e6b0       ?Insert@?$List@PAURPCNode@@@DataStructures@@QAEXQAURPCNode@@@Z 0041f6b0 f i RPCMap.obj
 0001:0001e720       ?Replace@?$List@PAURPCNode@@@DataStructures@@QAEXQAURPCNode@@0I@Z 0041f720 f i RPCMap.obj
 0001:0001e7c0       ?Size@?$List@PAURPCNode@@@DataStructures@@QBEIXZ 0041f7c0 f i RPCMap.obj
 0001:0001e7d0       ?Clear@?$List@PAURPCNode@@@DataStructures@@QAEX_N@Z 0041f7d0 f i RPCMap.obj
 0001:0001e810       ??0RPCMap@@QAE@XZ          0041f810 f   RPCMap.obj
 0001:0001e820       ?Clear@RPCMap@@QAEXXZ      0041f820 f   RPCMap.obj
 0001:0001e880       ?GetNodeFromIndex@RPCMap@@QAEPAURPCNode@@E@Z 0041f880 f   RPCMap.obj
 0001:0001e8a0       ?GetIndexFromFunctionName@RPCMap@@QAEEPAH@Z 0041f8a0 f   RPCMap.obj
 0001:0001e8d0       ?AddIdentifierWithFunction@RPCMap@@QAEXPAHPAX_N@Z 0041f8d0 f   RPCMap.obj
 0001:0001e950       ?AddIdentifierAtIndex@RPCMap@@QAEXE@Z 0041f950 f   RPCMap.obj
 0001:0001e9f0       ?RemoveNode@RPCMap@@QAEXPAH@Z 0041f9f0 f   RPCMap.obj
 0001:0001ea40       ??1RPCMap@@QAE@XZ          0041fa40 f   RPCMap.obj
 0001:0001eaa0       ?GetNodeFromFunctionName@RPCMap@@QAEPAURPCNode@@PAH@Z 0041faa0 f   RPCMap.obj
 0001:0001eae0       ?Reset@CSHA1@@QAEXXZ       0041fae0 f   SHA1.obj
 0001:0001eb10       ?Transform@CSHA1@@AAEXQAIQAE@Z 0041fb10 f   SHA1.obj
 0001:0001fee0       ?Update@CSHA1@@QAEXPAEI@Z  00420ee0 f   SHA1.obj
 0001:0001ffa0       ?HashFile@CSHA1@@QAE_NPAD@Z 00420fa0 f   SHA1.obj
 0001:00020080       ?Final@CSHA1@@QAEXXZ       00421080 f   SHA1.obj
 0001:00020180       ?ReportHash@CSHA1@@QAEXPADE@Z 00421180 f   SHA1.obj
 0001:000202f0       ?GetHash@CSHA1@@QAEXPAE@Z  004212f0 f   SHA1.obj
 0001:00020320       ?GetHash@CSHA1@@QBEPAEXZ   00421320 f   SHA1.obj
 0001:00020330       ??0CSHA1@@QAE@XZ           00421330 f   SHA1.obj
 0001:00020370       ??1CSHA1@@UAE@XZ           00421370 f   SHA1.obj
 0001:000203b0       ??_GCSHA1@@UAEPAXI@Z       004213b0 f i SHA1.obj
 0001:000203b0       ??_ECSHA1@@UAEPAXI@Z       004213b0 f i SHA1.obj
 0001:00020400       ??0SimpleMutex@@QAE@XZ     00421400 f   SimpleMutex.obj
 0001:00020410       ??1SimpleMutex@@QAE@XZ     00421410 f   SimpleMutex.obj
 0001:00020420       ?Lock@SimpleMutex@@QAEXXZ  00421420 f   SimpleMutex.obj
 0001:00020430       ?Unlock@SimpleMutex@@QAEXXZ 00421430 f   SimpleMutex.obj
 0001:00020440       ??0SocketLayer@@QAE@XZ     00421440 f   SocketLayer.obj
 0001:00020470       ??1SocketLayer@@QAE@XZ     00421470 f   SocketLayer.obj
 0001:00020490       ?Connect@SocketLayer@@QAEIIIG@Z 00421490 f   SocketLayer.obj
 0001:000204f0       ?CreateBoundSocket@SocketLayer@@QAEIG_NPBD@Z 004214f0 f   SocketLayer.obj
 0001:00020620       ?DomainNameToIP@SocketLayer@@QAEPBDPBD@Z 00421620 f   SocketLayer.obj
 0001:00020650       ?Write@SocketLayer@@QAEXIPBDH@Z 00421650 f   SocketLayer.obj
 0001:00020670       ?AssociateSocketWithCompletionPortAndRead@SocketLayer@@QAE_NIIGPAVRakPeer@@@Z 00421670 f   SocketLayer.obj
 0001:00020680       ?RecvFrom@SocketLayer@@QAEHIPAVRakPeer@@PAH@Z 00421680 f   SocketLayer.obj
 0001:00020750       ?SendTo@SocketLayer@@QAEHIPBDHIG@Z 00421750 f   SocketLayer.obj
 0001:000207f0       ?SendTo@SocketLayer@@QAEHIPBDHQADG@Z 004217f0 f   SocketLayer.obj
 0001:00020820       ?GetMyIP@SocketLayer@@QAEXQAY0BA@D@Z 00421820 f   SocketLayer.obj
 0001:000208a0       ?GetLocalPort@SocketLayer@@QAEGI@Z 004218a0 f   SocketLayer.obj
 0001:000208e0       ?Instance@StringCompressor@@SAPAV1@XZ 004218e0 f   StringCompressor.obj
 0001:000208f0       ??$defaultMapKeyComparison@H@DataStructures@@YAHABH0@Z 004218f0 f i StringCompressor.obj
 0001:00020910       ??0MapNode@?$Map@HPAVHuffmanEncodingTree@@$1??$defaultMapKeyComparison@H@DataStructures@@YAHABH0@Z@DataStructures@@QAE@HPAVHuffmanEncodingTree@@@Z 00421910 f i StringCompressor.obj
 0001:00020930       ?SaveLastSearch@?$Map@HPAVHuffmanEncodingTree@@$1??$defaultMapKeyComparison@H@DataStructures@@YAHABH0@Z@DataStructures@@IAEXABHI@Z 00421930 f i StringCompressor.obj
 0001:00020950       ?HasSavedSearchResult@?$Map@HPAVHuffmanEncodingTree@@$1??$defaultMapKeyComparison@H@DataStructures@@YAHABH0@Z@DataStructures@@IBE_NABH@Z 00421950 f i StringCompressor.obj
 0001:00020970       ?NodeComparisonFunc@?$Map@HPAVHuffmanEncodingTree@@$1??$defaultMapKeyComparison@H@DataStructures@@YAHABH0@Z@DataStructures@@SAHABHABUMapNode@12@@Z 00421970 f i StringCompressor.obj
 0001:00020990       ??0?$List@UMapNode@?$Map@HPAVHuffmanEncodingTree@@$1??$defaultMapKeyComparison@H@DataStructures@@YAHABH0@Z@DataStructures@@@DataStructures@@QAE@XZ 00421990 f i StringCompressor.obj
 0001:000209a0       ??1?$List@UMapNode@?$Map@HPAVHuffmanEncodingTree@@$1??$defaultMapKeyComparison@H@DataStructures@@YAHABH0@Z@DataStructures@@@DataStructures@@QAE@XZ 004219a0 f i StringCompressor.obj
 0001:000209b0       ??A?$List@UMapNode@?$Map@HPAVHuffmanEncodingTree@@$1??$defaultMapKeyComparison@H@DataStructures@@YAHABH0@Z@DataStructures@@@DataStructures@@QBEAAUMapNode@?$Map@HPAVHuffmanEncodingTree@@$1??$defaultMapKeyComparison@H@DataStructures@@YAHABH0@Z@1@I@Z 004219b0 f i StringCompressor.obj
 0001:000209c0       ?Size@?$List@UMapNode@?$Map@HPAVHuffmanEncodingTree@@$1??$defaultMapKeyComparison@H@DataStructures@@YAHABH0@Z@DataStructures@@@DataStructures@@QBEIXZ 004219c0 f i StringCompressor.obj
 0001:000209d0       ??_H@YGXPAXIHP6EPAX0@Z@Z   004219d0 f i StringCompressor.obj
 0001:00020a10       ??0MapNode@?$Map@HPAVHuffmanEncodingTree@@$1??$defaultMapKeyComparison@H@DataStructures@@YAHABH0@Z@DataStructures@@QAE@XZ 00421a10 f i StringCompressor.obj
 0001:00020a20       ?Clear@?$List@UMapNode@?$Map@HPAVHuffmanEncodingTree@@$1??$defaultMapKeyComparison@H@DataStructures@@YAHABH0@Z@DataStructures@@@DataStructures@@QAEX_N@Z 00421a20 f i StringCompressor.obj
 0001:00020a60       ?IMPLEMENT_DEFAULT_COMPARISON@?$Map@HPAVHuffmanEncodingTree@@$1??$defaultMapKeyComparison@H@DataStructures@@YAHABH0@Z@DataStructures@@SAXXZ 00421a60 f i StringCompressor.obj
 0001:00020a70       ??0?$OrderedList@HUMapNode@?$Map@HPAVHuffmanEncodingTree@@$1??$defaultMapKeyComparison@H@DataStructures@@YAHABH0@Z@DataStructures@@$1?NodeComparisonFunc@23@SAHABHABU123@@Z@DataStructures@@QAE@XZ 00421a70 f i StringCompressor.obj
 0001:00020a80       ?GetIndexFromKey@?$OrderedList@HUMapNode@?$Map@HPAVHuffmanEncodingTree@@$1??$defaultMapKeyComparison@H@DataStructures@@YAHABH0@Z@DataStructures@@$1?NodeComparisonFunc@23@SAHABHABU123@@Z@DataStructures@@QBEIABHPA_N@Z 00421a80 f i StringCompressor.obj
 0001:00020af0       ??A?$OrderedList@HUMapNode@?$Map@HPAVHuffmanEncodingTree@@$1??$defaultMapKeyComparison@H@DataStructures@@YAHABH0@Z@DataStructures@@$1?NodeComparisonFunc@23@SAHABHABU123@@Z@DataStructures@@QBEAAUMapNode@?$Map@HPAVHuffmanEncodingTree@@$1??$defaultMapKeyComparison@H@DataStructures@@YAHABH0@Z@1@I@Z 00421af0 f i StringCompressor.obj
 0001:00020b00       ?Size@?$OrderedList@HUMapNode@?$Map@HPAVHuffmanEncodingTree@@$1??$defaultMapKeyComparison@H@DataStructures@@YAHABH0@Z@DataStructures@@$1?NodeComparisonFunc@23@SAHABHABU123@@Z@DataStructures@@QBEIXZ 00421b00 f i StringCompressor.obj
 0001:00020b10       ?Clear@?$OrderedList@HUMapNode@?$Map@HPAVHuffmanEncodingTree@@$1??$defaultMapKeyComparison@H@DataStructures@@YAHABH0@Z@DataStructures@@$1?NodeComparisonFunc@23@SAHABHABU123@@Z@DataStructures@@QAEXXZ 00421b10 f i StringCompressor.obj
 0001:00020b50       ?Insert@?$List@UMapNode@?$Map@HPAVHuffmanEncodingTree@@$1??$defaultMapKeyComparison@H@DataStructures@@YAHABH0@Z@DataStructures@@@DataStructures@@QAEXUMapNode@?$Map@HPAVHuffmanEncodingTree@@$1??$defaultMapKeyComparison@H@DataStructures@@YAHABH0@Z@2@@Z 00421b50 f i StringCompressor.obj
 0001:00020bd0       ?Insert@?$List@UMapNode@?$Map@HPAVHuffmanEncodingTree@@$1??$defaultMapKeyComparison@H@DataStructures@@YAHABH0@Z@DataStructures@@@DataStructures@@QAEXUMapNode@?$Map@HPAVHuffmanEncodingTree@@$1??$defaultMapKeyComparison@H@DataStructures@@YAHABH0@Z@2@I@Z 00421bd0 f i StringCompressor.obj
 0001:00020c70       ?Get@?$Map@HPAVHuffmanEncodingTree@@$1??$defaultMapKeyComparison@H@DataStructures@@YAHABH0@Z@DataStructures@@QAEAAPAVHuffmanEncodingTree@@ABH@Z 00421c70 f i StringCompressor.obj
 0001:00020ce0       ?Has@?$Map@HPAVHuffmanEncodingTree@@$1??$defaultMapKeyComparison@H@DataStructures@@YAHABH0@Z@DataStructures@@QAE_NABH@Z 00421ce0 f i StringCompressor.obj
 0001:00020d30       ??A?$Map@HPAVHuffmanEncodingTree@@$1??$defaultMapKeyComparison@H@DataStructures@@YAHABH0@Z@DataStructures@@QBEAAPAVHuffmanEncodingTree@@I@Z 00421d30 f i StringCompressor.obj
 0001:00020d40       ?Size@?$Map@HPAVHuffmanEncodingTree@@$1??$defaultMapKeyComparison@H@DataStructures@@YAHABH0@Z@DataStructures@@QBEIXZ 00421d40 f i StringCompressor.obj
 0001:00020d50       ?Clear@?$Map@HPAVHuffmanEncodingTree@@$1??$defaultMapKeyComparison@H@DataStructures@@YAHABH0@Z@DataStructures@@QAEXXZ 00421d50 f i StringCompressor.obj
 0001:00020d90       ??1?$OrderedList@HUMapNode@?$Map@HPAVHuffmanEncodingTree@@$1??$defaultMapKeyComparison@H@DataStructures@@YAHABH0@Z@DataStructures@@$1?NodeComparisonFunc@23@SAHABHABU123@@Z@DataStructures@@QAE@XZ 00421d90 f i StringCompressor.obj
 0001:00020e10       ?Insert@?$OrderedList@HUMapNode@?$Map@HPAVHuffmanEncodingTree@@$1??$defaultMapKeyComparison@H@DataStructures@@YAHABH0@Z@DataStructures@@$1?NodeComparisonFunc@23@SAHABHABU123@@Z@DataStructures@@QAEIABHABUMapNode@?$Map@HPAVHuffmanEncodingTree@@$1??$defaultMapKeyComparison@H@DataStructures@@YAHABH0@Z@2@@Z 00421e10 f i StringCompressor.obj
 0001:00020e70       ?EncodeString@StringCompressor@@QAEXPBDHPAVBitStream@RakNet@@H@Z 00421e70 f   StringCompressor.obj
 0001:00020fd0       ?DecodeString@StringCompressor@@QAE_NPADHPAVBitStream@RakNet@@H@Z 00421fd0 f   StringCompressor.obj
 0001:000210a0       ??0?$Map@HPAVHuffmanEncodingTree@@$1??$defaultMapKeyComparison@H@DataStructures@@YAHABH0@Z@DataStructures@@QAE@XZ 004220a0 f i StringCompressor.obj
 0001:000210b0       ??1?$Map@HPAVHuffmanEncodingTree@@$1??$defaultMapKeyComparison@H@DataStructures@@YAHABH0@Z@DataStructures@@QAE@XZ 004220b0 f i StringCompressor.obj
 0001:00021120       ?Set@?$Map@HPAVHuffmanEncodingTree@@$1??$defaultMapKeyComparison@H@DataStructures@@YAHABH0@Z@DataStructures@@QAEXABHABQAVHuffmanEncodingTree@@@Z 00422120 f i StringCompressor.obj
 0001:000211c0       ??0StringCompressor@@AAE@XZ 004221c0 f   StringCompressor.obj
 0001:00021260       ?GenerateTreeFromStrings@StringCompressor@@QAEXPAEIH@Z 00422260 f   StringCompressor.obj
 0001:000213a0       ??1StringCompressor@@QAE@XZ 004223a0 f   StringCompressor.obj
 0001:00021420       ?AddReference@StringCompressor@@SAXXZ 00422420 f   StringCompressor.obj
 0001:00021490       ??_GStringCompressor@@QAEPAXI@Z 00422490 f i StringCompressor.obj
 0001:000214b0       ?RemoveReference@StringCompressor@@SAXXZ 004224b0 f   StringCompressor.obj
 0001:00021510       ?StrAndBoolComp@@YAHABQADABUStrAndBool@@@Z 00422510 f   StringTable.obj
 0001:00021550       ?Instance@StringTable@@SAPAV1@XZ 00422550 f   StringTable.obj
 0001:00021560       ?LogStringNotFound@StringTable@@IAEXPBD@Z 00422560 f   StringTable.obj
 0001:00021570       ??0?$List@UStrAndBool@@@DataStructures@@QAE@XZ 00422570 f i StringTable.obj
 0001:00021580       ??1?$List@UStrAndBool@@@DataStructures@@QAE@XZ 00422580 f i StringTable.obj
 0001:00021590       ??A?$List@UStrAndBool@@@DataStructures@@QBEAAUStrAndBool@@I@Z 00422590 f i StringTable.obj
 0001:000215a0       ?Insert@?$List@UStrAndBool@@@DataStructures@@QAEXUStrAndBool@@@Z 004225a0 f i StringTable.obj
 0001:00021620       ?Insert@?$List@UStrAndBool@@@DataStructures@@QAEXUStrAndBool@@I@Z 00422620 f i StringTable.obj
 0001:000216c0       ?Size@?$List@UStrAndBool@@@DataStructures@@QBEIXZ 004226c0 f i StringTable.obj
 0001:000216d0       ?Clear@?$List@UStrAndBool@@@DataStructures@@QAEX_N@Z 004226d0 f i StringTable.obj
 0001:00021710       ??0?$OrderedList@PADUStrAndBool@@$1?StrAndBoolComp@@YAHABQADABU1@@Z@DataStructures@@QAE@XZ 00422710 f i StringTable.obj
 0001:00021720       ?GetIndexFromKey@?$OrderedList@PADUStrAndBool@@$1?StrAndBoolComp@@YAHABQADABU1@@Z@DataStructures@@QBEIABQADPA_N@Z 00422720 f i StringTable.obj
 0001:00021810       ?Insert@?$OrderedList@PADUStrAndBool@@$1?StrAndBoolComp@@YAHABQADABU1@@Z@DataStructures@@QAEIABQADABUStrAndBool@@@Z 00422810 f i StringTable.obj
 0001:00021870       ??A?$OrderedList@PADUStrAndBool@@$1?StrAndBoolComp@@YAHABQADABU1@@Z@DataStructures@@QBEAAUStrAndBool@@I@Z 00422870 f i StringTable.obj
 0001:00021880       ?Size@?$OrderedList@PADUStrAndBool@@$1?StrAndBoolComp@@YAHABQADABU1@@Z@DataStructures@@QBEIXZ 00422880 f i StringTable.obj
 0001:00021890       ?Clear@?$OrderedList@PADUStrAndBool@@$1?StrAndBoolComp@@YAHABQADABU1@@Z@DataStructures@@QAEXXZ 00422890 f i StringTable.obj
 0001:000218d0       ?AddString@StringTable@@QAEXPBD_N@Z 004228d0 f   StringTable.obj
 0001:00021970       ?EncodeString@StringTable@@QAEXPBDHPAVBitStream@RakNet@@@Z 00422970 f   StringTable.obj
 0001:000219e0       ?DecodeString@StringTable@@QAE_NPADHPAVBitStream@RakNet@@@Z 004229e0 f   StringTable.obj
 0001:00021a90       ??1?$OrderedList@PADUStrAndBool@@$1?StrAndBoolComp@@YAHABQADABU1@@Z@DataStructures@@QAE@XZ 00422a90 f i StringTable.obj
 0001:00021b10       ??0StringTable@@IAE@XZ     00422b10 f   StringTable.obj
 0001:00021b20       ??1StringTable@@QAE@XZ     00422b20 f   StringTable.obj
 0001:00021b90       ?AddReference@StringTable@@SAXXZ 00422b90 f   StringTable.obj
 0001:00021bd0       ??_GStringTable@@QAEPAXI@Z 00422bd0 f i StringTable.obj
 0001:00021bf0       ?RemoveReference@StringTable@@SAXXZ 00422bf0 f   StringTable.obj
 0001:00021c50       ?GetList@SystemAddressList@@QAEPAV?$List@UPlayerID@@@DataStructures@@XZ 00422c50 f   SystemAddressList.obj
 0001:00021c60       ??0?$List@UPlayerID@@@DataStructures@@QAE@XZ 00422c60 f i SystemAddressList.obj
 0001:00021c70       ??1?$List@UPlayerID@@@DataStructures@@QAE@XZ 00422c70 f i SystemAddressList.obj
 0001:00021c80       ??A?$List@UPlayerID@@@DataStructures@@QBEAAUPlayerID@@I@Z 00422c80 f i SystemAddressList.obj
 0001:00021c90       ?Insert@?$List@UPlayerID@@@DataStructures@@QAEXUPlayerID@@@Z 00422c90 f i SystemAddressList.obj
 0001:00021d10       ?Del@?$List@UPlayerID@@@DataStructures@@QAEXI@Z 00422d10 f i SystemAddressList.obj
 0001:00021d20       ?Size@?$List@UPlayerID@@@DataStructures@@QBEIXZ 00422d20 f i SystemAddressList.obj
 0001:00021d30       ?Clear@?$List@UPlayerID@@@DataStructures@@QAEX_N@Z 00422d30 f i SystemAddressList.obj
 0001:00021d70       ??0SystemAddressList@@QAE@XZ 00422d70 f   SystemAddressList.obj
 0001:00021d80       ??0SystemAddressList@@QAE@UPlayerID@@@Z 00422d80 f   SystemAddressList.obj
 0001:00021dd0       ?AddSystem@SystemAddressList@@QAEXUPlayerID@@@Z 00422dd0 f   SystemAddressList.obj
 0001:00021df0       ?RandomizeOrder@SystemAddressList@@QAEXXZ 00422df0 f   SystemAddressList.obj
 0001:00021e60       ?Serialize@SystemAddressList@@QAEXPAVBitStream@RakNet@@@Z 00422e60 f   SystemAddressList.obj
 0001:00021ee0       ?Deserialize@SystemAddressList@@QAE_NPAVBitStream@RakNet@@@Z 00422ee0 f   SystemAddressList.obj
 0001:00021fc0       ?RemoveSystem@SystemAddressList@@QAEXUPlayerID@@@Z 00422fc0 f   SystemAddressList.obj
 0001:00022000       ?Save@SystemAddressList@@QAE_NPBD@Z 00423000 f   SystemAddressList.obj
 0001:000220e0       ?Load@SystemAddressList@@QAE_NPBD@Z 004230e0 f   SystemAddressList.obj
 0001:000221d0       ?Size@SystemAddressList@@QBEIXZ 004231d0 f   SystemAddressList.obj
 0001:000221e0       ??ASystemAddressList@@QBEAAUPlayerID@@I@Z 004231e0 f   SystemAddressList.obj
 0001:000221f0       ?Clear@SystemAddressList@@QAEXXZ 004231f0 f   SystemAddressList.obj
 0001:00022230       ??$Write@H@BitStream@RakNet@@QAEXH@Z 00423230 f i TableSerializer.obj
 0001:00022250       ??$Read@H@BitStream@RakNet@@QAE_NAAH@Z 00423250 f i TableSerializer.obj
 0001:00022270       ?SerializeCell@TableSerializer@@SAXPAVBitStream@RakNet@@PAUCell@Table@DataStructures@@W4ColumnType@56@@Z 00423270 f   TableSerializer.obj
 0001:00022320       ?DeserializeCell@TableSerializer@@SA_NPAVBitStream@RakNet@@PAUCell@Table@DataStructures@@W4ColumnType@56@@Z 00423320 f   TableSerializer.obj
 0001:00022470       ?SerializeRow@TableSerializer@@SAXPAURow@Table@DataStructures@@IAAV?$List@UColumnDescriptor@Table@DataStructures@@@4@PAVBitStream@RakNet@@@Z 00423470 f   TableSerializer.obj
 0001:000224d0       ?DeserializeRow@TableSerializer@@SA_NPAVBitStream@RakNet@@PAVTable@DataStructures@@@Z 004234d0 f   TableSerializer.obj
 0001:00022560       ?SerializeTable@TableSerializer@@SAXPAVTable@DataStructures@@PAVBitStream@RakNet@@@Z 00423560 f   TableSerializer.obj
 0001:00022670       ?DeserializeTable@TableSerializer@@SA_NPAEIPAVTable@DataStructures@@@Z 00423670 f   TableSerializer.obj
 0001:00022800       ?GetChar@@YADD@Z           00423800 f   samp_netencr.obj
 0001:00022810       ?DumpMem@@YAPADPAEH@Z      00423810 f   samp_netencr.obj
 0001:00022ae0       ?kyretardizeDatagram@@YAXPAEHHH@Z 00423ae0 f   samp_netencr.obj
 0001:00022bb0       ??0TiXmlString@@QAE@XZ     00423bb0 f i tinystr.obj
 0001:00022bc0       ?data@TiXmlString@@QBEPBDXZ 00423bc0 f i tinystr.obj
 0001:00022bd0       ?length@TiXmlString@@QBEIXZ 00423bd0 f i tinystr.obj
 0001:00022be0       ?capacity@TiXmlString@@QBEIXZ 00423be0 f i tinystr.obj
 0001:00022bf0       ?swap@TiXmlString@@QAEXAAV1@@Z 00423bf0 f i tinystr.obj
 0001:00022c10       ?set_size@TiXmlString@@AAEXI@Z 00423c10 f i tinystr.obj
 0001:00022c30       ?start@TiXmlString@@ABEPADXZ 00423c30 f i tinystr.obj
 0001:00022c40       ?finish@TiXmlString@@ABEPADXZ 00423c40 f i tinystr.obj
 0001:00022c50       ?init@TiXmlString@@AAEXII@Z 00423c50 f i tinystr.obj
 0001:00022ca0       ?quit@TiXmlString@@AAEXXZ  00423ca0 f i tinystr.obj
 0001:00022cc0       ??1TiXmlString@@QAE@XZ     00423cc0 f i tinystr.obj
 0001:00022ce0       ?init@TiXmlString@@AAEXI@Z 00423ce0 f i tinystr.obj
 0001:00022d30       ?reserve@TiXmlString@@QAEXI@Z 00423d30 f   tinystr.obj
 0001:00022dc0       ?assign@TiXmlString@@QAEAAV1@PBDI@Z 00423dc0 f   tinystr.obj
 0001:00022ea0       ?append@TiXmlString@@QAEAAV1@PBDI@Z 00423ea0 f   tinystr.obj
 0001:00022ef0       ??0TiXmlString@@QAE@ABV0@@Z 00423ef0 f i tinystr.obj
 0001:00022f60       ??YTiXmlString@@QAEAAV0@ABV0@@Z 00423f60 f i tinystr.obj
 0001:00022fb0       ??H@YA?AVTiXmlString@@ABV0@0@Z 00423fb0 f   tinystr.obj
 0001:00023030       ??H@YA?AVTiXmlString@@ABV0@PBD@Z 00424030 f   tinystr.obj
 0001:000230f0       ??H@YA?AVTiXmlString@@PBDABV0@@Z 004240f0 f   tinystr.obj
 0001:000231b0       ??4TiXmlString@@QAEAAV0@PBD@Z 004241b0 f i tinyxml.obj
 0001:000231e0       ??YTiXmlString@@QAEAAV0@PBD@Z 004241e0 f i tinyxml.obj
 0001:00023210       ??YTiXmlString@@QAEAAV0@D@Z 00424210 f i tinyxml.obj
 0001:00023220       ?c_str@TiXmlString@@QBEPBDXZ 00424220 f i tinyxml.obj
 0001:00023230       ?empty@TiXmlString@@QBE_NXZ 00424230 f i tinyxml.obj
 0001:00023240       ??ATiXmlString@@QBEAADI@Z  00424240 f i tinyxml.obj
 0001:00023270       ?find@TiXmlString@@QBEIDI@Z 00424270 f i tinyxml.obj
 0001:000232b0       ?Clear@TiXmlCursor@@QAEXXZ 004242b0 f i tinyxml.obj
 0001:000232c0       ??1TiXmlBase@@UAE@XZ       004242c0 f i tinyxml.obj
 0001:000232d0       ??_GTiXmlBase@@UAEPAXI@Z   004242d0 f i tinyxml.obj
 0001:000232d0       ??_ETiXmlBase@@UAEPAXI@Z   004242d0 f i tinyxml.obj
 0001:000232f0       ?Value@TiXmlNode@@QBEPBDXZ 004242f0 f i tinyxml.obj
 0001:00023300       ?ValueTStr@TiXmlNode@@QBEABVTiXmlString@@XZ 00424300 f i tinyxml.obj
 0001:00023310       ?SetValue@TiXmlNode@@QAEXPBD@Z 00424310 f i tinyxml.obj
 0001:00023340       ?FirstChild@TiXmlNode@@QBEPBV1@XZ 00424340 f i tinyxml.obj
 0001:00023350       ?FirstChild@TiXmlNode@@QAEPAV1@XZ 00424350 f i tinyxml.obj
 0001:00023360       ?LastChild@TiXmlNode@@QBEPBV1@XZ 00424360 f i tinyxml.obj
 0001:00023370       ?NextSibling@TiXmlNode@@QBEPBV1@XZ 00424370 f i tinyxml.obj
 0001:00023380       ?NextSibling@TiXmlNode@@QAEPAV1@XZ 00424380 f i tinyxml.obj
 0001:00023390       ?Type@TiXmlNode@@QBEHXZ    00424390 f i tinyxml.obj
 0001:000233a0       ?Name@TiXmlAttribute@@QBEPBDXZ 004243a0 f i tinyxml.obj
 0001:000233b0       ?Value@TiXmlAttribute@@QBEPBDXZ 004243b0 f i tinyxml.obj
 0001:000233c0       ?SetName@TiXmlAttribute@@QAEXPBD@Z 004243c0 f i tinyxml.obj
 0001:000233f0       ?SetValue@TiXmlAttribute@@QAEXPBD@Z 004243f0 f i tinyxml.obj
 0001:00023420       ?First@TiXmlAttributeSet@@QBEPBVTiXmlAttribute@@XZ 00424420 f i tinyxml.obj
 0001:00023430       ?First@TiXmlAttributeSet@@QAEPAVTiXmlAttribute@@XZ 00424430 f i tinyxml.obj
 0001:00023440       ?CDATA@TiXmlText@@QBE_NXZ  00424440 f i tinyxml.obj
 0001:00023450       ?Error@TiXmlDocument@@QBE_NXZ 00424450 f i tinyxml.obj
 0001:00023460       ?ClearError@TiXmlDocument@@QAEXXZ 00424460 f i tinyxml.obj
 0001:00023490       ??0TiXmlHandle@@QAE@PAVTiXmlNode@@@Z 00424490 f i tinyxml.obj
 0001:000234a0       ?TiXmlFOpen@@YAPAU_iobuf@@PBD0@Z 004244a0 f   tinyxml.obj
 0001:000234d0       ?CopyTo@TiXmlNode@@IBEXPAV1@@Z 004244d0 f   tinyxml.obj
 0001:00023510       ?Clear@TiXmlNode@@QAEXXZ   00424510 f   tinyxml.obj
 0001:00023540       ?RemoveChild@TiXmlNode@@QAE_NPAV1@@Z 00424540 f   tinyxml.obj
 0001:000235c0       ?FirstChild@TiXmlNode@@QBEPBV1@PBD@Z 004245c0 f   tinyxml.obj
 0001:00023610       ?LastChild@TiXmlNode@@QBEPBV1@PBD@Z 00424610 f   tinyxml.obj
 0001:00023660       ?IterateChildren@TiXmlNode@@QBEPBV1@PBV1@@Z 00424660 f   tinyxml.obj
 0001:000236a0       ?NextSibling@TiXmlNode@@QBEPBV1@PBD@Z 004246a0 f   tinyxml.obj
 0001:000236f0       ?PreviousSibling@TiXmlNode@@QBEPBV1@PBD@Z 004246f0 f   tinyxml.obj
 0001:00023740       ?FirstChildElement@TiXmlNode@@QBEPBVTiXmlElement@@XZ 00424740 f   tinyxml.obj
 0001:00023770       ?FirstChildElement@TiXmlNode@@QBEPBVTiXmlElement@@PBD@Z 00424770 f   tinyxml.obj
 0001:000237b0       ?NextSiblingElement@TiXmlNode@@QBEPBVTiXmlElement@@XZ 004247b0 f   tinyxml.obj
 0001:000237e0       ?NextSiblingElement@TiXmlNode@@QBEPBVTiXmlElement@@PBD@Z 004247e0 f   tinyxml.obj
 0001:00023820       ?GetDocument@TiXmlNode@@QBEPBVTiXmlDocument@@XZ 00424820 f   tinyxml.obj
 0001:00023850       ?Accept@TiXmlElement@@UBE_NPAVTiXmlVisitor@@@Z 00424850 f   tinyxml.obj
 0001:000238b0       ?GetText@TiXmlElement@@QBEPBDXZ 004248b0 f   tinyxml.obj
 0001:000238d0       ?LoadFile@TiXmlDocument@@QAE_NPAU_iobuf@@W4TiXmlEncoding@@@Z 004248d0 f   tinyxml.obj
 0001:00023a70       ?SaveFile@TiXmlDocument@@QBE_NPAU_iobuf@@@Z 00424a70 f   tinyxml.obj
 0001:00023ad0       ?Print@TiXmlDocument@@UBEXPAU_iobuf@@H@Z 00424ad0 f   tinyxml.obj
 0001:00023b30       ?Accept@TiXmlDocument@@UBE_NPAVTiXmlVisitor@@@Z 00424b30 f   tinyxml.obj
 0001:00023b80       ?Next@TiXmlAttribute@@QBEPBV1@XZ 00424b80 f   tinyxml.obj
 0001:00023ba0       ?Previous@TiXmlAttribute@@QBEPBV1@XZ 00424ba0 f   tinyxml.obj
 0001:00023bc0       ?QueryIntValue@TiXmlAttribute@@QBEHPAH@Z 00424bc0 f   tinyxml.obj
 0001:00023bf0       ?QueryDoubleValue@TiXmlAttribute@@QBEHPAN@Z 00424bf0 f   tinyxml.obj
 0001:00023c20       ?QueryVectorValue@TiXmlAttribute@@QBEHPAM@Z 00424c20 f   tinyxml.obj
 0001:00023c50       ?QueryPointerValue@TiXmlAttribute@@QBEHPAX@Z 00424c50 f   tinyxml.obj
 0001:00023ca0       ?QueryColorValue@TiXmlAttribute@@QBEHPAE00@Z 00424ca0 f   tinyxml.obj
 0001:00023cd0       ?IntValue@TiXmlAttribute@@QBEHXZ 00424cd0 f   tinyxml.obj
 0001:00023ce0       ?DoubleValue@TiXmlAttribute@@QBENXZ 00424ce0 f   tinyxml.obj
 0001:00023cf0       ?Print@TiXmlComment@@UBEXPAU_iobuf@@H@Z 00424cf0 f   tinyxml.obj
 0001:00023d50       ?CopyTo@TiXmlComment@@IBEXPAV1@@Z 00424d50 f   tinyxml.obj
 0001:00023d90       ?Accept@TiXmlComment@@UBE_NPAVTiXmlVisitor@@@Z 00424d90 f   tinyxml.obj
 0001:00023db0       ?CopyTo@TiXmlText@@IBEXPAV1@@Z 00424db0 f   tinyxml.obj
 0001:00023e00       ?Accept@TiXmlText@@UBE_NPAVTiXmlVisitor@@@Z 00424e00 f   tinyxml.obj
 0001:00023e20       ?Accept@TiXmlDeclaration@@UBE_NPAVTiXmlVisitor@@@Z 00424e20 f   tinyxml.obj
 0001:00023e40       ?Print@TiXmlUnknown@@UBEXPAU_iobuf@@H@Z 00424e40 f   tinyxml.obj
 0001:00023e80       ?CopyTo@TiXmlUnknown@@IBEXPAV1@@Z 00424e80 f   tinyxml.obj
 0001:00023ec0       ?Accept@TiXmlUnknown@@UBE_NPAVTiXmlVisitor@@@Z 00424ec0 f   tinyxml.obj
 0001:00023ee0       ?Remove@TiXmlAttributeSet@@QAEXPAVTiXmlAttribute@@@Z 00424ee0 f   tinyxml.obj
 0001:00023f40       ?Find@TiXmlAttributeSet@@QBEPAVTiXmlAttribute@@PBD@Z 00424f40 f   tinyxml.obj
 0001:00023f90       ?FirstChild@TiXmlHandle@@QBE?AV1@XZ 00424f90 f   tinyxml.obj
 0001:00023fc0       ?Child@TiXmlHandle@@QBE?AV1@H@Z 00424fc0 f   tinyxml.obj
 0001:00024000       ?VisitEnter@TiXmlPrinter@@UAE_NABVTiXmlDocument@@@Z 00425000 f   tinyxml.obj
 0001:00024010       ?VisitExit@TiXmlPrinter@@UAE_NABVTiXmlDocument@@@Z 00425010 f   tinyxml.obj
 0001:00024020       ??$_snprintf_s@$0CA@@@YAHAAY0CA@DIPBDZZ 00425020 f i tinyxml.obj
 0001:00024040       ??$_snprintf_s@$0EA@@@YAHAAY0EA@DIPBDZZ 00425040 f i tinyxml.obj
 0001:00024060       ??$_snprintf_s@$0BAA@@@YAHAAY0BAA@DIPBDZZ 00425060 f i tinyxml.obj
 0001:00024090       ??4TiXmlString@@QAEAAV0@ABV0@@Z 00425090 f i tinyxml.obj
 0001:000240b0       ?find@TiXmlString@@QBEID@Z 004250b0 f i tinyxml.obj
 0001:000240f0       ??0TiXmlCursor@@QAE@XZ     004250f0 f i tinyxml.obj
 0001:00024100       ??0TiXmlBase@@QAE@XZ       00425100 f i tinyxml.obj
 0001:00024120       ?FirstChild@TiXmlNode@@QAEPAV1@PBD@Z 00425120 f i tinyxml.obj
 0001:00024130       ?NextSibling@TiXmlNode@@QAEPAV1@PBD@Z 00425130 f i tinyxml.obj
 0001:00024140       ?NextSiblingElement@TiXmlNode@@QAEPAVTiXmlElement@@XZ 00425140 f i tinyxml.obj
 0001:00024170       ?NextSiblingElement@TiXmlNode@@QAEPAVTiXmlElement@@PBD@Z 00425170 f i tinyxml.obj
 0001:00024180       ?FirstChildElement@TiXmlNode@@QAEPAVTiXmlElement@@XZ 00425180 f i tinyxml.obj
 0001:000241b0       ?FirstChildElement@TiXmlNode@@QAEPAVTiXmlElement@@PBD@Z 004251b0 f i tinyxml.obj
 0001:000241c0       ?GetDocument@TiXmlNode@@QAEPAVTiXmlDocument@@XZ 004251c0 f i tinyxml.obj
 0001:000241f0       ??0TiXmlAttribute@@QAE@XZ  004251f0 f i tinyxml.obj
 0001:00024220       ??1TiXmlAttribute@@UAE@XZ  00425220 f i tinyxml.obj
 0001:00024290       ?DoIndent@TiXmlPrinter@@AAEXXZ 00425290 f i tinyxml.obj
 0001:000242c0       ?DoLineBreak@TiXmlPrinter@@AAEXXZ 004252c0 f i tinyxml.obj
 0001:000242e0       ?EncodeString@TiXmlBase@@SAXABVTiXmlString@@PAV2@@Z 004252e0 f   tinyxml.obj
 0001:00024490       ??0TiXmlNode@@IAE@W4NodeType@0@@Z 00425490 f   tinyxml.obj
 0001:000244d0       ?ToDocument@TiXmlNode@@UBEPBVTiXmlDocument@@XZ 004254d0 f i tinyxml.obj
 0001:000244e0       ?ToElement@TiXmlNode@@UBEPBVTiXmlElement@@XZ 004254e0 f i tinyxml.obj
 0001:000244f0       ?ToComment@TiXmlNode@@UBEPBVTiXmlComment@@XZ 004254f0 f i tinyxml.obj
 0001:00024500       ?ToUnknown@TiXmlNode@@UBEPBVTiXmlUnknown@@XZ 00425500 f i tinyxml.obj
 0001:00024510       ?ToText@TiXmlNode@@UBEPBVTiXmlText@@XZ 00425510 f i tinyxml.obj
 0001:00024520       ?ToDeclaration@TiXmlNode@@UBEPBVTiXmlDeclaration@@XZ 00425520 f i tinyxml.obj
 0001:00024530       ?ToDocument@TiXmlNode@@UAEPAVTiXmlDocument@@XZ 00425530 f i tinyxml.obj
 0001:00024540       ?ToElement@TiXmlNode@@UAEPAVTiXmlElement@@XZ 00425540 f i tinyxml.obj
 0001:00024550       ?ToComment@TiXmlNode@@UAEPAVTiXmlComment@@XZ 00425550 f i tinyxml.obj
 0001:00024560       ?ToUnknown@TiXmlNode@@UAEPAVTiXmlUnknown@@XZ 00425560 f i tinyxml.obj
 0001:00024570       ?ToText@TiXmlNode@@UAEPAVTiXmlText@@XZ 00425570 f i tinyxml.obj
 0001:00024580       ?ToDeclaration@TiXmlNode@@UAEPAVTiXmlDeclaration@@XZ 00425580 f i tinyxml.obj
 0001:00024590       ??1TiXmlNode@@UAE@XZ       00425590 f   tinyxml.obj
 0001:00024610       ?LinkEndChild@TiXmlNode@@QAEPAV1@PAV1@@Z 00425610 f   tinyxml.obj
 0001:00024760       ?InsertEndChild@TiXmlNode@@QAEPAV1@ABV1@@Z 00425760 f   tinyxml.obj
 0001:000247e0       ?InsertBeforeChild@TiXmlNode@@QAEPAV1@PAV1@ABV1@@Z 004257e0 f   tinyxml.obj
 0001:00024890       ?InsertAfterChild@TiXmlNode@@QAEPAV1@PAV1@ABV1@@Z 00425890 f   tinyxml.obj
 0001:00024940       ?ReplaceChild@TiXmlNode@@QAEPAV1@PAV1@ABV1@@Z 00425940 f   tinyxml.obj
 0001:000249e0       ?IterateChildren@TiXmlNode@@QBEPBV1@PBDPBV1@@Z 004259e0 f   tinyxml.obj
 0001:00024a30       ?RemoveAttribute@TiXmlElement@@QAEXPBD@Z 00425a30 f   tinyxml.obj
 0001:00024a60       ?ClearThis@TiXmlElement@@IAEXXZ 00425a60 f   tinyxml.obj
 0001:00024b00       ?Attribute@TiXmlElement@@QBEPBDPBD@Z 00425b00 f   tinyxml.obj
 0001:00024b20       ?Attribute@TiXmlElement@@QBEPBDPBDPAH@Z 00425b20 f   tinyxml.obj
 0001:00024b60       ?Attribute@TiXmlElement@@QBEPBDPBDPAN@Z 00425b60 f   tinyxml.obj
 0001:00024ba0       ?QueryIntAttribute@TiXmlElement@@QBEHPBDPAH@Z 00425ba0 f   tinyxml.obj
 0001:00024be0       ?QueryDoubleAttribute@TiXmlElement@@QBEHPBDPAN@Z 00425be0 f   tinyxml.obj
 0001:00024c20       ?QueryVectorAttribute@TiXmlElement@@QBEHPBDPAM@Z 00425c20 f   tinyxml.obj
 0001:00024c70       ?QueryPointerAttribute@TiXmlElement@@QBEHPBDPAX@Z 00425c70 f   tinyxml.obj
 0001:00024ca0       ?QueryColorAttribute@TiXmlElement@@QBEHPBDPAE11@Z 00425ca0 f   tinyxml.obj
 0001:00024cf0       ?Print@TiXmlElement@@UBEXPAU_iobuf@@H@Z 00425cf0 f   tinyxml.obj
 0001:00024e80       ??0TiXmlDocument@@QAE@XZ   00425e80 f   tinyxml.obj
 0001:00024f20       ?ToDocument@TiXmlDocument@@UBEPBV1@XZ 00425f20 f i tinyxml.obj
 0001:00024f30       ?ToDocument@TiXmlDocument@@UAEPAV1@XZ 00425f30 f i tinyxml.obj
 0001:00024f40       ??0TiXmlDocument@@QAE@PBD@Z 00425f40 f   tinyxml.obj
 0001:00025010       ?SaveFile@TiXmlDocument@@QBE_NPBD@Z 00426010 f   tinyxml.obj
 0001:00025070       ?CopyTo@TiXmlDocument@@ABEXPAV1@@Z 00426070 f   tinyxml.obj
 0001:00025110       ?Clone@TiXmlDocument@@MBEPAVTiXmlNode@@XZ 00426110 f   tinyxml.obj
 0001:00025190       ?Print@TiXmlAttribute@@QBEXPAU_iobuf@@HPAVTiXmlString@@@Z 00426190 f   tinyxml.obj
 0001:00025340       ?SetIntValue@TiXmlAttribute@@QAEXH@Z 00426340 f   tinyxml.obj
 0001:00025390       ?SetDoubleValue@TiXmlAttribute@@QAEXN@Z 00426390 f   tinyxml.obj
 0001:000253f0       ??0TiXmlComment@@QAE@ABV0@@Z 004263f0 f   tinyxml.obj
 0001:000254a0       ?ToComment@TiXmlComment@@UBEPBV1@XZ 004264a0 f i tinyxml.obj
 0001:000254b0       ?ToComment@TiXmlComment@@UAEPAV1@XZ 004264b0 f i tinyxml.obj
 0001:000254c0       ??4TiXmlComment@@QAEXABV0@@Z 004264c0 f   tinyxml.obj
 0001:00025530       ?Print@TiXmlText@@UBEXPAU_iobuf@@H@Z 00426530 f   tinyxml.obj
 0001:00025630       ??0TiXmlDeclaration@@QAE@PBD00@Z 00426630 f   tinyxml.obj
 0001:00025720       ?Print@TiXmlDeclaration@@UBEXPAU_iobuf@@H@Z 00426720 f i tinyxml.obj
 0001:00025740       ?ToDeclaration@TiXmlDeclaration@@UBEPBV1@XZ 00426740 f i tinyxml.obj
 0001:00025750       ?ToDeclaration@TiXmlDeclaration@@UAEPAV1@XZ 00426750 f i tinyxml.obj
 0001:00025760       ?Print@TiXmlDeclaration@@UBEXPAU_iobuf@@HPAVTiXmlString@@@Z 00426760 f   tinyxml.obj
 0001:000258b0       ?CopyTo@TiXmlDeclaration@@IBEXPAV1@@Z 004268b0 f   tinyxml.obj
 0001:00025930       ??0TiXmlAttributeSet@@QAE@XZ 00426930 f   tinyxml.obj
 0001:00025960       ??1TiXmlAttributeSet@@QAE@XZ 00426960 f   tinyxml.obj
 0001:000259b0       ?Add@TiXmlAttributeSet@@QAEXPAVTiXmlAttribute@@@Z 004269b0 f   tinyxml.obj
 0001:00025a00       ?FindOrCreate@TiXmlAttributeSet@@QAEPAVTiXmlAttribute@@PBD@Z 00426a00 f   tinyxml.obj
 0001:00025a80       ?FirstChild@TiXmlHandle@@QBE?AV1@PBD@Z 00426a80 f   tinyxml.obj
 0001:00025ab0       ?FirstChildElement@TiXmlHandle@@QBE?AV1@XZ 00426ab0 f   tinyxml.obj
 0001:00025b00       ?FirstChildElement@TiXmlHandle@@QBE?AV1@PBD@Z 00426b00 f   tinyxml.obj
 0001:00025b30       ?Child@TiXmlHandle@@QBE?AV1@PBDH@Z 00426b30 f   tinyxml.obj
 0001:00025b90       ?ChildElement@TiXmlHandle@@QBE?AV1@H@Z 00426b90 f   tinyxml.obj
 0001:00025c30       ?ChildElement@TiXmlHandle@@QBE?AV1@PBDH@Z 00426c30 f   tinyxml.obj
 0001:00025c90       ?VisitEnter@TiXmlPrinter@@UAE_NABVTiXmlElement@@PBVTiXmlAttribute@@@Z 00426c90 f   tinyxml.obj
 0001:00025dc0       ?VisitExit@TiXmlPrinter@@UAE_NABVTiXmlElement@@@Z 00426dc0 f   tinyxml.obj
 0001:00025e40       ?Visit@TiXmlPrinter@@UAE_NABVTiXmlText@@@Z 00426e40 f   tinyxml.obj
 0001:00025fa0       ?Visit@TiXmlPrinter@@UAE_NABVTiXmlDeclaration@@@Z 00426fa0 f   tinyxml.obj
 0001:00026000       ?Visit@TiXmlPrinter@@UAE_NABVTiXmlComment@@@Z 00427000 f   tinyxml.obj
 0001:00026080       ?Visit@TiXmlPrinter@@UAE_NABVTiXmlUnknown@@@Z 00427080 f   tinyxml.obj
 0001:00026100       ??0TiXmlString@@QAE@PBD@Z  00427100 f i tinyxml.obj
 0001:00026180       ?Print@TiXmlAttribute@@UBEXPAU_iobuf@@H@Z 00427180 f i tinyxml.obj
 0001:000261a0       ??_GTiXmlAttribute@@UAEPAXI@Z 004271a0 f i tinyxml.obj
 0001:000261a0       ??_ETiXmlAttribute@@UAEPAXI@Z 004271a0 f i tinyxml.obj
 0001:000261c0       ??0TiXmlComment@@QAE@XZ    004271c0 f i tinyxml.obj
 0001:00026200       ??1TiXmlComment@@UAE@XZ    00427200 f i tinyxml.obj
 0001:00026210       ??_GTiXmlComment@@UAEPAXI@Z 00427210 f i tinyxml.obj
 0001:00026210       ??_ETiXmlComment@@UAEPAXI@Z 00427210 f i tinyxml.obj
 0001:00026240       ??0TiXmlText@@QAE@PBD@Z    00427240 f i tinyxml.obj
 0001:000262d0       ?ToText@TiXmlText@@UBEPBV1@XZ 004272d0 f i tinyxml.obj
 0001:000262e0       ?ToText@TiXmlText@@UAEPAV1@XZ 004272e0 f i tinyxml.obj
 0001:000262f0       ??1TiXmlText@@UAE@XZ       004272f0 f i tinyxml.obj
 0001:00026300       ??_GTiXmlText@@UAEPAXI@Z   00427300 f i tinyxml.obj
 0001:00026300       ??_ETiXmlText@@UAEPAXI@Z   00427300 f i tinyxml.obj
 0001:00026330       ??0TiXmlDeclaration@@QAE@XZ 00427330 f i tinyxml.obj
 0001:00026370       ??1TiXmlDeclaration@@UAE@XZ 00427370 f i tinyxml.obj
 0001:00026400       ??_ETiXmlDeclaration@@UAEPAXI@Z 00427400 f i tinyxml.obj
 0001:00026400       ??_GTiXmlDeclaration@@UAEPAXI@Z 00427400 f i tinyxml.obj
 0001:00026420       ??0TiXmlUnknown@@QAE@XZ    00427420 f i tinyxml.obj
 0001:00026460       ?ToUnknown@TiXmlUnknown@@UBEPBV1@XZ 00427460 f i tinyxml.obj
 0001:00026470       ?ToUnknown@TiXmlUnknown@@UAEPAV1@XZ 00427470 f i tinyxml.obj
 0001:00026480       ??1TiXmlUnknown@@UAE@XZ    00427480 f i tinyxml.obj
 0001:00026490       ??_GTiXmlUnknown@@UAEPAXI@Z 00427490 f i tinyxml.obj
 0001:00026490       ??_ETiXmlUnknown@@UAEPAXI@Z 00427490 f i tinyxml.obj
 0001:000264c0       ??1TiXmlDocument@@UAE@XZ   004274c0 f i tinyxml.obj
 0001:00026520       ??_GTiXmlDocument@@UAEPAXI@Z 00427520 f i tinyxml.obj
 0001:00026520       ??_ETiXmlDocument@@UAEPAXI@Z 00427520 f i tinyxml.obj
 0001:00026540       ??_GTiXmlNode@@UAEPAXI@Z   00427540 f i tinyxml.obj
 0001:00026540       ??_ETiXmlNode@@UAEPAXI@Z   00427540 f i tinyxml.obj
 0001:00026560       ??0TiXmlElement@@QAE@PBD@Z 00427560 f   tinyxml.obj
 0001:00026610       ?ToElement@TiXmlElement@@UBEPBV1@XZ 00427610 f i tinyxml.obj
 0001:00026620       ?ToElement@TiXmlElement@@UAEPAV1@XZ 00427620 f i tinyxml.obj
 0001:00026630       ??1TiXmlElement@@UAE@XZ    00427630 f   tinyxml.obj
 0001:000266d0       ?SetAttribute@TiXmlElement@@QAEXPBDH@Z 004276d0 f   tinyxml.obj
 0001:00026730       ?SetDoubleAttribute@TiXmlElement@@QAEXPBDN@Z 00427730 f   tinyxml.obj
 0001:00026760       ?SetAttribute@TiXmlElement@@QAEXPBD0@Z 00427760 f   tinyxml.obj
 0001:000267a0       ?CopyTo@TiXmlElement@@IBEXPAV1@@Z 004277a0 f   tinyxml.obj
 0001:00026870       ?Clone@TiXmlElement@@UBEPAVTiXmlNode@@XZ 00427870 f   tinyxml.obj
 0001:00026900       ??0TiXmlDocument@@QAE@ABV0@@Z 00427900 f   tinyxml.obj
 0001:00026980       ??4TiXmlDocument@@QAEXABV0@@Z 00427980 f   tinyxml.obj
 0001:000269c0       ?SaveFile@TiXmlDocument@@QBE_NXZ 004279c0 f   tinyxml.obj
 0001:000269d0       ?LoadFile@TiXmlDocument@@QAE_NPBDW4TiXmlEncoding@@@Z 004279d0 f   tinyxml.obj
 0001:00026ad0       ?Clone@TiXmlComment@@UBEPAVTiXmlNode@@XZ 00427ad0 f   tinyxml.obj
 0001:00026b70       ?Clone@TiXmlText@@MBEPAVTiXmlNode@@XZ 00427b70 f   tinyxml.obj
 0001:00026c20       ??0TiXmlDeclaration@@QAE@ABV0@@Z 00427c20 f   tinyxml.obj
 0001:00026ca0       ??4TiXmlDeclaration@@QAEXABV0@@Z 00427ca0 f   tinyxml.obj
 0001:00026ce0       ?Clone@TiXmlDeclaration@@UBEPAVTiXmlNode@@XZ 00427ce0 f   tinyxml.obj
 0001:00026d50       ?Clone@TiXmlUnknown@@UBEPAVTiXmlNode@@XZ 00427d50 f   tinyxml.obj
 0001:00026df0       ??_ETiXmlElement@@UAEPAXI@Z 00427df0 f i tinyxml.obj
 0001:00026df0       ??_GTiXmlElement@@UAEPAXI@Z 00427df0 f i tinyxml.obj
 0001:00026e10       ??0TiXmlElement@@QAE@ABV0@@Z 00427e10 f   tinyxml.obj
 0001:00026eb0       ??4TiXmlElement@@QAEXABV0@@Z 00427eb0 f   tinyxml.obj
 0001:00026ed0       ?LoadFile@TiXmlDocument@@QAE_NW4TiXmlEncoding@@@Z 00427ed0 f   tinyxml.obj
 0001:00026ef0       ?IsWhiteSpaceCondensed@TiXmlBase@@SA_NXZ 00427ef0 f i tinyxmlparser.obj
 0001:00026f00       ?IsWhiteSpace@TiXmlBase@@KA_ND@Z 00427f00 f i tinyxmlparser.obj
 0001:00026f30       ?ToLower@TiXmlBase@@KAHHW4TiXmlEncoding@@@Z 00427f30 f i tinyxmlparser.obj
 0001:00026f50       ?SetDocument@TiXmlAttribute@@QAEXPAVTiXmlDocument@@@Z 00427f50 f i tinyxmlparser.obj
 0001:00026f60       ?SetCDATA@TiXmlText@@QAEX_N@Z 00427f60 f i tinyxmlparser.obj
 0001:00026f70       ?Encoding@TiXmlDeclaration@@QBEPBDXZ 00427f70 f i tinyxmlparser.obj
 0001:00026f80       ?TabSize@TiXmlDocument@@QBEHXZ 00427f80 f i tinyxmlparser.obj
 0001:00026f90       ?ConvertUTF32ToUTF8@TiXmlBase@@KAXKPADPAH@Z 00427f90 f   tinyxmlparser.obj
 0001:00027090       ?IsAlpha@TiXmlBase@@KAHEW4TiXmlEncoding@@@Z 00428090 f   tinyxmlparser.obj
 0001:000270b0       ?IsAlphaNum@TiXmlBase@@KAHEW4TiXmlEncoding@@@Z 004280b0 f   tinyxmlparser.obj
 0001:000270d0       ?Cursor@TiXmlParsingData@@QAEABUTiXmlCursor@@XZ 004280d0 f i tinyxmlparser.obj
 0001:000270e0       ?Stamp@TiXmlParsingData@@QAEXPBDW4TiXmlEncoding@@@Z 004280e0 f   tinyxmlparser.obj
 0001:00027380       ?SkipWhiteSpace@TiXmlBase@@KAPBDPBDW4TiXmlEncoding@@@Z 00428380 f   tinyxmlparser.obj
 0001:00027430       ?ReadName@TiXmlBase@@KAPBDPBDPAVTiXmlString@@W4TiXmlEncoding@@@Z 00428430 f   tinyxmlparser.obj
 0001:000274e0       ?StringEqual@TiXmlBase@@KA_NPBD0_NW4TiXmlEncoding@@@Z 004284e0 f   tinyxmlparser.obj
 0001:000275c0       ?SetError@TiXmlDocument@@QAEXHPBDPAVTiXmlParsingData@@W4TiXmlEncoding@@@Z 004285c0 f   tinyxmlparser.obj
 0001:00027650       ?Parse@TiXmlUnknown@@UAEPBDPBDPAVTiXmlParsingData@@W4TiXmlEncoding@@@Z 00428650 f   tinyxmlparser.obj
 0001:000277a0       ?Parse@TiXmlComment@@UAEPBDPBDPAVTiXmlParsingData@@W4TiXmlEncoding@@@Z 004287a0 f   tinyxmlparser.obj
 0001:00027900       ?Blank@TiXmlText@@IBE_NXZ  00428900 f   tinyxmlparser.obj
 0001:00027970       ??0TiXmlParsingData@@AAE@PBDHHH@Z 00428970 f i tinyxmlparser.obj
 0001:000279c0       ?GetEntity@TiXmlBase@@KAPBDPBDPADPAHW4TiXmlEncoding@@@Z 004289c0 f   tinyxmlparser.obj
 0001:00027c10       ?Identify@TiXmlNode@@IAEPAV1@PBDW4TiXmlEncoding@@@Z 00428c10 f   tinyxmlparser.obj
 0001:00027e10       ?ReadValue@TiXmlElement@@IAEPBDPBDPAVTiXmlParsingData@@W4TiXmlEncoding@@@Z 00428e10 f   tinyxmlparser.obj
 0001:00027fb0       ?GetChar@TiXmlBase@@KAPBDPBDPADPAHW4TiXmlEncoding@@@Z 00428fb0 f i tinyxmlparser.obj
 0001:00028080       ?ReadText@TiXmlBase@@KAPBDPBDPAVTiXmlString@@_N02W4TiXmlEncoding@@@Z 00429080 f   tinyxmlparser.obj
 0001:00028250       ?Parse@TiXmlDocument@@UAEPBDPBDPAVTiXmlParsingData@@W4TiXmlEncoding@@@Z 00429250 f   tinyxmlparser.obj
 0001:00028490       ?Parse@TiXmlElement@@UAEPBDPBDPAVTiXmlParsingData@@W4TiXmlEncoding@@@Z 00429490 f   tinyxmlparser.obj
 0001:00028840       ?Parse@TiXmlAttribute@@UAEPBDPBDPAVTiXmlParsingData@@W4TiXmlEncoding@@@Z 00429840 f   tinyxmlparser.obj
 0001:000289d0       ?Parse@TiXmlText@@UAEPBDPBDPAVTiXmlParsingData@@W4TiXmlEncoding@@@Z 004299d0 f   tinyxmlparser.obj
 0001:00028bd0       ?Parse@TiXmlDeclaration@@UAEPBDPBDPAVTiXmlParsingData@@W4TiXmlEncoding@@@Z 00429bd0 f   tinyxmlparser.obj
 0001:00028f70       ?RunCommand@@YAHPADH@Z     00429f70 f   cmds.obj
 0001:00029af0       ?sync_with_stdio@ios_base@std@@SA_N_N@Z 0042aaf0 f i console.obj
 0001:00029b20       ?inputThread@@YGKPAX@Z     0042ab20 f   console.obj
 0001:00029b90       ?CtrlHandler@@YAHK@Z       0042ab90 f   console.obj
 0001:00029bd0       ?SetUpConsole@@YAXXZ       0042abd0 f   console.obj
 0001:00029d00       ??$Write@K@BitStream@RakNet@@QAEXK@Z 0042ad00 f i localplayer.obj
 0001:00029d20       ?SendInCarFullSyncData@@YAXPAU_INCAR_SYNC_DATA@@HG@Z 0042ad20 f   localplayer.obj
 0001:00029f80       ?SendPassengerFullSyncData@@YAXG@Z 0042af80 f   localplayer.obj
 0001:0002a0b0       ?SendAimSyncData@@YAXPAU_AIM_SYNC_DATA@@KHG@Z 0042b0b0 f   localplayer.obj
 0001:0002a240       ?SendUnoccupiedSyncData@@YAXPAU_UNOCCUPIED_SYNC_DATA@@@Z 0042b240 f   localplayer.obj
 0001:0002a310       ?SendSpectatorData@@YAXPAU_SPECTATOR_SYNC_DATA@@@Z 0042b310 f   localplayer.obj
 0001:0002a3b0       ?SendEnterVehicleNotification@@YAXGH@Z 0042b3b0 f   localplayer.obj
 0001:0002a480       ?SendExitVehicleNotification@@YAXG@Z 0042b480 f   localplayer.obj
 0001:0002a530       ?SendWastedNotification@@YAXEG@Z 0042b530 f   localplayer.obj
 0001:0002a5f0       ?NotifyVehicleDeath@@YAXG@Z 0042b5f0 f   localplayer.obj
 0001:0002a6a0       ?SendDamageVehicle@@YAXGKKEE@Z 0042b6a0 f   localplayer.obj
 0001:0002a7c0       ?SendOnFootFullSyncData@@YAXPAU_ONFOOT_SYNC_DATA@@HG@Z 0042b7c0 f   localplayer.obj
 0001:0002a9d0       ?Log@@YAXPADZZ             0042b9d0 f   main.obj
 0001:0002ab80       ?gen_random@@YAXPADH@Z     0042bb80 f   main.obj
 0001:0002abd0       _WinMain@16                0042bbd0 f   main.obj
 0001:0002b130       _fabsf                     0042c130 f i math_stuff.obj
 0001:0002b140       _cosf                      0042c140 f i math_stuff.obj
 0001:0002b160       _floorf                    0042c160 f i math_stuff.obj
 0001:0002b180       _sinf                      0042c180 f i math_stuff.obj
 0001:0002b1a0       _sqrtf                     0042c1a0 f i math_stuff.obj
 0001:0002b1c0       ?fabs@@YAMM@Z              0042c1c0 f i math_stuff.obj
 0001:0002b1d0       ?sqrt@@YAMM@Z              0042c1d0 f i math_stuff.obj
 0001:0002b1f0       ?near_zero@@YAHM@Z         0042c1f0 f   math_stuff.obj
 0001:0002b230       ?vect2_normalize@@YAXQBMQAM@Z 0042c230 f   math_stuff.obj
 0001:0002b280       ?vect2_length@@YAMQBM@Z    0042c280 f   math_stuff.obj
 0001:0002b2b0       ?vect2_near_zero@@YAHQBM@Z 0042c2b0 f   math_stuff.obj
 0001:0002b330       ?vect3_zero@@YAXQAM@Z      0042c330 f   math_stuff.obj
 0001:0002b340       ?vect2_copy@@YAXQBEQAE@Z   0042c340 f   math_stuff.obj
 0001:0002b350       ?vect3_normalize@@YAXQBMQAM@Z 0042c350 f   math_stuff.obj
 0001:0002b3b0       ?vect3_length@@YAMQBM@Z    0042c3b0 f   math_stuff.obj
 0001:0002b3f0       ?vect3_div@@YAXQBMMQAM@Z   0042c3f0 f   math_stuff.obj
 0001:0002b420       ?vect3_mult@@YAXQBMMQAM@Z  0042c420 f   math_stuff.obj
 0001:0002b450       ?vect3_vect3_mult@@YAXQBM0QAM@Z 0042c450 f   math_stuff.obj
 0001:0002b480       ?vect3_vect3_add@@YAXQBM0QAM@Z 0042c480 f   math_stuff.obj
 0001:0002b4b0       ?vect3_vect3_sub@@YAXQBM0QAM@Z 0042c4b0 f   math_stuff.obj
 0001:0002b4e0       ?vect3_invert@@YAXQBMQAM@Z 0042c4e0 f   math_stuff.obj
 0001:0002b500       ?vect3_near_zero@@YAHQBM@Z 0042c500 f   math_stuff.obj
 0001:0002b5a0       ?vect3_copy@@YAXQBMQAM@Z   0042c5a0 f   math_stuff.obj
 0001:0002b5c0       ?vect3_dist@@YAMQBM0@Z     0042c5c0 f   math_stuff.obj
 0001:0002b620       ?vect4_near_zero@@YAHQBM@Z 0042c620 f   math_stuff.obj
 0001:0002b6d0       ?vect4_copy@@YAXQBEQAE@Z   0042c6d0 f   math_stuff.obj
 0001:0002b6e0       ?vect4_copy@@YAXQBMQAM@Z   0042c6e0 f   math_stuff.obj
 0001:0002b700       ?matrix_copy@@YAXQBMQAM@Z  0042c700 f   math_stuff.obj
 0001:0002b720       ?vect3_dot_product@@YAMQBM0@Z 0042c720 f   math_stuff.obj
 0001:0002b750       ?vect3_cross_product@@YAXQBM0QAM@Z 0042c750 f   math_stuff.obj
 0001:0002b790       ?matrix_vect4_mult@@YAXQBM0QAM@Z 0042c790 f   math_stuff.obj
 0001:0002b840       ?matrix_matrix_mult@@YAXQBM0QAM@Z 0042c840 f   math_stuff.obj
 0001:0002b910       ?matrix_vect3_rotate@@YAXQBM0MQAM@Z 0042c910 f   math_stuff.obj
 0001:0002baa0       ?matrix_vect3_switchXY@@YAXQBMQAM@Z 0042caa0 f   math_stuff.obj
 0001:0002bb30       ?matrix_identity@@YAXQAM@Z 0042cb30 f   math_stuff.obj
 0001:0002bb50       ?roundf@@YAMM@Z            0042cb50 f   math_stuff.obj
 0001:0002bb80       ?GetOrthMatrix@@YAXMMMMMMMMMPAM000@Z 0042cb80 f   math_stuff.obj
 0001:0002bd40       ?MakeOrthMatrix@@YAXMMMMPAM00000000@Z 0042cd40 f   math_stuff.obj
 0001:0002be50       ?matrix_vect3_mult@@YAXQBM0QAM@Z 0042ce50 f   math_stuff.obj
 0001:0002bea0       ?onFootUpdateAtNormalPos@@YAXXZ 0042cea0 f   misc_funcs.obj
 0001:0002bf40       ?onFootUpdateFollow@@YAXG@Z 0042cf40 f   misc_funcs.obj
 0001:0002bfa0       ?inCarUpdateFollow@@YAXGG@Z 0042cfa0 f   misc_funcs.obj
 0001:0002c0d0       ?sampConnect@@YAHPADH00@Z  0042d0d0 f   misc_funcs.obj
 0001:0002c140       ?sampDisconnect@@YAXH@Z    0042d140 f   misc_funcs.obj
 0001:0002c180       ?sampSpawn@@YAXXZ          0042d180 f   misc_funcs.obj
 0001:0002c270       ?isPlayerConnected@@YAHG@Z 0042d270 f   misc_funcs.obj
 0001:0002c2a0       ?getPlayerID@@YAHPAD@Z     0042d2a0 f   misc_funcs.obj
 0001:0002c300       ?getPlayerName@@YAPADG@Z   0042d300 f   misc_funcs.obj
 0001:0002c330       ?getPlayerPos@@YAHGPAM@Z   0042d330 f   misc_funcs.obj
 0001:0002c380       ?getPlayerIDFromPlayerName@@YAGPAD@Z 0042d380 f   misc_funcs.obj
 0001:0002c3f0       ?getPlayerCount@@YAGXZ     0042d3f0 f   misc_funcs.obj
 0001:0002c440       ?gta_vehicle_get_by_id@@YAPBUvehicle_entry@@H@Z 0042d440 f   misc_funcs.obj
 0001:0002c460       ?sampRequestClass@@YAXH@Z  0042d460 f   misc_funcs.obj
 0001:0002c510       ?sampSmth@@YAXXZ           0042d510 f   misc_funcs.obj
 0001:0002c6b0       ?sampFakeNpc@@YAXXZ        0042d6b0 f   misc_funcs.obj
 0001:0002c860       ?sendServerCommand@@YAXPAD@Z 0042d860 f   misc_funcs.obj
 0001:0002c930       ?sendChat@@YAXPAD@Z        0042d930 f   misc_funcs.obj
 0001:0002ca00       ?SendScmEvent@@YAXHKKK@Z   0042da00 f   misc_funcs.obj
 0001:0002cb00       ?sendDialogResponse@@YAXGEGPAD@Z 0042db00 f   misc_funcs.obj
 0001:0002cc30       ?sampReg@@YAXXZ            0042dc30 f   misc_funcs.obj
 0001:0002ce30       ??$ReadCompressed@_N@BitStream@RakNet@@QAE_NAA_N@Z 0042de30 f i netgame.obj
 0001:0002ce40       ?resetPools@@YAXHK@Z       0042de40 f   netgame.obj
 0001:0002ce90       ?UpdatePlayerScoresAndPings@@YAXHH@Z 0042de90 f   netgame.obj
 0001:0002cfc0       ??$Read@K@BitStream@RakNet@@QAE_NAAK@Z 0042dfc0 f i netgame.obj
 0001:0002cfe0       ??$Read@M@BitStream@RakNet@@QAE_NAAM@Z 0042dfe0 f i netgame.obj
 0001:0002d000       ??$ReadNormQuat@M@BitStream@RakNet@@QAE_NAAM000@Z 0042e000 f i netgame.obj
 0001:0002d150       ??$ReadCompressed@M@BitStream@RakNet@@QAE_NAAM@Z 0042e150 f i netgame.obj
 0001:0002d190       ?Packet_ConnectionSucceeded@@YAXPAUPacket@@@Z 0042e190 f   netgame.obj
 0001:0002d400       ?Packet_UnoccupiedSync@@YAXPAUPacket@@@Z 0042e400 f   netgame.obj
 0001:0002d4c0       ?Packet_AimSync@@YAXPAUPacket@@@Z 0042e4c0 f   netgame.obj
 0001:0002d580       ?Packet_PassengerSync@@YAXPAUPacket@@@Z 0042e580 f   netgame.obj
 0001:0002d6b0       ?Packet_TrailerSync@@YAXPAUPacket@@@Z 0042e6b0 f   netgame.obj
 0001:0002d740       ?Packet_MarkersSync@@YAXPAUPacket@@@Z 0042e740 f   netgame.obj
 0001:0002d900       ??$ReadVector@M@BitStream@RakNet@@QAE_NAAM00@Z 0042e900 f i netgame.obj
 0001:0002da30       ?Packet_PlayerSync@@YAXPAUPacket@@@Z 0042ea30 f   netgame.obj
 0001:0002ddf0       ?Packet_VehicleSync@@YAXPAUPacket@@@Z 0042edf0 f   netgame.obj
 0001:0002e190       ?UpdateNetwork@@YAXXZ      0042f190 f   netgame.obj
 0001:0002e470       ?strstr@@YAPADPADPBD@Z     0042f470 f i netrpc.obj
 0001:0002e480       ?WorldVehicleAdd@@YAXPAURPCParameters@@@Z 0042f480 f   netrpc.obj
 0001:0002e560       ?SAMPDlgProc@@YGJPAUHWND__@@IIJ@Z 0042f560 f   netrpc.obj
 0001:0002e910       ?DialogBoxThread@@YGKPAX@Z 0042f910 f   netrpc.obj
 0001:0002ead0       ?UnRegisterRPCs@@YAXPAVRakClientInterface@@@Z 0042fad0 f   netrpc.obj
 0001:0002ebc0       ?ServerJoin@@YAXPAURPCParameters@@@Z 0042fbc0 f   netrpc.obj
 0001:0002ed10       ?ServerQuit@@YAXPAURPCParameters@@@Z 0042fd10 f   netrpc.obj
 0001:0002ee00       ?InitGame@@YAXPAURPCParameters@@@Z 0042fe00 f   netrpc.obj
 0001:0002f100       ?WorldPlayerAdd@@YAXPAURPCParameters@@@Z 00430100 f   netrpc.obj
 0001:0002f280       ?WorldPlayerDeath@@YAXPAURPCParameters@@@Z 00430280 f   netrpc.obj
 0001:0002f320       ?WorldPlayerRemove@@YAXPAURPCParameters@@@Z 00430320 f   netrpc.obj
 0001:0002f3f0       ?WorldVehicleRemove@@YAXPAURPCParameters@@@Z 004303f0 f   netrpc.obj
 0001:0002f4c0       ?ConnectionRejected@@YAXPAURPCParameters@@@Z 004304c0 f   netrpc.obj
 0001:0002f5e0       ?ClientMessage@@YAXPAURPCParameters@@@Z 004305e0 f   netrpc.obj
 0001:0002f730       ?Chat@@YAXPAURPCParameters@@@Z 00430730 f   netrpc.obj
 0001:0002f8b0       ?UpdateScoresPingsIPs@@YAXPAURPCParameters@@@Z 004308b0 f   netrpc.obj
 0001:0002f9b0       ?ScrInitMenu@@YAXPAURPCParameters@@@Z 004309b0 f   netrpc.obj
 0001:0002fc20       ?ScrDialogBox@@YAXPAURPCParameters@@@Z 00430c20 f   netrpc.obj
 0001:0002fe00       ?ScrGameText@@YAXPAURPCParameters@@@Z 00430e00 f   netrpc.obj
 0001:0002fef0       ?ScrPlayAudioStream@@YAXPAURPCParameters@@@Z 00430ef0 f   netrpc.obj
 0001:0002ffb0       ?RegisterRPCs@@YAXPAVRakClientInterface@@@Z 00430fb0 f   netrpc.obj
 0001:000300f0       ?sendRconCommand@@YAXPADH@Z 004310f0 f   rcon.obj
 0001:000301e0       ?RCONReceiveLoop@@YAHXZ    004311e0 f   rcon.obj
 0001:00030390       ?rec_sqlite_optimizeDatabase@@YA_NXZ 00431390 f   vehplayer.obj
 0001:00030440       ?vehicle_playback_handler@@YAXXZ 00431440 f   vehplayer.obj
 0001:00030650       ??$_snprintf_s@$0EAA@@@YAHAAY0EAA@DIPBDZZ 00431650 f i vehplayer.obj
 0001:00030680       ?sqliteDB_checkTableExists@@YAHPAUsqlite3@@PAD@Z 00431680 f   vehplayer.obj
 0001:00030770       ?sqliteDB_getNumTables@@YAHPAUsqlite3@@_N@Z 00431770 f   vehplayer.obj
 0001:00030850       ?sqliteDB_dropTable@@YA_NPAUsqlite3@@PAD@Z 00431850 f   vehplayer.obj
 0001:00030900       ?rec_sqlite_getNumTables@@YAHXZ 00431900 f   vehplayer.obj
 0001:00030960       ?rec_sqlite_getTableName@@YAPADH@Z 00431960 f   vehplayer.obj
 0001:00030a80       ?rec_sqlite_loadTable@@YA_NPAD@Z 00431a80 f   vehplayer.obj
 0001:00030d50       ?rec_sqlite_dropTable@@YA_NPAD@Z 00431d50 f   vehplayer.obj
 0001:00030dd0       ?rec_sqlite_writeTable@@YA_NXZ 00431dd0 f   vehplayer.obj
 0001:00031100       ?CalcWindowTextSize@@YAHPAUHWND__@@PAUtagRECT@@@Z 00432100 f   window.obj
 0001:00031190       ?CenterWindow@@YAHPAUHWND__@@0@Z 00432190 f   window.obj
 0001:00031300       ?MainWindowProc@@YGJPAUHWND__@@IIJ@Z 00432300 f   window.obj
 0001:00031a10       ?windowThread@@YGKPAX@Z    00432a10 f   window.obj
 0001:00031be0       ?SetUpWindow@@YAXPAUHINSTANCE__@@@Z 00432be0 f   window.obj
 0001:00031c00       ?QueryFloatAttribute@TiXmlElement@@QBEHPBDPAM@Z 00432c00 f i xmlsets.obj
 0001:00031c30       ?LoadSettings@@YAHXZ       00432c30 f   xmlsets.obj
 0001:00032050       ?UnLoadSettings@@YAHXZ     00433050 f   xmlsets.obj
 0001:00032070       ?ReloadSettings@@YAHXZ     00433070 f   xmlsets.obj
 0001:000320b0       _inet_ntoa@4               004330b0 f   ws2_32:WS2_32.dll
 0001:000320b6       _inet_addr@4               004330b6 f   ws2_32:WS2_32.dll
 0001:000320bc       _closesocket@4             004330bc f   ws2_32:WS2_32.dll
 0001:000320c2       _WSAStartup@8              004330c2 f   ws2_32:WS2_32.dll
 0001:000320c8       _WSACleanup@0              004330c8 f   ws2_32:WS2_32.dll
 0001:000320ce       _connect@12                004330ce f   ws2_32:WS2_32.dll
 0001:000320d4       _htons@4                   004330d4 f   ws2_32:WS2_32.dll
 0001:000320da       _bind@12                   004330da f   ws2_32:WS2_32.dll
 0001:000320e0       _ioctlsocket@12            004330e0 f   ws2_32:WS2_32.dll
 0001:000320e6       _setsockopt@20             004330e6 f   ws2_32:WS2_32.dll
 0001:000320ec       _socket@12                 004330ec f   ws2_32:WS2_32.dll
 0001:000320f2       _gethostbyname@4           004330f2 f   ws2_32:WS2_32.dll
 0001:000320f8       _send@16                   004330f8 f   ws2_32:WS2_32.dll
 0001:000320fe       _ntohs@4                   004330fe f   ws2_32:WS2_32.dll
 0001:00032104       _recvfrom@24               00433104 f   ws2_32:WS2_32.dll
 0001:0003210a       _WSAGetLastError@0         0043310a f   ws2_32:WS2_32.dll
 0001:00032110       _sendto@24                 00433110 f   ws2_32:WS2_32.dll
 0001:00032116       _gethostname@8             00433116 f   ws2_32:WS2_32.dll
 0001:0003211c       _getsockname@12            0043311c f   ws2_32:WS2_32.dll
 0001:00032122       _InitCommonControls@0      00433122 f   comctl32:COMCTL32.dll
 0001:00032128       _QueryPerformanceCounter@4 00433128 f   kernel32:KERNEL32.dll
 0001:0003212e       _QueryPerformanceFrequency@4 0043312e f   kernel32:KERNEL32.dll
 0001:00032134       _SetWaitableTimer@24       00433134 f   kernel32:KERNEL32.dll
 0001:0003213a       _CreateWaitableTimerA@12   0043313a f   kernel32:KERNEL32.dll
 0001:00032140       _CloseHandle@4             00433140 f   kernel32:KERNEL32.dll
 0001:00032146       _Sleep@4                   00433146 f   kernel32:KERNEL32.dll
 0001:0003214c       _InitializeCriticalSection@4 0043314c f   kernel32:KERNEL32.dll
 0001:00032152       _DeleteCriticalSection@4   00433152 f   kernel32:KERNEL32.dll
 0001:00032158       _EnterCriticalSection@4    00433158 f   kernel32:KERNEL32.dll
 0001:0003215e       _LeaveCriticalSection@4    0043315e f   kernel32:KERNEL32.dll
 0001:00032164       _ExitProcess@4             00433164 f   kernel32:KERNEL32.dll
 0001:0003216a       _ReadConsoleA@20           0043316a f   kernel32:KERNEL32.dll
 0001:00032170       _FlushConsoleInputBuffer@4 00433170 f   kernel32:KERNEL32.dll
 0001:00032176       _SetConsoleMode@8          00433176 f   kernel32:KERNEL32.dll
 0001:0003217c       _GetStdHandle@4            0043317c f   kernel32:KERNEL32.dll
 0001:00032182       _SetConsoleCtrlHandler@8   00433182 f   kernel32:KERNEL32.dll
 0001:00032188       _CreateThread@24           00433188 f   kernel32:KERNEL32.dll
 0001:0003218e       _SetConsoleTitleA@4        0043318e f   kernel32:KERNEL32.dll
 0001:00032194       _AllocConsole@0            00433194 f   kernel32:KERNEL32.dll
 0001:0003219a       _GetTickCount@0            0043319a f   kernel32:KERNEL32.dll
 0001:000321a0       _GetLocalTime@4            004331a0 f   kernel32:KERNEL32.dll
 0001:000321a6       _GetModuleHandleA@4        004331a6 f   kernel32:KERNEL32.dll
 0001:000321ac       _TerminateThread@8         004331ac f   kernel32:KERNEL32.dll
 0001:000321b2       _GetConsoleWindow@0        004331b2 f   kernel32:KERNEL32.dll
 0001:000321b8       _lstrlenA@4                004331b8 f   kernel32:KERNEL32.dll
 0001:000321be       _MulDiv@12                 004331be f   kernel32:KERNEL32.dll
 0001:000321c4       _wvsprintfA@12             004331c4 f   user32:USER32.dll
 0001:000321ca       _SendMessageA@16           004331ca f   user32:USER32.dll
 0001:000321d0       _SetWindowTextA@8          004331d0 f   user32:USER32.dll
 0001:000321d6       _PostQuitMessage@4         004331d6 f   user32:USER32.dll
 0001:000321dc       _GetWindowTextA@12         004331dc f   user32:USER32.dll
 0001:000321e2       _DefWindowProcA@16         004331e2 f   user32:USER32.dll
 0001:000321e8       _EndPaint@8                004331e8 f   user32:USER32.dll
 0001:000321ee       _DrawTextA@20              004331ee f   user32:USER32.dll
 0001:000321f4       _BeginPaint@8              004331f4 f   user32:USER32.dll
 0001:000321fa       _GetClientRect@8           004331fa f   user32:USER32.dll
 0001:00032200       _CreateWindowExA@48        00433200 f   user32:USER32.dll
 0001:00032206       _GetDlgItem@8              00433206 f   user32:USER32.dll
 0001:0003220c       _UnregisterClassA@8        0043320c f   user32:USER32.dll
 0001:00032212       _DestroyWindow@4           00433212 f   user32:USER32.dll
 0001:00032218       _DispatchMessageA@4        00433218 f   user32:USER32.dll
 0001:0003221e       _TranslateMessage@4        0043321e f   user32:USER32.dll
 0001:00032224       _GetMessageA@16            00433224 f   user32:USER32.dll
 0001:0003222a       _SetForegroundWindow@4     0043322a f   user32:USER32.dll
 0001:00032230       _UpdateWindow@4            00433230 f   user32:USER32.dll
 0001:00032236       _ShowWindow@8              00433236 f   user32:USER32.dll
 0001:0003223c       _RegisterClassExA@4        0043323c f   user32:USER32.dll
 0001:00032242       _LoadCursorA@8             00433242 f   user32:USER32.dll
 0001:00032248       _LoadIconA@8               00433248 f   user32:USER32.dll
 0001:0003224e       _GetWindowRect@8           0043324e f   user32:USER32.dll
 0001:00032254       _ReleaseDC@8               00433254 f   user32:USER32.dll
 0001:0003225a       _GetDC@4                   0043325a f   user32:USER32.dll
 0001:00032260       _GetWindowTextLengthA@4    00433260 f   user32:USER32.dll
 0001:00032266       _SetWindowPos@28           00433266 f   user32:USER32.dll
 0001:0003226c       _MapWindowPoints@16        0043326c f   user32:USER32.dll
 0001:00032272       _SystemParametersInfoA@16  00433272 f   user32:USER32.dll
 0001:00032278       _GetWindow@8               00433278 f   user32:USER32.dll
 0001:0003227e       _GetParent@4               0043327e f   user32:USER32.dll
 0001:00032284       _GetWindowLongA@8          00433284 f   user32:USER32.dll
 0001:0003228a       _GetKeyState@4             0043328a f   user32:USER32.dll
 0001:00032290       _GetFocus@0                00433290 f   user32:USER32.dll
 0001:00032296       _RedrawWindow@16           00433296 f   user32:USER32.dll
 0001:0003229c       _EndDeferWindowPos@4       0043329c f   user32:USER32.dll
 0001:000322a2       _DeferWindowPos@32         004332a2 f   user32:USER32.dll
 0001:000322a8       _BeginDeferWindowPos@4     004332a8 f   user32:USER32.dll
 0001:000322ae       _DrawFocusRect@8           004332ae f   user32:USER32.dll
 0001:000322b4       _SetFocus@4                004332b4 f   user32:USER32.dll
 0001:000322ba       _IsDialogMessageA@8        004332ba f   user32:USER32.dll
 0001:000322c0       _MessageBoxA@16            004332c0 f   user32:USER32.dll
 0001:000322c6       _DeleteDC@4                004332c6 f   gdi32:GDI32.dll
 0001:000322cc       _SelectObject@8            004332cc f   gdi32:GDI32.dll
 0001:000322d2       _CreateCompatibleDC@4      004332d2 f   gdi32:GDI32.dll
 0001:000322d8       _CreateFontA@56            004332d8 f   gdi32:GDI32.dll
 0001:000322de       _GetTextMetricsA@8         004332de f   gdi32:GDI32.dll
 0001:000322e4       _ExtTextOutA@32            004332e4 f   gdi32:GDI32.dll
 0001:000322ea       _SetTextColor@8            004332ea f   gdi32:GDI32.dll
 0001:000322f0       _SetBkColor@8              004332f0 f   gdi32:GDI32.dll
 0001:000322f6       _DeleteObject@4            004332f6 f   gdi32:GDI32.dll
 0001:000322fc       _GetDeviceCaps@8           004332fc f   gdi32:GDI32.dll
 0001:00032302       _V6_HeapAlloc              00433302 f   LIBCMT:malloc.obj
 0001:00032351       __heap_alloc               00433351 f i LIBCMT:malloc.obj
 0001:000323cb       _malloc                    004333cb f   LIBCMT:malloc.obj
 0001:000324a0       _memcpy                    004334a0 f   LIBCMT:memcpy.obj
 0001:00032805       _free                      00433805 f   LIBCMT:free.obj
 0001:000328a0       _memset                    004338a0 f   LIBCMT:memset.obj
 0001:0003291a       _realloc                   0043391a f   LIBCMT:realloc.obj
 0001:00032b35       __invoke_watson_if_error   00433b35 f i LIBCMT:wassert.obj
 0001:00032b77       __wassert                  00433b77 f   LIBCMT:wassert.obj
 0001:000332c9       __fputchar                 004342c9 f   LIBCMT:fputchar.obj
 0001:000332e3       _putchar                   004342e3 f   LIBCMT:fputchar.obj
 0001:000332ee       _printf                    004342ee f   LIBCMT:printf.obj
 0001:0003339d       __printf_l                 0043439d f   LIBCMT:printf.obj
 0001:000333b6       __printf_s_l               004343b6 f   LIBCMT:printf.obj
 0001:000333cf       _printf_s                  004343cf f   LIBCMT:printf.obj
 0001:000333e7       __printf_p_l               004343e7 f   LIBCMT:printf.obj
 0001:00033400       __printf_p                 00434400 f   LIBCMT:printf.obj
 0001:00033418       __set_printf_count_output  00434418 f   LIBCMT:printf.obj
 0001:00033442       __get_printf_count_output  00434442 f   LIBCMT:printf.obj
 0001:00033458       ??0bad_alloc@std@@QAE@XZ   00434458 f i LIBCMT:new.obj
 0001:00033473       ??1bad_alloc@std@@UAE@XZ   00434473 f i LIBCMT:new.obj
 0001:0003347e       ??_Ebad_alloc@std@@UAEPAXI@Z 0043447e f i LIBCMT:new.obj
 0001:0003347e       ??_Gbad_alloc@std@@UAEPAXI@Z 0043447e f i LIBCMT:new.obj
 0001:000334a5       ??0bad_alloc@std@@QAE@ABV01@@Z 004344a5 f i LIBCMT:new.obj
 0001:000334c2       ??2@YAPAXI@Z               004344c2 f   LIBCMT:new.obj
 0001:00033530       _memmove                   00434530 f   LIBCMT:memmove.obj
 0001:00033895       ?_JumpToContinuation@@YGXPAXPAUEHRegistrationNode@@@Z 00434895 f   LIBCMT:_trnsctrl_.obj
 0001:000338c7       ?_CallMemberFunction0@@YGXPAX0@Z 004348c7 f   LIBCMT:_trnsctrl_.obj
 0001:000338ce       ?_CallMemberFunction1@@YGXPAX00@Z 004348ce f   LIBCMT:_trnsctrl_.obj
 0001:000338d5       ?_CallMemberFunction2@@YGXPAX00H@Z 004348d5 f   LIBCMT:_trnsctrl_.obj
 0001:000338dc       ?_UnwindNestedFrames@@YGXPAUEHRegistrationNode@@PAUEHExceptionRecord@@@Z 004348dc f   LIBCMT:_trnsctrl_.obj
 0001:00033930       ___CxxFrameHandler         00434930 f   LIBCMT:_trnsctrl_.obj
 0001:00033966       ___CxxFrameHandler3        00434966 f   LIBCMT:_trnsctrl_.obj
 0001:0003399c       ___CxxFrameHandler2        0043499c f   LIBCMT:_trnsctrl_.obj
 0001:000339d2       ___CxxLongjmpUnwind@4      004349d2 f   LIBCMT:_trnsctrl_.obj
 0001:00033a24       ?_CallSETranslator@@YAHPAUEHExceptionRecord@@PAUEHRegistrationNode@@PAX2PBU_s_FuncInfo@@H1@Z 00434a24 f   LIBCMT:_trnsctrl_.obj
 0001:00033b9a       ?_GetRangeOfTrysToCheck@@YAPBU_s_TryBlockMapEntry@@PBU_s_FuncInfo@@HHPAI1@Z 00434b9a f   LIBCMT:_trnsctrl_.obj
 0001:00033c0f       __CreateFrameInfo          00434c0f f   LIBCMT:_trnsctrl_.obj
 0001:00033c3b       __IsExceptionObjectToBeDestroyed 00434c3b f   LIBCMT:_trnsctrl_.obj
 0001:00033c62       __FindAndUnlinkFrame       00434c62 f   LIBCMT:_trnsctrl_.obj
 0001:00033cb4       ?_CallCatchBlock2@@YAPAXPAUEHRegistrationNode@@PBU_s_FuncInfo@@PAXHK@Z 00434cb4 f   LIBCMT:_trnsctrl_.obj
 0001:00033d14       ??3@YAXPAX@Z               00434d14 f   LIBCMT:delete.obj
 0001:00033d31       ?__ArrayUnwind@@YGXPAXIHP6EX0@Z@Z 00434d31 f   LIBCMT:ehvecdtr.obj
 0001:00033d8f       ??_M@YGXPAXIHP6EX0@Z@Z     00434d8f f   LIBCMT:ehvecdtr.obj
 0001:00033df2       _sprintf                   00434df2 f   LIBCMT:sprintf.obj
 0001:00033e6f       __sprintf_l                00434e6f f   LIBCMT:sprintf.obj
 0001:00033e8b       _sprintf_s                 00434e8b f   LIBCMT:sprintf.obj
 0001:00033ea9       __sprintf_s_l              00434ea9 f   LIBCMT:sprintf.obj
 0001:00033ec8       __snprintf_s               00434ec8 f   LIBCMT:sprintf.obj
 0001:00033ee9       __snprintf_s_l             00434ee9 f   LIBCMT:sprintf.obj
 0001:00033f0b       __sprintf_p                00434f0b f   LIBCMT:sprintf.obj
 0001:00033f29       __sprintf_p_l              00434f29 f   LIBCMT:sprintf.obj
 0001:00033f48       __scprintf                 00434f48 f   LIBCMT:sprintf.obj
 0001:00033f5d       __scprintf_p               00434f5d f   LIBCMT:sprintf.obj
 0001:00033f72       __scprintf_l               00434f72 f   LIBCMT:sprintf.obj
 0001:00033f8b       __scprintf_p_l             00434f8b f   LIBCMT:sprintf.obj
 0001:00033fb0       _strncpy                   00434fb0 f   LIBCMT:strncpy.obj
 0001:000340d4       ??_L@YGXPAXIHP6EX0@Z1@Z    004350d4 f   LIBCMT:ehvecctr.obj
 0001:00034140       __alldiv                   00435140 f   LIBCMT:lldiv.obj
 0001:000341f0       __allmul                   004351f0 f   LIBCMT:llmul.obj
 0001:00034230       __alldvrm                  00435230 f   LIBCMT:lldvrm.obj
 0001:0003430f       ?name@type_info@@QBEPBDPAU__type_info_node@@@Z 0043530f f   LIBCMT:typinfo.obj
 0001:00034323       ??1type_info@@UAE@XZ       00435323 f   LIBCMT:typinfo.obj
 0001:00034333       ??_Etype_info@@UAEPAXI@Z   00435333 f i LIBCMT:typinfo.obj
 0001:00034333       ??_Gtype_info@@UAEPAXI@Z   00435333 f i LIBCMT:typinfo.obj
 0001:00034354       ?_name_internal_method@type_info@@QBEPBDPAU__type_info_node@@@Z 00435354 f   LIBCMT:typinfo.obj
 0001:00034368       ?_type_info_dtor_internal_method@type_info@@QAEXXZ 00435368 f   LIBCMT:typinfo.obj
 0001:00034372       ??8type_info@@QBE_NABV0@@Z 00435372 f   LIBCMT:typinfo.obj
 0001:00034392       ??9type_info@@QBE_NABV0@@Z 00435392 f   LIBCMT:typinfo.obj
 0001:000343b3       ?before@type_info@@QBEHABV1@@Z 004353b3 f   LIBCMT:typinfo.obj
 0001:000343d7       ?raw_name@type_info@@QBEPBDXZ 004353d7 f   LIBCMT:typinfo.obj
 0001:000343db       ??0type_info@@AAE@ABV0@@Z  004353db f   LIBCMT:typinfo.obj
 0001:000343e6       ??4type_info@@AAEAAV0@ABV0@@Z 004353e6 f   LIBCMT:typinfo.obj
 0001:000343eb       __purecall                 004353eb f   LIBCMT:purevirt.obj
 0001:00034415       __set_purecall_handler     00435415 f   LIBCMT:purevirt.obj
 0001:0003443c       __get_purecall_handler     0043543c f   LIBCMT:purevirt.obj
 0001:00034503       ___onexitinit              00435503 f   LIBCMT:onexit.obj
 0001:00034534       __onexit                   00435534 f   LIBCMT:onexit.obj
 0001:00034570       _atexit                    00435570 f   LIBCMT:onexit.obj
 0001:000345cb       __itoa                     004355cb f   LIBCMT:xtoa.obj
 0001:000345f5       __ltoa                     004355f5 f   LIBCMT:xtoa.obj
 0001:0003461c       __ultoa                    0043561c f   LIBCMT:xtoa.obj
 0001:000346a5       __i64toa                   004356a5 f   LIBCMT:xtoa.obj
 0001:000346d8       __ui64toa                  004356d8 f   LIBCMT:xtoa.obj
 0001:000346f5       __fpclear                  004356f5 f   LIBCMT:_fpinit_.obj
 0001:000346f6       __cfltcvt_init             004356f6 f   LIBCMT:_fpinit_.obj
 0001:00034756       ___setfflag                00435756 f   LIBCMT:_fpinit_.obj
 0001:0003476b       __fpmath                   0043576b f   LIBCMT:_fpinit_.obj
 0001:00034790       __alloca_probe_16          00435790 f   LIBCMT:alloca16.obj
 0001:000347a6       __alloca_probe_8           004357a6     LIBCMT:alloca16.obj
 0001:000347c0       __alloca_probe             004357c0     LIBCMT:chkstk.obj
 0001:000347c0       __chkstk                   004357c0 f   LIBCMT:chkstk.obj
 0001:000347eb       __endthreadex              004357eb f   LIBCMT:threadex.obj
 0001:000348ec       __beginthreadex            004358ec f   LIBCMT:threadex.obj
 0001:0003499c       __fclose_nolock            0043599c f   LIBCMT:fclose.obj
 0001:00034a13       _fclose                    00435a13 f   LIBCMT:fclose.obj
 0001:00034a8f       __fread_nolock_s           00435a8f f   LIBCMT:fread.obj
 0001:00034c99       __fread_nolock             00435c99 f   LIBCMT:fread.obj
 0001:00034cb6       _fread_s                   00435cb6 f   LIBCMT:fread.obj
 0001:00034d4c       _fread                     00435d4c f   LIBCMT:fread.obj
 0001:00034d69       _div                       00435d69 f   LIBCMT:div.obj
 0001:00034d77       __ftell_nolock             00435d77 f   LIBCMT:ftell.obj
 0001:00034f14       _ftell                     00435f14 f   LIBCMT:ftell.obj
 0001:00034f82       __fseek_nolock             00435f82 f   LIBCMT:fseek.obj
 0001:0003500c       _fseek                     0043600c f   LIBCMT:fseek.obj
 0001:00035091       __fsopen                   00436091 f   LIBCMT:fopen.obj
 0001:00035155       _fopen                     00436155 f   LIBCMT:fopen.obj
 0001:0003516c       _fopen_s                   0043616c f   LIBCMT:fopen.obj
 0001:000351bf       __fwrite_nolock            004361bf f   LIBCMT:fwrite.obj
 0001:00035321       _fwrite                    00436321 f   LIBCMT:fwrite.obj
 0001:000353a3       _feof                      004363a3 f   LIBCMT:feoferr.obj
 0001:000353d7       _ferror                    004363d7 f   LIBCMT:feoferr.obj
 0001:0003540b       _fputc                     0043640b f   LIBCMT:fputc.obj
 0001:00035517       _putc                      00436517 f   LIBCMT:fputc.obj
 0001:00035623       _fprintf                   00436623 f   LIBCMT:fprintf.obj
 0001:0003573f       __fprintf_l                0043673f f   LIBCMT:fprintf.obj
 0001:0003575b       __fprintf_s_l              0043675b f   LIBCMT:fprintf.obj
 0001:00035777       _fprintf_s                 00436777 f   LIBCMT:fprintf.obj
 0001:00035792       __fprintf_p_l              00436792 f   LIBCMT:fprintf.obj
 0001:000357ae       __fprintf_p                004367ae f   LIBCMT:fprintf.obj
 0001:00035833       _sscanf                    00436833 f   LIBCMT:sscanf.obj
 0001:00035855       __sscanf_l                 00436855 f   LIBCMT:sscanf.obj
 0001:00035878       _sscanf_s                  00436878 f   LIBCMT:sscanf.obj
 0001:0003589a       __sscanf_s_l               0043689a f   LIBCMT:sscanf.obj
 0001:000358bd       _atol                      004368bd f   LIBCMT:atox.obj
 0001:000358d3       __atol_l                   004368d3 f   LIBCMT:atox.obj
 0001:000358ec       _atoi                      004368ec f   LIBCMT:atox.obj
 0001:000358f7       __atoi_l                   004368f7 f   LIBCMT:atox.obj
 0001:00035902       __atoi64                   00436902 f   LIBCMT:atox.obj
 0001:00035918       __atoi64_l                 00436918 f   LIBCMT:atox.obj
 0001:00035931       ??0_LocaleUpdate@@QAE@PAUlocaleinfo_struct@@@Z 00436931 f i LIBCMT:atof.obj
 0001:000359b8       ??1_LocaleUpdate@@QAE@XZ   004369b8 f i LIBCMT:atof.obj
 0001:000359c6       ?GetLocaleT@_LocaleUpdate@@QAEPAUlocaleinfo_struct@@XZ 004369c6 f i LIBCMT:atof.obj
 0001:000359c9       __atof_l                   004369c9 f   LIBCMT:atof.obj
 0001:00035a74       _atof                      00436a74 f   LIBCMT:atof.obj
 0001:00035a87       ___strgtold12              00436a87 f   LIBCMT:atof.obj
 0001:00035ac9       ___STRINGTOLD              00436ac9 f   LIBCMT:atof.obj
 0001:00035b02       __vsnprintf_helper         00436b02 f   LIBCMT:vsnprnc.obj
 0001:00035bce       __vsnprintf_c              00436bce f   LIBCMT:vsnprnc.obj
 0001:00035bf7       __vsnprintf_c_l            00436bf7 f   LIBCMT:vsnprnc.obj
 0001:00035c21       __vsprintf_s_l             00436c21 f   LIBCMT:vsnprnc.obj
 0001:00035ca9       _vsprintf_s                00436ca9 f   LIBCMT:vsnprnc.obj
 0001:00035cc6       __vsnprintf_s_l            00436cc6 f   LIBCMT:vsnprnc.obj
 0001:00035dcd       __vsnprintf_s              00436dcd f   LIBCMT:vsnprnc.obj
 0001:00035ded       __vsprintf_p               00436ded f   LIBCMT:vsnprnc.obj
 0001:00035e16       __vsprintf_p_l             00436e16 f   LIBCMT:vsnprnc.obj
 0001:00035e40       __isalpha_l                00436e40 f i LIBCMT:_ctype.obj
 0001:00035e96       _isalpha                   00436e96 f i LIBCMT:_ctype.obj
 0001:00035ec6       __isupper_l                00436ec6 f i LIBCMT:_ctype.obj
 0001:00035f17       _isupper                   00436f17 f i LIBCMT:_ctype.obj
 0001:00035f45       __islower_l                00436f45 f i LIBCMT:_ctype.obj
 0001:00035f96       _islower                   00436f96 f i LIBCMT:_ctype.obj
 0001:00035fc4       __isdigit_l                00436fc4 f i LIBCMT:_ctype.obj
 0001:00036015       _isdigit                   00437015 f i LIBCMT:_ctype.obj
 0001:00036043       __isxdigit_l               00437043 f i LIBCMT:_ctype.obj
 0001:00036099       _isxdigit                  00437099 f i LIBCMT:_ctype.obj
 0001:000360c9       __isspace_l                004370c9 f i LIBCMT:_ctype.obj
 0001:0003611a       _isspace                   0043711a f i LIBCMT:_ctype.obj
 0001:00036148       __ispunct_l                00437148 f i LIBCMT:_ctype.obj
 0001:00036199       _ispunct                   00437199 f i LIBCMT:_ctype.obj
 0001:000361c7       __isalnum_l                004371c7 f i LIBCMT:_ctype.obj
 0001:0003621d       _isalnum                   0043721d f i LIBCMT:_ctype.obj
 0001:0003624d       __isprint_l                0043724d f i LIBCMT:_ctype.obj
 0001:000362a3       _isprint                   004372a3 f i LIBCMT:_ctype.obj
 0001:000362d3       __isgraph_l                004372d3 f i LIBCMT:_ctype.obj
 0001:00036329       _isgraph                   00437329 f i LIBCMT:_ctype.obj
 0001:00036359       __iscntrl_l                00437359 f i LIBCMT:_ctype.obj
 0001:000363aa       _iscntrl                   004373aa f i LIBCMT:_ctype.obj
 0001:000363d8       ___isascii                 004373d8 f i LIBCMT:_ctype.obj
 0001:000363ea       ___toascii                 004373ea f i LIBCMT:_ctype.obj
 0001:000363f7       __iscsymf_l                004373f7 f i LIBCMT:_ctype.obj
 0001:0003641a       ___iscsymf                 0043741a f i LIBCMT:_ctype.obj
 0001:00036439       __iscsym_l                 00437439 f i LIBCMT:_ctype.obj
 0001:0003645c       ___iscsym                  0043745c f i LIBCMT:_ctype.obj
 0001:0003647d       __tolower                  0043747d f   LIBCMT:tolower.obj
 0001:0003648a       __tolower_l                0043748a f   LIBCMT:tolower.obj
 0001:0003659f       _tolower                   0043759f f   LIBCMT:tolower.obj
 0001:000365cb       _strncmp                   004375cb f   LIBCMT:strncmp.obj
 0001:000366a0       _strchr                    004376a0 f   LIBCMT:strchr.obj
 0001:000366a6       ___from_strstr_to_strchr   004376a6     LIBCMT:strchr.obj
 0001:0003675e       _setvbuf                   0043775e f   LIBCMT:setvbuf.obj
 0001:0003685c       ___iob_func                0043785c f   LIBCMT:_file.obj
 0001:00036862       ___initstdio               00437862 f   LIBCMT:_file.obj
 0001:00036913       ___endstdio                00437913 f   LIBCMT:_file.obj
 0001:00036933       __lock_file                00437933 f   LIBCMT:_file.obj
 0001:00036974       __lock_file2               00437974 f   LIBCMT:_file.obj
 0001:000369a6       __unlock_file              004379a6 f   LIBCMT:_file.obj
 0001:000369e2       __unlock_file2             004379e2 f   LIBCMT:_file.obj
 0001:00036a11       __fdopen                   00437a11 f   LIBCMT:fdopen.obj
 0001:00036b97       __set_osfhnd               00437b97 f   LIBCMT:osfinfo.obj
 0001:00036c18       __free_osfhnd              00437c18 f   LIBCMT:osfinfo.obj
 0001:00036c9e       __get_osfhandle            00437c9e f   LIBCMT:osfinfo.obj
 0001:00036d15       ___lock_fhandle            00437d15 f   LIBCMT:osfinfo.obj
 0001:00036db5       __unlock_fhandle           00437db5 f   LIBCMT:osfinfo.obj
 0001:00036ddc       __alloc_osfhnd             00437ddc f   LIBCMT:osfinfo.obj
 0001:00036f76       __open_osfhandle           00437f76 f   LIBCMT:osfinfo.obj
 0001:0003708c       __flush                    0043808c f   LIBCMT:fflush.obj
 0001:000370f4       __fflush_nolock            004380f4 f   LIBCMT:fflush.obj
 0001:00037216       _fflush                    00438216 f   LIBCMT:fflush.obj
 0001:00037269       __flushall                 00438269 f   LIBCMT:fflush.obj
 0001:00037272       _vprintf_helper            00438272 f   LIBCMT:vprintf.obj
 0001:00037302       __vprintf_l                00438302 f   LIBCMT:vprintf.obj
 0001:0003731f       __vprintf_s_l              0043831f f   LIBCMT:vprintf.obj
 0001:0003733c       __vprintf_p_l              0043833c f   LIBCMT:vprintf.obj
 0001:00037359       _vprintf                   00438359 f   LIBCMT:vprintf.obj
 0001:00037375       _vprintf_s                 00438375 f   LIBCMT:vprintf.obj
 0001:00037391       __vprintf_p                00438391 f   LIBCMT:vprintf.obj
 0001:000373ad       _vfprintf_helper           004383ad f   LIBCMT:vfprintf.obj
 0001:000374c8       __vfprintf_l               004384c8 f   LIBCMT:vfprintf.obj
 0001:000374e8       __vfprintf_s_l             004384e8 f   LIBCMT:vfprintf.obj
 0001:00037508       __vfprintf_p_l             00438508 f   LIBCMT:vfprintf.obj
 0001:00037528       _vfprintf                  00438528 f   LIBCMT:vfprintf.obj
 0001:00037547       _vfprintf_s                00438547 f   LIBCMT:vfprintf.obj
 0001:00037566       __vfprintf_p               00438566 f   LIBCMT:vfprintf.obj
 0001:00037585       _srand                     00438585 f   LIBCMT:rand.obj
 0001:00037597       _rand                      00438597 f   LIBCMT:rand.obj
 0001:000375b9       __fgetchar                 004385b9 f   LIBCMT:fgetchar.obj
 0001:000375c6       _getchar                   004385c6 f   LIBCMT:fgetchar.obj
 0001:000375d0       _cos                       004385d0 f   LIBCMT:_cos_.obj
 0001:00037610       __CIcos                    00438610 f   LIBCMT:_cos_.obj
 0001:0003764b       __CIcos_default            0043864b f   LIBCMT:_cos_.obj
 0001:0003765f       __cos_default              0043865f     LIBCMT:_cos_.obj
 0001:00037700       _floor                     00438700 f   LIBCMT:_floor_pentium4_.obj
 0001:00037740       __floor_pentium4           00438740 f   LIBCMT:_floor_pentium4_.obj
 0001:00037830       _sin                       00438830 f   LIBCMT:_sin_.obj
 0001:00037870       __CIsin                    00438870 f   LIBCMT:_sin_.obj
 0001:000378ab       __CIsin_default            004388ab f   LIBCMT:_sin_.obj
 0001:000378bf       __sin_default              004388bf     LIBCMT:_sin_.obj
 0001:00037960       __CIsqrt                   00438960 f   LIBCMT:_sqrt_.obj
 0001:00037974       _sqrt                      00438974     LIBCMT:_sqrt_.obj
 0001:00037a1a       __copysign                 00438a1a f   LIBCMT:_ieeemisc_.obj
 0001:00037a42       __chgsign                  00438a42 f   LIBCMT:_ieeemisc_.obj
 0001:00037a6f       __scalb                    00438a6f f   LIBCMT:_ieeemisc_.obj
 0001:00037a89       __logb                     00438a89 f   LIBCMT:_ieeemisc_.obj
 0001:00037b72       __nextafter                00438b72 f   LIBCMT:_ieeemisc_.obj
 0001:00037e1a       __finite                   00438e1a f   LIBCMT:_ieeemisc_.obj
 0001:00037e36       __isnan                    00438e36 f   LIBCMT:_ieeemisc_.obj
 0001:00037e6a       __fpclass                  00438e6a f   LIBCMT:_ieeemisc_.obj
 0001:00037f00       _strstr                    00438f00 f   LIBCMT:strstr.obj
 0001:00037f86       _strtok                    00438f86 f   LIBCMT:strtok.obj
 0001:00038235       _WinMainCRTStartup         00439235 f   LIBCMT:wincrt0.obj
 0001:0003823f       __mtinitlocks              0043923f f   LIBCMT:mlock.obj
 0001:0003828a       __mtdeletelocks            0043928a f   LIBCMT:mlock.obj
 0001:000382e1       __unlock                   004392e1 f   LIBCMT:mlock.obj
 0001:000382f8       __lockerr_exit             004392f8 f   LIBCMT:mlock.obj
 0001:00038310       __mtinitlocknum            00439310 f   LIBCMT:mlock.obj
 0001:000383d3       __lock                     004393d3 f   LIBCMT:mlock.obj
 0001:00038406       __get_sbh_threshold        00439406 f   LIBCMT:sbheap.obj
 0001:00038427       __set_amblksiz             00439427 f   LIBCMT:sbheap.obj
 0001:00038472       __get_amblksiz             00439472 f   LIBCMT:sbheap.obj
 0001:000384b3       ___sbh_heap_init           004394b3 f   LIBCMT:sbheap.obj
 0001:00038501       ___sbh_find_block          00439501 f   LIBCMT:sbheap.obj
 0001:00038531       ___sbh_free_block          00439531 f   LIBCMT:sbheap.obj
 0001:00038847       ___sbh_alloc_new_region    00439847 f   LIBCMT:sbheap.obj
 0001:000388f7       ___sbh_alloc_new_group     004398f7 f   LIBCMT:sbheap.obj
 0001:000389ff       ___sbh_resize_block        004399ff f   LIBCMT:sbheap.obj
 0001:00038ce0       ___sbh_heapmin             00439ce0 f   LIBCMT:sbheap.obj
 0001:00038dad       ___sbh_heap_check          00439dad f   LIBCMT:sbheap.obj
 0001:00039091       __set_sbh_threshold        0043a091 f   LIBCMT:sbheap.obj
 0001:00039140       ___sbh_alloc_block         0043a140 f   LIBCMT:sbheap.obj
 0001:00039428       __SEH_prolog4              0043a428 f   LIBCMT:sehprolg4.obj
 0001:0003946d       __SEH_epilog4              0043a46d f   LIBCMT:sehprolg4.obj
 0001:000394c0       __except_handler4          0043a4c0 f   LIBCMT:chandler4.obj
 0001:0003964c       ___heap_select             0043a64c f   LIBCMT:heapinit.obj
 0001:00039650       __heap_init                0043a650 f   LIBCMT:heapinit.obj
 0001:00039680       __heap_term                0043a680 f   LIBCMT:heapinit.obj
 0001:000396f4       __get_heap_handle          0043a6f4 f   LIBCMT:heapinit.obj
 0001:000396fa       __crt_waiting_on_module_handle 0043a6fa f   LIBCMT:crt0dat.obj
 0001:0003972a       __amsg_exit                0043a72a f   LIBCMT:crt0dat.obj
 0001:00039753       ___crtCorExitProcess       0043a753 f   LIBCMT:crt0dat.obj
 0001:0003977e       ___crtExitProcess          0043a77e f   LIBCMT:crt0dat.obj
 0001:00039796       __lockexit                 0043a796 f   LIBCMT:crt0dat.obj
 0001:0003979f       __unlockexit               0043a79f f   LIBCMT:crt0dat.obj
 0001:000397c5       __initterm_e               0043a7c5 f   LIBCMT:crt0dat.obj
 0001:000397e9       __get_wpgmptr              0043a7e9 f   LIBCMT:crt0dat.obj
 0001:00039825       __get_pgmptr               0043a825 f   LIBCMT:crt0dat.obj
 0001:00039861       __cinit                    0043a861 f   LIBCMT:crt0dat.obj
 0001:00039a12       _exit                      0043aa12 f   LIBCMT:crt0dat.obj
 0001:00039a28       __exit                     0043aa28 f   LIBCMT:crt0dat.obj
 0001:00039a3e       __cexit                    0043aa3e f   LIBCMT:crt0dat.obj
 0001:00039a4d       __c_exit                   0043aa4d f   LIBCMT:crt0dat.obj
 0001:00039a5c       __init_pointers            0043aa5c f   LIBCMT:crt0dat.obj
 0001:00039aaa       __NMSG_WRITE               0043aaaa f   LIBCMT:crt0msg.obj
 0001:00039c55       __GET_RTERRMSG             0043ac55 f   LIBCMT:crt0msg.obj
 0001:00039c7b       __FF_MSGBANNER             0043ac7b f   LIBCMT:crt0msg.obj
 0001:00039cb4       __get_errno_from_oserr     0043acb4 f   LIBCMT:dosmap.obj
 0001:00039cf6       __errno                    0043acf6 f   LIBCMT:dosmap.obj
 0001:00039d09       ___doserrno                0043ad09 f   LIBCMT:dosmap.obj
 0001:00039d1c       __dosmaperr                0043ad1c f   LIBCMT:dosmap.obj
 0001:00039d3f       __set_errno                0043ad3f f   LIBCMT:dosmap.obj
 0001:00039d60       __get_errno                0043ad60 f   LIBCMT:dosmap.obj
 0001:00039d8f       __set_doserrno             0043ad8f f   LIBCMT:dosmap.obj
 0001:00039db0       __get_doserrno             0043adb0 f   LIBCMT:dosmap.obj
 0001:00039ddf       __initp_heap_handler       0043addf f   LIBCMT:handler.obj
 0001:00039dee       ?_set_new_handler@@YAP6AHI@ZP6AHI@Z@Z 0043adee f   LIBCMT:handler.obj
 0001:00039e24       ?_set_new_handler@@YAP6AHI@ZH@Z 0043ae24 f   LIBCMT:handler.obj
 0001:00039e2d       ?_query_new_handler@@YAP6AHI@ZXZ 0043ae2d f   LIBCMT:handler.obj
 0001:00039e3a       __callnewh                 0043ae3a f   LIBCMT:handler.obj
 0001:00039ee9       __VEC_memcpy               0043aee9 f   LIBCMT:p4_memcpy.obj
 0001:0003a01c       __get_sse2_info            0043b01c f   LIBCMT:cpu_disp.obj
 0001:0003a07e       ___sse2_available_init     0043b07e f   LIBCMT:cpu_disp.obj
 0001:0003a0e2       __VEC_memzero              0043b0e2 f   LIBCMT:p4_memset.obj
 0001:0003a171       __initp_misc_invarg        0043b171 f   LIBCMT:invarg.obj
 0001:0003a180       __invoke_watson            0043b180 f   LIBCMT:invarg.obj
 0001:0003a2a8       __set_invalid_parameter_handler 0043b2a8 f   LIBCMT:invarg.obj
 0001:0003a2cf       __get_invalid_parameter_handler 0043b2cf f   LIBCMT:invarg.obj
 0001:0003a2dc       ?_invoke_watson@@YAXPBG00II@Z 0043b2dc f   LIBCMT:invarg.obj
 0001:0003a2e7       __invalid_parameter        0043b2e7 f   LIBCMT:invarg.obj
 0001:0003a30d       __invalid_parameter_noinfo 0043b30d f   LIBCMT:invarg.obj
 0001:0003a31d       ?_invalid_parameter@@YAXPBG00II@Z 0043b31d f   LIBCMT:invarg.obj
 0001:0003a328       __vswprintf_helper         0043b328 f   LIBCMT:vswprnc.obj
 0001:0003a420       __vswprintf_c              0043b420 f   LIBCMT:vswprnc.obj
 0001:0003a449       __vswprintf_c_l            0043b449 f   LIBCMT:vswprnc.obj
 0001:0003a473       __vswprintf_s_l            0043b473 f   LIBCMT:vswprnc.obj
 0001:0003a4fe       _vswprintf_s               0043b4fe f   LIBCMT:vswprnc.obj
 0001:0003a51b       __vsnwprintf_s_l           0043b51b f   LIBCMT:vswprnc.obj
 0001:0003a627       __vsnwprintf_s             0043b627 f   LIBCMT:vswprnc.obj
 0001:0003a647       __vswprintf_p              0043b647 f   LIBCMT:vswprnc.obj
 0001:0003a670       __vswprintf_p_l            0043b670 f   LIBCMT:vswprnc.obj
 0001:0003a69a       _fwprintf                  0043b69a f   LIBCMT:fwprintf.obj
 0001:0003a72e       __fwprintf_l               0043b72e f   LIBCMT:fwprintf.obj
 0001:0003a74a       __fwprintf_s_l             0043b74a f   LIBCMT:fwprintf.obj
 0001:0003a766       _fwprintf_s                0043b766 f   LIBCMT:fwprintf.obj
 0001:0003a781       __fwprintf_p_l             0043b781 f   LIBCMT:fwprintf.obj
 0001:0003a79d       __fwprintf_p               0043b79d f   LIBCMT:fwprintf.obj
 0001:0003a7b8       _abort                     0043b7b8 f   LIBCMT:abort.obj
 0001:0003a8cf       __set_abort_behavior       0043b8cf f   LIBCMT:abort.obj
 0001:0003a8f0       __initp_misc_winsig        0043b8f0 f   LIBCMT:winsig.obj
 0001:0003a9e0       ___get_sigabrt             0043b9e0 f   LIBCMT:winsig.obj
 0001:0003a9ed       ___fpecode                 0043b9ed f   LIBCMT:winsig.obj
 0001:0003a9f6       ___pxcptinfoptrs           0043b9f6 f   LIBCMT:winsig.obj
 0001:0003a9ff       _signal                    0043b9ff f   LIBCMT:winsig.obj
 0001:0003ac3c       _raise                     0043bc3c f   LIBCMT:winsig.obj
 0001:0003adec       ___crtMessageBoxW          0043bdec f   LIBCMT:crtmboxw.obj
 0001:0003b04b       __itow_s                   0043c04b f   LIBCMT:xtows.obj
 0001:0003b077       __ltow_s                   0043c077 f   LIBCMT:xtows.obj
 0001:0003b09e       __ultow_s                  0043c09e f   LIBCMT:xtows.obj
 0001:0003b1be       __i64tow_s                 0043c1be f   LIBCMT:xtows.obj
 0001:0003b1f3       __ui64tow_s                0043c1f3 f   LIBCMT:xtows.obj
 0001:0003b212       _wcsncat_s                 0043c212 f   LIBCMT:wcsncat_s.obj
 0001:0003b300       _wcsncpy_s                 0043c300 f   LIBCMT:wcsncpy_s.obj
 0001:0003b3d3       _wcslen                    0043c3d3 f   LIBCMT:wcslen.obj
 0001:0003b3ed       _wcscat_s                  0043c3ed f   LIBCMT:wcscat_s.obj
 0001:0003b46a       _wcscpy_s                  0043c46a f   LIBCMT:wcscpy_s.obj
 0001:0003b4d9       __set_error_mode           0043c4d9 f   LIBCMT:errmode.obj
 0001:0003b524       ___set_app_type            0043c524 f   LIBCMT:errmode.obj
 0001:0003b533       ___get_app_type            0043c533 f   LIBCMT:errmode.obj
 0001:0003b539       @__security_check_cookie@4 0043c539 f   LIBCMT:secchk.obj
 0001:0003b548       __stbuf                    0043c548 f   LIBCMT:_sftbuf.obj
 0001:0003b5e4       __ftbuf                    0043c5e4 f   LIBCMT:_sftbuf.obj
 0001:0003b6be       _get_int_arg               0043c6be f i LIBCMT:output.obj
 0001:0003b6d0       _get_int64_arg             0043c6d0 f i LIBCMT:output.obj
 0001:0003b6e5       _get_short_arg             0043c6e5 f i LIBCMT:output.obj
 0001:0003b6f8       __output_l                 0043c6f8 f   LIBCMT:output.obj
 0001:0003c290       ??0exception@std@@QAE@XZ   0043d290 f   LIBCMT:stdexcpt.obj
 0001:0003c2a1       ??0exception@std@@QAE@ABQBD@Z 0043d2a1 f   LIBCMT:stdexcpt.obj
 0001:0003c2f4       ??0exception@std@@QAE@ABQBDH@Z 0043d2f4 f   LIBCMT:stdexcpt.obj
 0001:0003c311       ??0exception@std@@QAE@ABV01@@Z 0043d311 f   LIBCMT:stdexcpt.obj
 0001:0003c36e       ??4exception@std@@QAEAAV01@ABV01@@Z 0043d36e f   LIBCMT:stdexcpt.obj
 0001:0003c3c9       ??1exception@std@@UAE@XZ   0043d3c9 f   LIBCMT:stdexcpt.obj
 0001:0003c3df       ?what@exception@std@@UBEPBDXZ 0043d3df f   LIBCMT:stdexcpt.obj
 0001:0003c3ec       ??0bad_cast@std@@QAE@PBD@Z 0043d3ec f   LIBCMT:stdexcpt.obj
 0001:0003c40a       ??0bad_cast@std@@QAE@ABV01@@Z 0043d40a f   LIBCMT:stdexcpt.obj
 0001:0003c427       ??1bad_cast@std@@UAE@XZ    0043d427 f   LIBCMT:stdexcpt.obj
 0001:0003c432       ??0bad_typeid@std@@QAE@PBD@Z 0043d432 f   LIBCMT:stdexcpt.obj
 0001:0003c450       ??0bad_typeid@std@@QAE@ABV01@@Z 0043d450 f   LIBCMT:stdexcpt.obj
 0001:0003c46d       ??1bad_typeid@std@@UAE@XZ  0043d46d f   LIBCMT:stdexcpt.obj
 0001:0003c478       ??0__non_rtti_object@std@@QAE@PBD@Z 0043d478 f   LIBCMT:stdexcpt.obj
 0001:0003c495       ??0__non_rtti_object@std@@QAE@ABV01@@Z 0043d495 f   LIBCMT:stdexcpt.obj
 0001:0003c4b2       ??1__non_rtti_object@std@@UAE@XZ 0043d4b2 f   LIBCMT:stdexcpt.obj
 0001:0003c4bd       ??_Gexception@std@@UAEPAXI@Z 0043d4bd f i LIBCMT:stdexcpt.obj
 0001:0003c4bd       ??_Eexception@std@@UAEPAXI@Z 0043d4bd f i LIBCMT:stdexcpt.obj
 0001:0003c4de       ??_Gbad_cast@std@@UAEPAXI@Z 0043d4de f i LIBCMT:stdexcpt.obj
 0001:0003c4de       ??_Ebad_cast@std@@UAEPAXI@Z 0043d4de f i LIBCMT:stdexcpt.obj
 0001:0003c505       ??_Gbad_typeid@std@@UAEPAXI@Z 0043d505 f i LIBCMT:stdexcpt.obj
 0001:0003c505       ??_Ebad_typeid@std@@UAEPAXI@Z 0043d505 f i LIBCMT:stdexcpt.obj
 0001:0003c52c       ??_E__non_rtti_object@std@@UAEPAXI@Z 0043d52c f i LIBCMT:stdexcpt.obj
 0001:0003c52c       ??_G__non_rtti_object@std@@UAEPAXI@Z 0043d52c f i LIBCMT:stdexcpt.obj
 0001:0003c553       __CxxThrowException@8      0043d553 f   LIBCMT:throw.obj
 0001:0003c59f       ??0bad_exception@std@@QAE@PBD@Z 0043d59f f i LIBCMT:frame.obj
 0001:0003c5bd       ??1bad_exception@std@@UAE@XZ 0043d5bd f i LIBCMT:frame.obj
 0001:0003c5c8       ??_Gbad_exception@std@@UAEPAXI@Z 0043d5c8 f i LIBCMT:frame.obj
 0001:0003c5c8       ??_Ebad_exception@std@@UAEPAXI@Z 0043d5c8 f i LIBCMT:frame.obj
 0001:0003c5ef       ___TypeMatch               0043d5ef f   LIBCMT:frame.obj
 0001:0003c64e       ___FrameUnwindFilter       0043d64e f   LIBCMT:frame.obj
 0001:0003c697       ___FrameUnwindToState      0043d697 f   LIBCMT:frame.obj
 0001:0003c7bd       ___DestructExceptionObject 0043d7bd f   LIBCMT:frame.obj
 0001:0003c812       ___AdjustPointer           0043d812 f   LIBCMT:frame.obj
 0001:0003c83b       ?__uncaught_exception@@YA_NXZ 0043d83b f   LIBCMT:frame.obj
 0001:0003c84e       ___CxxRegisterExceptionObject 0043d84e f   LIBCMT:frame.obj
 0001:0003c905       ___CxxDetectRethrow        0043d905 f   LIBCMT:frame.obj
 0001:0003c957       ___CxxUnregisterExceptionObject 0043d957 f   LIBCMT:frame.obj
 0001:0003ca96       ___CxxQueryExceptionSize   0043da96 f   LIBCMT:frame.obj
 0001:0003ca9a       ___CxxCallUnwindDtor       0043da9a f   LIBCMT:frame.obj
 0001:0003cacc       ___CxxCallUnwindDelDtor    0043dacc f   LIBCMT:frame.obj
 0001:0003caff       ___CxxCallUnwindStdDelDtor 0043daff f   LIBCMT:frame.obj
 0001:0003cb31       ___CxxCallUnwindVecDtor    0043db31 f   LIBCMT:frame.obj
 0001:0003cc62       ?_is_exception_typeof@@YAHABVtype_info@@PAU_EXCEPTION_POINTERS@@@Z 0043dc62 f   LIBCMT:frame.obj
 0001:0003ce84       ___BuildCatchObjectHelper  0043de84 f   LIBCMT:frame.obj
 0001:0003d003       ___BuildCatchObject        0043e003 f   LIBCMT:frame.obj
 0001:0003d095       ___CxxExceptionFilter      0043e095 f   LIBCMT:frame.obj
 0001:0003d683       ??0bad_exception@std@@QAE@ABV01@@Z 0043e683 f i LIBCMT:frame.obj
 0001:0003d6a0       ___InternalCxxFrameHandler 0043e6a0 f   LIBCMT:frame.obj
 0001:0003d786       __crt_wait_module_handle   0043e786 f i LIBCMT:tidtable.obj
 0001:0003d7a0       __encode_pointer           0043e7a0 f   LIBCMT:tidtable.obj
 0001:0003d812       __encoded_null             0043e812 f   LIBCMT:tidtable.obj
 0001:0003d81b       __decode_pointer           0043e81b f   LIBCMT:tidtable.obj
 0001:0003d88d       ___crtTlsAlloc@4           0043e88d f   LIBCMT:tidtable.obj
 0001:0003d896       ___fls_getvalue@4          0043e896 f   LIBCMT:tidtable.obj
 0001:0003d8b0       ___get_flsindex            0043e8b0 f   LIBCMT:tidtable.obj
 0001:0003d8b6       ___set_flsgetvalue         0043e8b6 f   LIBCMT:tidtable.obj
 0001:0003d8ea       ___fls_setvalue@8          0043e8ea f   LIBCMT:tidtable.obj
 0001:0003d907       __mtterm                   0043e907 f   LIBCMT:tidtable.obj
 0001:0003d944       __initptd                  0043e944 f   LIBCMT:tidtable.obj
 0001:0003da2b       __getptd_noexit            0043ea2b f   LIBCMT:tidtable.obj
 0001:0003daa4       __getptd                   0043eaa4 f   LIBCMT:tidtable.obj
 0001:0003dabe       __freefls@4                0043eabe f   LIBCMT:tidtable.obj
 0001:0003dbed       __freeptd                  0043ebed f   LIBCMT:tidtable.obj
 0001:0003dc5b       ___threadid                0043ec5b f   LIBCMT:tidtable.obj
 0001:0003dc61       ___threadhandle            0043ec61 f   LIBCMT:tidtable.obj
 0001:0003dc67       __mtinit                   0043ec67 f   LIBCMT:tidtable.obj
 0001:0003ddf4       ?terminate@@YAXXZ          0043edf4 f   LIBCMT:hooks.obj
 0001:0003de2d       ?unexpected@@YAXXZ         0043ee2d f   LIBCMT:hooks.obj
 0001:0003de40       ?_inconsistency@@YAXXZ     0043ee40 f   LIBCMT:hooks.obj
 0001:0003de78       __initp_eh_hooks           0043ee78 f   LIBCMT:hooks.obj
 0001:0003de90       __CallSettingFrame@12      0043ee90 f   LIBCMT:lowhelpr.obj
 0001:0003deb7       __NLG_Return               0043eeb7     LIBCMT:lowhelpr.obj
 0001:0003dedc       __flsbuf                   0043eedc f   LIBCMT:_flsbuf.obj
 0001:0003e040       __vsprintf_l               0043f040 f   LIBCMT:vsprintf.obj
 0001:0003e0be       _vsprintf                  0043f0be f   LIBCMT:vsprintf.obj
 0001:0003e0d8       __vscprintf_helper         0043f0d8 f   LIBCMT:vsprintf.obj
 0001:0003e12f       __vscprintf                0043f12f f   LIBCMT:vsprintf.obj
 0001:0003e14b       __vscprintf_l              0043f14b f   LIBCMT:vsprintf.obj
 0001:0003e168       __vscprintf_p              0043f168 f   LIBCMT:vsprintf.obj
 0001:0003e184       __vscprintf_p_l            0043f184 f   LIBCMT:vsprintf.obj
 0001:0003e1a1       ?_Type_info_dtor@type_info@@CAXPAV1@@Z 0043f1a1 f   LIBCMT:typname.obj
 0001:0003e211       ?_Name_base@type_info@@CAPBDPBV1@PAU__type_info_node@@@Z 0043f211 f   LIBCMT:typname.obj
 0001:0003e306       ?_Type_info_dtor_internal@type_info@@CAXPAV1@@Z 0043f306 f   LIBCMT:typname.obj
 0001:0003e376       ___unDNameHelper           0043f376 f   LIBCMT:typname.obj
 0001:0003e3a9       ?_Name_base_internal@type_info@@CAPBDPBV1@PAU__type_info_node@@@Z 0043f3a9 f   LIBCMT:typname.obj
 0001:0003e4b8       ___clean_type_info_names_internal 0043f4b8 f   LIBCMT:typname.obj
 0001:0003e510       _strcmp                    0043f510 f   LIBCMT:strcmp.obj
 0001:0003e598       ___getlocaleinfo           0043f598 f   LIBCMT:inithelp.obj
 0001:0003e717       __initp_misc_purevirt      0043f717 f   LIBCMT:inithelp.obj
 0001:0003e726       _wait_a_bit                0043f726 f i LIBCMT:crtheap.obj
 0001:0003e74c       __set_malloc_crt_max_wait  0043f74c f   LIBCMT:crtheap.obj
 0001:0003e761       __malloc_crt               0043f761 f   LIBCMT:crtheap.obj
 0001:0003e7a6       __calloc_crt               0043f7a6 f   LIBCMT:crtheap.obj
 0001:0003e7f2       __realloc_crt              0043f7f2 f   LIBCMT:crtheap.obj
 0001:0003e840       __recalloc_crt             0043f840 f   LIBCMT:crtheap.obj
 0001:0003e892       __msize                    0043f892 f   LIBCMT:msize.obj
 0001:0003e940       __aulldvrm                 0043f940 f   LIBCMT:ulldvrm.obj
 0001:0003e9d5       ?strrchr@@YAPADPADH@Z      0043f9d5 f i LIBCMT:cvt.obj
 0001:0003e9e0       __forcdecpt_l              0043f9e0 f   LIBCMT:cvt.obj
 0001:0003ea53       __cropzeros_l              0043fa53 f   LIBCMT:cvt.obj
 0001:0003ead5       __positive                 0043fad5 f   LIBCMT:cvt.obj
 0001:0003eaf1       __fassign_l                0043faf1 f   LIBCMT:cvt.obj
 0001:0003eb33       __fassign                  0043fb33 f   LIBCMT:cvt.obj
 0001:0003eb6c       __forcdecpt                0043fb6c f   LIBCMT:cvt.obj
 0001:0003eb7f       __cropzeros                0043fb7f f   LIBCMT:cvt.obj
 0001:0003ed01       __cftoe_l                  0043fd01 f   LIBCMT:cvt.obj
 0001:0003edd1       __cftoe                    0043fdd1 f   LIBCMT:cvt.obj
 0001:0003edf1       __cftoa_l                  0043fdf1 f   LIBCMT:cvt.obj
 0001:0003f164       __cftoa                    00440164 f   LIBCMT:cvt.obj
 0001:0003f27b       __cftof_l                  0044027b f   LIBCMT:cvt.obj
 0001:0003f336       __cftof                    00440336 f   LIBCMT:cvt.obj
 0001:0003f353       __cftog_l                  00440353 f   LIBCMT:cvt.obj
 0001:0003f44d       __cftog                    0044044d f   LIBCMT:cvt.obj
 0001:0003f46d       __cfltcvt_l                0044046d f   LIBCMT:cvt.obj
 0001:0003f4f5       __cfltcvt                  004404f5 f   LIBCMT:cvt.obj
 0001:0003f518       __initp_misc_cfltcvt_tab   00440518 f   LIBCMT:cmiscdat.obj
 0001:0003f539       __setdefaultprecision      00440539 f   LIBCMT:fp8.obj
 0001:0003f564       __ms_p5_test_fdiv          00440564 f   LIBCMT:_testfdiv_.obj
 0001:0003f5a2       __ms_p5_mp_test_fdiv       004405a2 f   LIBCMT:_testfdiv_.obj
 0001:0003f5d0       __ValidateImageBase        004405d0 f   LIBCMT:pesect.obj
 0001:0003f610       __FindPESection            00440610 f   LIBCMT:pesect.obj
 0001:0003f660       __IsNonwritableInCurrentImage 00440660 f   LIBCMT:pesect.obj
 0001:0003f71d       __initp_misc_winxfltr      0044071d f   LIBCMT:winxfltr.obj
 0001:0003f753       __XcptFilter               00440753 f   LIBCMT:winxfltr.obj
 0001:0003f8b3       ___CppXcptFilter           004408b3 f   LIBCMT:winxfltr.obj
 0001:0003f8d3       __close_nolock             004408d3 f   LIBCMT:close.obj
 0001:0003f96f       __close                    0044096f f   LIBCMT:close.obj
 0001:0003fa3c       __fileno                   00440a3c f   LIBCMT:fileno.obj
 0001:0003fa6e       __freebuf                  00440a6e f   LIBCMT:_freebuf.obj
 0001:0003fa9f       __filbuf                   00440a9f f   LIBCMT:_filbuf.obj
 0001:0003fbca       __read_nolock              00440bca f   LIBCMT:read.obj
 0001:0004018c       __read                     0044118c f   LIBCMT:read.obj
 0001:00040289       _memcpy_s                  00441289 f   LIBCMT:memcpy_s.obj
 0001:00040306       __ioinit                   00441306 f   LIBCMT:ioinit.obj
 0001:0004055a       __ioterm                   0044155a f   LIBCMT:ioinit.obj
 0001:000405a8       __lseek_nolock             004415a8 f   LIBCMT:lseek.obj
 0001:0004061d       __lseek                    0044161d f   LIBCMT:lseek.obj
 0001:000406f9       __openfile                 004416f9 f   LIBCMT:_open.obj
 0001:000409c2       __getstream                004419c2 f   LIBCMT:stream.obj
 0001:00040afc       __local_unwind4            00441afc f   LIBCMT:exsup4.obj
 0001:00040bd2       __seh_longjmp_unwind4@4    00441bd2 f   LIBCMT:exsup4.obj
 0001:00040bee       @_EH4_CallFilterFunc@8     00441bee f   LIBCMT:exsup4.obj
 0001:00040c05       @_EH4_TransferToHandler@8  00441c05 f   LIBCMT:exsup4.obj
 0001:00040c1e       @_EH4_GlobalUnwind@4       00441c1e f   LIBCMT:exsup4.obj
 0001:00040c38       @_EH4_LocalUnwind@16       00441c38 f   LIBCMT:exsup4.obj
 0001:00040c4f       __write_nolock             00441c4f f   LIBCMT:write.obj
 0001:00041382       __write                    00442382 f   LIBCMT:write.obj
 0001:00041460       _strlen                    00442460 f   LIBCMT:strlen.obj
 0001:00041542       __INTRN_LOCALE_CONV        00442542 f i LIBCMT:input.obj
 0001:000415c7       __input_l                  004425c7 f   LIBCMT:input.obj
 0001:0004264e       __input_s_l                0044364e f   LIBCMT:inputs.obj
 0001:000439a1       _strtol                    004449a1 f   LIBCMT:strtol.obj
 0001:000439cc       __strtol_l                 004449cc f   LIBCMT:strtol.obj
 0001:000439e9       _strtoul                   004449e9 f   LIBCMT:strtol.obj
 0001:00043a15       __strtoul_l                00444a15 f   LIBCMT:strtol.obj
 0001:00043cc9       __strtoi64                 00444cc9 f   LIBCMT:strtoq.obj
 0001:00043cf4       __strtoi64_l               00444cf4 f   LIBCMT:strtoq.obj
 0001:00043d11       __strtoui64                00444d11 f   LIBCMT:strtoq.obj
 0001:00043d3d       __strtoui64_l              00444d3d f   LIBCMT:strtoq.obj
 0001:00043f80       ___updatetmbcinfo          00444f80 f   LIBCMT:mbctype.obj
 0001:000440a0       __setmbcp_nolock           004450a0 f   LIBCMT:mbctype.obj
 0001:00044285       __getmbcp                  00445285 f   LIBCMT:mbctype.obj
 0001:000442c3       __setmbcp                  004452c3 f   LIBCMT:mbctype.obj
 0001:0004445d       ___initmbctable            0044545d f   LIBCMT:mbctype.obj
 0001:0004447b       ____setlc_active_func      0044547b f   LIBCMT:setlocal.obj
 0001:00044481       ____unguarded_readlc_active_add_func 00445481 f   LIBCMT:setlocal.obj
 0001:00044487       ___freetlocinfo            00445487 f   LIBCMT:setlocal.obj
 0001:000445d0       ___addlocaleref            004455d0 f   LIBCMT:setlocal.obj
 0001:0004465f       ___removelocaleref         0044565f f   LIBCMT:setlocal.obj
 0001:0004475c       ___updatetlocinfo          0044575c f   LIBCMT:setlocal.obj
 0001:000447d2       __configthreadlocale       004457d2 f   LIBCMT:setlocal.obj
 0001:0004488f       __free_locale              0044588f f   LIBCMT:setlocal.obj
 0001:00044951       ___free_locale             00445951 f   LIBCMT:setlocal.obj
 0001:0004495c       __get_current_locale       0044595c f   LIBCMT:setlocal.obj
 0001:00044a0b       ___get_current_locale      00445a0b f   LIBCMT:setlocal.obj
 0001:00044a10       ___init_dummy              00445a10 f   LIBCMT:setlocal.obj
 0001:00044a13       __strcats                  00445a13 f   LIBCMT:setlocal.obj
 0001:00044a53       ___lc_strtolc              00445a53 f   LIBCMT:setlocal.obj
 0001:00044b7c       ___lc_lctostr              00445b7c f   LIBCMT:setlocal.obj
 0001:00044d66       __expandlocale             00445d66 f   LIBCMT:setlocal.obj
 0001:000454b4       __create_locale            004464b4 f   LIBCMT:setlocal.obj
 0001:000455a9       ___create_locale           004465a9 f   LIBCMT:setlocal.obj
 0001:000455b4       _setlocale                 004465b4 f   LIBCMT:setlocal.obj
 0001:00045724       __fltin2                   00446724 f   LIBCMT:_cfin_.obj
 0001:000457cb       __isctype_l                004467cb f   LIBCMT:isctype.obj
 0001:00045883       __isctype                  00446883 f   LIBCMT:isctype.obj
 0001:000458b5       ___addl                    004468b5 f i LIBCMT:_strgtold_.obj
 0001:000458d9       ___shl_12                  004468d9 f i LIBCMT:_strgtold_.obj
 0001:0004590c       ___shr_12                  0044690c f i LIBCMT:_strgtold_.obj
 0001:0004593e       ___ld12mul                 0044693e f i LIBCMT:_strgtold_.obj
 0001:00045bb9       ___multtenpow12            00446bb9 f i LIBCMT:_strgtold_.obj
 0001:00045ebe       ___strgtold12_l            00446ebe f   LIBCMT:_strgtold_.obj
 0001:000465b6       ___STRINGTOLD_L            004475b6 f   LIBCMT:_strgtold_.obj
 0001:000466b7       __output_s_l               004476b7 f   LIBCMT:outputs.obj
 0001:00047287       __validate_param_reuseA    00448287 f   LIBCMT:outputp.obj
 0001:00047458       _get_crtdouble_arg         00448458 f i LIBCMT:outputp.obj
 0001:0004746d       __output_p_l               0044846d f   LIBCMT:outputp.obj
 0001:0004872d       __MarkAllocaS              0044972d f i LIBCMT:a_map.obj
 0001:00048743       __freea                    00449743 f i LIBCMT:a_map.obj
 0001:00048b26       ___crtLCMapStringA         00449b26 f   LIBCMT:a_map.obj
 0001:00048b6b       __isleadbyte_l             00449b6b f i LIBCMT:_wctype.obj
 0001:00048ba3       _isleadbyte                00449ba3 f i LIBCMT:_wctype.obj
 0001:00048bb6       __iswalpha_l               00449bb6 f i LIBCMT:_wctype.obj
 0001:00048bd0       _iswalpha                  00449bd0 f i LIBCMT:_wctype.obj
 0001:00048be6       __iswupper_l               00449be6 f i LIBCMT:_wctype.obj
 0001:00048bfd       _iswupper                  00449bfd f i LIBCMT:_wctype.obj
 0001:00048c10       __iswlower_l               00449c10 f i LIBCMT:_wctype.obj
 0001:00048c27       _iswlower                  00449c27 f i LIBCMT:_wctype.obj
 0001:00048c3a       __iswdigit_l               00449c3a f i LIBCMT:_wctype.obj
 0001:00048c51       _iswdigit                  00449c51 f i LIBCMT:_wctype.obj
 0001:00048c64       __iswxdigit_l              00449c64 f i LIBCMT:_wctype.obj
 0001:00048c7e       _iswxdigit                 00449c7e f i LIBCMT:_wctype.obj
 0001:00048c94       __iswspace_l               00449c94 f i LIBCMT:_wctype.obj
 0001:00048cab       _iswspace                  00449cab f i LIBCMT:_wctype.obj
 0001:00048cbe       __iswpunct_l               00449cbe f i LIBCMT:_wctype.obj
 0001:00048cd5       _iswpunct                  00449cd5 f i LIBCMT:_wctype.obj
 0001:00048ce8       __iswalnum_l               00449ce8 f i LIBCMT:_wctype.obj
 0001:00048d02       _iswalnum                  00449d02 f i LIBCMT:_wctype.obj
 0001:00048d18       __iswprint_l               00449d18 f i LIBCMT:_wctype.obj
 0001:00048d32       _iswprint                  00449d32 f i LIBCMT:_wctype.obj
 0001:00048d48       __iswgraph_l               00449d48 f i LIBCMT:_wctype.obj
 0001:00048d62       _iswgraph                  00449d62 f i LIBCMT:_wctype.obj
 0001:00048d78       __iswcntrl_l               00449d78 f i LIBCMT:_wctype.obj
 0001:00048d8f       _iswcntrl                  00449d8f f i LIBCMT:_wctype.obj
 0001:00048da2       _iswascii                  00449da2 f i LIBCMT:_wctype.obj
 0001:00048db6       __iswcsym_l                00449db6 f i LIBCMT:_wctype.obj
 0001:00048de0       ___iswcsym                 00449de0 f i LIBCMT:_wctype.obj
 0001:00048e06       __iswcsymf_l               00449e06 f i LIBCMT:_wctype.obj
 0001:00048e30       ___iswcsymf                00449e30 f i LIBCMT:_wctype.obj
 0001:00048e56       __fcloseall                00449e56 f   LIBCMT:closeall.obj
 0001:00048ef5       __initp_misc_initcrit      00449ef5 f   LIBCMT:initcrit.obj
 0001:00048f04       ___crtInitCritSecAndSpinCount 00449f04 f   LIBCMT:initcrit.obj
 0001:00048f64       __commit                   00449f64 f   LIBCMT:commit.obj
 0001:00049045       _fgetc                     0044a045 f   LIBCMT:fgetc.obj
 0001:00049149       _getc                      0044a149 f   LIBCMT:fgetc.obj
 0001:0004924d       __getc_nolock              0044a24d f   LIBCMT:fgetc.obj
 0001:0004926d       __sse2_mathfcns_init       0044a26d f   LIBCMT:_mathfcns_.obj
 0001:00049281       __set_SSE2_enable          0044a281 f   LIBCMT:_mathfcns_.obj
 0001:000492a0       __CIcos_pentium4           0044a2a0 f   LIBCMT:_cos_pentium4_.obj
 0001:000492b8       __cos_pentium4             0044a2b8     LIBCMT:_cos_pentium4_.obj
 0001:00049450       __trandisp1                0044a450 f   LIBCMT:_87disp_.obj
 0001:000494b7       __trandisp2                0044a4b7 f   LIBCMT:_87disp_.obj
 0001:00049543       __rttospopde               0044a543     LIBCMT:_87disp_.obj
 0001:00049548       __rttospop                 0044a548     LIBCMT:_87disp_.obj
 0001:0004954a       __rtnospop                 0044a54a     LIBCMT:_87disp_.obj
 0001:0004954c       __rttosnpop                0044a54c     LIBCMT:_87disp_.obj
 0001:0004954d       __rtnospopde               0044a54d     LIBCMT:_87disp_.obj
 0001:00049554       __rtzeropop                0044a554     LIBCMT:_87disp_.obj
 0001:00049556       __rtzeronpop               0044a556     LIBCMT:_87disp_.obj
 0001:0004955b       __rtonepop                 0044a55b     LIBCMT:_87disp_.obj
 0001:0004955d       __rtonenpop                0044a55d     LIBCMT:_87disp_.obj
 0001:00049562       __tosnan1                  0044a562     LIBCMT:_87disp_.obj
 0001:0004958d       __nosnan2                  0044a58d     LIBCMT:_87disp_.obj
 0001:0004958f       __tosnan2                  0044a58f     LIBCMT:_87disp_.obj
 0001:000495b7       __nan2                     0044a5b7     LIBCMT:_87disp_.obj
 0001:000495f6       __rtindfpop                0044a5f6     LIBCMT:_87disp_.obj
 0001:000495f8       __rtindfnpop               0044a5f8     LIBCMT:_87disp_.obj
 0001:00049609       __rttosnpopde              0044a609     LIBCMT:_87disp_.obj
 0001:00049613       __rtchsifneg               0044a613     LIBCMT:_87disp_.obj
 0001:00049620       __twoToTOS                 0044a620 f   LIBCMT:_common_.obj
 0001:00049635       __load_CW                  0044a635 f   LIBCMT:_common_.obj
 0001:0004964c       __convertTOStoQNaN         0044a64c f   LIBCMT:_common_.obj
 0001:00049665       __fload_withFB             0044a665 f   LIBCMT:_common_.obj
 0001:000496a8       __checkTOS_withFB          0044a6a8 f   LIBCMT:_common_.obj
 0001:000496be       __fast_exit                0044a6be f   LIBCMT:_common_.obj
 0001:000496cb       __math_exit                0044a6cb f   LIBCMT:_common_.obj
 0001:000496f5       __check_overflow_exit      0044a6f5 f   LIBCMT:_common_.obj
 0001:00049709       __check_range_exit         0044a709 f   LIBCMT:_common_.obj
 0001:000497b0       __startTwoArgErrorHandling 0044a7b0 f   LIBCMT:_genexcep_.obj
 0001:000497c7       __startOneArgErrorHandling 0044a7c7 f   LIBCMT:_genexcep_.obj
 0001:00049803       ___libm_setusermatherr     0044a803 f   LIBCMT:_libm_error_.obj
 0001:00049831       ___libm_error_support      0044a831 f   LIBCMT:_libm_error_.obj
 0001:00049ae1       __floor_default            0044aae1 f   LIBCMT:_floor_.obj
 0001:00049bc0       __CIsin_pentium4           0044abc0 f   LIBCMT:_sin_pentium4_.obj
 0001:00049bd8       __sin_pentium4             0044abd8     LIBCMT:_sin_pentium4_.obj
 0001:00049d88       _ldexp                     0044ad88 f   LIBCMT:_ldexp_.obj
 0001:00049f3a       __set_exp                  0044af3a f   LIBCMT:_util_.obj
 0001:00049f66       __get_exp                  0044af66 f   LIBCMT:_util_.obj
 0001:00049f7e       __add_exp                  0044af7e f   LIBCMT:_util_.obj
 0001:00049fab       __set_bexp                 0044afab f   LIBCMT:_util_.obj
 0001:00049fd2       __sptype                   0044afd2 f   LIBCMT:_util_.obj
 0001:0004a032       __decomp                   0044b032 f   LIBCMT:_util_.obj
 0001:0004a0eb       __raise_exc_ex             0044b0eb f   LIBCMT:_fpexcept_.obj
 0001:0004a3c7       __raise_exc                0044b3c7 f   LIBCMT:_fpexcept_.obj
 0001:0004a3ea       __raise_excf               0044b3ea f   LIBCMT:_fpexcept_.obj
 0001:0004a40d       __handle_exc               0044b40d f   LIBCMT:_fpexcept_.obj
 0001:0004a5ef       __set_errno_from_matherr   0044b5ef f   LIBCMT:_fpexcept_.obj
 0001:0004a642       __errcode                  0044b642 f   LIBCMT:_fpexcept_.obj
 0001:0004a676       __umatherr                 0044b676 f   LIBCMT:_fpexcept_.obj
 0001:0004a716       __handle_qnan1             0044b716 f   LIBCMT:_fpexcept_.obj
 0001:0004a76b       __handle_qnan2             0044b76b f   LIBCMT:_fpexcept_.obj
 0001:0004a7cc       __except1                  0044b7cc f   LIBCMT:_fpexcept_.obj
 0001:0004a895       __except2                  0044b895 f   LIBCMT:_fpexcept_.obj
 0001:0004a96d       __statfp                   0044b96d f   LIBCMT:_fpctrl_.obj
 0001:0004a97d       __clrfp                    0044b97d f   LIBCMT:_fpctrl_.obj
 0001:0004a98e       __ctrlfp                   0044b98e f   LIBCMT:_fpctrl_.obj
 0001:0004a9b7       __set_statfp               0044b9b7 f   LIBCMT:_fpctrl_.obj
 0001:0004aa0f       ___get_fpsr_sse2           0044ba0f f   LIBCMT:_fpctrl_.obj
 0001:0004aa2d       ___set_fpsr_sse2           0044ba2d f   LIBCMT:_fpctrl_.obj
 0001:0004aa9f       ___fclrf_sse2              0044ba9f f   LIBCMT:_fpctrl_.obj
 0001:0004aabc       ___statfp_sse2             0044babc f   LIBCMT:_fpctrl_.obj
 0001:0004aacf       ___clrfp_sse2              0044bacf f   LIBCMT:_fpctrl_.obj
 0001:0004aae7       ___ctrlfp_sse2             0044bae7 f   LIBCMT:_fpctrl_.obj
 0001:0004ab1e       ___set_statfp_sse2         0044bb1e f   LIBCMT:_fpctrl_.obj
 0001:0004ab39       ?__CxxUnhandledExceptionFilter@@YGJPAU_EXCEPTION_POINTERS@@@Z 0044bb39 f   LIBCMT:unhandld.obj
 0001:0004ab7b       ___CxxSetUnhandledExceptionFilter 0044bb7b f   LIBCMT:unhandld.obj
 0001:0004ab89       __wincmdln                 0044bb89 f   LIBCMT:wincmdln.obj
 0001:0004abe8       __setenvp                  0044bbe8 f   LIBCMT:stdenvp.obj
 0001:0004acc6       __set_pgmptr               0044bcc6 f i LIBCMT:stdargv.obj
 0001:0004ae6f       __setargv                  0044be6f f   LIBCMT:stdargv.obj
 0001:0004af2a       ___crtGetEnvironmentStringsA 0044bf2a f   LIBCMT:a_env.obj
 0001:0004b061       __RTC_Initialize           0044c061 f   LIBCMT:_initsect_.obj
 0001:0004b087       __RTC_Terminate            0044c087 f   LIBCMT:_initsect_.obj
 0001:0004b0ad       ___security_init_cookie    0044c0ad f   LIBCMT:gs_support.obj
 0001:0004b143       __initp_misc_rand_s        0044c143 f   LIBCMT:rand_s.obj
 0001:0004b152       _rand_s                    0044c152 f   LIBCMT:rand_s.obj
 0001:0004b25a       ___crtMessageBoxA          0044c25a f   LIBCMT:crtmbox.obj
 0001:0004b3c3       _strcat_s                  0044c3c3 f   LIBCMT:strcat_s.obj
 0001:0004b437       _strncpy_s                 0044c437 f   LIBCMT:strncpy_s.obj
 0001:0004b4ec       _strcpy_s                  0044c4ec f   LIBCMT:strcpy_s.obj
 0001:0004b554       __crt_debugger_hook        0044c554 f   LIBCMT:dbghook.obj
 0001:0004b604       __woutput_l                0044c604 f   LIBCMT:woutput.obj
 0001:0004c244       __woutput_s_l              0044d244 f   LIBCMT:woutputs.obj
 0001:0004cde4       __validate_param_reuseW    0044dde4 f   LIBCMT:woutputp.obj
 0001:0004cfe2       __woutput_p_l              0044dfe2 f   LIBCMT:woutputp.obj
 0001:0004e2a2       _vfwprintf_helper          0044f2a2 f   LIBCMT:vfwprint.obj
 0001:0004e335       __vfwprintf_l              0044f335 f   LIBCMT:vfwprint.obj
 0001:0004e355       __vfwprintf_s_l            0044f355 f   LIBCMT:vfwprint.obj
 0001:0004e375       __vfwprintf_p_l            0044f375 f   LIBCMT:vfwprint.obj
 0001:0004e395       _vfwprintf                 0044f395 f   LIBCMT:vfwprint.obj
 0001:0004e3b4       _vfwprintf_s               0044f3b4 f   LIBCMT:vfwprint.obj
 0001:0004e3d3       __vfwprintf_p              0044f3d3 f   LIBCMT:vfwprint.obj
 0001:0004e3f2       ___report_gsfailure        0044f3f2 f   LIBCMT:gs_report.obj
 0001:0004e4f8       __isatty                   0044f4f8 f   LIBCMT:isatty.obj
 0001:0004e55c       __wctomb_s_l               0044f55c f   LIBCMT:wctomb.obj
 0001:0004e6c8       _wctomb_s                  0044f6c8 f   LIBCMT:wctomb.obj
 0001:0004e6e5       __wctomb_l                 0044f6e5 f   LIBCMT:wctomb.obj
 0001:0004e736       _wctomb                    0044f736 f   LIBCMT:wctomb.obj
 0001:0004e768       __EH_prolog3               0044f768 f   LIBCMT:ehprolg3.obj
 0001:0004e79b       __EH_prolog3_catch         0044f79b f   LIBCMT:ehprolg3.obj
 0001:0004e7d1       __EH_prolog3_GS            0044f7d1 f   LIBCMT:ehprolg3.obj
 0001:0004e807       __EH_prolog3_catch_GS      0044f807 f   LIBCMT:ehprolg3.obj
 0001:0004e840       __EH_epilog3               0044f840 f   LIBCMT:ehprolg3.obj
 0001:0004e854       __EH_epilog3_GS            0044f854 f   LIBCMT:ehprolg3.obj
 0001:0004e863       __EH_epilog3_catch_GS      0044f863 f   LIBCMT:ehprolg3.obj
 0001:0004e872       ?_ValidateRead@@YAHPBXI@Z  0044f872 f   LIBCMT:validate.obj
 0001:0004e884       ?_ValidateWrite@@YAHPAXI@Z 0044f884 f   LIBCMT:validate.obj
 0001:0004e896       ?_ValidateExecute@@YAHP6GHXZ@Z 0044f896 f   LIBCMT:validate.obj
 0001:0004e8a8       __global_unwind2           0044f8a8 f   LIBCMT:exsup.obj
 0001:0004e90d       __local_unwind2            0044f90d f   LIBCMT:exsup.obj
 0001:0004e991       __abnormal_termination     0044f991 f   LIBCMT:exsup.obj
 0001:0004e9b4       __NLG_Notify1              0044f9b4 f   LIBCMT:exsup.obj
 0001:0004e9bd       __NLG_Notify               0044f9bd f   LIBCMT:exsup.obj
 0001:0004e9d4       __NLG_Dispatch             0044f9d4     LIBCMT:exsup.obj
 0001:0004e9d4       __NLG_Dispatch2            0044f9d4     LIBCMT:exsup.obj
 0001:0004e9dc       __NLG_Call                 0044f9dc f   LIBCMT:exsup.obj
 0001:0004e9de       __NLG_Return2              0044f9de     LIBCMT:exsup.obj
 0001:0004e9df       __lseeki64_nolock          0044f9df f   LIBCMT:lseeki64.obj
 0001:0004ea64       __lseeki64                 0044fa64 f   LIBCMT:lseeki64.obj
 0001:0004eb7d       __getbuf                   0044fb7d f   LIBCMT:_getbuf.obj
 0001:0004ebc6       ??0Block@HeapManager@@QAE@XZ 0044fbc6 f i LIBCMT:undname.obj
 0001:0004ebcc       ?Constructor@HeapManager@@QAEXP6APAXI@ZP6AXPAX@Z@Z 0044fbcc f i LIBCMT:undname.obj
 0001:0004ebeb       ?Destructor@HeapManager@@QAEXXZ 0044fbeb f i LIBCMT:undname.obj
 0001:0004ec13       ?getNumberOfDimensions@UnDecorator@@CAHXZ 0044fc13 f   LIBCMT:undname.obj
 0001:0004ec76       ?getTypeEncoding@UnDecorator@@CAHXZ 0044fc76 f i LIBCMT:undname.obj
 0001:0004f162       ?doUnderScore@UnDecorator@@SAHXZ 00450162 f i LIBCMT:undname.obj
 0001:0004f16d       ?doMSKeywords@UnDecorator@@SAHXZ 0045016d f i LIBCMT:undname.obj
 0001:0004f17a       ?doPtr64@UnDecorator@@SAHXZ 0045017a f i LIBCMT:undname.obj
 0001:0004f188       ?doFunctionReturns@UnDecorator@@SAHXZ 00450188 f i LIBCMT:undname.obj
 0001:0004f196       ?doAllocationModel@UnDecorator@@SAHXZ 00450196 f i LIBCMT:undname.obj
 0001:0004f1a4       ?doAllocationLanguage@UnDecorator@@SAHXZ 004501a4 f i LIBCMT:undname.obj
 0001:0004f1b2       ?doThisTypes@UnDecorator@@SAHXZ 004501b2 f i LIBCMT:undname.obj
 0001:0004f1c4       ?doAccessSpecifiers@UnDecorator@@SAHXZ 004501c4 f i LIBCMT:undname.obj
 0001:0004f1d2       ?doThrowTypes@UnDecorator@@SAHXZ 004501d2 f i LIBCMT:undname.obj
 0001:0004f1e0       ?doMemberTypes@UnDecorator@@SAHXZ 004501e0 f i LIBCMT:undname.obj
 0001:0004f1ee       ?doNameOnly@UnDecorator@@SAHXZ 004501ee f i LIBCMT:undname.obj
 0001:0004f1f9       ?doTypeOnly@UnDecorator@@SAHXZ 004501f9 f i LIBCMT:undname.obj
 0001:0004f204       ?haveTemplateParameters@UnDecorator@@SAHXZ 00450204 f i LIBCMT:undname.obj
 0001:0004f20f       ?doEcsu@UnDecorator@@SAHXZ 0045020f f i LIBCMT:undname.obj
 0001:0004f21d       ?doNoIdentCharCheck@UnDecorator@@SAHXZ 0045021d f i LIBCMT:undname.obj
 0001:0004f228       ?doEllipsis@UnDecorator@@SAHXZ 00450228 f i LIBCMT:undname.obj
 0001:0004f236       ?UScore@UnDecorator@@SAPBDW4Tokens@@@Z 00450236 f   LIBCMT:undname.obj
 0001:0004f254       ?getMemory@HeapManager@@QAEPAXIH@Z 00450254 f   LIBCMT:undname.obj
 0001:0004f2dc       ??0DName@@QAE@XZ           004502dc f i LIBCMT:undname.obj
 0001:0004f2ed       ??0DName@@QAE@ABV0@@Z      004502ed f i LIBCMT:undname.obj
 0001:0004f305       ?isValid@DName@@QBEHXZ     00450305 f i LIBCMT:undname.obj
 0001:0004f30f       ?isEmpty@DName@@QBEHXZ     0045030f f i LIBCMT:undname.obj
 0001:0004f317       ?status@DName@@QBE?AW4DNameStatus@@XZ 00450317 f i LIBCMT:undname.obj
 0001:0004f31c       ?setPtrRef@DName@@QAEAAV1@XZ 0045031c f i LIBCMT:undname.obj
 0001:0004f326       ?isPtrRef@DName@@QBEHXZ    00450326 f i LIBCMT:undname.obj
 0001:0004f330       ?isUDC@DName@@QBEHXZ       00450330 f i LIBCMT:undname.obj
 0001:0004f341       ?setIsUDC@DName@@QAEXXZ    00450341 f i LIBCMT:undname.obj
 0001:0004f34e       ?isUDTThunk@DName@@QBEHXZ  0045034e f i LIBCMT:undname.obj
 0001:0004f35f       ?setIsArray@DName@@QAEXXZ  0045035f f i LIBCMT:undname.obj
 0001:0004f367       ?isArray@DName@@QBEHXZ     00450367 f i LIBCMT:undname.obj
 0001:0004f371       ?isNoTE@DName@@QBEHXZ      00450371 f i LIBCMT:undname.obj
 0001:0004f37b       ?setIsNoTE@DName@@QAEXXZ   0045037b f i LIBCMT:undname.obj
 0001:0004f383       ?isPinPtr@DName@@QBEHXZ    00450383 f i LIBCMT:undname.obj
 0001:0004f38d       ?setIsPinPtr@DName@@QAEXXZ 0045038d f i LIBCMT:undname.obj
 0001:0004f395       ?isComArray@DName@@QBEHXZ  00450395 f i LIBCMT:undname.obj
 0001:0004f39f       ?setIsComArray@DName@@QAEXXZ 0045039f f i LIBCMT:undname.obj
 0001:0004f3a7       ?isVCallThunk@DName@@QBEHXZ 004503a7 f i LIBCMT:undname.obj
 0001:0004f3b1       ?setIsVCallThunk@DName@@QAEXXZ 004503b1 f i LIBCMT:undname.obj
 0001:0004f3b9       ?length@DName@@QBEHXZ      004503b9 f i LIBCMT:undname.obj
 0001:0004f3c6       ?getLastChar@DName@@QBEDXZ 004503c6 f i LIBCMT:undname.obj
 0001:0004f3d4       ?getString@DName@@QBEPADPAD0@Z 004503d4 f i LIBCMT:undname.obj
 0001:0004f3ec       ??_5DName@@QAEAAV0@ABV0@@Z 004503ec f   LIBCMT:undname.obj
 0001:0004f40b       ??4DName@@QAEAAV0@ABV0@@Z  0045040b f   LIBCMT:undname.obj
 0001:0004f423       ?isFull@Replicator@@QBEHXZ 00450423 f i LIBCMT:undname.obj
 0001:0004f42c       ??0Replicator@@QAE@XZ      0045042c f i LIBCMT:undname.obj
 0001:0004f432       ??0DNameNode@@IAE@XZ       00450432 f   LIBCMT:undname.obj
 0001:0004f43b       ??0charNode@@QAE@D@Z       0045043b f   LIBCMT:undname.obj
 0001:0004f452       ?length@charNode@@UBEHXZ   00450452 f i LIBCMT:undname.obj
 0001:0004f456       ?getLastChar@charNode@@UBEDXZ 00450456 f i LIBCMT:undname.obj
 0001:0004f45a       ?getString@charNode@@UBEPADPAD0@Z 0045045a f i LIBCMT:undname.obj
 0001:0004f471       ??0pDNameNode@@QAE@PAVDName@@@Z 00450471 f   LIBCMT:undname.obj
 0001:0004f49b       ?length@pDNameNode@@UBEHXZ 0045049b f i LIBCMT:undname.obj
 0001:0004f4b1       ?getLastChar@pDNameNode@@UBEDXZ 004504b1 f i LIBCMT:undname.obj
 0001:0004f4c8       ?getString@pDNameNode@@UBEPADPAD0@Z 004504c8 f i LIBCMT:undname.obj
 0001:0004f4e1       ??0DNameStatusNode@@AAE@W4DNameStatus@@@Z 004504e1 f   LIBCMT:undname.obj
 0001:0004f506       ?length@DNameStatusNode@@UBEHXZ 00450506 f i LIBCMT:undname.obj
 0001:0004f50a       ?getLastChar@DNameStatusNode@@UBEDXZ 0045050a f i LIBCMT:undname.obj
 0001:0004f516       ?make@DNameStatusNode@@SAPAV1@W4DNameStatus@@@Z 00450516 f i LIBCMT:undname.obj
 0001:0004f59c       ??0pairNode@@QAE@PAVDNameNode@@0@Z 0045059c f   LIBCMT:undname.obj
 0001:0004f5bd       ?length@pairNode@@UBEHXZ   004505bd f i LIBCMT:undname.obj
 0001:0004f5e8       ?getLastChar@pairNode@@UBEDXZ 004505e8 f i LIBCMT:undname.obj
 0001:0004f604       ?getString@pairNode@@UBEPADPAD0@Z 00450604 f i LIBCMT:undname.obj
 0001:0004f67e       ??0UnDecorator@@QAE@PADPBDHP6APADJ@ZK@Z 0045067e f i LIBCMT:undname.obj
 0001:0004f6ed       ?getDataIndirectType@UnDecorator@@CA?AVDName@@XZ 004506ed f i LIBCMT:undname.obj
 0001:0004f722       ?getThisType@UnDecorator@@CA?AVDName@@XZ 00450722 f i LIBCMT:undname.obj
 0001:0004f758       ??2@YAPAXIAAVHeapManager@@H@Z 00450758 f i LIBCMT:undname.obj
 0001:0004f76f       ?getStringHelper@@YAPADPAD00H@Z 0045076f f i LIBCMT:undname.obj
 0001:0004f7a6       ??0DName@@QAE@PAV0@@Z      004507a6 f   LIBCMT:undname.obj
 0001:0004f7f9       ??0DName@@QAE@W4DNameStatus@@@Z 004507f9 f   LIBCMT:undname.obj
 0001:0004f83e       ?getString@DName@@QBEPADPADH@Z 0045083e f i LIBCMT:undname.obj
 0001:0004f896       ?append@DName@@AAEXPAVDNameNode@@@Z 00450896 f   LIBCMT:undname.obj
 0001:0004f8d5       ??4DName@@QAEAAV0@PAV0@@Z  004508d5 f   LIBCMT:undname.obj
 0001:0004f922       ??4DName@@QAEAAV0@W4DNameStatus@@@Z 00450922 f   LIBCMT:undname.obj
 0001:0004f959       ??YReplicator@@QAEAAV0@ABVDName@@@Z 00450959 f   LIBCMT:undname.obj
 0001:0004f9a3       ??AReplicator@@QBE?AVDName@@H@Z 004509a3 f   LIBCMT:undname.obj
 0001:0004f9e3       ??0pcharNode@@QAE@PBDH@Z   004509e3 f   LIBCMT:undname.obj
 0001:0004fa3a       ?length@pcharNode@@UBEHXZ  00450a3a f i LIBCMT:undname.obj
 0001:0004fa3e       ?getLastChar@pcharNode@@UBEDXZ 00450a3e f i LIBCMT:undname.obj
 0001:0004fa50       ?getString@pcharNode@@UBEPADPAD0@Z 00450a50 f i LIBCMT:undname.obj
 0001:0004fa6d       ?getString@DNameStatusNode@@UBEPADPAD0@Z 00450a6d f i LIBCMT:undname.obj
 0001:0004fa96       ?getReturnType@UnDecorator@@CA?AVDName@@PAV2@@Z 00450a96 f   LIBCMT:undname.obj
 0001:0004fac7       ?getStorageConvention@UnDecorator@@CA?AVDName@@XZ 00450ac7 f i LIBCMT:undname.obj
 0001:0004fada       ??YDName@@QAEAAV0@W4DNameStatus@@@Z 00450ada f   LIBCMT:undname.obj
 0001:0004fb1c       ?doPchar@DName@@AAEXPBDH@Z 00450b1c f   LIBCMT:undname.obj
 0001:0004fb98       ??0DName@@QAE@D@Z          00450b98 f   LIBCMT:undname.obj
 0001:0004fbc5       ??0DName@@QAE@PBD@Z        00450bc5 f   LIBCMT:undname.obj
 0001:0004fbfe       ??0DName@@QAE@AAPBDD@Z     00450bfe f   LIBCMT:undname.obj
 0001:0004fcbd       ??0DName@@QAE@_K@Z         00450cbd f   LIBCMT:undname.obj
 0001:0004fd2b       ??0DName@@QAE@_J@Z         00450d2b f   LIBCMT:undname.obj
 0001:0004fdc6       ??HDName@@QBE?AV0@W4DNameStatus@@@Z 00450dc6 f   LIBCMT:undname.obj
 0001:0004fdea       ??YDName@@QAEAAV0@ABV0@@Z  00450dea f   LIBCMT:undname.obj
 0001:0004fe2d       ??YDName@@QAEAAV0@PAV0@@Z  00450e2d f   LIBCMT:undname.obj
 0001:0004fe94       ??4DName@@QAEAAV0@D@Z      00450e94 f i LIBCMT:undname.obj
 0001:0004fec1       ??4DName@@QAEAAV0@PBD@Z    00450ec1 f   LIBCMT:undname.obj
 0001:0004fef6       ?getCallingConvention@UnDecorator@@CA?AVDName@@XZ 00450ef6 f   LIBCMT:undname.obj
 0001:0004ffa0       ?getVCallThunkType@UnDecorator@@CA?AVDName@@XZ 00450fa0 f i LIBCMT:undname.obj
 0001:0004ffd9       ??HDName@@QBE?AV0@ABV0@@Z  00450fd9 f   LIBCMT:undname.obj
 0001:0004fffd       ??HDName@@QBE?AV0@PAV0@@Z  00450ffd f   LIBCMT:undname.obj
 0001:00050021       ??YDName@@QAEAAV0@D@Z      00451021 f   LIBCMT:undname.obj
 0001:00050073       ??YDName@@QAEAAV0@PBD@Z    00451073 f   LIBCMT:undname.obj
 0001:000500d7       ?getArgumentList@UnDecorator@@CA?AVDName@@XZ 004510d7 f   LIBCMT:undname.obj
 0001:000501d9       ?getVdispMapType@UnDecorator@@CA?AVDName@@ABV2@@Z 004511d9 f i LIBCMT:undname.obj
 0001:0005022d       ??H@YA?AVDName@@DABV0@@Z   0045122d f i LIBCMT:undname.obj
 0001:00050251       ??H@YA?AVDName@@W4DNameStatus@@ABV0@@Z 00451251 f i LIBCMT:undname.obj
 0001:00050275       ??H@YA?AVDName@@PBDABV0@@Z 00451275 f i LIBCMT:undname.obj
 0001:00050299       ??HDName@@QBE?AV0@D@Z      00451299 f   LIBCMT:undname.obj
 0001:000502bd       ??HDName@@QBE?AV0@PBD@Z    004512bd f   LIBCMT:undname.obj
 0001:000502e1       ?getDimension@UnDecorator@@CA?AVDName@@_N@Z 004512e1 f   LIBCMT:undname.obj
 0001:00050433       ?getEnumType@UnDecorator@@CA?AVDName@@XZ 00451433 f i LIBCMT:undname.obj
 0001:00050507       ?getArgumentTypes@UnDecorator@@CA?AVDName@@XZ 00451507 f   LIBCMT:undname.obj
 0001:000505e3       ?getThrowTypes@UnDecorator@@CA?AVDName@@XZ 004515e3 f   LIBCMT:undname.obj
 0001:00050662       ?getExtendedDataIndirectType@UnDecorator@@CA?AVDName@@AADAA_NH@Z 00451662 f   LIBCMT:undname.obj
 0001:000507df       ?getArrayType@UnDecorator@@CA?AVDName@@ABV2@@Z 004517df f i LIBCMT:undname.obj
 0001:00050959       ?getLexicalFrame@UnDecorator@@CA?AVDName@@XZ 00451959 f i LIBCMT:undname.obj
 0001:0005098c       ?getDisplacement@UnDecorator@@CA?AVDName@@XZ 0045198c f i LIBCMT:undname.obj
 0001:000509a2       ?getCallIndex@UnDecorator@@CA?AVDName@@XZ 004519a2 f i LIBCMT:undname.obj
 0001:000509b8       ?getGuardNumber@UnDecorator@@CA?AVDName@@XZ 004519b8 f i LIBCMT:undname.obj
 0001:000509ce       ?getVfTableType@UnDecorator@@CA?AVDName@@ABV2@@Z 004519ce f i LIBCMT:undname.obj
 0001:00050b05       ?getStringEncoding@UnDecorator@@CA?AVDName@@PADH@Z 00451b05 f   LIBCMT:undname.obj
 0001:00050ba9       ?getSignedDimension@UnDecorator@@CA?AVDName@@XZ 00451ba9 f   LIBCMT:undname.obj
 0001:00050bfb       ?getTemplateConstant@UnDecorator@@CA?AVDName@@XZ 00451bfb f   LIBCMT:undname.obj
 0001:00050ec8       ?getPtrRefDataType@UnDecorator@@CA?AVDName@@ABV2@H@Z 00451ec8 f i LIBCMT:undname.obj
 0001:00050fa6       ?getVbTableType@UnDecorator@@CA?AVDName@@ABV2@@Z 00451fa6 f i LIBCMT:undname.obj
 0001:00050fbd       ?getTemplateArgumentList@UnDecorator@@CA?AVDName@@XZ 00451fbd f   LIBCMT:undname.obj
 0001:00051181       ?getOperatorName@UnDecorator@@CA?AVDName@@_NPA_N@Z 00452181 f i LIBCMT:undname.obj
 0001:0005171e       ?getTemplateName@UnDecorator@@CA?AVDName@@_N@Z 0045271e f   LIBCMT:undname.obj
 0001:00051865       ?getZName@UnDecorator@@CA?AVDName@@_N0@Z 00452865 f   LIBCMT:undname.obj
 0001:00051a5b       ?getScopedName@UnDecorator@@CA?AVDName@@XZ 00452a5b f   LIBCMT:undname.obj
 0001:00051b2c       ?getECSUName@UnDecorator@@CA?AVDName@@XZ 00452b2c f i LIBCMT:undname.obj
 0001:00051b3f       ?getECSUDataType@UnDecorator@@CA?AVDName@@XZ 00452b3f f   LIBCMT:undname.obj
 0001:00051c46       ?getSymbolName@UnDecorator@@CA?AVDName@@XZ 00452c46 f i LIBCMT:undname.obj
 0001:00051c90       ?getBasedType@UnDecorator@@CA?AVDName@@XZ 00452c90 f   LIBCMT:undname.obj
 0001:00051d28       ?composeDeclaration@UnDecorator@@CA?AVDName@@ABV2@@Z 00452d28 f i LIBCMT:undname.obj
 0001:000528c3       ?getDecoratedName@UnDecorator@@CA?AVDName@@XZ 004538c3 f   LIBCMT:undname.obj
 0001:00052adb       ?getScope@UnDecorator@@CA?AVDName@@XZ 00453adb f   LIBCMT:undname.obj
 0001:00052d4b       ?getFunctionIndirectType@UnDecorator@@CA?AVDName@@ABV2@@Z 00453d4b f   LIBCMT:undname.obj
 0001:0005309f       ?getDataIndirectType@UnDecorator@@CA?AVDName@@ABV2@D0H@Z 0045409f f   LIBCMT:undname.obj
 0001:00053566       ??BUnDecorator@@QAEPADXZ   00454566 f i LIBCMT:undname.obj
 0001:00053697       ?getPtrRefType@UnDecorator@@CA?AVDName@@ABV2@0D@Z 00454697 f   LIBCMT:undname.obj
 0001:00053790       ?getPointerType@UnDecorator@@CA?AVDName@@ABV2@0@Z 00454790 f i LIBCMT:undname.obj
 0001:000537ad       ?getPointerTypeArray@UnDecorator@@CA?AVDName@@ABV2@0@Z 004547ad f i LIBCMT:undname.obj
 0001:000537ca       ?getReferenceType@UnDecorator@@CA?AVDName@@ABV2@0@Z 004547ca f i LIBCMT:undname.obj
 0001:000537e7       ___unDName                 004547e7 f   LIBCMT:undname.obj
 0001:00053881       ___unDNameEx               00454881 f   LIBCMT:undname.obj
 0001:0005391b       ?getBasicDataType@UnDecorator@@CA?AVDName@@ABV2@@Z 0045491b f   LIBCMT:undname.obj
 0001:00053cd2       ?getPrimaryDataType@UnDecorator@@CA?AVDName@@ABV2@@Z 00454cd2 f   LIBCMT:undname.obj
 0001:00053e0a       ?getDataType@UnDecorator@@CA?AVDName@@PAV2@@Z 00454e0a f   LIBCMT:undname.obj
 0001:00053eca       ?getExternalDataType@UnDecorator@@CA?AVDName@@ABV2@@Z 00454eca f i LIBCMT:undname.obj
 0001:00053f51       ___crtGetLocaleInfoW       00454f51 f   LIBCMT:w_loc.obj
 0001:000540c4       ___crtGetLocaleInfoA       004550c4 f   LIBCMT:a_loc.obj
 0001:00054101       __calloc_impl              00455101 f   LIBCMT:calloc_impl.obj
 0001:0005421f       __recalloc                 0045521f f   LIBCMT:recalloc.obj
 0001:000542a0       _strrchr                   004552a0 f   LIBCMT:strrchr.obj
 0001:000542cd       __atodbl_l                 004552cd f   LIBCMT:atodbl.obj
 0001:00054375       __atodbl                   00455375 f   LIBCMT:atodbl.obj
 0001:0005438c       __atoldbl_l                0045538c f   LIBCMT:atodbl.obj
 0001:00054435       __atoldbl                  00455435 f   LIBCMT:atodbl.obj
 0001:0005444c       __atoflt_l                 0045544c f   LIBCMT:atodbl.obj
 0001:000544f4       __atoflt                   004554f4 f   LIBCMT:atodbl.obj
 0001:0005450b       __set_output_format        0045550b f   LIBCMT:outputformat.obj
 0001:00054547       __get_output_format        00455547 f   LIBCMT:outputformat.obj
 0001:0005454d       __fptostr                  0045554d f   LIBCMT:_fptostr.obj
 0001:0005460c       ___dtold                   0045560c f   LIBCMT:_cfout_.obj
 0001:000546c9       __fltout2                  004556c9 f   LIBCMT:_cfout_.obj
 0001:00054760       __aullshr                  00455760 f   LIBCMT:ullshr.obj
 0001:0005477f       __fptrap                   0045577f f   LIBCMT:crt0fp.obj
 0001:00054788       __controlfp_s              00455788 f   LIBCMT:_contrlfp_.obj
 0001:00054f13       __open                     00455f13 f   LIBCMT:open.obj
 0001:00054fc9       __sopen_helper             00455fc9 f   LIBCMT:open.obj
 0001:00055095       __sopen                    00456095 f   LIBCMT:open.obj
 0001:000550c7       __sopen_s                  004560c7 f   LIBCMT:open.obj
 0001:000550e7       __mbsnbicmp_l              004560e7 f   LIBCMT:mbsnbicm.obj
 0001:00055312       __mbsnbicmp                00456312 f   LIBCMT:mbsnbicm.obj
 0001:0005532c       __mbsnbcmp_l               0045632c f   LIBCMT:mbsnbcmp.obj
 0001:00055496       __mbsnbcmp                 00456496 f   LIBCMT:mbsnbcmp.obj
 0001:000554b0       __putwch_nolock            004564b0 f   LIBCMT:putwch.obj
 0001:00055575       __cputws                   00456575 f   LIBCMT:putwch.obj
 0001:00055614       __putwch                   00456614 f   LIBCMT:putwch.obj
 0001:0005565a       __mbtowc_l                 0045665a f   LIBCMT:mbtowc.obj
 0001:00055771       _mbtowc                    00456771 f   LIBCMT:mbtowc.obj
 0001:0005578b       __ungetc_nolock            0045678b f   LIBCMT:ungetc.obj
 0001:0005587c       _ungetc                    0045687c f   LIBCMT:ungetc.obj
 0001:00055aa8       ___crtGetStringTypeA       00456aa8 f   LIBCMT:a_str.obj
 0001:00055aea       ___pwctype_func            00456aea f   LIBCMT:ctype.obj
 0001:00055af0       ___pctype_func             00456af0 f   LIBCMT:ctype.obj
 0001:00055f34       ___free_lc_time            00456f34 f   LIBCMT:inittime.obj
 0001:000560c9       ___init_time               004570c9 f   LIBCMT:inittime.obj
 0001:00056175       ___free_lconv_num          00457175 f   LIBCMT:initnum.obj
 0001:000561ba       ___init_numeric            004571ba f   LIBCMT:initnum.obj
 0001:000563b7       ___free_lconv_mon          004573b7 f   LIBCMT:initmon.obj
 0001:00056445       ___init_monetary           00457445 f   LIBCMT:initmon.obj
 0001:0005670b       ___init_ctype              0045770b f   LIBCMT:initctyp.obj
 0001:00056aad       ____mb_cur_max_func        00457aad f   LIBCMT:initctyp.obj
 0001:00056ad6       ____mb_cur_max_l_func      00457ad6 f   LIBCMT:initctyp.obj
 0001:00056af2       ____lc_codepage_func       00457af2 f   LIBCMT:initctyp.obj
 0001:00056b18       ____lc_collate_cp_func     00457b18 f   LIBCMT:initctyp.obj
 0001:00056b3e       ____lc_handle_func         00457b3e f   LIBCMT:initctyp.obj
 0001:00056b64       ___init_collate            00457b64 f   LIBCMT:initcoll.obj
 0001:00056b67       __Getdays_l                00457b67 f   LIBCMT:strftime.obj
 0001:00056c67       __Getdays                  00457c67 f   LIBCMT:strftime.obj
 0001:00056c70       __Getmonths_l              00457c70 f   LIBCMT:strftime.obj
 0001:00056d70       __Getmonths                00457d70 f   LIBCMT:strftime.obj
 0001:00056d79       __Gettnames_l              00457d79 f   LIBCMT:strftime.obj
 0001:000570d0       __Gettnames                004580d0 f   LIBCMT:strftime.obj
 0001:000579f3       __Strftime_l               004589f3 f   LIBCMT:strftime.obj
 0001:00057b97       __strftime_l               00458b97 f   LIBCMT:strftime.obj
 0001:00057bb7       _strftime                  00458bb7 f   LIBCMT:strftime.obj
 0001:00057bd6       __Strftime                 00458bd6 f   LIBCMT:strftime.obj
 0001:00057bf6       _localeconv                00458bf6 f   LIBCMT:lconv.obj
 0001:00057c20       _strcspn                   00458c20 f   LIBCMT:strcspn.obj
 0001:00058261       ___get_qualified_locale    00459261 f   LIBCMT:getqloc.obj
 0001:000599c8       _memcmp                    0045a9c8 f   LIBCMT:memcmp.obj
 0001:0005b050       _strpbrk                   0045c050 f   LIBCMT:strpbrk.obj
 0001:0005b090       __ZeroTail                 0045c090 f i LIBCMT:_intrncvt_.obj
 0001:0005b0d9       __IncMan                   0045c0d9 f i LIBCMT:_intrncvt_.obj
 0001:0005b146       __RoundMan                 0045c146 f i LIBCMT:_intrncvt_.obj
 0001:0005b236       __CopyMan                  0045c236 f i LIBCMT:_intrncvt_.obj
 0001:0005b255       __FillZeroMan              0045c255 f i LIBCMT:_intrncvt_.obj
 0001:0005b266       __IsZeroMan                0045c266 f i LIBCMT:_intrncvt_.obj
 0001:0005b285       __ShrMan                   0045c285 f i LIBCMT:_intrncvt_.obj
 0001:0005b31f       __ld12cvt                  0045c31f f i LIBCMT:_intrncvt_.obj
 0001:0005b84a       __ld12tod                  0045c84a f   LIBCMT:_intrncvt_.obj
 0001:0005bd8e       __ld12tof                  0045cd8e f   LIBCMT:_intrncvt_.obj
 0001:0005c2d2       __ld12told                 0045d2d2 f   LIBCMT:_intrncvt_.obj
 0001:0005c399       ___add_12                  0045d399 f i LIBCMT:_mantold_.obj
 0001:0005c40a       ___mtold12                 0045d40a f   LIBCMT:_mantold_.obj
 0001:0005c5d8       ___ansicp                  0045d5d8 f   LIBCMT:convrtcp.obj
 0001:0005c621       ___convertcp               0045d621 f   LIBCMT:convrtcp.obj
 0001:0005c7d5       __iswctype_l               0045d7d5 f   LIBCMT:iswctype.obj
 0001:0005c85f       _iswctype                  0045d85f f   LIBCMT:iswctype.obj
 0001:0005c8d5       _is_wctype                 0045d8d5 f   LIBCMT:iswctype.obj
 0001:0005c8e0       __87except                 0045d8e0 f   LIBCMT:_87except_.obj
 0001:0005ca1f       __matherr                  0045da1f f   LIBCMT:_matherr_.obj
 0001:0005ca22       __frnd                     0045da22 f   LIBCMT:_frnd_.obj
 0001:0005ca89       __ismbbkalnum_l            0045da89 f   LIBCMT:ismbbyte.obj
 0001:0005caa2       __ismbbkalnum              0045daa2 f   LIBCMT:ismbbyte.obj
 0001:0005caba       __ismbbkprint_l            0045daba f   LIBCMT:ismbbyte.obj
 0001:0005cad3       __ismbbkprint              0045dad3 f   LIBCMT:ismbbyte.obj
 0001:0005caeb       __ismbbkpunct_l            0045daeb f   LIBCMT:ismbbyte.obj
 0001:0005cb04       __ismbbkpunct              0045db04 f   LIBCMT:ismbbyte.obj
 0001:0005cb1c       __ismbbalnum_l             0045db1c f   LIBCMT:ismbbyte.obj
 0001:0005cb38       __ismbbalnum               0045db38 f   LIBCMT:ismbbyte.obj
 0001:0005cb53       __ismbbalpha_l             0045db53 f   LIBCMT:ismbbyte.obj
 0001:0005cb6f       __ismbbalpha               0045db6f f   LIBCMT:ismbbyte.obj
 0001:0005cb8a       __ismbbgraph_l             0045db8a f   LIBCMT:ismbbyte.obj
 0001:0005cba6       __ismbbgraph               0045dba6 f   LIBCMT:ismbbyte.obj
 0001:0005cbc1       __ismbbprint_l             0045dbc1 f   LIBCMT:ismbbyte.obj
 0001:0005cbdd       __ismbbprint               0045dbdd f   LIBCMT:ismbbyte.obj
 0001:0005cbf8       __ismbbpunct_l             0045dbf8 f   LIBCMT:ismbbyte.obj
 0001:0005cc11       __ismbbpunct               0045dc11 f   LIBCMT:ismbbyte.obj
 0001:0005cc29       __ismbblead_l              0045dc29 f   LIBCMT:ismbbyte.obj
 0001:0005cc42       __ismbblead                0045dc42 f   LIBCMT:ismbbyte.obj
 0001:0005cc5a       __ismbbtrail_l             0045dc5a f   LIBCMT:ismbbyte.obj
 0001:0005cc73       __ismbbtrail               0045dc73 f   LIBCMT:ismbbyte.obj
 0001:0005cc8b       __ismbbkana_l              0045dc8b f   LIBCMT:ismbbyte.obj
 0001:0005cce0       __ismbbkana                0045dce0 f   LIBCMT:ismbbyte.obj
 0001:0005ccf3       __fputwc_nolock            0045dcf3 f   LIBCMT:fputwc.obj
 0001:0005ce7a       _fputwc                    0045de7a f   LIBCMT:fputwc.obj
 0001:0005cef3       _putwc                     0045def3 f   LIBCMT:fputwc.obj
 0001:0005d0f8       _wcstol                    0045e0f8 f   LIBCMT:wcstol.obj
 0001:0005d123       __wcstol_l                 0045e123 f   LIBCMT:wcstol.obj
 0001:0005d140       _wcstoul                   0045e140 f   LIBCMT:wcstol.obj
 0001:0005d16c       __wcstoul_l                0045e16c f   LIBCMT:wcstol.obj
 0001:0005d189       _$I10_OUTPUT               0045e189 f   LIBCMT:_x10fout_.obj
 0001:0005daad       __set_controlfp            0045eaad f   LIBCMT:_ieee87_.obj
 0001:0005de21       __statusfp                 0045ee21 f   LIBCMT:_ieee87_.obj
 0001:0005deb3       __fpreset                  0045eeb3 f   LIBCMT:_ieee87_.obj
 0001:0005e0ec       __statusfp2                0045f0ec f   LIBCMT:_ieee87_.obj
 0001:0005e146       __clearfp                  0045f146 f   LIBCMT:_ieee87_.obj
 0001:0005e21f       ___control87_2             0045f21f f   LIBCMT:_ieee87_.obj
 0001:0005e533       __control87                0045f533 f i LIBCMT:_ieee87_.obj
 0001:0005e842       __controlfp                0045f842 f   LIBCMT:_ieee87_.obj
 0001:0005eb54       __chsize_nolock            0045fb54 f   LIBCMT:chsize.obj
 0001:0005ed0a       __chsize_s                 0045fd0a f   LIBCMT:chsize.obj
 0001:0005edf7       __chsize                   0045fdf7 f   LIBCMT:chsize.obj
 0001:0005ee13       __setmode_nolock           0045fe13 f   LIBCMT:setmode.obj
 0001:0005eecf       __set_fmode                0045fecf f   LIBCMT:setmode.obj
 0001:0005ef1b       __get_fmode                0045ff1b f   LIBCMT:setmode.obj
 0001:0005ef54       __setmode                  0045ff54 f   LIBCMT:setmode.obj
 0001:0005f04b       __strnicmp_l               0046004b f   LIBCMT:strnicmp.obj
 0001:0005f13d       __strnicmp                 0046013d f   LIBCMT:strnicmp.obj
 0001:0005f19b       ___initconin               0046019b f   LIBCMT:initcon.obj
 0001:0005f1ba       ___initconout              004601ba f   LIBCMT:initcon.obj
 0001:0005f1d9       ___termcon                 004601d9 f   LIBCMT:initcon.obj
 0001:0005f206       __get_daylight             00460206 f   LIBCMT:timeset.obj
 0001:0005f23f       __get_dstbias              0046023f f   LIBCMT:timeset.obj
 0001:0005f278       __get_timezone             00460278 f   LIBCMT:timeset.obj
 0001:0005f2b1       __get_tzname               004602b1 f   LIBCMT:timeset.obj
 0001:0005f355       ___daylight                00460355 f   LIBCMT:timeset.obj
 0001:0005f35b       ___dstbias                 0046035b f   LIBCMT:timeset.obj
 0001:0005f361       ___timezone                00460361 f   LIBCMT:timeset.obj
 0001:0005f367       ___tzname                  00460367 f   LIBCMT:timeset.obj
 0001:0005f36d       __set_daylight             0046036d f i LIBCMT:tzset.obj
 0001:0005f37e       __set_dstbias              0046037e f i LIBCMT:tzset.obj
 0001:0005f38f       __set_timezone             0046038f f i LIBCMT:tzset.obj
 0001:0005fab5       ___tzset                   00460ab5 f   LIBCMT:tzset.obj
 0001:0005fb04       __tzset                    00460b04 f   LIBCMT:tzset.obj
 0001:0005fb3c       __isindst                  00460b3c f   LIBCMT:tzset.obj
 0001:0005fb7d       ___ascii_stricmp           00460b7d f   LIBCMT:stricmp.obj
 0001:0005fbb6       __stricmp_l                00460bb6 f   LIBCMT:stricmp.obj
 0001:0005fc8b       __stricmp                  00460c8b f   LIBCMT:stricmp.obj
 0001:0005fdba       __itoa_s                   00460dba f   LIBCMT:xtoas.obj
 0001:0005fde4       __ltoa_s                   00460de4 f   LIBCMT:xtoas.obj
 0001:0005fe0b       __ultoa_s                  00460e0b f   LIBCMT:xtoas.obj
 0001:0005ff1d       __i64toa_s                 00460f1d f   LIBCMT:xtoas.obj
 0001:0005ff52       __ui64toa_s                00460f52 f   LIBCMT:xtoas.obj
 0001:0005ff94       ___crtGetStringTypeW       00460f94 f   LIBCMT:w_str.obj
 0001:0005ffd2       __flswbuf                  00460fd2 f   LIBCMT:_flswbuf.obj
 0001:00060146       __wchartodigit             00461146 f   LIBCMT:wchtodig.obj
 0001:00060330       ___ascii_strnicmp          00461330 f   LIBCMT:_strnicm.obj
 0001:00060391       __getenv_helper_nolock     00461391 f   LIBCMT:getenv.obj
 0001:00060551       _getenv                    00461551 f   LIBCMT:getenv.obj
 0001:000605d4       _getenv_s                  004615d4 f   LIBCMT:getenv.obj
 0001:000606ac       __dupenv_s                 004616ac f   LIBCMT:getenv.obj
 0001:00060792       __mbsnbicoll_l             00461792 f   LIBCMT:mbsnbico.obj
 0001:00060880       __mbsnbicoll               00461880 f   LIBCMT:mbsnbico.obj
 0001:0006089a       ___wtomb_environ           0046189a f   LIBCMT:wtombenv.obj
 0001:00060931       _calloc                    00461931 f   LIBCMT:calloc.obj
 0001:00060971       _strnlen                   00461971 f   LIBCMT:strlen_s.obj
 0001:00060d1c       ___crtCompareStringA       00461d1c f   LIBCMT:a_cmp.obj
 0001:00060d5e       __strnicoll_l              00461d5e f   LIBCMT:strnicol.obj
 0001:00060e58       __strnicoll                00461e58 f   LIBCMT:strnicol.obj
 0001:00060f2d       ___crtsetenv               00461f2d f   LIBCMT:setenv.obj
 0001:00061178       __strdup                   00462178 f   LIBCMT:strdup.obj
 0001:000611cd       __mbschr_l                 004621cd f   LIBCMT:mbschr.obj
 0001:00061289       __mbschr                   00462289 f   LIBCMT:mbschr.obj
 0001:000612a0       _sqlite3_exec              004622a0 f   sqlite3:sqlite3.dll
 0001:000612a6       _sqlite3_close             004622a6 f   sqlite3:sqlite3.dll
 0001:000612ac       _sqlite3_errmsg            004622ac f   sqlite3:sqlite3.dll
 0001:000612b2       _sqlite3_open              004622b2 f   sqlite3:sqlite3.dll
 0001:000612b8       _sqlite3_finalize          004622b8 f   sqlite3:sqlite3.dll
 0001:000612be       _sqlite3_column_text       004622be f   sqlite3:sqlite3.dll
 0001:000612c4       _sqlite3_step              004622c4 f   sqlite3:sqlite3.dll
 0001:000612ca       _sqlite3_prepare_v2        004622ca f   sqlite3:sqlite3.dll
 0001:000612d0       _sqlite3_column_double     004622d0 f   sqlite3:sqlite3.dll
 0001:000612d6       _sqlite3_column_int        004622d6 f   sqlite3:sqlite3.dll
 0001:000612dc       ??0_Init_locks@std@@QAE@XZ 004622dc f   libcpmt:xlock.obj
 0001:0006130d       ??1_Init_locks@std@@QAE@XZ 0046230d f   libcpmt:xlock.obj
 0001:00061336       ?_Init_locks_ctor@_Init_locks@std@@CAXPAV12@@Z 00462336 f   libcpmt:xlock.obj
 0001:0006135f       ?_Init_locks_dtor@_Init_locks@std@@CAXPAV12@@Z 0046235f f   libcpmt:xlock.obj
 0001:00061388       ??0_Lockit@std@@QAE@XZ     00462388 f   libcpmt:xlock.obj
 0001:0006139f       ??0_Lockit@std@@QAE@H@Z    0046239f f   libcpmt:xlock.obj
 0001:000613c7       ??1_Lockit@std@@QAE@XZ     004623c7 f   libcpmt:xlock.obj
 0001:000613de       ?_Lockit_ctor@_Lockit@std@@CAXPAV12@@Z 004623de f   libcpmt:xlock.obj
 0001:000613ea       ?_Lockit_ctor@_Lockit@std@@CAXPAV12@H@Z 004623ea f   libcpmt:xlock.obj
 0001:0006140b       ?_Lockit_dtor@_Lockit@std@@CAXPAV12@@Z 0046240b f   libcpmt:xlock.obj
 0001:00061426       ?_Lockit_ctor@_Lockit@std@@SAXH@Z 00462426 f   libcpmt:xlock.obj
 0001:00061442       ?_Lockit_dtor@_Lockit@std@@SAXH@Z 00462442 f   libcpmt:xlock.obj
 0001:0006145e       ?_Decref@facet@locale@std@@QAEPAV123@XZ 0046245e f i libcpmt:ios.obj
 0001:0006149b       ??1locale@std@@QAE@XZ      0046249b f i libcpmt:ios.obj
 0001:000614b3       ?_Callfns@ios_base@std@@AAEXW4event@12@@Z 004624b3 f i libcpmt:ios.obj
 0001:000614da       ?_Tidy@ios_base@std@@AAAXXZ 004624da f i libcpmt:ios.obj
 0001:00061525       ?_Fpz_func@std@@YAAA_JXZ   00462525 f   libcpmt:ios.obj
 0001:0006152b       ?_BADOFF_func@std@@YAABJXZ 0046252b f   libcpmt:ios.obj
 0001:00061531       ?_Index_func@ios_base@std@@CAAAHXZ 00462531 f   libcpmt:ios.obj
 0001:00061537       ?_Sync_func@ios_base@std@@CAAA_NXZ 00462537 f   libcpmt:ios.obj
 0001:0006153d       ??_Glocale@std@@QAEPAXI@Z  0046253d f i libcpmt:ios.obj
 0001:0006155e       ?_Addstd@ios_base@std@@SAXPAV12@@Z 0046255e f   libcpmt:ios.obj
 0001:000615b0       ?_Ios_base_dtor@ios_base@std@@CAXPAV12@@Z 004625b0 f   libcpmt:ios.obj
 0001:000615ec       __Once                     004625ec f   libcpmt:xmtx.obj
 0001:00061627       __Mtxinit                  00462627 f   libcpmt:xmtx.obj
 0001:00061637       __Mtxdst                   00462637 f   libcpmt:xmtx.obj
 0001:00061647       __Mtxlock                  00462647 f   libcpmt:xmtx.obj
 0001:00061657       __Mtxunlock                00462657 f   libcpmt:xmtx.obj
 0001:00061668       _HeapAlloc@12              00462668 f   kernel32:KERNEL32.dll
 0001:0006166e       _GetLastError@0            0046266e f   kernel32:KERNEL32.dll
 0001:00061674       _HeapFree@12               00462674 f   kernel32:KERNEL32.dll
 0001:0006167a       _HeapReAlloc@16            0046267a f   kernel32:KERNEL32.dll
 0001:00061680       _WriteConsoleW@20          00462680 f   kernel32:KERNEL32.dll
 0001:00061686       _GetFileType@4             00462686 f   kernel32:KERNEL32.dll
 0001:0006168c       _GetModuleFileNameW@12     0046268c f   kernel32:KERNEL32.dll
 0001:00061692       _RtlUnwind@16              00462692 f   kernel32:KERNEL32.dll
 0001:00061698       _ExitThread@4              00462698 f   kernel32:KERNEL32.dll
 0001:0006169e       _GetCurrentThreadId@0      0046269e f   kernel32:KERNEL32.dll
 0001:000616a4       _SetStdHandle@8            004626a4 f   kernel32:KERNEL32.dll
 0001:000616aa       _GetCommandLineA@0         004626aa f   kernel32:KERNEL32.dll
 0001:000616b0       _GetStartupInfoA@4         004626b0 f   kernel32:KERNEL32.dll
 0001:000616b6       _FatalAppExitA@8           004626b6 f   kernel32:KERNEL32.dll
 0001:000616bc       _VirtualFree@12            004626bc f   kernel32:KERNEL32.dll
 0001:000616c2       _VirtualAlloc@16           004626c2 f   kernel32:KERNEL32.dll
 0001:000616c8       _HeapCreate@12             004626c8 f   kernel32:KERNEL32.dll
 0001:000616ce       _HeapDestroy@4             004626ce f   kernel32:KERNEL32.dll
 0001:000616d4       _GetModuleHandleW@4        004626d4 f   kernel32:KERNEL32.dll
 0001:000616da       _GetProcAddress@8          004626da f   kernel32:KERNEL32.dll
 0001:000616e0       _WriteFile@20              004626e0 f   kernel32:KERNEL32.dll
 0001:000616e6       _GetModuleFileNameA@12     004626e6 f   kernel32:KERNEL32.dll
 0001:000616ec       _TerminateProcess@8        004626ec f   kernel32:KERNEL32.dll
 0001:000616f2       _GetCurrentProcess@0       004626f2 f   kernel32:KERNEL32.dll
 0001:000616f8       _UnhandledExceptionFilter@4 004626f8 f   kernel32:KERNEL32.dll
 0001:000616fe       _SetUnhandledExceptionFilter@4 004626fe f   kernel32:KERNEL32.dll
 0001:00061704       _IsDebuggerPresent@0       00462704 f   kernel32:KERNEL32.dll
 0001:0006170a       _LoadLibraryW@4            0046270a f   kernel32:KERNEL32.dll
 0001:00061710       _RaiseException@16         00462710 f   kernel32:KERNEL32.dll
 0001:00061716       _TlsGetValue@4             00462716 f   kernel32:KERNEL32.dll
 0001:0006171c       _TlsAlloc@0                0046271c f   kernel32:KERNEL32.dll
 0001:00061722       _TlsSetValue@8             00462722 f   kernel32:KERNEL32.dll
 0001:00061728       _TlsFree@4                 00462728 f   kernel32:KERNEL32.dll
 0001:0006172e       _InterlockedIncrement@4    0046272e f   kernel32:KERNEL32.dll
 0001:00061734       _SetLastError@4            00462734 f   kernel32:KERNEL32.dll
 0001:0006173a       _InterlockedDecrement@4    0046273a f   kernel32:KERNEL32.dll
 0001:00061740       _GetCurrentThread@0        00462740 f   kernel32:KERNEL32.dll
 0001:00061746       _HeapSize@12               00462746 f   kernel32:KERNEL32.dll
 0001:0006174c       _MultiByteToWideChar@24    0046274c f   kernel32:KERNEL32.dll
 0001:00061752       _ReadFile@20               00462752 f   kernel32:KERNEL32.dll
 0001:00061758       _SetHandleCount@4          00462758 f   kernel32:KERNEL32.dll
 0001:0006175e       _SetFilePointer@16         0046275e f   kernel32:KERNEL32.dll
 0001:00061764       _WideCharToMultiByte@32    00462764 f   kernel32:KERNEL32.dll
 0001:0006176a       _GetConsoleCP@0            0046276a f   kernel32:KERNEL32.dll
 0001:00061770       _GetConsoleMode@8          00462770 f   kernel32:KERNEL32.dll
 0001:00061776       _GetCPInfo@8               00462776 f   kernel32:KERNEL32.dll
 0001:0006177c       _GetACP@0                  0046277c f   kernel32:KERNEL32.dll
 0001:00061782       _GetOEMCP@0                00462782 f   kernel32:KERNEL32.dll
 0001:00061788       _IsValidCodePage@4         00462788 f   kernel32:KERNEL32.dll
 0001:0006178e       _LCMapStringA@24           0046278e f   kernel32:KERNEL32.dll
 0001:00061794       _LCMapStringW@24           00462794 f   kernel32:KERNEL32.dll
 0001:0006179a       _InitializeCriticalSectionAndSpinCount@8 0046279a f   kernel32:KERNEL32.dll
 0001:000617a0       _FlushFileBuffers@4        004627a0 f   kernel32:KERNEL32.dll
 0001:000617a6       _FreeEnvironmentStringsA@4 004627a6 f   kernel32:KERNEL32.dll
 0001:000617ac       _GetEnvironmentStrings@0   004627ac f   kernel32:KERNEL32.dll
 0001:000617b2       _FreeEnvironmentStringsW@4 004627b2 f   kernel32:KERNEL32.dll
 0001:000617b8       _GetEnvironmentStringsW@0  004627b8 f   kernel32:KERNEL32.dll
 0001:000617be       _GetCurrentProcessId@0     004627be f   kernel32:KERNEL32.dll
 0001:000617c4       _GetSystemTimeAsFileTime@4 004627c4 f   kernel32:KERNEL32.dll
 0001:000617ca       _FreeLibrary@4             004627ca f   kernel32:KERNEL32.dll
 0001:000617d0       _InterlockedExchange@8     004627d0 f   kernel32:KERNEL32.dll
 0001:000617d6       _LoadLibraryA@4            004627d6 f   kernel32:KERNEL32.dll
 0001:000617dc       _GetLocaleInfoW@16         004627dc f   kernel32:KERNEL32.dll
 0001:000617e2       _GetLocaleInfoA@16         004627e2 f   kernel32:KERNEL32.dll
 0001:000617e8       _CreateFileA@28            004627e8 f   kernel32:KERNEL32.dll
 0001:000617ee       _WriteConsoleA@20          004627ee f   kernel32:KERNEL32.dll
 0001:000617f4       _GetConsoleOutputCP@0      004627f4 f   kernel32:KERNEL32.dll
 0001:000617fa       _GetStringTypeA@20         004627fa f   kernel32:KERNEL32.dll
 0001:00061800       _GetStringTypeW@16         00462800 f   kernel32:KERNEL32.dll
 0001:00061806       _GetTimeFormatA@24         00462806 f   kernel32:KERNEL32.dll
 0001:0006180c       _GetDateFormatA@24         0046280c f   kernel32:KERNEL32.dll
 0001:00061812       _GetUserDefaultLCID@0      00462812 f   kernel32:KERNEL32.dll
 0001:00061818       _EnumSystemLocalesA@8      00462818 f   kernel32:KERNEL32.dll
 0001:0006181e       _IsValidLocale@8           0046281e f   kernel32:KERNEL32.dll
 0001:00061824       _SetEndOfFile@4            00462824 f   kernel32:KERNEL32.dll
 0001:0006182a       _GetProcessHeap@0          0046282a f   kernel32:KERNEL32.dll
 0001:00061830       _GetTimeZoneInformation@4  00462830 f   kernel32:KERNEL32.dll
 0001:00061836       _CompareStringA@24         00462836 f   kernel32:KERNEL32.dll
 0001:0006183c       _CompareStringW@24         0046283c f   kernel32:KERNEL32.dll
 0001:00061842       _SetEnvironmentVariableA@8 00462842 f   kernel32:KERNEL32.dll
 0002:00000000       __imp__InitCommonControls@0 00465000     comctl32:COMCTL32.dll
 0002:00000004       \177COMCTL32_NULL_THUNK_DATA 00465004     comctl32:COMCTL32.dll
 0002:00000008       __imp__DeleteObject@4      00465008     gdi32:GDI32.dll
 0002:0000000c       __imp__SetBkColor@8        0046500c     gdi32:GDI32.dll
 0002:00000010       __imp__SetTextColor@8      00465010     gdi32:GDI32.dll
 0002:00000014       __imp__ExtTextOutA@32      00465014     gdi32:GDI32.dll
 0002:00000018       __imp__GetDeviceCaps@8     00465018     gdi32:GDI32.dll
 0002:0000001c       __imp__CreateCompatibleDC@4 0046501c     gdi32:GDI32.dll
 0002:00000020       __imp__SelectObject@8      00465020     gdi32:GDI32.dll
 0002:00000024       __imp__DeleteDC@4          00465024     gdi32:GDI32.dll
 0002:00000028       __imp__CreateFontA@56      00465028     gdi32:GDI32.dll
 0002:0000002c       __imp__GetTextMetricsA@8   0046502c     gdi32:GDI32.dll
 0002:00000030       \177GDI32_NULL_THUNK_DATA  00465030     gdi32:GDI32.dll
 0002:00000034       __imp__GetConsoleOutputCP@0 00465034     kernel32:KERNEL32.dll
 0002:00000038       __imp__WriteConsoleA@20    00465038     kernel32:KERNEL32.dll
 0002:0000003c       __imp__CreateFileA@28      0046503c     kernel32:KERNEL32.dll
 0002:00000040       __imp__GetLocaleInfoA@16   00465040     kernel32:KERNEL32.dll
 0002:00000044       __imp__GetLocaleInfoW@16   00465044     kernel32:KERNEL32.dll
 0002:00000048       __imp__LoadLibraryA@4      00465048     kernel32:KERNEL32.dll
 0002:0000004c       __imp__InterlockedExchange@8 0046504c     kernel32:KERNEL32.dll
 0002:00000050       __imp__GetStringTypeA@20   00465050     kernel32:KERNEL32.dll
 0002:00000054       __imp__GetStringTypeW@16   00465054     kernel32:KERNEL32.dll
 0002:00000058       __imp__QueryPerformanceCounter@4 00465058     kernel32:KERNEL32.dll
 0002:0000005c       __imp__QueryPerformanceFrequency@4 0046505c     kernel32:KERNEL32.dll
 0002:00000060       __imp__SetWaitableTimer@24 00465060     kernel32:KERNEL32.dll
 0002:00000064       __imp__CreateWaitableTimerA@12 00465064     kernel32:KERNEL32.dll
 0002:00000068       __imp__CloseHandle@4       00465068     kernel32:KERNEL32.dll
 0002:0000006c       __imp__Sleep@4             0046506c     kernel32:KERNEL32.dll
 0002:00000070       __imp__InitializeCriticalSection@4 00465070     kernel32:KERNEL32.dll
 0002:00000074       __imp__DeleteCriticalSection@4 00465074     kernel32:KERNEL32.dll
 0002:00000078       __imp__EnterCriticalSection@4 00465078     kernel32:KERNEL32.dll
 0002:0000007c       __imp__LeaveCriticalSection@4 0046507c     kernel32:KERNEL32.dll
 0002:00000080       __imp__ExitProcess@4       00465080     kernel32:KERNEL32.dll
 0002:00000084       __imp__ReadConsoleA@20     00465084     kernel32:KERNEL32.dll
 0002:00000088       __imp__FlushConsoleInputBuffer@4 00465088     kernel32:KERNEL32.dll
 0002:0000008c       __imp__SetConsoleMode@8    0046508c     kernel32:KERNEL32.dll
 0002:00000090       __imp__GetStdHandle@4      00465090     kernel32:KERNEL32.dll
 0002:00000094       __imp__SetConsoleCtrlHandler@8 00465094     kernel32:KERNEL32.dll
 0002:00000098       __imp__CreateThread@24     00465098     kernel32:KERNEL32.dll
 0002:0000009c       __imp__SetConsoleTitleA@4  0046509c     kernel32:KERNEL32.dll
 0002:000000a0       __imp__AllocConsole@0      004650a0     kernel32:KERNEL32.dll
 0002:000000a4       __imp__GetTickCount@0      004650a4     kernel32:KERNEL32.dll
 0002:000000a8       __imp__GetLocalTime@4      004650a8     kernel32:KERNEL32.dll
 0002:000000ac       __imp__GetModuleHandleA@4  004650ac     kernel32:KERNEL32.dll
 0002:000000b0       __imp__TerminateThread@8   004650b0     kernel32:KERNEL32.dll
 0002:000000b4       __imp__GetConsoleWindow@0  004650b4     kernel32:KERNEL32.dll
 0002:000000b8       __imp__lstrlenA@4          004650b8     kernel32:KERNEL32.dll
 0002:000000bc       __imp__MulDiv@12           004650bc     kernel32:KERNEL32.dll
 0002:000000c0       __imp__FreeLibrary@4       004650c0     kernel32:KERNEL32.dll
 0002:000000c4       __imp__GetSystemTimeAsFileTime@4 004650c4     kernel32:KERNEL32.dll
 0002:000000c8       __imp__GetCurrentProcessId@0 004650c8     kernel32:KERNEL32.dll
 0002:000000cc       __imp__GetTimeFormatA@24   004650cc     kernel32:KERNEL32.dll
 0002:000000d0       __imp__FreeEnvironmentStringsW@4 004650d0     kernel32:KERNEL32.dll
 0002:000000d4       __imp__GetEnvironmentStrings@0 004650d4     kernel32:KERNEL32.dll
 0002:000000d8       __imp__FreeEnvironmentStringsA@4 004650d8     kernel32:KERNEL32.dll
 0002:000000dc       __imp__FlushFileBuffers@4  004650dc     kernel32:KERNEL32.dll
 0002:000000e0       __imp__InitializeCriticalSectionAndSpinCount@8 004650e0     kernel32:KERNEL32.dll
 0002:000000e4       __imp__LCMapStringW@24     004650e4     kernel32:KERNEL32.dll
 0002:000000e8       __imp__LCMapStringA@24     004650e8     kernel32:KERNEL32.dll
 0002:000000ec       __imp__IsValidCodePage@4   004650ec     kernel32:KERNEL32.dll
 0002:000000f0       __imp__GetOEMCP@0          004650f0     kernel32:KERNEL32.dll
 0002:000000f4       __imp__GetACP@0            004650f4     kernel32:KERNEL32.dll
 0002:000000f8       __imp__GetCPInfo@8         004650f8     kernel32:KERNEL32.dll
 0002:000000fc       __imp__GetConsoleMode@8    004650fc     kernel32:KERNEL32.dll
 0002:00000100       __imp__GetConsoleCP@0      00465100     kernel32:KERNEL32.dll
 0002:00000104       __imp__WideCharToMultiByte@32 00465104     kernel32:KERNEL32.dll
 0002:00000108       __imp__SetFilePointer@16   00465108     kernel32:KERNEL32.dll
 0002:0000010c       __imp__SetHandleCount@4    0046510c     kernel32:KERNEL32.dll
 0002:00000110       __imp__ReadFile@20         00465110     kernel32:KERNEL32.dll
 0002:00000114       __imp__MultiByteToWideChar@24 00465114     kernel32:KERNEL32.dll
 0002:00000118       __imp__HeapSize@12         00465118     kernel32:KERNEL32.dll
 0002:0000011c       __imp__GetCurrentThread@0  0046511c     kernel32:KERNEL32.dll
 0002:00000120       __imp__InterlockedDecrement@4 00465120     kernel32:KERNEL32.dll
 0002:00000124       __imp__SetLastError@4      00465124     kernel32:KERNEL32.dll
 0002:00000128       __imp__InterlockedIncrement@4 00465128     kernel32:KERNEL32.dll
 0002:0000012c       __imp__TlsFree@4           0046512c     kernel32:KERNEL32.dll
 0002:00000130       __imp__TlsSetValue@8       00465130     kernel32:KERNEL32.dll
 0002:00000134       __imp__TlsAlloc@0          00465134     kernel32:KERNEL32.dll
 0002:00000138       __imp__TlsGetValue@4       00465138     kernel32:KERNEL32.dll
 0002:0000013c       __imp__RaiseException@16   0046513c     kernel32:KERNEL32.dll
 0002:00000140       __imp__LoadLibraryW@4      00465140     kernel32:KERNEL32.dll
 0002:00000144       __imp__IsDebuggerPresent@0 00465144     kernel32:KERNEL32.dll
 0002:00000148       __imp__SetUnhandledExceptionFilter@4 00465148     kernel32:KERNEL32.dll
 0002:0000014c       __imp__UnhandledExceptionFilter@4 0046514c     kernel32:KERNEL32.dll
 0002:00000150       __imp__GetCurrentProcess@0 00465150     kernel32:KERNEL32.dll
 0002:00000154       __imp__TerminateProcess@8  00465154     kernel32:KERNEL32.dll
 0002:00000158       __imp__GetModuleFileNameA@12 00465158     kernel32:KERNEL32.dll
 0002:0000015c       __imp__WriteFile@20        0046515c     kernel32:KERNEL32.dll
 0002:00000160       __imp__GetProcAddress@8    00465160     kernel32:KERNEL32.dll
 0002:00000164       __imp__GetModuleHandleW@4  00465164     kernel32:KERNEL32.dll
 0002:00000168       __imp__HeapDestroy@4       00465168     kernel32:KERNEL32.dll
 0002:0000016c       __imp__HeapCreate@12       0046516c     kernel32:KERNEL32.dll
 0002:00000170       __imp__GetDateFormatA@24   00465170     kernel32:KERNEL32.dll
 0002:00000174       __imp__GetUserDefaultLCID@0 00465174     kernel32:KERNEL32.dll
 0002:00000178       __imp__EnumSystemLocalesA@8 00465178     kernel32:KERNEL32.dll
 0002:0000017c       __imp__IsValidLocale@8     0046517c     kernel32:KERNEL32.dll
 0002:00000180       __imp__SetEnvironmentVariableA@8 00465180     kernel32:KERNEL32.dll
 0002:00000184       __imp__SetEndOfFile@4      00465184     kernel32:KERNEL32.dll
 0002:00000188       __imp__GetProcessHeap@0    00465188     kernel32:KERNEL32.dll
 0002:0000018c       __imp__GetTimeZoneInformation@4 0046518c     kernel32:KERNEL32.dll
 0002:00000190       __imp__CompareStringA@24   00465190     kernel32:KERNEL32.dll
 0002:00000194       __imp__CompareStringW@24   00465194     kernel32:KERNEL32.dll
 0002:00000198       __imp__GetEnvironmentStringsW@0 00465198     kernel32:KERNEL32.dll
 0002:0000019c       __imp__VirtualAlloc@16     0046519c     kernel32:KERNEL32.dll
 0002:000001a0       __imp__VirtualFree@12      004651a0     kernel32:KERNEL32.dll
 0002:000001a4       __imp__FatalAppExitA@8     004651a4     kernel32:KERNEL32.dll
 0002:000001a8       __imp__GetStartupInfoA@4   004651a8     kernel32:KERNEL32.dll
 0002:000001ac       __imp__GetCommandLineA@0   004651ac     kernel32:KERNEL32.dll
 0002:000001b0       __imp__SetStdHandle@8      004651b0     kernel32:KERNEL32.dll
 0002:000001b4       __imp__GetCurrentThreadId@0 004651b4     kernel32:KERNEL32.dll
 0002:000001b8       __imp__ExitThread@4        004651b8     kernel32:KERNEL32.dll
 0002:000001bc       __imp__RtlUnwind@16        004651bc     kernel32:KERNEL32.dll
 0002:000001c0       __imp__GetModuleFileNameW@12 004651c0     kernel32:KERNEL32.dll
 0002:000001c4       __imp__GetFileType@4       004651c4     kernel32:KERNEL32.dll
 0002:000001c8       __imp__HeapAlloc@12        004651c8     kernel32:KERNEL32.dll
 0002:000001cc       __imp__GetLastError@0      004651cc     kernel32:KERNEL32.dll
 0002:000001d0       __imp__HeapFree@12         004651d0     kernel32:KERNEL32.dll
 0002:000001d4       __imp__HeapReAlloc@16      004651d4     kernel32:KERNEL32.dll
 0002:000001d8       __imp__WriteConsoleW@20    004651d8     kernel32:KERNEL32.dll
 0002:000001dc       \177KERNEL32_NULL_THUNK_DATA 004651dc     kernel32:KERNEL32.dll
 0002:000001e0       __imp__SetForegroundWindow@4 004651e0     user32:USER32.dll
 0002:000001e4       __imp__SendMessageA@16     004651e4     user32:USER32.dll
 0002:000001e8       __imp__SetWindowTextA@8    004651e8     user32:USER32.dll
 0002:000001ec       __imp__PostQuitMessage@4   004651ec     user32:USER32.dll
 0002:000001f0       __imp__GetWindowTextA@12   004651f0     user32:USER32.dll
 0002:000001f4       __imp__DefWindowProcA@16   004651f4     user32:USER32.dll
 0002:000001f8       __imp__EndPaint@8          004651f8     user32:USER32.dll
 0002:000001fc       __imp__DrawTextA@20        004651fc     user32:USER32.dll
 0002:00000200       __imp__BeginPaint@8        00465200     user32:USER32.dll
 0002:00000204       __imp__GetClientRect@8     00465204     user32:USER32.dll
 0002:00000208       __imp__CreateWindowExA@48  00465208     user32:USER32.dll
 0002:0000020c       __imp__MessageBoxA@16      0046520c     user32:USER32.dll
 0002:00000210       __imp__IsDialogMessageA@8  00465210     user32:USER32.dll
 0002:00000214       __imp__SetFocus@4          00465214     user32:USER32.dll
 0002:00000218       __imp__DrawFocusRect@8     00465218     user32:USER32.dll
 0002:0000021c       __imp__BeginDeferWindowPos@4 0046521c     user32:USER32.dll
 0002:00000220       __imp__DeferWindowPos@32   00465220     user32:USER32.dll
 0002:00000224       __imp__EndDeferWindowPos@4 00465224     user32:USER32.dll
 0002:00000228       __imp__RedrawWindow@16     00465228     user32:USER32.dll
 0002:0000022c       __imp__GetFocus@0          0046522c     user32:USER32.dll
 0002:00000230       __imp__GetKeyState@4       00465230     user32:USER32.dll
 0002:00000234       __imp__GetWindowLongA@8    00465234     user32:USER32.dll
 0002:00000238       __imp__GetParent@4         00465238     user32:USER32.dll
 0002:0000023c       __imp__GetWindow@8         0046523c     user32:USER32.dll
 0002:00000240       __imp__SystemParametersInfoA@16 00465240     user32:USER32.dll
 0002:00000244       __imp__MapWindowPoints@16  00465244     user32:USER32.dll
 0002:00000248       __imp__SetWindowPos@28     00465248     user32:USER32.dll
 0002:0000024c       __imp__GetWindowTextLengthA@4 0046524c     user32:USER32.dll
 0002:00000250       __imp__GetDC@4             00465250     user32:USER32.dll
 0002:00000254       __imp__ReleaseDC@8         00465254     user32:USER32.dll
 0002:00000258       __imp__GetWindowRect@8     00465258     user32:USER32.dll
 0002:0000025c       __imp__LoadIconA@8         0046525c     user32:USER32.dll
 0002:00000260       __imp__LoadCursorA@8       00465260     user32:USER32.dll
 0002:00000264       __imp__RegisterClassExA@4  00465264     user32:USER32.dll
 0002:00000268       __imp__ShowWindow@8        00465268     user32:USER32.dll
 0002:0000026c       __imp__UpdateWindow@4      0046526c     user32:USER32.dll
 0002:00000270       __imp__GetDlgItem@8        00465270     user32:USER32.dll
 0002:00000274       __imp__GetMessageA@16      00465274     user32:USER32.dll
 0002:00000278       __imp__TranslateMessage@4  00465278     user32:USER32.dll
 0002:0000027c       __imp__DispatchMessageA@4  0046527c     user32:USER32.dll
 0002:00000280       __imp__DestroyWindow@4     00465280     user32:USER32.dll
 0002:00000284       __imp__UnregisterClassA@8  00465284     user32:USER32.dll
 0002:00000288       __imp__wvsprintfA@12       00465288     user32:USER32.dll
 0002:0000028c       \177USER32_NULL_THUNK_DATA 0046528c     user32:USER32.dll
 0002:00000290       __imp__socket@12           00465290     ws2_32:WS2_32.dll
 0002:00000294       __imp__setsockopt@20       00465294     ws2_32:WS2_32.dll
 0002:00000298       __imp__ioctlsocket@12      00465298     ws2_32:WS2_32.dll
 0002:0000029c       __imp__bind@12             0046529c     ws2_32:WS2_32.dll
 0002:000002a0       __imp__htons@4             004652a0     ws2_32:WS2_32.dll
 0002:000002a4       __imp__connect@12          004652a4     ws2_32:WS2_32.dll
 0002:000002a8       __imp__WSACleanup@0        004652a8     ws2_32:WS2_32.dll
 0002:000002ac       __imp__WSAStartup@8        004652ac     ws2_32:WS2_32.dll
 0002:000002b0       __imp__closesocket@4       004652b0     ws2_32:WS2_32.dll
 0002:000002b4       __imp__inet_addr@4         004652b4     ws2_32:WS2_32.dll
 0002:000002b8       __imp__inet_ntoa@4         004652b8     ws2_32:WS2_32.dll
 0002:000002bc       __imp__getsockname@12      004652bc     ws2_32:WS2_32.dll
 0002:000002c0       __imp__gethostname@8       004652c0     ws2_32:WS2_32.dll
 0002:000002c4       __imp__sendto@24           004652c4     ws2_32:WS2_32.dll
 0002:000002c8       __imp__WSAGetLastError@0   004652c8     ws2_32:WS2_32.dll
 0002:000002cc       __imp__recvfrom@24         004652cc     ws2_32:WS2_32.dll
 0002:000002d0       __imp__ntohs@4             004652d0     ws2_32:WS2_32.dll
 0002:000002d4       __imp__send@16             004652d4     ws2_32:WS2_32.dll
 0002:000002d8       __imp__gethostbyname@4     004652d8     ws2_32:WS2_32.dll
 0002:000002dc       \177WS2_32_NULL_THUNK_DATA 004652dc     ws2_32:WS2_32.dll
 0002:000002e0       __imp__sqlite3_exec        004652e0     sqlite3:sqlite3.dll
 0002:000002e4       __imp__sqlite3_close       004652e4     sqlite3:sqlite3.dll
 0002:000002e8       __imp__sqlite3_errmsg      004652e8     sqlite3:sqlite3.dll
 0002:000002ec       __imp__sqlite3_open        004652ec     sqlite3:sqlite3.dll
 0002:000002f0       __imp__sqlite3_finalize    004652f0     sqlite3:sqlite3.dll
 0002:000002f4       __imp__sqlite3_column_text 004652f4     sqlite3:sqlite3.dll
 0002:000002f8       __imp__sqlite3_step        004652f8     sqlite3:sqlite3.dll
 0002:000002fc       __imp__sqlite3_prepare_v2  004652fc     sqlite3:sqlite3.dll
 0002:00000300       __imp__sqlite3_column_double 00465300     sqlite3:sqlite3.dll
 0002:00000304       __imp__sqlite3_column_int  00465304     sqlite3:sqlite3.dll
 0002:00000308       \177sqlite3_NULL_THUNK_DATA 00465308     sqlite3:sqlite3.dll
 0002:0000030c       ___xc_a                    0046530c     LIBCMT:crt0init.obj
 0002:00000340       ___xc_z                    00465340     LIBCMT:crt0init.obj
 0002:00000344       ___xi_a                    00465344     LIBCMT:crt0init.obj
 0002:00000360       ___xi_z                    00465360     LIBCMT:crt0init.obj
 0002:00000364       ___xp_a                    00465364     LIBCMT:crt0init.obj
 0002:00000370       ___xp_z                    00465370     LIBCMT:crt0init.obj
 0002:00000374       ___xt_a                    00465374     LIBCMT:crt0init.obj
 0002:00000378       ___xt_z                    00465378     LIBCMT:crt0init.obj
 0002:0000039c       ??_C@_1DO@BPODHJKO@?$AAr?$AAe?$AAa?$AAd?$AAO?$AAf?$AAf?$AAs?$AAe?$AAt?$AA?5?$AA?$DN?$AA?$DN?$AA?5?$AAn?$AAu?$AAm?$AAb?$AAe?$AAr?$AAO?$AAf?$AAB?$AAi?$AAt?$AAs?$AAU?$AAs?$AAe?$AAd?$AA?$AA@ 0046539c     BitStream.obj
 0002:000003dc       ??_C@_1DG@NPGAOJOM@?$AA?4?$AA?4?$AA?2?$AA?4?$AA?4?$AA?2?$AAr?$AAa?$AAk?$AAn?$AAe?$AAt?$AA?2?$AAB?$AAi?$AAt?$AAS?$AAt?$AAr?$AAe?$AAa?$AAm?$AA?4?$AAc?$AAp?$AAp?$AA?$AA@ 004653dc     BitStream.obj
 0002:00000414       ??_C@_08FAMLAKGK@No?5bits?6?$AA@ 00465414     BitStream.obj
 0002:00000420       ??_C@_1CK@LGOIMEII@?$AAi?$AAn?$AAp?$AAu?$AAt?$AA?5?$AA?$CG?$AA?$CG?$AA?5?$AAi?$AAn?$AAp?$AAu?$AAt?$AAL?$AAe?$AAn?$AAg?$AAt?$AAh?$AA?$AA@ 00465420     DataBlockEncryptor.obj
 0002:00000450       ??_C@_1EI@MOBCDLAM@?$AA?4?$AA?4?$AA?2?$AA?4?$AA?4?$AA?2?$AAr?$AAa?$AAk?$AAn?$AAe?$AAt?$AA?2?$AAD?$AAa?$AAt?$AAa?$AAB?$AAl?$AAo?$AAc?$AAk?$AAE?$AAn?$AAc?$AAr?$AAy?$AAp?$AAt?$AAo?$AAr?$AA?4@ 00465450     DataBlockEncryptor.obj
 0002:00000498       ??_C@_1CG@MPAKJGI@?$AAs?$AAi?$AAz?$AAe?$AAI?$AAn?$AAB?$AAy?$AAt?$AAe?$AAs?$AA?5?$AA?$DO?$AA?5?$AA2?$AA0?$AA4?$AA8?$AA?$AA@ 00465498     DataCompressor.obj
 0002:000004c0       ??_C@_1EA@LOKAMDEN@?$AA?4?$AA?4?$AA?2?$AA?4?$AA?4?$AA?2?$AAr?$AAa?$AAk?$AAn?$AAe?$AAt?$AA?2?$AAD?$AAa?$AAt?$AAa?$AAC?$AAo?$AAm?$AAp?$AAr?$AAe?$AAs?$AAs?$AAo?$AAr?$AA?4?$AAc?$AAp?$AAp?$AA?$AA@ 004654c0     DataCompressor.obj
 0002:00000500       ??_C@_1FE@KFPEALKF@?$AAd?$AAe?$AAc?$AAo?$AAm?$AAp?$AAr?$AAe?$AAs?$AAs?$AAe?$AAd?$AAB?$AAy?$AAt?$AAe?$AAs?$AA?$DN?$AA?$DN?$AAd?$AAe?$AAs?$AAt?$AAi?$AAn?$AAa?$AAt?$AAi?$AAo?$AAn?$AAS?$AAi@ 00465500     DataCompressor.obj
 0002:00000554       ??_C@_01EEMJAFIK@?6?$AA@   00465554     DS_ByteQueue.obj
 0002:00000558       ??_C@_03JLNFKLOC@?$CFi?5?$AA@ 00465558     DS_ByteQueue.obj
 0002:0000055c       ??_C@_1BA@MHHNNPBM@?$AAi?$AAs?$AAE?$AAm?$AAp?$AAt?$AAy?$AA?$AA@ 0046555c     DS_Table.obj
 0002:0000056c       ??_C@_1DE@LGNMBKFF@?$AA?4?$AA?4?$AA?2?$AA?4?$AA?4?$AA?2?$AAr?$AAa?$AAk?$AAn?$AAe?$AAt?$AA?2?$AAD?$AAS?$AA_?$AAT?$AAa?$AAb?$AAl?$AAe?$AA?4?$AAc?$AAp?$AAp?$AA?$AA@ 0046556c     DS_Table.obj
 0002:000005a0       ??_C@_1BO@OLJOILKC@?$AAi?$AAs?$AAE?$AAm?$AAp?$AAt?$AAy?$AA?$DN?$AA?$DN?$AAf?$AAa?$AAl?$AAs?$AAe?$AA?$AA@ 004655a0     DS_Table.obj
 0002:000005c0       ??_C@_1BK@CAFOCCOP@?$AAp?$AAa?$AAg?$AAe?$AA?9?$AA?$DO?$AAs?$AAi?$AAz?$AAe?$AA?$DO?$AA0?$AA?$AA@ 004655c0     DS_Table.obj
 0002:000005e0       ??_C@_1GK@LCACLEJK@?$AAc?$AA?3?$AA?2?$AAu?$AAs?$AAe?$AAr?$AAs?$AA?2?$AE?$DP?$AEC?$AEH?$AE?$DO?$AE?3?$AA?2?$AAd?$AAe?$AAs?$AAk?$AAt?$AAo?$AAp?$AA?2?$AAr?$AAa?$AAk?$AAs?$AAa?$AAm?$AAp?$AA?2?$AAr@ 004655e0     DS_Table.obj
 0002:0000064c       ??_C@_02IKAHHCAI@?$CFi?$AA@ 0046564c     DS_Table.obj
 0002:00000650       ??_C@_0CJ@PKINFIOI@Cell?5width?5does?5not?5match?5column@ 00465650     DS_Table.obj
 0002:0000067c       ??_C@_1BC@GBMFMLDI@?$AAb?$AA?$DN?$AA?$DN?$AAf?$AAa?$AAl?$AAs?$AAe?$AA?$AA@ 0046567c     DS_Table.obj
 0002:00000690       ??_C@_1GO@DFNPOHCN@?$AAr?$AAe?$AAt?$AAu?$AAr?$AAn?$AAA?$AAc?$AAt?$AAi?$AAo?$AAn?$AA?9?$AA?$DO?$AAa?$AAc?$AAt?$AAi?$AAo?$AAn?$AA?$DN?$AA?$DN?$AAR?$AAe?$AAt?$AAu?$AAr?$AAn?$AAA?$AAc?$AAt?$AAi@ 00465690     DS_Table.obj
 0002:00000700       ??_C@_1FC@CHFBNAKC@?$AAc?$AAo?$AAl?$AAu?$AAm?$AAn?$AAs?$AA?$FL?$AAc?$AAo?$AAl?$AAu?$AAm?$AAn?$AAI?$AAn?$AAd?$AAe?$AAx?$AA?$FN?$AA?4?$AAc?$AAo?$AAl?$AAu?$AAm?$AAn?$AAT?$AAy?$AAp?$AAe?$AA?$DN@ 00465700     DS_Table.obj
 0002:00000758       ??_C@_1FA@KGODCHJF@?$AAc?$AAo?$AAl?$AAu?$AAm?$AAn?$AAs?$AA?$FL?$AAc?$AAo?$AAl?$AAu?$AAm?$AAn?$AAI?$AAn?$AAd?$AAe?$AAx?$AA?$FN?$AA?4?$AAc?$AAo?$AAl?$AAu?$AAm?$AAn?$AAT?$AAy?$AAp?$AAe?$AA?$DN@ 00465758     DS_Table.obj
 0002:000007a8       ??_C@_1FA@OFEMIOAC@?$AAc?$AAo?$AAl?$AAu?$AAm?$AAn?$AAs?$AA?$FL?$AAc?$AAo?$AAl?$AAu?$AAm?$AAn?$AAI?$AAn?$AAd?$AAe?$AAx?$AA?$FN?$AA?4?$AAc?$AAo?$AAl?$AAu?$AAm?$AAn?$AAT?$AAy?$AAp?$AAe?$AA?$DN@ 004657a8     DS_Table.obj
 0002:000007f8       ??_C@_1GM@PECFPFGO@?$AAr?$AAe?$AAt?$AAu?$AAr?$AAn?$AAA?$AAc?$AAt?$AAi?$AAo?$AAn?$AA?4?$AAa?$AAc?$AAt?$AAi?$AAo?$AAn?$AA?$DN?$AA?$DN?$AAR?$AAe?$AAt?$AAu?$AAr?$AAn?$AAA?$AAc?$AAt?$AAi?$AAo@ 004657f8     DS_Table.obj
 0002:00000868       ??_7NetworkIDGenerator@@6B@ 00465868     NetworkIDGenerator.obj
 0002:00000884       ??_C@_1DO@FONFJDEJ@?$AAp?$AAl?$AAa?$AAy?$AAe?$AAr?$AAI?$AAd?$AA?$CB?$AA?$DN?$AAU?$AAN?$AAA?$AAS?$AAS?$AAI?$AAG?$AAN?$AAE?$AAD?$AA_?$AAP?$AAL?$AAA?$AAY?$AAE?$AAR?$AA_?$AAI?$AAD?$AA?$AA@ 00465884     NetworkIDGenerator.obj
 0002:000008c8       ??_C@_1EI@EHANPGDC@?$AA?4?$AA?4?$AA?2?$AA?4?$AA?4?$AA?2?$AAr?$AAa?$AAk?$AAn?$AAe?$AAt?$AA?2?$AAN?$AAe?$AAt?$AAw?$AAo?$AAr?$AAk?$AAI?$AAD?$AAG?$AAe?$AAn?$AAe?$AAr?$AAa?$AAt?$AAo?$AAr?$AA?4@ 004658c8     NetworkIDGenerator.obj
 0002:00000914       ??_7?$BinarySearchTree@UNetworkIDNode@@@DataStructures@@6B@ 00465914     NetworkIDGenerator.obj
 0002:0000091c       ??_7?$AVLBalancedBinarySearchTree@UNetworkIDNode@@@DataStructures@@6B@ 0046591c     NetworkIDGenerator.obj
 0002:00000920       ??_C@_1EO@EECHBJKE@?$AAe?$AAx?$AAt?$AAe?$AAr?$AAn?$AAa?$AAl?$AAP?$AAl?$AAa?$AAy?$AAe?$AAr?$AAI?$AAd?$AA?$CB?$AA?$DN?$AAU?$AAN?$AAA?$AAS?$AAS?$AAI?$AAG?$AAN?$AAE?$AAD?$AA_?$AAP?$AAL?$AAA@ 00465920     NetworkIDGenerator.obj
 0002:00000970       ??_C@_1CO@EKDMJBHP@?$AAI?$AAs?$AAN?$AAe?$AAt?$AAw?$AAo?$AAr?$AAk?$AAI?$AAD?$AAA?$AAu?$AAt?$AAh?$AAo?$AAr?$AAi?$AAt?$AAy?$AA?$CI?$AA?$CJ?$AA?$AA@ 00465970     NetworkIDGenerator.obj
 0002:000009a0       ??_C@_0BB@JCEFLFJE@0123456789abcdef?$AA@ 004659a0     NetworkTypes.obj
 0002:000009b4       ??_C@_01JLIPDDHJ@?3?$AA@   004659b4     NetworkTypes.obj
 0002:000009bc       ??_7RakClientInterface@@6B@ 004659bc     RakClient.obj
 0002:00000a9c       ??_7RakClient@@6BRakClientInterface@@@ 00465a9c     RakClient.obj
 0002:00000b7c       ??_7RakClient@@6BRakPeer@@@ 00465b7c     RakClient.obj
 0002:00000c88       ??_C@_0EPJ@GHCCKPPI@Bytes?5sent?3?7?7?7?7?$CFu?6Messages?5in?5se@ 00465c88     RakNetStatistics.obj
 0002:00001188       ??_C@_0BGM@MAJEJOFP@Messages?5in?5Send?5buffer?3?5?$CFu?6Mess@ 00466188     RakNetStatistics.obj
 0002:000012f8       __real@41f0000000000000    004662f8     RakNetStatistics.obj
 0002:00001300       __real@408f400000000000    00466300     RakNetStatistics.obj
 0002:00001308       ??_C@_0EC@LDIFCIKH@Total?5bytes?5sent?3?5?$CFu?6Total?5bytes@ 00466308     RakNetStatistics.obj
 0002:00001350       __real@4059000000000000    00466350     RakNetStatistics.obj
 0002:00001358       __real@4f800000            00466358     RakNetStatistics.obj
 0002:0000135c       ??_C@_0CK@JHPDEPLM@stats?5is?5a?5NULL?5pointer?5in?5stats@ 0046635c     RakNetStatistics.obj
 0002:0000158c       ??_7RakPeerInterface@@6B@  0046658c     RakPeer.obj
 0002:00001698       ??_C@_1BK@PNPFLKAA@?$AAl?$AAe?$AAn?$AAg?$AAt?$AAh?$AA?5?$AA?$DM?$AA?5?$AA4?$AA0?$AA0?$AA?$AA@ 00466698     RakPeer.obj
 0002:000016b4       ??_C@_1DC@LCCFDLOH@?$AA?4?$AA?4?$AA?2?$AA?4?$AA?4?$AA?2?$AAr?$AAa?$AAk?$AAn?$AAe?$AAt?$AA?2?$AAR?$AAa?$AAk?$AAP?$AAe?$AAe?$AAr?$AA?4?$AAc?$AAp?$AAp?$AA?$AA@ 004666b4     RakPeer.obj
 0002:000016e8       __real@00000000            004666e8     RakPeer.obj
 0002:000016f0       __real@0000000000000000    004666f0     RakPeer.obj
 0002:000016f8       ??_C@_1DA@FABPCGM@?$AAw?$AAr?$AAi?$AAt?$AAe?$AAA?$AAh?$AAe?$AAa?$AAd?$AAP?$AAo?$AAi?$AAn?$AAt?$AAe?$AAr?$AA?9?$AA?$DO?$AAn?$AAe?$AAx?$AAt?$AA?$AA@ 004666f8     RakPeer.obj
 0002:00001728       ??_C@_1HO@LEEIPPOO@?$AAc?$AA?3?$AA?2?$AAu?$AAs?$AAe?$AAr?$AAs?$AA?2?$AE?$DP?$AEC?$AEH?$AE?$DO?$AE?3?$AA?2?$AAd?$AAe?$AAs?$AAk?$AAt?$AAo?$AAp?$AA?2?$AAr?$AAa?$AAk?$AAs?$AAa?$AAm?$AAp?$AA?2?$AAr@ 00466728     RakPeer.obj
 0002:000017a8       ??_C@_1BM@DNMMOAPD@?$AAd?$AAa?$AAt?$AAa?$AAL?$AAe?$AAn?$AAg?$AAt?$AAh?$AA?$DO?$AA?$DN?$AA0?$AA?$AA@ 004667a8     RakPeer.obj
 0002:000017c8       ??_C@_1EM@PPGDKCEI@?$AAd?$AAa?$AAt?$AAa?$AAL?$AAe?$AAn?$AAg?$AAt?$AAh?$AA?5?$AA?$DM?$AA?$DN?$AA?5?$AAM?$AAA?$AAX?$AA_?$AAO?$AAF?$AAF?$AAL?$AAI?$AAN?$AAE?$AA_?$AAD?$AAA?$AAT?$AAA?$AA_?$AAL@ 004667c8     RakPeer.obj
 0002:00001818       ??_C@_1IK@PCGACABH@?$AAr?$AAe?$AAm?$AAo?$AAt?$AAe?$AAS?$AAy?$AAs?$AAt?$AAe?$AAm?$AAL?$AAi?$AAs?$AAt?$AA?$FL?$AAr?$AAe?$AAm?$AAo?$AAt?$AAe?$AAS?$AAy?$AAs?$AAt?$AAe?$AAm?$AAL?$AAo?$AAo@ 00466818     RakPeer.obj
 0002:000018a4       ??_C@_13COJANIEC@?$AA0?$AA?$AA@ 004668a4     RakPeer.obj
 0002:000018a8       ??_C@_1CG@FNLJFNDG@?$AAo?$AAb?$AAj?$AAe?$AAc?$AAt?$AAE?$AAx?$AAi?$AAs?$AAt?$AAs?$AA?$DN?$AA?$DN?$AAt?$AAr?$AAu?$AAe?$AA?$AA@ 004668a8     RakPeer.obj
 0002:000018d0       ??_C@_1GO@GCMPONFE@?$AAc?$AA?3?$AA?2?$AAu?$AAs?$AAe?$AAr?$AAs?$AA?2?$AE?$DP?$AEC?$AEH?$AE?$DO?$AE?3?$AA?2?$AAd?$AAe?$AAs?$AAk?$AAt?$AAo?$AAp?$AA?2?$AAr?$AAa?$AAk?$AAs?$AAa?$AAm?$AAp?$AA?2?$AAr@ 004668d0     RakPeer.obj
 0002:00001944       ??_7RakPeer@@6B@           00466944     RakPeer.obj
 0002:00001a50       ??_C@_1DE@MHEPBEIO@?$AAp?$AAa?$AAs?$AAs?$AAw?$AAo?$AAr?$AAd?$AAD?$AAa?$AAt?$AAa?$AAL?$AAe?$AAn?$AAg?$AAt?$AAh?$AA?5?$AA?$DM?$AA?$DN?$AA?5?$AA2?$AA5?$AA6?$AA?$AA@ 00466a50     RakPeer.obj
 0002:00001a88       ??_C@_1HO@KBDHKDHK@?$AAr?$AAc?$AAs?$AA?9?$AA?$DO?$AAa?$AAc?$AAt?$AAi?$AAo?$AAn?$AAT?$AAo?$AAT?$AAa?$AAk?$AAe?$AA?$DN?$AA?$DN?$AAR?$AAa?$AAk?$AAP?$AAe?$AAe?$AAr?$AA?3?$AA?3?$AAR?$AAe?$AAq?$AAu@ 00466a88     RakPeer.obj
 0002:00001b08       ??_C@_07OHKHACFK@0?40?40?40?$AA@ 00466b08     RakPeer.obj
 0002:00001b10       ??_C@_09PFCHIMEP@127?40?40?41?$AA@ 00466b10     RakPeer.obj
 0002:00001b1c       ??_C@_1BK@CNLEAJJK@?$AAp?$AAi?$AAn?$AAg?$AA?5?$AA?$DM?$AA?5?$AA1?$AA0?$AA0?$AA0?$AA0?$AA?$AA@ 00466b1c     RakPeer.obj
 0002:00001b38       ??_C@_1BA@ICANLBCA@?$AAs?$AAu?$AAc?$AAc?$AAe?$AAs?$AAs?$AA?$AA@ 00466b38     RakPeer.obj
 0002:00001b48       ??_C@_1BI@JFBHHBPJ@?$AAt?$AAi?$AAm?$AAe?$AAr?$AAH?$AAa?$AAn?$AAd?$AAl?$AAe?$AA?$AA@ 00466b48     RakPeer.obj
 0002:00001b60       ??_C@_1CG@FBMJBJBI@?$AAm?$AAa?$AAx?$AAC?$AAo?$AAn?$AAn?$AAe?$AAc?$AAt?$AAi?$AAo?$AAn?$AAs?$AA?5?$AA?$DO?$AA?5?$AA0?$AA?$AA@ 00466b60     RakPeer.obj
 0002:00001b8c       ??_7RakServerInterface@@6B@ 00466b8c     rakserver.obj
 0002:00001c9c       ??_7RakServer@@6BRakPeer@@@ 00466c9c     rakserver.obj
 0002:00001dac       ??_7RakServer@@6BRakServerInterface@@@ 00466dac     rakserver.obj
 0002:00001eb8       __real@3df0000000000000    00466eb8     Rand.obj
 0002:00001ed8       ??_C@_1CK@KNPFILPK@?$AA?$CI?$AA?5?$AAl?$AAe?$AAn?$AAg?$AAt?$AAh?$AA?5?$AA?$CF?$AA?5?$AA1?$AA6?$AA?5?$AA?$CJ?$AA?5?$AA?$DN?$AA?$DN?$AA?5?$AA0?$AA?$AA@ 00466ed8     ReliabilityLayer.obj
 0002:00001f08       ??_C@_1EE@DEJIGJPH@?$AA?4?$AA?4?$AA?2?$AA?4?$AA?4?$AA?2?$AAr?$AAa?$AAk?$AAn?$AAe?$AAt?$AA?2?$AAR?$AAe?$AAl?$AAi?$AAa?$AAb?$AAi?$AAl?$AAi?$AAt?$AAy?$AAL?$AAa?$AAy?$AAe?$AAr?$AA?4?$AAc?$AAp@ 00466f08     ReliabilityLayer.obj
 0002:00001f50       ??_C@_1EG@DIEFEKLO@?$AAr?$AAa?$AAn?$AAg?$AAe?$AAs?$AA?4?$AAS?$AAi?$AAz?$AAe?$AA?$CI?$AA?$CJ?$AA?5?$AA?$DM?$AA?5?$AA?$CI?$AAu?$AAn?$AAs?$AAi?$AAg?$AAn?$AAe?$AAd?$AA?5?$AAs?$AAh?$AAo?$AAr?$AAt?$AA?$CJ@ 00466f50     ReliabilityLayer.obj
 0002:00001f98       ??_C@_1GK@BNOGMKDK@?$AAc?$AA?3?$AA?2?$AAu?$AAs?$AAe?$AAr?$AAs?$AA?2?$AE?$DP?$AEC?$AEH?$AE?$DO?$AE?3?$AA?2?$AAd?$AAe?$AAs?$AAk?$AAt?$AAo?$AAp?$AA?2?$AAr?$AAa?$AAk?$AAs?$AAa?$AAm?$AAp?$AA?2?$AAr@ 00466f98     ReliabilityLayer.obj
 0002:00002004       __real@3d23d70a            00467004     ReliabilityLayer.obj
 0002:00002008       __real@3ff0cccccccccccd    00467008     ReliabilityLayer.obj
 0002:00002010       __real@3ff8000000000000    00467010     ReliabilityLayer.obj
 0002:00002018       __real@40ac200000000000    00467018     ReliabilityLayer.obj
 0002:00002020       __real@3feccccccccccccd    00467020     ReliabilityLayer.obj
 0002:00002028       __real@3fe0000000000000    00467028     ReliabilityLayer.obj
 0002:00002030       __real@3fc999999999999a    00467030     ReliabilityLayer.obj
 0002:00002038       __real@412e848000000000    00467038     ReliabilityLayer.obj
 0002:00002040       ??_C@_02JDPG@rb?$AA@       00467040     SHA1.obj
 0002:00002044       ??_C@_01LOCGONAA@?$AA?$AA@ 00467044     SHA1.obj
 0002:00002048       ??_C@_01IFKFHFEL@?$IA?$AA@ 00467048     SHA1.obj
 0002:0000204c       ??_C@_0BM@DLILFBO@Error?3?5Unknown?5report?5type?$CB?$AA@ 0046704c     SHA1.obj
 0002:00002068       ??_C@_03BCEHIGGF@?5?$CFu?$AA@ 00467068     SHA1.obj
 0002:0000206c       ??_C@_02GMHACPFF@?$CFu?$AA@ 0046706c     SHA1.obj
 0002:00002070       ??_C@_05OFBGOFBN@?5?$CF02X?$AA@ 00467070     SHA1.obj
 0002:00002078       ??_C@_04JFFKLGJF@?$CF02X?$AA@ 00467078     SHA1.obj
 0002:00002084       ??_7CSHA1@@6B@             00467084     SHA1.obj
 0002:00002088       ??_C@_1DM@IOFBKPGG@?$AAw?$AAr?$AAi?$AAt?$AAe?$AAS?$AAo?$AAc?$AAk?$AAe?$AAt?$AA?5?$AA?$CB?$AA?$DN?$AA?5?$AAI?$AAN?$AAV?$AAA?$AAL?$AAI?$AAD?$AA_?$AAS?$AAO?$AAC?$AAK?$AAE?$AAT?$AA?$AA@ 00467088     SocketLayer.obj
 0002:000020c4       ??_C@_1DK@LDBDLLFF@?$AA?4?$AA?4?$AA?2?$AA?4?$AA?4?$AA?2?$AAr?$AAa?$AAk?$AAn?$AAe?$AAt?$AA?2?$AAS?$AAo?$AAc?$AAk?$AAe?$AAt?$AAL?$AAa?$AAy?$AAe?$AAr?$AA?4?$AAc?$AAp?$AAp?$AA?$AA@ 004670c4     SocketLayer.obj
 0002:00002100       ??_C@_1BK@EBNJALNF@?$AAo?$AAb?$AAj?$AAe?$AAc?$AAt?$AAE?$AAx?$AAi?$AAs?$AAt?$AAs?$AA?$AA@ 00467100     StringCompressor.obj
 0002:00002120       ??_C@_1FO@NDOKBCKF@?$AAc?$AA?3?$AA?2?$AAu?$AAs?$AAe?$AAr?$AAs?$AA?2?$AE?$DP?$AEC?$AEH?$AE?$DO?$AE?3?$AA?2?$AAd?$AAe?$AAs?$AAk?$AAt?$AAo?$AAp?$AA?2?$AAr?$AAa?$AAk?$AAs?$AAa?$AAm?$AAp?$AA?2?$AAr@ 00467120     StringCompressor.obj
 0002:00002180       ??_C@_1CG@DEPNCJGC@?$AAr?$AAe?$AAf?$AAe?$AAr?$AAe?$AAn?$AAc?$AAe?$AAC?$AAo?$AAu?$AAn?$AAt?$AA?5?$AA?$DO?$AA?5?$AA0?$AA?$AA@ 00467180     StringCompressor.obj
 0002:000021a8       ??_C@_1EE@FIBGJMEG@?$AA?4?$AA?4?$AA?2?$AA?4?$AA?4?$AA?2?$AAr?$AAa?$AAk?$AAn?$AAe?$AAt?$AA?2?$AAS?$AAt?$AAr?$AAi?$AAn?$AAg?$AAC?$AAo?$AAm?$AAp?$AAr?$AAe?$AAs?$AAs?$AAo?$AAr?$AA?4?$AAc?$AAp@ 004671a8     StringCompressor.obj
 0002:000021f0       ??_C@_1FO@HDKNIFHI@?$AAo?$AAr?$AAd?$AAe?$AAr?$AAe?$AAd?$AAS?$AAt?$AAr?$AAi?$AAn?$AAg?$AAL?$AAi?$AAs?$AAt?$AA?4?$AAS?$AAi?$AAz?$AAe?$AA?$CI?$AA?$CJ?$AA?5?$AA?$DM?$AA?5?$AA?$CI?$AAS?$AAt?$AAr?$AAi@ 004671f0     StringTable.obj
 0002:00002250       ??_C@_1DK@LNCDDKPM@?$AA?4?$AA?4?$AA?2?$AA?4?$AA?4?$AA?2?$AAr?$AAa?$AAk?$AAn?$AAe?$AAt?$AA?2?$AAS?$AAt?$AAr?$AAi?$AAn?$AAg?$AAT?$AAa?$AAb?$AAl?$AAe?$AA?4?$AAc?$AAp?$AAp?$AA?$AA@ 00467250     StringTable.obj
 0002:0000228c       ??_C@_1CE@IIKHMION@?$AAm?$AAa?$AAx?$AAC?$AAh?$AAa?$AAr?$AAs?$AAT?$AAo?$AAW?$AAr?$AAi?$AAt?$AAe?$AA?$DO?$AA0?$AA?$AA@ 0046728c     StringTable.obj
 0002:000022b0       ??_C@_02GMLFBBN@wb?$AA@    004672b0     SystemAddressList.obj
 0002:000022b8       ??_C@_1FE@LFCOHDLN@?$AAc?$AAo?$AAl?$AAu?$AAm?$AAn?$AAT?$AAy?$AAp?$AAe?$AA?$DN?$AA?$DN?$AAD?$AAa?$AAt?$AAa?$AAS?$AAt?$AAr?$AAu?$AAc?$AAt?$AAu?$AAr?$AAe?$AAs?$AA?3?$AA?3?$AAT?$AAa?$AAb?$AAl@ 004672b8     TableSerializer.obj
 0002:00002310       ??_C@_1EC@LMHEOMDL@?$AA?4?$AA?4?$AA?2?$AA?4?$AA?4?$AA?2?$AAr?$AAa?$AAk?$AAn?$AAe?$AAt?$AA?2?$AAT?$AAa?$AAb?$AAl?$AAe?$AAS?$AAe?$AAr?$AAi?$AAa?$AAl?$AAi?$AAz?$AAe?$AAr?$AA?4?$AAc?$AAp?$AAp@ 00467310     TableSerializer.obj
 0002:00002354       ??_C@_02DKCKIIND@?$CFs?$AA@ 00467354     samp_netencr.obj
 0002:00002358       ??_C@_01CLKCMJKC@?5?$AA@   00467358     samp_netencr.obj
 0002:0000235c       ??_C@_05BFHEBJNP@?$CF02X?5?$AA@ 0046735c     samp_netencr.obj
 0002:00002364       ??_C@_06MJENIHFP@?$CF08X?5?5?$AA@ 00467364     samp_netencr.obj
 0002:0000236c       ??_C@_02PHMGELLB@?6?6?$AA@ 0046736c     samp_netencr.obj
 0002:00002370       ?npos@TiXmlString@@2IB     00467370     tinystr.obj
 0002:00002374       ??_C@_1CC@PEHEJHGC@?$AAi?$AAn?$AAd?$AAe?$AAx?$AA?5?$AA?$DM?$AA?5?$AAl?$AAe?$AAn?$AAg?$AAt?$AAh?$AA?$CI?$AA?$CJ?$AA?$AA@ 00467374     tinyxml.obj
 0002:00002398       ??_C@_1GC@CPEGOIEK@?$AAc?$AA?3?$AA?2?$AAu?$AAs?$AAe?$AAr?$AAs?$AA?2?$AE?$DP?$AEC?$AEH?$AE?$DO?$AE?3?$AA?2?$AAd?$AAe?$AAs?$AAk?$AAt?$AAo?$AAp?$AA?2?$AAr?$AAa?$AAk?$AAs?$AAa?$AAm?$AAp?$AA?2?$AAt@ 00467398     tinyxml.obj
 0002:00002400       ??_7TiXmlBase@@6B@         00467400     tinyxml.obj
 0002:0000240c       ??_C@_00CNPNBAHC@?$AA@     0046740c     tinyxml.obj
 0002:00002410       ??_C@_1DE@OBBJJOCM@?$AA?4?$AA?4?$AA?2?$AA?4?$AA?4?$AA?2?$AAt?$AAi?$AAn?$AAy?$AAx?$AAm?$AAl?$AA?2?$AAt?$AAi?$AAn?$AAy?$AAx?$AAm?$AAl?$AA?4?$AAc?$AAp?$AAp?$AA?$AA@ 00467410     tinyxml.obj
 0002:00002444       ??_C@_1DC@LEADHCOJ@?$AAp?$AAr?$AAe?$AAv?$AAi?$AAo?$AAu?$AAs?$AA?9?$AA?$DO?$AAp?$AAa?$AAr?$AAe?$AAn?$AAt?$AA?5?$AA?$DN?$AA?$DN?$AA?5?$AAt?$AAh?$AAi?$AAs?$AA?$AA@ 00467444     tinyxml.obj
 0002:00002478       ??_C@_1O@EBIBIOED@?$AAq?$AA?5?$AA?$DM?$AA?$DN?$AA?5?$AAp?$AA?$AA@ 00467478     tinyxml.obj
 0002:00002488       ??_C@_1CE@GCHNJGEH@?$AAq?$AA?5?$AA?$DM?$AA?$DN?$AA?5?$AA?$CI?$AAb?$AAu?$AAf?$AA?$CL?$AAl?$AAe?$AAn?$AAg?$AAt?$AAh?$AA?$CJ?$AA?$AA@ 00467488     tinyxml.obj
 0002:000024ac       ??_C@_1CC@BHFGGFMK@?$AAp?$AA?5?$AA?$DM?$AA?5?$AA?$CI?$AAb?$AAu?$AAf?$AA?$CL?$AAl?$AAe?$AAn?$AAg?$AAt?$AAh?$AA?$CJ?$AA?$AA@ 004674ac     tinyxml.obj
 0002:000024d0       ??_C@_1M@LLHFIANP@?$AAc?$AAf?$AAi?$AAl?$AAe?$AA?$AA@ 004674d0     tinyxml.obj
 0002:000024dc       ??_C@_02DPKJAMEF@?$CFd?$AA@ 004674dc     tinyxml.obj
 0002:000024e0       ??_C@_03DLDNIBIK@?$CFlf?$AA@ 004674e0     tinyxml.obj
 0002:000024e4       ??_C@_08OEKJENGB@?$CFf?5?$CFf?5?$CFf?$AA@ 004674e4     tinyxml.obj
 0002:000024f0       ??_C@_02BBAHNLBA@?$CFp?$AA@ 004674f0     tinyxml.obj
 0002:000024f4       ??_C@_04CHMOMFOK@0x?$CFp?$AA@ 004674f4     tinyxml.obj
 0002:000024fc       ??_C@_08FADCNHGJ@?$CFu?5?$CFu?5?$CFu?$AA@ 004674fc     tinyxml.obj
 0002:00002508       ??_C@_09PNDCPLLD@?$DM?$CB?9?9?$CFs?9?9?$DO?$AA@ 00467508     tinyxml.obj
 0002:00002514       ??_C@_04PFOHOKJK@?5?5?5?5?$AA@ 00467514     tinyxml.obj
 0002:0000251c       ??_C@_04NNJCMPBN@?$DM?$CFs?$DO?$AA@ 0046751c     tinyxml.obj
 0002:00002528       ??_7TiXmlAttribute@@6B@    00467528     tinyxml.obj
 0002:00002534       ??_C@_08LCBMGHJI@?$CG?$CDx?$CF02X?$DL?$AA@ 00467534     tinyxml.obj
 0002:00002544       ??_7TiXmlNode@@6B@         00467544     tinyxml.obj
 0002:00002588       ??_C@_1IO@GOJOIIEP@?$AAn?$AAo?$AAd?$AAe?$AA?9?$AA?$DO?$AAG?$AAe?$AAt?$AAD?$AAo?$AAc?$AAu?$AAm?$AAe?$AAn?$AAt?$AA?$CI?$AA?$CJ?$AA?5?$AA?$DN?$AA?$DN?$AA?5?$AA0?$AA?5?$AA?$HM?$AA?$HM?$AA?5?$AAn?$AAo?$AAd?$AAe@ 00467588     tinyxml.obj
 0002:00002618       ??_C@_1FE@KCNOEABA@?$AAn?$AAo?$AAd?$AAe?$AA?9?$AA?$DO?$AAp?$AAa?$AAr?$AAe?$AAn?$AAt?$AA?5?$AA?$DN?$AA?$DN?$AA?5?$AA0?$AA?5?$AA?$HM?$AA?$HM?$AA?5?$AAn?$AAo?$AAd?$AAe?$AA?9?$AA?$DO?$AAp?$AAa?$AAr?$AAe?$AAn@ 00467618     tinyxml.obj
 0002:0000266c       ??_C@_1DC@BIKDOIFI@?$AAf?$AAi?$AAr?$AAs?$AAt?$AAC?$AAh?$AAi?$AAl?$AAd?$AA?5?$AA?$DN?$AA?$DN?$AA?5?$AAb?$AAe?$AAf?$AAo?$AAr?$AAe?$AAT?$AAh?$AAi?$AAs?$AA?$AA@ 0046766c     tinyxml.obj
 0002:000026a0       ??_C@_1CO@NMILEPCN@?$AAl?$AAa?$AAs?$AAt?$AAC?$AAh?$AAi?$AAl?$AAd?$AA?5?$AA?$DN?$AA?$DN?$AA?5?$AAa?$AAf?$AAt?$AAe?$AAr?$AAT?$AAh?$AAi?$AAs?$AA?$AA@ 004676a0     tinyxml.obj
 0002:000026d0       ??_C@_05POIKLDCH@?$DM?1?$CFs?$DO?$AA@ 004676d0     tinyxml.obj
 0002:000026d8       ??_C@_01PPODPGHN@?$DO?$AA@ 004676d8     tinyxml.obj
 0002:000026dc       ??_C@_03MFNJFHN@?5?1?$DO?$AA@ 004676dc     tinyxml.obj
 0002:000026e0       ??_C@_03FONCMJME@?$DM?$CFs?$AA@ 004676e0     tinyxml.obj
 0002:000026ec       ??_7TiXmlDocument@@6B@     004676ec     tinyxml.obj
 0002:00002730       ??_C@_01NOFIACDB@w?$AA@    00467730     tinyxml.obj
 0002:00002734       ??_C@_01GEODFPGF@?8?$AA@   00467734     tinyxml.obj
 0002:00002738       ??_C@_02PGMIOCEL@?$DN?8?$AA@ 00467738     tinyxml.obj
 0002:0000273c       ??_C@_07CGFAFKBF@?$CFs?$DN?8?$CFs?8?$AA@ 0046773c     tinyxml.obj
 0002:00002744       ??_C@_01BJJEKLCA@?$CC?$AA@ 00467744     tinyxml.obj
 0002:00002748       ??_C@_02ILLPBGAO@?$DN?$CC?$AA@ 00467748     tinyxml.obj
 0002:0000274c       ??_C@_07JDMHCBCA@?$CFs?$DN?$CC?$CFs?$CC?$AA@ 0046774c     tinyxml.obj
 0002:00002754       ??_C@_02BEIEFPIG@?$CFg?$AA@ 00467754     tinyxml.obj
 0002:0000275c       ??_7TiXmlComment@@6B@      0046775c     tinyxml.obj
 0002:000027a0       ??_C@_0BA@HEAAMLOF@?$DM?$CB?$FLCDATA?$FL?$CFs?$FN?$FN?$DO?6?$AA@ 004677a0     tinyxml.obj
 0002:000027b4       ??_7TiXmlDeclaration@@6B@  004677b4     tinyxml.obj
 0002:000027fc       ??_C@_02GOEMJPDN@?$DP?$DO?$AA@ 004677fc     tinyxml.obj
 0002:00002800       ??_C@_0N@IHAMHLOK@standalone?$DN?$CC?$AA@ 00467800     tinyxml.obj
 0002:00002810       ??_C@_0BB@OAOJGGEI@standalone?$DN?$CC?$CFs?$CC?5?$AA@ 00467810     tinyxml.obj
 0002:00002824       ??_C@_0L@ENAAEPMN@encoding?$DN?$CC?$AA@ 00467824     tinyxml.obj
 0002:00002830       ??_C@_0P@CJGKNICB@encoding?$DN?$CC?$CFs?$CC?5?$AA@ 00467830     tinyxml.obj
 0002:00002840       ??_C@_02KOPDJAMB@?$CC?5?$AA@ 00467840     tinyxml.obj
 0002:00002844       ??_C@_09KGECPEDL@version?$DN?$CC?$AA@ 00467844     tinyxml.obj
 0002:00002850       ??_C@_0O@LGPLJGNM@version?$DN?$CC?$CFs?$CC?5?$AA@ 00467850     tinyxml.obj
 0002:00002860       ??_C@_06CMNLMIOJ@?$DM?$DPxml?5?$AA@ 00467860     tinyxml.obj
 0002:00002868       ??_C@_1DG@LFHPEILE@?$AAs?$AAe?$AAn?$AAt?$AAi?$AAn?$AAe?$AAl?$AA?4?$AAp?$AAr?$AAe?$AAv?$AA?5?$AA?$DN?$AA?$DN?$AA?5?$AA?$CG?$AAs?$AAe?$AAn?$AAt?$AAi?$AAn?$AAe?$AAl?$AA?$AA@ 00467868     tinyxml.obj
 0002:000028a0       ??_C@_1DG@DBLLEBDG@?$AAs?$AAe?$AAn?$AAt?$AAi?$AAn?$AAe?$AAl?$AA?4?$AAn?$AAe?$AAx?$AAt?$AA?5?$AA?$DN?$AA?$DN?$AA?5?$AA?$CG?$AAs?$AAe?$AAn?$AAt?$AAi?$AAn?$AAe?$AAl?$AA?$AA@ 004678a0     tinyxml.obj
 0002:000028d8       ??_C@_1CO@FPCHJIP@?$AA?$CB?$AAF?$AAi?$AAn?$AAd?$AA?$CI?$AA?5?$AAa?$AAd?$AAd?$AAM?$AAe?$AA?9?$AA?$DO?$AAN?$AAa?$AAm?$AAe?$AA?$CI?$AA?$CJ?$AA?5?$AA?$CJ?$AA?$AA@ 004678d8     tinyxml.obj
 0002:00002908       ??_C@_01MNNFJEPP@?$DM?$AA@ 00467908     tinyxml.obj
 0002:0000290c       ??_C@_02DPNDACHE@?$DM?1?$AA@ 0046790c     tinyxml.obj
 0002:00002910       ??_C@_03MCHNFBAC@?$FN?$FN?$DO?$AA@ 00467910     tinyxml.obj
 0002:00002914       ??_C@_09BLLNCBLF@?$DM?$CB?$FLCDATA?$FL?$AA@ 00467914     tinyxml.obj
 0002:00002920       ??_C@_03PNLDJJMO@?9?9?$DO?$AA@ 00467920     tinyxml.obj
 0002:00002924       ??_C@_04FFDNBKGC@?$DM?$CB?9?9?$AA@ 00467924     tinyxml.obj
 0002:00002934       ??_7TiXmlText@@6B@         00467934     tinyxml.obj
 0002:0000297c       ??_7TiXmlUnknown@@6B@      0046797c     tinyxml.obj
 0002:000029c4       ??_7TiXmlElement@@6B@      004679c4     tinyxml.obj
 0002:00002a08       ??_C@_0FL@BMBPKIGK@Error?5when?5TiXmlDocument?5added?5t@ 00467a08     tinyxmlerror.obj
 0002:00002a64       ??_C@_0BF@HJPECPBG@Error?5parsing?5CDATA?4?$AA@ 00467a64     tinyxmlerror.obj
 0002:00002a7c       ??_C@_0DI@GMJJAOBO@Error?5null?5?$CI0?$CJ?5or?5unexpected?5EOF@ 00467a7c     tinyxmlerror.obj
 0002:00002ab4       ??_C@_0BG@FFJMEOCN@Error?5document?5empty?4?$AA@ 00467ab4     tinyxmlerror.obj
 0002:00002acc       ??_C@_0BL@BMCKJPKK@Error?5parsing?5Declaration?4?$AA@ 00467acc     tinyxmlerror.obj
 0002:00002ae8       ??_C@_0BH@MPJHJCKO@Error?5parsing?5Comment?4?$AA@ 00467ae8     tinyxmlerror.obj
 0002:00002b00       ??_C@_0BH@EPLDMIEN@Error?5parsing?5Unknown?4?$AA@ 00467b00     tinyxmlerror.obj
 0002:00002b18       ??_C@_0BH@JJGGDJOP@Error?5reading?5end?5tag?4?$AA@ 00467b18     tinyxmlerror.obj
 0002:00002b30       ??_C@_0BC@HMFFDDLH@Error?3?5empty?5tag?4?$AA@ 00467b30     tinyxmlerror.obj
 0002:00002b44       ??_C@_0BK@JPCMNIIK@Error?5reading?5Attributes?4?$AA@ 00467b44     tinyxmlerror.obj
 0002:00002b60       ??_C@_0BN@KKMBBCED@Error?5reading?5Element?5value?4?$AA@ 00467b60     tinyxmlerror.obj
 0002:00002b80       ??_C@_0BM@NCHBIJBE@Failed?5to?5read?5Element?5name?$AA@ 00467b80     tinyxmlerror.obj
 0002:00002b9c       ??_C@_0BH@BONKCKA@Error?5parsing?5Element?4?$AA@ 00467b9c     tinyxmlerror.obj
 0002:00002bb4       ??_C@_0BE@HJPJFJPJ@Failed?5to?5open?5file?$AA@ 00467bb4     tinyxmlerror.obj
 0002:00002bc8       ??_C@_05NAOIJFC@Error?$AA@ 00467bc8     tinyxmlerror.obj
 0002:00002bd0       ??_C@_08INEPGKHH@No?5error?$AA@ 00467bd0     tinyxmlerror.obj
 0002:00002bdc       ??_C@_06PNMEMOHD@?$CGapos?$DL?$AA@ 00467bdc     tinyxmlparser.obj
 0002:00002be4       ??_C@_06DDLNFFBN@?$CGquot?$DL?$AA@ 00467be4     tinyxmlparser.obj
 0002:00002bec       ??_C@_04LOOHDCEI@?$CGgt?$DL?$AA@ 00467bec     tinyxmlparser.obj
 0002:00002bf4       ??_C@_04GJOGLFEJ@?$CGlt?$DL?$AA@ 00467bf4     tinyxmlparser.obj
 0002:00002bfc       ??_C@_05JKJFEODM@?$CGamp?$DL?$AA@ 00467bfc     tinyxmlparser.obj
 0002:00002c08       ?utf8ByteTable@TiXmlBase@@2QBHB 00467c08     tinyxmlparser.obj
 0002:00003008       ??_C@_1M@OLEIFDEL@?$AAs?$AAt?$AAa?$AAm?$AAp?$AA?$AA@ 00468008     tinyxmlparser.obj
 0002:00003014       ??_C@_1CC@DMFNEMDE@?$AAc?$AAu?$AAr?$AAs?$AAo?$AAr?$AA?4?$AAc?$AAo?$AAl?$AA?5?$AA?$DO?$AA?$DN?$AA?5?$AA?9?$AA1?$AA?$AA@ 00468014     tinyxmlparser.obj
 0002:00003038       ??_C@_1CC@FAAMJHE@?$AAc?$AAu?$AAr?$AAs?$AAo?$AAr?$AA?4?$AAr?$AAo?$AAw?$AA?5?$AA?$DO?$AA?$DN?$AA?5?$AA?9?$AA1?$AA?$AA@ 00468038     tinyxmlparser.obj
 0002:0000305c       ??_C@_13LFIEIAHP@?$AAp?$AA?$AA@ 0046805c     tinyxmlparser.obj
 0002:00003060       ??_C@_17FAPGLHLF@?$AAn?$AAo?$AAw?$AA?$AA@ 00468060     tinyxmlparser.obj
 0002:00003068       ??_C@_1EA@IBJHAIBD@?$AA?4?$AA?4?$AA?2?$AA?4?$AA?4?$AA?2?$AAt?$AAi?$AAn?$AAy?$AAx?$AAm?$AAl?$AA?2?$AAt?$AAi?$AAn?$AAy?$AAx?$AAm?$AAl?$AAp?$AAa?$AAr?$AAs?$AAe?$AAr?$AA?4?$AAc?$AAp?$AAp?$AA?$AA@ 00468068     tinyxmlparser.obj
 0002:000030a8       ??_C@_17NHJOKMLJ@?$AAt?$AAa?$AAg?$AA?$AA@ 004680a8     tinyxmlparser.obj
 0002:000030b0       ??_C@_1FE@EHOANJMC@?$AAe?$AAr?$AAr?$AA?5?$AA?$DO?$AA?5?$AA0?$AA?5?$AA?$CG?$AA?$CG?$AA?5?$AAe?$AAr?$AAr?$AA?5?$AA?$DM?$AA?5?$AAT?$AAI?$AAX?$AAM?$AAL?$AA_?$AAE?$AAR?$AAR?$AAO?$AAR?$AA_?$AAS?$AAT?$AAR@ 004680b0     tinyxmlparser.obj
 0002:00003104       ??_C@_1M@JGKKHEFC@?$AAs?$AAt?$AAa?$AAr?$AAt?$AA?$AA@ 00468104     tinyxmlparser.obj
 0002:00003110       ??_C@_1FO@HPPHIJHG@?$AAs?$AAt?$AAr?$AAl?$AAe?$AAn?$AA?$CI?$AA?5?$AAe?$AAn?$AAt?$AAi?$AAt?$AAy?$AA?$FL?$AAi?$AA?$FN?$AA?4?$AAs?$AAt?$AAr?$AA?5?$AA?$CJ?$AA?5?$AA?$DN?$AA?$DN?$AA?5?$AAe?$AAn?$AAt?$AAi?$AAt@ 00468110     tinyxmlparser.obj
 0002:00003170       ??_C@_02KBFACPPK@?$DM?$CB?$AA@ 00468170     tinyxmlparser.obj
 0002:00003174       ??_C@_05DJDIECHG@?$DM?$DPxml?$AA@ 00468174     tinyxmlparser.obj
 0002:0000317c       ??_C@_1DI@JGFAPJP@?$AA?$CK?$AAl?$AAe?$AAn?$AAg?$AAt?$AAh?$AA?5?$AA?$DO?$AA?$DN?$AA?5?$AA0?$AA?5?$AA?$CG?$AA?$CG?$AA?5?$AA?$CK?$AAl?$AAe?$AAn?$AAg?$AAt?$AAh?$AA?5?$AA?$DM?$AA?5?$AA5?$AA?$AA@ 0046817c     tinyxmlparser.obj
 0002:000031b8       ??_C@_1GC@OMFOMFHP@?$AAc?$AA?3?$AA?2?$AAu?$AAs?$AAe?$AAr?$AAs?$AA?2?$AE?$DP?$AEC?$AEH?$AE?$DO?$AE?3?$AA?2?$AAd?$AAe?$AAs?$AAk?$AAt?$AAo?$AAp?$AA?2?$AAr?$AAa?$AAk?$AAs?$AAa?$AAm?$AAp?$AA?2?$AAt@ 004681b8     tinyxmlparser.obj
 0002:0000321c       ??_C@_04OOMJJNCF@UTF8?$AA@ 0046821c     tinyxmlparser.obj
 0002:00003224       ??_C@_05EGJIMALK@UTF?98?$AA@ 00468224     tinyxmlparser.obj
 0002:0000322c       ??_C@_17BJLLLIIO@?$AAe?$AAn?$AAc?$AA?$AA@ 0046822c     tinyxmlparser.obj
 0002:00003234       ??_C@_0L@FLHGMILF@standalone?$AA@ 00468234     tinyxmlparser.obj
 0002:00003240       ??_C@_08MLPGAEIK@encoding?$AA@ 00468240     tinyxmlparser.obj
 0002:0000324c       ??_C@_07CPCPJPKL@version?$AA@ 0046824c     tinyxmlparser.obj
 0002:00003254       ??_C@_0BE@ENHMBMKD@?$DN?$DN?$DN?5?$FLCOUNT?3?5?$CFd?$FN?5?$DN?$DN?$DN?$AA@ 00468254     cmds.obj
 0002:00003268       ??_C@_0O@GGACFFFI@?$CI?$CFd?$CJ?5?$CFs?5?$CFd?5?$CFd?$AA@ 00468268     cmds.obj
 0002:00003278       ??_C@_0BD@EAIFIKLP@ID?5Name?5Ping?5Score?$AA@ 00468278     cmds.obj
 0002:0000328c       ??_C@_0BE@MMHNGKME@?$DN?$DN?$DN?5PLAYER?5LIST?5?$DN?$DN?$DN?$AA@ 0046828c     cmds.obj
 0002:000032a0       ??_C@_0CD@HKNOBLPB@?$FLGOTO?$FN?5Player?5?$CFd?5is?5not?5connecte@ 004682a0     cmds.obj
 0002:000032c4       ??_C@_0CG@MDCJBJI@?$FLIMITATE?$FN?5Player?5?$CFs?5is?5not?5conne@ 004682c4     cmds.obj
 0002:000032ec       ??_C@_0CE@HNFPHDCF@?$FLIMITATE?$FN?5Imitate?5ID?5set?5to?5?$CFd?5?$CI@ 004682ec     cmds.obj
 0002:00003310       ??_C@_0CA@DKCGBFFF@?$FLIMITATE?$FN?5Imitate?5was?5disabled?4?$AA@ 00468310     cmds.obj
 0002:00003330       ??_C@_02PGHGPEOM@?91?$AA@  00468330     cmds.obj
 0002:00003334       ??_C@_0BA@IMAHEAPE@?$FLVLIST?$FN?5?$CFd?5?$CI?$CFs?$CJ?$AA@ 00468334     cmds.obj
 0002:00003344       ??_C@_0BP@GIMALHHO@?$FLVDEATH?$FN?5Sent?5to?5vehicle?5ID?5?$CFd?$AA@ 00468344     cmds.obj
 0002:00003364       ??_C@_0CG@CGHPHHKN@?$FLSELVEH?$FN?5Changed?5to?5vehicle?5ID?5t@ 00468364     cmds.obj
 0002:0000338c       ??_C@_0M@PPCLIDLP@ID?5?$CFd?3?5?8?$CFs?8?$AA@ 0046838c     cmds.obj
 0002:00003398       ??_C@_0BA@MKPEOKGE@No?5Saved?5Routes?$AA@ 00468398     cmds.obj
 0002:000033a8       ??_C@_0BH@LPLHDFBO@Error?5Reading?5Database?$AA@ 004683a8     cmds.obj
 0002:000033c0       ??_C@_0BE@OLCGOFDP@Started?5flooding?4?4?4?$AA@ 004683c0     cmds.obj
 0002:000033d4       ??_C@_0L@ENGCKLF@Stopped?4?4?4?$AA@ 004683d4     cmds.obj
 0002:000033e0       ??_C@_0M@CJDBNIPN@Started?5?3?9?$CJ?$AA@ 004683e0     cmds.obj
 0002:000033ec       ??_C@_0BE@PCAGCLPG@Stopped?5flooding?4?4?4?$AA@ 004683ec     cmds.obj
 0002:00003400       ??_C@_0BF@JAMGFEMD@Started?5flooding?5?3?9?$CJ?$AA@ 00468400     cmds.obj
 0002:00003418       ??_C@_0BD@FAEPPLLL@Stopped?5lagging?4?4?4?$AA@ 00468418     cmds.obj
 0002:0000342c       ??_C@_0BE@GDIILECN@Started?5lagging?5?3?9?$CJ?$AA@ 0046842c     cmds.obj
 0002:00003440       ??_C@_07FAOBPMFB@Done?4?4?4?$AA@ 00468440     cmds.obj
 0002:00003448       ??_C@_0BF@EAPNOEP@Connecting?5as?5NPC?4?4?4?$AA@ 00468448     cmds.obj
 0002:00003460       ??_C@_0BK@JAKFGHKE@Command?5?$CFs?5was?5not?5found?4?$AA@ 00468460     cmds.obj
 0002:0000347c       ??_C@_03BCJIDNJL@NPC?$AA@  0046847c     cmds.obj
 0002:00003480       ??_C@_03BPGDPAOH@npc?$AA@  00468480     cmds.obj
 0002:00003484       ??_C@_04OIKJMBFP@TEST?$AA@ 00468484     cmds.obj
 0002:0000348c       ??_C@_04CEJDCDCH@test?$AA@ 0046848c     cmds.obj
 0002:00003494       ??_C@_03MBBJPJFD@LAG?$AA@  00468494     cmds.obj
 0002:00003498       ??_C@_03MMOCDECP@lag?$AA@  00468498     cmds.obj
 0002:0000349c       ??_C@_04NFKOACKA@KILL?$AA@ 0046849c     cmds.obj
 0002:000034a4       ??_C@_04BJJEOANI@kill?$AA@ 004684a4     cmds.obj
 0002:000034ac       ??_C@_03HGNGHBCD@REG?$AA@  004684ac     cmds.obj
 0002:000034b0       ??_C@_03HLCNLMFP@reg?$AA@  004684b0     cmds.obj
 0002:000034b4       ??_C@_04PJFINEKF@JOIN?$AA@ 004684b4     cmds.obj
 0002:000034bc       ??_C@_04DFGCDGNN@join?$AA@ 004684bc     cmds.obj
 0002:000034c4       ??_C@_07IPCGJLN@MENUSEL?$AA@ 004684c4     cmds.obj
 0002:000034cc       ??_C@_07PFKPNFDJ@menusel?$AA@ 004684cc     cmds.obj
 0002:000034d4       ??_C@_06EHPADLPO@STOPRT?$AA@ 004684d4     cmds.obj
 0002:000034dc       ??_C@_06EDNLOFCM@stoprt?$AA@ 004684dc     cmds.obj
 0002:000034e4       ??_C@_06FLKFFAHO@PLAYRT?$AA@ 004684e4     cmds.obj
 0002:000034ec       ??_C@_06FPIOIOKM@playrt?$AA@ 004684ec     cmds.obj
 0002:000034f4       ??_C@_06NPDMFLCI@LOADRT?$AA@ 004684f4     cmds.obj
 0002:000034fc       ??_C@_06NLBHIFPK@loadrt?$AA@ 004684fc     cmds.obj
 0002:00003504       ??_C@_06IKPEDILI@RTLIST?$AA@ 00468504     cmds.obj
 0002:0000350c       ??_C@_06IONPOGGK@rtlist?$AA@ 0046850c     cmds.obj
 0002:00003514       ??_C@_06BCKPCHGE@SELVEH?$AA@ 00468514     cmds.obj
 0002:0000351c       ??_C@_06BGIEPJLG@selveh?$AA@ 0046851c     cmds.obj
 0002:00003524       ??_C@_02BOKMBMMM@fu?$AA@   00468524     cmds.obj
 0002:00003528       ??_C@_06FGPBBPHG@VDEATH?$AA@ 00468528     cmds.obj
 0002:00003530       ??_C@_06FCNKMBKE@vdeath?$AA@ 00468530     cmds.obj
 0002:00003538       ??_C@_05FPNIBPPA@VLIST?$AA@ 00468538     cmds.obj
 0002:00003540       ??_C@_05JEEOPILO@vlist?$AA@ 00468540     cmds.obj
 0002:00003548       ??_C@_07KJAENNDC@IMITATE?$AA@ 00468548     cmds.obj
 0002:00003550       ??_C@_07FEFJGBLG@imitate?$AA@ 00468550     cmds.obj
 0002:00003558       ??_C@_04MCNBBHG@GOTO?$AA@  00468558     cmds.obj
 0002:00003560       ??_C@_04MABHPDAO@goto?$AA@ 00468560     cmds.obj
 0002:00003568       ??_C@_07OPDDOEGI@PLAYERS?$AA@ 00468568     cmds.obj
 0002:00003570       ??_C@_07BCGOFIOM@players?$AA@ 00468570     cmds.obj
 0002:00003578       ??_C@_06DCHFNDBF@RELOAD?$AA@ 00468578     cmds.obj
 0002:00003580       ??_C@_06DGFOANMH@reload?$AA@ 00468580     cmds.obj
 0002:00003588       ??_C@_09PCJAMJNI@RECONNECT?$AA@ 00468588     cmds.obj
 0002:00003594       ??_C@_09MCGBPECP@reconnect?$AA@ 00468594     cmds.obj
 0002:000035a0       ??_C@_04GBOBDPBG@QUIT?$AA@ 004685a0     cmds.obj
 0002:000035a8       ??_C@_04KNNLNNGO@quit?$AA@ 004685a8     cmds.obj
 0002:000035b0       ??_C@_04GOLNGIJ@EXIT?$AA@  004685b0     cmds.obj
 0002:000035b8       ??_C@_04MKNBDEPB@exit?$AA@ 004685b8     cmds.obj
 0002:000035c0       ??_C@_0BD@KEPLIKPA@RCON?5password?5set?4?$AA@ 004685c0     cmds.obj
 0002:000035d4       ??_C@_0DB@ELLEKLDJ@RCON?5password?5was?5not?5set?4?5Type?5@ 004685d4     cmds.obj
 0002:00003608       ??_C@_05PLHGOPJD@LOGIN?$AA@ 00468608     cmds.obj
 0002:00003610       ??_C@_05DAOAAINN@login?$AA@ 00468610     cmds.obj
 0002:00003618       ??_C@_0BF@DLOCBHB@StreetSweeperTrailer?$AA@ 00468618     common.obj
 0002:00003630       ??_C@_0M@EKEKPONH@FarmTrailer?$AA@ 00468630     common.obj
 0002:0000363c       ??_C@_0O@ONKOADP@BlackBoxville?$AA@ 0046863c     common.obj
 0002:0000364c       ??_C@_0N@FEGCOPJO@TugStaircase?$AA@ 0046864c     common.obj
 0002:0000365c       ??_C@_0BA@PNHIGFJ@BaggageTrailer2?$AA@ 0046865c     common.obj
 0002:0000366c       ??_C@_0P@BPKIDMMJ@BaggageTrailer?$AA@ 0046866c     common.obj
 0002:0000367c       ??_C@_0O@GMDPAIOI@DamagedSadler?$AA@ 0046867c     common.obj
 0002:0000368c       ??_C@_0BA@DPGBENJN@DamagedGlendale?$AA@ 0046868c     common.obj
 0002:0000369c       ??_C@_07KEMLBHAB@Phoenix?$AA@ 0046869c     common.obj
 0002:000036a4       ??_C@_05IHOGHNDL@Alpha?$AA@ 004686a4     common.obj
 0002:000036ac       ??_C@_04LPDLPFEF@SWAT?$AA@ 004686ac     common.obj
 0002:000036b4       ??_C@_07BBCBAOFC@Picador?$AA@ 004686b4     common.obj
 0002:000036bc       ??_C@_0N@INBKHFMG@PoliceRanger?$AA@ 004686bc     common.obj
 0002:000036cc       ??_C@_0M@LOEFNGCH@PoliceCarLV?$AA@ 004686cc     common.obj
 0002:000036d8       ??_C@_0M@ODPNCADL@PoliceCarSF?$AA@ 004686d8     common.obj
 0002:000036e4       ??_C@_0M@MDDCCCGC@PoliceCarLS?$AA@ 004686e4     common.obj
 0002:000036f0       ??_C@_06CPOOJICK@Launch?$AA@ 004686f0     common.obj
 0002:000036f8       ??_C@_05MPJGBH@RCCam?$AA@  004686f8     common.obj
 0002:00003700       ??_C@_04FKFAAFKK@Dodo?$AA@ 00468700     common.obj
 0002:00003708       ??_C@_09POFIGJGN@Andromada?$AA@ 00468708     common.obj
 0002:00003714       ??_C@_0P@JJNKGFBC@ArtictTrailer3?$AA@ 00468714     common.obj
 0002:00003724       ??_C@_0BD@EKLECLGJ@FreightTrainBoxcar?$AA@ 00468724     common.obj
 0002:00003738       ??_C@_04FCIPMBFO@Club?$AA@ 00468738     common.obj
 0002:00003740       ??_C@_06DNPEPBDG@Hotdog?$AA@ 00468740     common.obj
 0002:00003748       ??_C@_05KGDFGEAD@Euros?$AA@ 00468748     common.obj
 0002:00003750       ??_C@_08ICKIDKCB@Wayfarer?$AA@ 00468750     common.obj
 0002:0000375c       ??_C@_07NEIFMLLI@Emperor?$AA@ 0046875c     common.obj
 0002:00003764       ??_C@_0O@NONOPHOF@PetrolTrailer?$AA@ 00468764     common.obj
 0002:00003774       ??_C@_03OCFCOPMN@Tug?$AA@  00468774     common.obj
 0002:00003778       ??_C@_07ILBMIDCN@NewsVan?$AA@ 00468778     common.obj
 0002:00003780       ??_C@_05FPHKOEEH@BF400?$AA@ 00468780     common.obj
 0002:00003788       ??_C@_08KKIMNFLL@Stafford?$AA@ 00468788     common.obj
 0002:00003794       ??_C@_07CBEIKNKI@Huntley?$AA@ 00468794     common.obj
 0002:0000379c       ??_C@_05LAEDEOAA@DFT30?$AA@ 0046879c     common.obj
 0002:000037a4       ??_C@_05MDMOFCAL@AT400?$AA@ 004687a4     common.obj
 0002:000037ac       ??_C@_07HIIGAALC@Tornado?$AA@ 004687ac     common.obj
 0002:000037b4       ??_C@_08JEADJMMO@Broadway?$AA@ 004687b4     common.obj
 0002:000037c0       ??_C@_07FJHKOOOB@Sweeper?$AA@ 004687c0     common.obj
 0002:000037c8       ??_C@_04JCIMNPAN@Dune?$AA@ 004687c8     common.obj
 0002:000037d0       ??_C@_05EDGECNOI@Mower?$AA@ 004687d0     common.obj
 0002:000037d8       ??_C@_04IJECPBBA@Kart?$AA@ 004687d8     common.obj
 0002:000037e0       ??_C@_0M@ENALKDLN@BrownStreak?$AA@ 004687e0     common.obj
 0002:000037ec       ??_C@_0BE@HNNCNFMJ@FreightTrainFlatbed?$AA@ 004687ec     common.obj
 0002:00003800       ??_C@_07HFFLBCJN@Bandito?$AA@ 00468800     common.obj
 0002:00003808       ??_C@_07PAMKBPDP@Savanna?$AA@ 00468808     common.obj
 0002:00003810       ??_C@_06IAEPOIJG@Tahoma?$AA@ 00468810     common.obj
 0002:00003818       ??_C@_05LDPHIKKB@Flash?$AA@ 00468818     common.obj
 0002:00003820       ??_C@_07OOEDJBB@RCTiger?$AA@ 00468820     common.obj
 0002:00003828       ??_C@_09EAHEKBCJ@Raindance?$AA@ 00468828     common.obj
 0002:00003834       ??_C@_05PCPHEHOE@Elegy?$AA@ 00468834     common.obj
 0002:0000383c       ??_C@_07NNNPFKCG@Stratum?$AA@ 0046883c     common.obj
 0002:00003844       ??_C@_06CBLFAFGA@Sultan?$AA@ 00468844     common.obj
 0002:0000384c       ??_C@_06NDOLCLDE@Jester?$AA@ 0046884c     common.obj
 0002:00003854       ??_C@_06HMBHBEBI@Uranus?$AA@ 00468854     common.obj
 0002:0000385c       ??_C@_08MKGLGNPB@Monster3?$AA@ 0046885c     common.obj
 0002:00003868       ??_C@_08NDHAFMLA@Monster2?$AA@ 00468868     common.obj
 0002:00003874       ??_C@_07KCFEPEMD@Windsor?$AA@ 00468874     common.obj
 0002:0000387c       ??_C@_08CHILKOCP@Yosemite?$AA@ 0046887c     common.obj
 0002:00003888       ??_C@_06OIKOAMFP@Nevada?$AA@ 00468888     common.obj
 0002:00003890       ??_C@_0L@DDOFOLID@UtilityVan?$AA@ 00468890     common.obj
 0002:0000389c       ??_C@_05GBEKJLJJ@Merit?$AA@ 0046889c     common.obj
 0002:000038a4       ??_C@_07EGNLAHNI@Sunrise?$AA@ 004688a4     common.obj
 0002:000038ac       ??_C@_05JMCLFHCI@Tampa?$AA@ 004688ac     common.obj
 0002:000038b4       ??_C@_08BCKDNAHK@Cargobob?$AA@ 004688b4     common.obj
 0002:000038c0       ??_C@_05CFOFHCJG@Primo?$AA@ 004688c0     common.obj
 0002:000038c8       ??_C@_08CGAIKJCC@Intruder?$AA@ 004688c8     common.obj
 0002:000038d4       ??_C@_07HNPEGFCG@Hustler?$AA@ 004688d4     common.obj
 0002:000038dc       ??_C@_0BE@NJLJEOGM@FireTruckwithladder?$AA@ 004688dc     common.obj
 0002:000038f0       ??_C@_06PNFBIENN@Sadler?$AA@ 004688f0     common.obj
 0002:000038f8       ??_C@_06GOGFINCH@Clover?$AA@ 004688f8     common.obj
 0002:00003900       ??_C@_06MCJFLPGN@Bullet?$AA@ 00468900     common.obj
 0002:00003908       ??_C@_07PODEONLP@Vincent?$AA@ 00468908     common.obj
 0002:00003910       ??_C@_06BFIBDPNC@Vortex?$AA@ 00468910     common.obj
 0002:00003918       ??_C@_0BC@CNKCCCJH@BrownStreakEngine?$AA@ 00468918     common.obj
 0002:0000392c       ??_C@_07GJKFEIPL@Freight?$AA@ 0046892c     common.obj
 0002:00003934       ??_C@_05IEKBADAP@Blade?$AA@ 00468934     common.obj
 0002:0000393c       ??_C@_07FDFHIFFP@Slamvan?$AA@ 0046893c     common.obj
 0002:00003944       ??_C@_09KHOEIBMD@Remington?$AA@ 00468944     common.obj
 0002:00003950       ??_C@_07IIFCFDNH@Feltzer?$AA@ 00468950     common.obj
 0002:00003958       ??_C@_0BB@MDNJHDPD@CombineHarvester?$AA@ 00468958     common.obj
 0002:0000396c       ??_C@_07JHKDGNGI@Tractor?$AA@ 0046896c     common.obj
 0002:00003974       ??_C@_08LJJEDEPF@Forklift?$AA@ 00468974     common.obj
 0002:00003980       ??_C@_07CNJKAEOJ@Willard?$AA@ 00468980     common.obj
 0002:00003988       ??_C@_08IKCBAKBD@FBITruck?$AA@ 00468988     common.obj
 0002:00003994       ??_C@_07FNJDAHLD@Cadrona?$AA@ 00468994     common.obj
 0002:0000399c       ??_C@_07EEELBEFD@Fortune?$AA@ 0046899c     common.obj
 0002:000039a4       ??_C@_08JFJEMMFK@Towtruck?$AA@ 004689a4     common.obj
 0002:000039b0       ??_C@_0M@IJILAFIF@CementTruck?$AA@ 004689b0     common.obj
 0002:000039bc       ??_C@_07OOAEBGH@HPV1000?$AA@ 004689bc     common.obj
 0002:000039c4       ??_C@_06OBOKNIPA@NRG500?$AA@ 004689c4     common.obj
 0002:000039cc       ??_C@_06PIFJOAOD@FCR900?$AA@ 004689cc     common.obj
 0002:000039d4       ??_C@_05MGCDNCGP@Hydra?$AA@ 004689d4     common.obj
 0002:000039dc       ??_C@_06HJEKKKAD@Shamal?$AA@ 004689dc     common.obj
 0002:000039e4       ??_C@_09GCHDDHPD@Buccaneer?$AA@ 004689e4     common.obj
 0002:000039f0       ??_C@_08OGMEHHJ@Majestic?$AA@ 004689f0     common.obj
 0002:000039fc       ??_C@_06KMKGKMGN@Nebula?$AA@ 004689fc     common.obj
 0002:00003a04       ??_C@_09GNLFJNMC@Roadtrain?$AA@ 00468a04     common.obj
 0002:00003a10       ??_C@_06OPJBJKEL@Tanker?$AA@ 00468a10     common.obj
 0002:00003a18       ??_C@_0L@GDENGONM@Stuntplane?$AA@ 00468a18     common.obj
 0002:00003a24       ??_C@_0L@CLMIPAFC@Cropduster?$AA@ 00468a24     common.obj
 0002:00003a30       ??_C@_06LCNKOGNJ@Beagle?$AA@ 00468a30     common.obj
 0002:00003a38       ??_C@_0N@LFHMCMMA@MountainBike?$AA@ 00468a38     common.obj
 0002:00003a48       ??_C@_04BMIAAGB@Bike?$AA@  00468a48     common.obj
 0002:00003a50       ??_C@_07OMJLKGCG@Journey?$AA@ 00468a50     common.obj
 0002:00003a58       ??_C@_07EOBNDFIE@Elegant?$AA@ 00468a58     common.obj
 0002:00003a60       ??_C@_07MPOALFMB@SuperGT?$AA@ 00468a60     common.obj
 0002:00003a68       ??_C@_0BA@GDCGHDGN@BloodringBanger?$AA@ 00468a68     common.obj
 0002:00003a78       ??_C@_0O@JBMOBKMA@HotringRacer3?$AA@ 00468a78     common.obj
 0002:00003a88       ??_C@_0O@IINFCLIB@HotringRacer2?$AA@ 00468a88     common.obj
 0002:00003a98       ??_C@_08LEDEGLMH@RCGoblin?$AA@ 00468a98     common.obj
 0002:00003aa4       ??_C@_04LPBHBPME@Mesa?$AA@ 00468aa4     common.obj
 0002:00003aac       ??_C@_06OEDNGFC@Benson?$AA@ 00468aac     common.obj
 0002:00003ab4       ??_C@_08FODAPCHG@Boxville?$AA@ 00468ab4     common.obj
 0002:00003ac0       ??_C@_0P@EOAPNKHK@PoliceMaverick?$AA@ 00468ac0     common.obj
 0002:00003ad0       ??_C@_0O@GJFHFIAL@BlistaCompact?$AA@ 00468ad0     common.obj
 0002:00003ae0       ??_C@_08MGLNKJKM@Sandking?$AA@ 00468ae0     common.obj
 0002:00003aec       ??_C@_0N@BFKGDGFI@HotringRacer?$AA@ 00468aec     common.obj
 0002:00003afc       ??_C@_06LBDMKPGH@Jetmax?$AA@ 00468afc     common.obj
 0002:00003b04       ??_C@_09KHJADKIA@Greenwood?$AA@ 00468b04     common.obj
 0002:00003b10       ??_C@_05GOADGCFA@Virgo?$AA@ 00468b10     common.obj
 0002:00003b18       ??_C@_0L@DJNCOCHA@FBIRancher?$AA@ 00468b18     common.obj
 0002:00003b24       ??_C@_07OBPEDNJI@Rancher?$AA@ 00468b24     common.obj
 0002:00003b2c       ??_C@_0M@IGFBCOBK@NewsChopper?$AA@ 00468b2c     common.obj
 0002:00003b38       ??_C@_08PEEPBIOP@Maverick?$AA@ 00468b38     common.obj
 0002:00003b44       ??_C@_05JGABKEPN@Dozer?$AA@ 00468b44     common.obj
 0002:00003b4c       ??_C@_07DEMPOEMJ@Baggage?$AA@ 00468b4c     common.obj
 0002:00003b54       ??_C@_07JICJFPHK@Marquis?$AA@ 00468b54     common.obj
 0002:00003b5c       ??_C@_06INFAJCEF@Camper?$AA@ 00468b5c     common.obj
 0002:00003b64       ??_C@_07HNHOAKIC@Burrito?$AA@ 00468b64     common.obj
 0002:00003b6c       ??_C@_03OFIGHJJK@BMX?$AA@  00468b6c     common.obj
 0002:00003b70       ??_C@_05BAJAFMOF@Comet?$AA@ 00468b70     common.obj
 0002:00003b78       ??_C@_06NNHDOJOO@Regina?$AA@ 00468b78     common.obj
 0002:00003b80       ??_C@_06EHCDEMPE@Walton?$AA@ 00468b80     common.obj
 0002:00003b88       ??_C@_05LOIDKPKB@ZR350?$AA@ 00468b88     common.obj
 0002:00003b90       ??_C@_07JAIPEIMF@Rustler?$AA@ 00468b90     common.obj
 0002:00003b98       ??_C@_05LOKFGGKM@Sabre?$AA@ 00468b98     common.obj
 0002:00003ba0       ??_C@_06ENBODKPJ@Hermes?$AA@ 00468ba0     common.obj
 0002:00003ba8       ??_C@_06MFOGHBMI@Dinghy?$AA@ 00468ba8     common.obj
 0002:00003bb0       ??_C@_0L@HLGDELAK@Coastguard?$AA@ 00468bb0     common.obj
 0002:00003bbc       ??_C@_08NPBPAMAK@Quadbike?$AA@ 00468bbc     common.obj
 0002:00003bc8       ??_C@_07LPGNOABP@Patriot?$AA@ 00468bc8     common.obj
 0002:00003bd0       ??_C@_07PGFGAPD@Sparrow?$AA@ 00468bd0     common.obj
 0002:00003bd8       ??_C@_07OFIHLHAO@Sanchez?$AA@ 00468bd8     common.obj
 0002:00003be0       ??_C@_07POHKCOEA@Oceanic?$AA@ 00468be0     common.obj
 0002:00003be8       ??_C@_08HJFONBEO@Glendale?$AA@ 00468be8     common.obj
 0002:00003bf4       ??_C@_08OGNBAEBJ@RCRaider?$AA@ 00468bf4     common.obj
 0002:00003c00       ??_C@_07GHDMOMHA@RCBaron?$AA@ 00468c00     common.obj
 0002:00003c08       ??_C@_07EGDDLHKH@Freeway?$AA@ 00468c08     common.obj
 0002:00003c10       ??_C@_06KOGAFPBN@Faggio?$AA@ 00468c10     common.obj
 0002:00003c18       ??_C@_06PEKEIFAC@PCJ600?$AA@ 00468c18     common.obj
 0002:00003c20       ??_C@_07BMMFBMKD@Skimmer?$AA@ 00468c20     common.obj
 0002:00003c28       ??_C@_0O@JHGDIOAD@BerkleysRCVan?$AA@ 00468c28     common.obj
 0002:00003c38       ??_C@_06MFLIPNF@Solair?$AA@ 00468c38     common.obj
 0002:00003c40       ??_C@_05GGMELJHE@Caddy?$AA@ 00468c40     common.obj
 0002:00003c48       ??_C@_06ILMFHPBN@Yankee?$AA@ 00468c48     common.obj
 0002:00003c50       ??_C@_07CIGBMPHN@Flatbed?$AA@ 00468c50     common.obj
 0002:00003c58       ??_C@_06IKGIMJCE@Tropic?$AA@ 00468c58     common.obj
 0002:00003c60       ??_C@_06JCGKAEKL@Reefer?$AA@ 00468c60     common.obj
 0002:00003c68       ??_C@_07EDKGBAKH@Speeder?$AA@ 00468c68     common.obj
 0002:00003c70       ??_C@_07PMMJLLLJ@Turismo?$AA@ 00468c70     common.obj
 0002:00003c78       ??_C@_0P@IAMBFEFD@ArtictTrailer2?$AA@ 00468c78     common.obj
 0002:00003c88       ??_C@_06CGEBBJDD@Trolly?$AA@ 00468c88     common.obj
 0002:00003c90       ??_C@_08GOJIDAJM@PizzaBoy?$AA@ 00468c90     common.obj
 0002:00003c9c       ??_C@_0L@GFDMINNG@Seasparrow?$AA@ 00468c9c     common.obj
 0002:00003ca8       ??_C@_06KBNALHDK@Squalo?$AA@ 00468ca8     common.obj
 0002:00003cb0       ??_C@_07GBDAGOAA@Admiral?$AA@ 00468cb0     common.obj
 0002:00003cb8       ??_C@_07GOHPBKOH@Monster?$AA@ 00468cb8     common.obj
 0002:00003cc0       ??_C@_06ODEOHKOJ@Packer?$AA@ 00468cc0     common.obj
 0002:00003cc8       ??_C@_06PHDBBKAL@Romero?$AA@ 00468cc8     common.obj
 0002:00003cd0       ??_C@_08GMGPBKCF@RCBandit?$AA@ 00468cd0     common.obj
 0002:00003cdc       ??_C@_05EBJBKIPJ@Rumpo?$AA@ 00468cdc     common.obj
 0002:00003ce4       ??_C@_08IKNNGJAJ@Stallion?$AA@ 00468ce4     common.obj
 0002:00003cf0       ??_C@_06PJIJOHHC@Cabbie?$AA@ 00468cf0     common.obj
 0002:00003cf8       ??_C@_05LILMMCLC@Coach?$AA@ 00468cf8     common.obj
 0002:00003d00       ??_C@_07GEHMOLGJ@Previon?$AA@ 00468d00     common.obj
 0002:00003d08       ??_C@_0O@GMOEMJBF@ArtictTrailer?$AA@ 00468d08     common.obj
 0002:00003d18       ??_C@_08DLJPKKCN@Hotknife?$AA@ 00468d18     common.obj
 0002:00003d24       ??_C@_08FJPAFNJ@Barracks?$AA@ 00468d24     common.obj
 0002:00003d30       ??_C@_05EADLOCOH@Rhino?$AA@ 00468d30     common.obj
 0002:00003d38       ??_C@_03LJIODANL@Bus?$AA@  00468d38     common.obj
 0002:00003d3c       ??_C@_08NBLHOMJL@Predator?$AA@ 00468d3c     common.obj
 0002:00003d48       ??_C@_07PICMBPKH@Banshee?$AA@ 00468d48     common.obj
 0002:00003d50       ??_C@_09BHNBGNIF@Securicar?$AA@ 00468d50     common.obj
 0002:00003d5c       ??_C@_08KAMCCCDN@Enforcer?$AA@ 00468d5c     common.obj
 0002:00003d68       ??_C@_07JIKMJFHB@Premier?$AA@ 00468d68     common.obj
 0002:00003d70       ??_C@_06NPNCGLLF@Hunter?$AA@ 00468d70     common.obj
 0002:00003d78       ??_C@_0M@HEMNCDHI@BFInjection?$AA@ 00468d78     common.obj
 0002:00003d84       ??_C@_09JBLHGDDB@MrWhoopee?$AA@ 00468d84     common.obj
 0002:00003d90       ??_C@_06IAICJIHL@Bobcat?$AA@ 00468d90     common.obj
 0002:00003d98       ??_C@_0L@GKJCJMFK@Washington?$AA@ 00468d98     common.obj
 0002:00003da4       ??_C@_04JJAJBIIJ@Taxi?$AA@ 00468da4     common.obj
 0002:00003dac       ??_C@_09FAMKJDEM@Esperanto?$AA@ 00468dac     common.obj
 0002:00003db8       ??_C@_08GKMHINB@Moonbeam?$AA@ 00468db8     common.obj
 0002:00003dc4       ??_C@_09HJBFIHEP@Leviathan?$AA@ 00468dc4     common.obj
 0002:00003dd0       ??_C@_09LODJDONJ@Ambulance?$AA@ 00468dd0     common.obj
 0002:00003ddc       ??_C@_07IMBBPGLN@Cheetah?$AA@ 00468ddc     common.obj
 0002:00003de4       ??_C@_04JMBIGJBC@Mule?$AA@ 00468de4     common.obj
 0002:00003dec       ??_C@_04NODPAEOJ@Pony?$AA@ 00468dec     common.obj
 0002:00003df4       ??_C@_06NFPMDKDO@Voodoo?$AA@ 00468df4     common.obj
 0002:00003dfc       ??_C@_08BADKLIKD@Infernus?$AA@ 00468dfc     common.obj
 0002:00003e08       ??_C@_06BPNAANEB@Manana?$AA@ 00468e08     common.obj
 0002:00003e10       ??_C@_07ENIDNHGB@Stretch?$AA@ 00468e10     common.obj
 0002:00003e18       ??_C@_0M@MJOPNGDA@Trashmaster?$AA@ 00468e18     common.obj
 0002:00003e24       ??_C@_09MMJOEMML@FireTruck?$AA@ 00468e24     common.obj
 0002:00003e30       ??_C@_06NALAOMEG@Dumper?$AA@ 00468e30     common.obj
 0002:00003e38       ??_C@_08EJJHPIDO@Sentinel?$AA@ 00468e38     common.obj
 0002:00003e44       ??_C@_09FGOBLKLG@Perennial?$AA@ 00468e44     common.obj
 0002:00003e50       ??_C@_0L@OHIEBILL@Linerunner?$AA@ 00468e50     common.obj
 0002:00003e5c       ??_C@_07KHNIKBGK@Buffalo?$AA@ 00468e5c     common.obj
 0002:00003e64       ??_C@_07EINKFLOC@Bravura?$AA@ 00468e64     common.obj
 0002:00003e6c       ??_C@_0M@PEBICIDH@Landstalker?$AA@ 00468e6c     common.obj
 0002:00003e78       ??_C@_0P@GHFPNOJB@bad?5allocation?$AA@ 00468e78     console.obj
 0002:00003e88       ?collate@?$_Locbase@H@std@@2HB 00468e88     console.obj
 0002:00003e8c       ?ctype@?$_Locbase@H@std@@2HB 00468e8c     console.obj
 0002:00003e90       ?monetary@?$_Locbase@H@std@@2HB 00468e90     console.obj
 0002:00003e94       ?numeric@?$_Locbase@H@std@@2HB 00468e94     console.obj
 0002:00003e98       ?time@?$_Locbase@H@std@@2HB 00468e98     console.obj
 0002:00003e9c       ?messages@?$_Locbase@H@std@@2HB 00468e9c     console.obj
 0002:00003ea0       ?all@?$_Locbase@H@std@@2HB 00468ea0     console.obj
 0002:00003ea4       ?none@?$_Locbase@H@std@@2HB 00468ea4     console.obj
 0002:00003ea8       ?table_size@?$ctype@D@std@@2IB 00468ea8     console.obj
 0002:00003eac       ?skipws@?$_Iosb@H@std@@2W4_Fmtflags@12@B 00468eac     console.obj
 0002:00003eb0       ?unitbuf@?$_Iosb@H@std@@2W4_Fmtflags@12@B 00468eb0     console.obj
 0002:00003eb4       ?uppercase@?$_Iosb@H@std@@2W4_Fmtflags@12@B 00468eb4     console.obj
 0002:00003eb8       ?showbase@?$_Iosb@H@std@@2W4_Fmtflags@12@B 00468eb8     console.obj
 0002:00003ebc       ?showpoint@?$_Iosb@H@std@@2W4_Fmtflags@12@B 00468ebc     console.obj
 0002:00003ec0       ?showpos@?$_Iosb@H@std@@2W4_Fmtflags@12@B 00468ec0     console.obj
 0002:00003ec4       ?left@?$_Iosb@H@std@@2W4_Fmtflags@12@B 00468ec4     console.obj
 0002:00003ec8       ?right@?$_Iosb@H@std@@2W4_Fmtflags@12@B 00468ec8     console.obj
 0002:00003ecc       ?internal@?$_Iosb@H@std@@2W4_Fmtflags@12@B 00468ecc     console.obj
 0002:00003ed0       ?dec@?$_Iosb@H@std@@2W4_Fmtflags@12@B 00468ed0     console.obj
 0002:00003ed4       ?oct@?$_Iosb@H@std@@2W4_Fmtflags@12@B 00468ed4     console.obj
 0002:00003ed8       ?hex@?$_Iosb@H@std@@2W4_Fmtflags@12@B 00468ed8     console.obj
 0002:00003edc       ?scientific@?$_Iosb@H@std@@2W4_Fmtflags@12@B 00468edc     console.obj
 0002:00003ee0       ?fixed@?$_Iosb@H@std@@2W4_Fmtflags@12@B 00468ee0     console.obj
 0002:00003ee4       ?hexfloat@?$_Iosb@H@std@@2W4_Fmtflags@12@B 00468ee4     console.obj
 0002:00003ee8       ?boolalpha@?$_Iosb@H@std@@2W4_Fmtflags@12@B 00468ee8     console.obj
 0002:00003eec       ?_Stdio@?$_Iosb@H@std@@2W4_Fmtflags@12@B 00468eec     console.obj
 0002:00003ef0       ?adjustfield@?$_Iosb@H@std@@2W4_Fmtflags@12@B 00468ef0     console.obj
 0002:00003ef4       ?basefield@?$_Iosb@H@std@@2W4_Fmtflags@12@B 00468ef4     console.obj
 0002:00003ef8       ?floatfield@?$_Iosb@H@std@@2W4_Fmtflags@12@B 00468ef8     console.obj
 0002:00003efc       ?goodbit@?$_Iosb@H@std@@2W4_Iostate@12@B 00468efc     console.obj
 0002:00003f00       ?eofbit@?$_Iosb@H@std@@2W4_Iostate@12@B 00468f00     console.obj
 0002:00003f04       ?failbit@?$_Iosb@H@std@@2W4_Iostate@12@B 00468f04     console.obj
 0002:00003f08       ?badbit@?$_Iosb@H@std@@2W4_Iostate@12@B 00468f08     console.obj
 0002:00003f0c       ?_Hardfail@?$_Iosb@H@std@@2W4_Iostate@12@B 00468f0c     console.obj
 0002:00003f10       ?in@?$_Iosb@H@std@@2W4_Openmode@12@B 00468f10     console.obj
 0002:00003f14       ?out@?$_Iosb@H@std@@2W4_Openmode@12@B 00468f14     console.obj
 0002:00003f18       ?ate@?$_Iosb@H@std@@2W4_Openmode@12@B 00468f18     console.obj
 0002:00003f1c       ?app@?$_Iosb@H@std@@2W4_Openmode@12@B 00468f1c     console.obj
 0002:00003f20       ?trunc@?$_Iosb@H@std@@2W4_Openmode@12@B 00468f20     console.obj
 0002:00003f24       ?_Nocreate@?$_Iosb@H@std@@2W4_Openmode@12@B 00468f24     console.obj
 0002:00003f28       ?_Noreplace@?$_Iosb@H@std@@2W4_Openmode@12@B 00468f28     console.obj
 0002:00003f2c       ?binary@?$_Iosb@H@std@@2W4_Openmode@12@B 00468f2c     console.obj
 0002:00003f30       ?beg@?$_Iosb@H@std@@2W4_Seekdir@12@B 00468f30     console.obj
 0002:00003f34       ?cur@?$_Iosb@H@std@@2W4_Seekdir@12@B 00468f34     console.obj
 0002:00003f38       ?end@?$_Iosb@H@std@@2W4_Seekdir@12@B 00468f38     console.obj
 0002:00003f3c       ??_C@_0BC@DKELIMCI@RakSAMP?5v0?45?90?43e?$AA@ 00468f3c     console.obj
 0002:00003f50       ??_C@_01KDCPPGHE@r?$AA@    00468f50     console.obj
 0002:00003f54       ??_C@_0BH@MHMFGIDG@?$FL?$CF02d?3?$CF02d?3?$CF02d?4?$CF03d?$FN?5?$AA@ 00468f54     main.obj
 0002:00003f6c       ??_C@_0BC@NKPJKMNH@RakSAMPClient?4log?$AA@ 00468f6c     main.obj
 0002:00003f80       ??_C@_01MCMALHOG@a?$AA@    00468f80     main.obj
 0002:00003fc4       ??_C@_0BD@MCJHHNAM@Loading?5autorun?4?4?4?$AA@ 00468fc4     main.obj
 0002:00003fd8       ??_C@_0DK@LJNGGDOC@Hostname?3?5?$CFs?5?5?5?5?5Players?3?5?$CFd?5?5?5?5@ 00468fd8     main.obj
 0002:00004014       ??_C@_0BP@FKEOEDEB@jlfm?0?5eider?0?5PAWNIAK?0?5Wkurzacz?$AA@ 00469014     main.obj
 0002:00004034       ??_C@_0CK@HMJEDEOK@?5?5Authors?3?5jlfm?0?5eider?0?5PAWNIAK?0@ 00469034     main.obj
 0002:00004060       ??_C@_0EB@PHCNNEJJ@?5?5RakSAMP?5v0?45?90?43e?5initialized?5@ 00469060     main.obj
 0002:000040a4       ??_C@_0DK@BGGFMNFL@?$CK?5?$DN?$DN?$DN?$DN?$DN?$DN?$DN?$DN?$DN?$DN?$DN?$DN?$DN?$DN?$DN?$DN?$DN?$DN?$DN?$DN?$DN?$DN?$DN?$DN?$DN?$DN?$DN?$DN?$DN?$DN@ 004690a4     main.obj
 0002:000040e0       ??_C@_0BI@FBAJJJML@Failed?5to?5load?5settings?$AA@ 004690e0     main.obj
 0002:000040f8       __real@3f50624dd2f1a9fc    004690f8     math_stuff.obj
 0002:00004100       __real@3f800000            00469100     math_stuff.obj
 0002:00004108       __real@3ff0000000000000    00469108     math_stuff.obj
 0002:00004150       __real@4000000000000000    00469150     math_stuff.obj
 0002:00004158       __real@3e800000            00469158     misc_funcs.obj
 0002:0000415c       ??_C@_0BE@DBMLHJCG@Connecting?5to?5?$CFs?3?$CFd?$AA@ 0046915c     misc_funcs.obj
 0002:00004170       ??_C@_0N@NFBNFHML@Disconnected?$AA@ 00469170     misc_funcs.obj
 0002:00004180       ??_C@_0CM@KHHAAPKL@354A1F8D95B8384F9C365E2D7418C7EC@ 00469180     misc_funcs.obj
 0002:000041ac       ??_C@_0CM@MJJPPCGG@hacked?5hacked?5hacked?$CB21121111111@ 004691ac     misc_funcs.obj
 0002:000041d8       ??_C@_05DJDHLJAH@12345?$AA@ 004691d8     misc_funcs.obj
 0002:000041e0       ??_C@_0BA@DCBKDFNK@?1register?512345?$AA@ 004691e0     misc_funcs.obj
 0002:000041f0       __real@40efffe000000000    004691f0     netgame.obj
 0002:000041f8       __real@40dfffe000000000    004691f8     netgame.obj
 0002:00004200       ??_C@_04OGLGKMEC@0?43e?$AA@ 00469200     netgame.obj
 0002:00004208       ??_C@_0BP@LEJJCCNB@Connected?4?5Joining?5the?5game?4?4?4?$AA@ 00469208     netgame.obj
 0002:00004228       __real@447a0000            00469228     netgame.obj
 0002:0000422c       ??_C@_0DP@CKOOEMAB@?$FLRAKSAMP?$FN?5The?5connection?5was?5los@ 0046922c     netgame.obj
 0002:0000426c       ??_C@_0DI@LHILJMPB@?$FLRAKSAMP?$FN?5Invalid?5password?4?5Reco@ 0046926c     netgame.obj
 0002:000042a4       ??_C@_0DK@FOBIBNO@?$FLRAKSAMP?$FN?5The?5server?5is?5full?4?5Re@ 004692a4     netgame.obj
 0002:000042e0       ??_C@_0EB@DOMMOCNL@?$FLRAKSAMP?$FN?5Connection?5attempt?5fai@ 004692e0     netgame.obj
 0002:00004324       ??_C@_0DG@COCILCOE@?$FLRAKSAMP?$FN?5You?5are?5banned?4?5Reconn@ 00469324     netgame.obj
 0002:00004360       ??_C@_0EL@MBNLFGMP@?$FLRAKSAMP?$FN?5Connection?5was?5closed?5@ 00469360     netgame.obj
 0002:000043ac       ??_C@_04BMCEDOKO@EDIT?$AA@ 004693ac     netrpc.obj
 0002:000043b4       ??_C@_06HBIEIEBN@BUTTON?$AA@ 004693b4     netrpc.obj
 0002:000043bc       ??_C@_07EKEMFJNL@LISTBOX?$AA@ 004693bc     netrpc.obj
 0002:000043c4       ??_C@_0M@GOBBANAF@dlgWndClass?$AA@ 004693c4     netrpc.obj
 0002:000043d0       ??_C@_0BD@KFGPICNB@Connected?5to?5?$CF?464s?$AA@ 004693d0     netrpc.obj
 0002:000043e4       ??_C@_0BF@KIECBJDM@?$CFs?5?$CI?$CFd?$CJ?5?9?5RakSAMP?5?$CFs?$AA@ 004693e4     netrpc.obj
 0002:000043fc       ??_C@_0BE@LJOGFEK@Connected?5to?5?$CF?464s?6?$AA@ 004693fc     netrpc.obj
 0002:00004410       ??_C@_0BN@MHMOMKKO@?$CFs?5?$CI?$CFd?$CJ?5?9?5?$CF?416s?5?9?5RakSAMP?5?$CFs?$AA@ 00469410     netrpc.obj
 0002:00004430       ??_C@_09LLONOKFN@v0?45?90?43e?$AA@ 00469430     netrpc.obj
 0002:0000443c       ??_C@_0BM@MPENFOKD@ConnectionRejected?3?5unknown?$AA@ 0046943c     netrpc.obj
 0002:00004458       ??_C@_0BJ@CBLEPFBJ@?$FLRAKSAMP?$FN?5Bad?5player?5ID?4?$AA@ 00469458     netrpc.obj
 0002:00004474       ??_C@_0BL@EHBLDKJD@?$FLRAKSAMP?$FN?5Bad?5mod?5version?4?$AA@ 00469474     netrpc.obj
 0002:00004490       ??_C@_0CM@GJFJLAGD@?$FLRAKSAMP?$FN?5Bad?5nickname?4?5Changing@ 00469490     netrpc.obj
 0002:000044bc       ??_C@_05ONEOBAM@?$CFs_?$CFs?$AA@ 004694bc     netrpc.obj
 0002:000044c4       ??_C@_0BN@PCHMDGD@?$FLRAKSAMP?$FN?5Bad?5SA?9MP?5version?4?$AA@ 004694c4     netrpc.obj
 0002:000044e4       ??_C@_09FCEDMBEM@?$FLCMSG?$FN?5?$CFs?$AA@ 004694e4     netrpc.obj
 0002:000044f0       ??_C@_0O@MMAJKGDK@?$FLCHAT?$FN?5?$CFs?3?5?$CFs?$AA@ 004694f0     netrpc.obj
 0002:00004500       ??_C@_0N@OPGFBPIO@?$FLMENU?3?$CFd?$FN?5?$CFs?$AA@ 00469500     netrpc.obj
 0002:00004510       ??_C@_09BHDFPPF@?$FLMENU?$FN?5?$CFs?$AA@ 00469510     netrpc.obj
 0002:0000451c       ??_C@_0O@NLMDLJJA@?$FLGAMETEXT?$FN?5?$CFs?$AA@ 0046951c     netrpc.obj
 0002:0000452c       ??_C@_0BC@IFGCBGEG@?$FLAUDIO_STREAM?$FN?5?$CFs?$AA@ 0046952c     netrpc.obj
 0002:00004540       ??_C@_0EK@PMBHOKFK@RCON?5mode?5initialized?5?$CI?$CFs?3?$CFd?$CJ?4?5T@ 00469540     rcon.obj
 0002:0000458c       ??_C@_0BM@MLBJODBJ@Database?5has?5been?5optimized?$AA@ 0046958c     vehplayer.obj
 0002:000045a8       ??_C@_0BO@GJEMFPDN@SQLite?5?9?5Error?5?$CIoptimize?$CJ?3?5?$CFs?$AA@ 004695a8     vehplayer.obj
 0002:000045c8       ??_C@_06CKLCCFNP@VACUUM?$AA@ 004695c8     vehplayer.obj
 0002:000045d0       ??_C@_0CE@EPBCCPPD@SQLite?5?9?5Error?5while?5connecting?3@ 004695d0     vehplayer.obj
 0002:000045f4       ??_C@_0BB@DFPAJAPJ@mod_sa_routes?4db?$AA@ 004695f4     vehplayer.obj
 0002:00004608       __real@bf800000            00469608     vehplayer.obj
 0002:0000460c       ??_C@_0CH@DHLELAHP@sqliteDB_checkTableExists?3?5recei@ 0046960c     vehplayer.obj
 0002:00004634       ??_C@_0BB@JKBONAAJ@tableName?5?$DN?5NULL?$AA@ 00469634     vehplayer.obj
 0002:00004648       ??_C@_09LPNOFEEG@db?5?$DN?5NULL?$AA@ 00469648     vehplayer.obj
 0002:00004654       ??_C@_0DM@EPFGBEFK@SQLite?5?9?5Error?5?$CIpreparing?5statem@ 00469654     vehplayer.obj
 0002:00004690       ??_C@_0EB@OKALLEFH@SELECT?5name?5FROM?5sqlite_master?5W@ 00469690     vehplayer.obj
 0002:000046d4       ??_C@_07IOGLMIPM@sqlite_?$AA@ 004696d4     vehplayer.obj
 0002:000046dc       ??_C@_0DJ@JHAOIJBM@SQLite?5?9?5Error?5?$CIpreparing?5statem@ 004696dc     vehplayer.obj
 0002:00004718       ??_C@_0DD@BBHHPPCJ@SELECT?5name?5FROM?5sqlite_master?5W@ 00469718     vehplayer.obj
 0002:0000474c       ??_C@_0CK@HMJOJADI@sqliteDB_getNumTables?3?5received?5@ 0046974c     vehplayer.obj
 0002:00004778       ??_C@_0CA@NEFMCAGJ@sqliteDB_dropTable?3?5received?5?$CFs?$AA@ 00469778     vehplayer.obj
 0002:00004798       ??_C@_0CK@EKIEHJDL@SQLite?5?9?5Error?5?$CIexec?5drop?5table?5@ 00469798     vehplayer.obj
 0002:000047c4       ??_C@_0BB@BCIBMJOE@DROP?5TABLE?5?8?$CFs?8?$DL?$AA@ 004697c4     vehplayer.obj
 0002:000047d8       ??_C@_0DJ@DNDEIIDH@SQLite?5?9?5Error?5?$CIpreparing?5statem@ 004697d8     vehplayer.obj
 0002:00004818       ??_C@_0FI@PPHFDDLP@Recording?5?9?5load?5table?5?8?$CFs?8?3?5rec@ 00469818     vehplayer.obj
 0002:00004870       ??_C@_0P@KDDBDKEH@failed?5to?5load?$AA@ 00469870     vehplayer.obj
 0002:00004880       ??_C@_0ED@BJOJMNGP@Problem?5while?5loading?5Recording?5@ 00469880     vehplayer.obj
 0002:000048c4       ??_C@_0BD@ONJJJFBM@Not?5at?5end?5of?5rows?$AA@ 004698c4     vehplayer.obj
 0002:000048d8       ??_C@_0M@CHEPKMAD@End?5of?5rows?$AA@ 004698d8     vehplayer.obj
 0002:000048e8       ??_C@_0EK@EPJIADPD@SQLite?5?9?5Error?5?$CIprepare?5statemen@ 004698e8     vehplayer.obj
 0002:00004934       ??_C@_0BK@NLDJPMAG@successfully?5loaded?5route?$AA@ 00469934     vehplayer.obj
 0002:00004950       ??_C@_0DP@FDMJPDLP@SQLite?5?9?5Error?5?$CIprepare?5statemen@ 00469950     vehplayer.obj
 0002:00004990       ??_C@_0BE@DNCEAMNL@SELECT?5?$CK?5FROM?5?8?$CFs?8?$DL?$AA@ 00469990     vehplayer.obj
 0002:000049a4       ??_C@_0BE@GNNPIGIN@table?5doesn?8t?5exist?$AA@ 004699a4     vehplayer.obj
 0002:000049b8       ??_C@_0BD@MMCBFDGC@Dropped?5table?5?8?$CFs?8?$AA@ 004699b8     vehplayer.obj
 0002:000049cc       ??_C@_0DF@IMOACJLB@SQLite?5?9?5Error?5?$CIexecuting?5INSERT@ 004699cc     vehplayer.obj
 0002:00004a04       ??_C@_0BD@NKFOGAPN@saved?5to?5?8route?$CFi?8?$AA@ 00469a04     vehplayer.obj
 0002:00004a18       ??_C@_0GJ@BMEJLGNJ@?$CFs?5?$CF0?42f?0?5?$CF0?42f?0?5?$CF0?42f?0?5?$CF0?42f?0?$CF0@ 00469a18     vehplayer.obj
 0002:00004a84       ??_C@_0CI@PPNIDHOP@INSERT?5INTO?5?8route?$CFi?8?5VALUES?$CI?5nu@ 00469a84     vehplayer.obj
 0002:00004aac       ??_C@_0CK@ECDMDEAP@INSERT?5INTO?5?8route?$CFi?8?5VALUES?$CI?5nu@ 00469aac     vehplayer.obj
 0002:00004ad8       ??_C@_0DG@KBKOFHNK@SQLite?5?9?5Error?5?$CIexecuting?5CREATE@ 00469ad8     vehplayer.obj
 0002:00004b10       ??_C@_0BKL@MGLLCEGG@?$CFs?5?8index?8?5INTEGER?5NOT?5NULL?5PRIM@ 00469b10     vehplayer.obj
 0002:00004cbc       ??_C@_0BI@MJKNHCLJ@CREATE?5TABLE?5?8route?$CFi?8?$CI?$AA@ 00469cbc     vehplayer.obj
 0002:00004cd4       ??_C@_07NIKKADNO@route?$CFi?$AA@ 00469cd4     vehplayer.obj
 0002:00004cdc       ??_C@_0BF@IKFNNNE@Nothing?5to?5be?5saved?4?$AA@ 00469cdc     vehplayer.obj
 0002:00004cf4       ??_C@_0BM@BFGODOMO@Can?8t?5save?5while?5recording?4?$AA@ 00469cf4     vehplayer.obj
 0002:00004d10       ??_C@_07NMCEPFIO@?$FLCMSG?$FN?5?$AA@ 00469d10     window.obj
 0002:00004d18       ??_C@_07NEGFFIKO@?$FLCHAT?$FN?5?$AA@ 00469d18     window.obj
 0002:00004d20       ??_C@_06LKBCGDFD@Button?$AA@ 00469d20     window.obj
 0002:00004d28       ??_C@_05KPFLECNE@?$CGSend?$AA@ 00469d28     window.obj
 0002:00004d30       ??_C@_04BBNPPDNC@Edit?$AA@ 00469d30     window.obj
 0002:00004d38       ??_C@_07OOFFCIDH@ListBox?$AA@ 00469d38     window.obj
 0002:00004d40       ??_C@_06KJMEDNIB@Static?$AA@ 00469d40     window.obj
 0002:00004d48       ??_C@_0L@PKBKLDDM@MainWindow?$AA@ 00469d48     window.obj
 0002:00004d54       ??_C@_0L@OBMBIFBF@text_color?$AA@ 00469d54     xmlsets.obj
 0002:00004d60       ??_C@_08IJAPCFHK@bk_color?$AA@ 00469d60     xmlsets.obj
 0002:00004d6c       ??_C@_03BANJEMDJ@say?$AA@  00469d6c     xmlsets.obj
 0002:00004d70       ??_C@_04CIMGMMMG@text?$AA@ 00469d70     xmlsets.obj
 0002:00004d78       ??_C@_08PJBINIIG@play_pos?$AA@ 00469d78     xmlsets.obj
 0002:00004d84       ??_C@_08OHGOKOGA@rotation?$AA@ 00469d84     xmlsets.obj
 0002:00004d90       ??_C@_08OAGMDKAF@position?$AA@ 00469d90     xmlsets.obj
 0002:00004d9c       ??_C@_0L@OHJPCEDH@normal_pos?$AA@ 00469d9c     xmlsets.obj
 0002:00004da8       ??_C@_08NLHBPEGP@password?$AA@ 00469da8     xmlsets.obj
 0002:00004db4       ??_C@_08GHIDDNMN@nickname?$AA@ 00469db4     xmlsets.obj
 0002:00004dc0       ??_C@_06HJHJCKIO@server?$AA@ 00469dc0     xmlsets.obj
 0002:00004dc8       ??_C@_0M@FEDFAMDF@imitatechat?$AA@ 00469dc8     xmlsets.obj
 0002:00004dd4       ??_C@_0O@HCNPKHCE@followZOffset?$AA@ 00469dd4     xmlsets.obj
 0002:00004de4       ??_C@_0O@PMFAKAMH@followYOffset?$AA@ 00469de4     xmlsets.obj
 0002:00004df4       ??_C@_0O@DAPKKAFJ@followXOffset?$AA@ 00469df4     xmlsets.obj
 0002:00004e04       ??_C@_0BK@HBDPBCKC@followplayerwithvehicleid?$AA@ 00469e04     xmlsets.obj
 0002:00004e20       ??_C@_0N@MCCPMFCE@followplayer?$AA@ 00469e20     xmlsets.obj
 0002:00004e30       ??_C@_0O@FOBBCBCF@clientmsg_rgb?$AA@ 00469e30     xmlsets.obj
 0002:00004e40       ??_C@_0O@BDHIBEFG@chatcolor_rgb?$AA@ 00469e40     xmlsets.obj
 0002:00004e50       ??_C@_0BB@GLCKHNMB@print_timestamps?$AA@ 00469e50     xmlsets.obj
 0002:00004e64       ??_C@_0P@NIABBIBP@select_classid?$AA@ 00469e64     xmlsets.obj
 0002:00004e74       ??_C@_04CKFJHKAP@find?$AA@ 00469e74     xmlsets.obj
 0002:00004e7c       ??_C@_07NLGPFEPB@autorun?$AA@ 00469e7c     xmlsets.obj
 0002:00004e84       ??_C@_07KNLFIPGK@runmode?$AA@ 00469e84     xmlsets.obj
 0002:00004e8c       ??_C@_07PMJAFAE@console?$AA@ 00469e8c     xmlsets.obj
 0002:00004e94       ??_C@_0O@BDEOGKOI@RakSAMPClient?$AA@ 00469e94     xmlsets.obj
 0002:00004ea4       ??_C@_0BP@HFCMMJC@Failed?5to?5load?5the?5config?5file?$AA@ 00469ea4     xmlsets.obj
 0002:00004ec4       ??_C@_0BC@OFPCGBLK@RakSAMPClient?4xml?$AA@ 00469ec4     xmlsets.obj
 0002:00004ed8       ??_C@_0BK@CACBKOLI@Failed?5to?5reload?5settings?$AA@ 00469ed8     xmlsets.obj
 0002:00004ef4       ??_C@_0BC@OIMIGJAK@Settings?5reloaded?$AA@ 00469ef4     xmlsets.obj
 0002:00004f08       ??_C@_15IABLJNFO@?$AA?6?$AA?6?$AA?$AA@ 00469f08     LIBCMT:wassert.obj
 0002:00004f10       ??_C@_13LBAGMAIH@?$AA?6?$AA?$AA@ 00469f10     LIBCMT:wassert.obj
 0002:00004f14       ??_C@_17LGKOMLJ@?$AA?4?$AA?4?$AA?4?$AA?$AA@ 00469f14     LIBCMT:wassert.obj
 0002:00004f20       ??_C@_1EK@MBDPDCGA@?$AAM?$AAi?$AAc?$AAr?$AAo?$AAs?$AAo?$AAf?$AAt?$AA?5?$AAV?$AAi?$AAs?$AAu?$AAa?$AAl?$AA?5?$AAC?$AA?$CL?$AA?$CL?$AA?5?$AAR?$AAu?$AAn?$AAt?$AAi?$AAm?$AAe?$AA?5?$AAL?$AAi?$AAb@ 00469f20     LIBCMT:wassert.obj
 0002:00004f70       ??_C@_1HK@POCJMFGK@?$AA?$CI?$AAP?$AAr?$AAe?$AAs?$AAs?$AA?5?$AAR?$AAe?$AAt?$AAr?$AAy?$AA?5?$AAt?$AAo?$AA?5?$AAd?$AAe?$AAb?$AAu?$AAg?$AA?5?$AAt?$AAh?$AAe?$AA?5?$AAa?$AAp?$AAp?$AAl?$AAi?$AAc@ 00469f70     LIBCMT:wassert.obj
 0002:00004ff0       ??_C@_1OA@EGMLFBHJ@?$AAF?$AAo?$AAr?$AA?5?$AAi?$AAn?$AAf?$AAo?$AAr?$AAm?$AAa?$AAt?$AAi?$AAo?$AAn?$AA?5?$AAo?$AAn?$AA?5?$AAh?$AAo?$AAw?$AA?5?$AAy?$AAo?$AAu?$AAr?$AA?5?$AAp?$AAr?$AAo?$AAg@ 00469ff0     LIBCMT:wassert.obj
 0002:000050d0       ??_C@_1BK@PEDCIPMA@?$AAE?$AAx?$AAp?$AAr?$AAe?$AAs?$AAs?$AAi?$AAo?$AAn?$AA?3?$AA?5?$AA?$AA@ 0046a0d0     LIBCMT:wassert.obj
 0002:000050ec       ??_C@_1O@KCAFKHJE@?$AAL?$AAi?$AAn?$AAe?$AA?3?$AA?5?$AA?$AA@ 0046a0ec     LIBCMT:wassert.obj
 0002:000050fc       ??_C@_1O@HEMHKNDC@?$AAF?$AAi?$AAl?$AAe?$AA?3?$AA?5?$AA?$AA@ 0046a0fc     LIBCMT:wassert.obj
 0002:0000510c       ??_C@_1CO@EAEJAADC@?$AA?$DM?$AAp?$AAr?$AAo?$AAg?$AAr?$AAa?$AAm?$AA?5?$AAn?$AAa?$AAm?$AAe?$AA?5?$AAu?$AAn?$AAk?$AAn?$AAo?$AAw?$AAn?$AA?$DO?$AA?$AA@ 0046a10c     LIBCMT:wassert.obj
 0002:0000513c       ??_C@_1BE@PHKBBGE@?$AAP?$AAr?$AAo?$AAg?$AAr?$AAa?$AAm?$AA?3?$AA?5?$AA?$AA@ 0046a13c     LIBCMT:wassert.obj
 0002:00005150       ??_C@_1CE@OJBNHDMO@?$AAA?$AAs?$AAs?$AAe?$AAr?$AAt?$AAi?$AAo?$AAn?$AA?5?$AAf?$AAa?$AAi?$AAl?$AAe?$AAd?$AA?$CB?$AA?$AA@ 0046a150     LIBCMT:wassert.obj
 0002:00005178       ??_7bad_alloc@std@@6B@     0046a178     LIBCMT:new.obj
 0002:00005180       ?ProcessDetach@NativeDll@<CrtImplementationDetails>@@0IB 0046a180     LIBCMT:_trnsctrl_.obj
 0002:00005184       ?ProcessAttach@NativeDll@<CrtImplementationDetails>@@0IB 0046a184     LIBCMT:_trnsctrl_.obj
 0002:00005188       ?ThreadAttach@NativeDll@<CrtImplementationDetails>@@0IB 0046a188     LIBCMT:_trnsctrl_.obj
 0002:0000518c       ?ThreadDetach@NativeDll@<CrtImplementationDetails>@@0IB 0046a18c     LIBCMT:_trnsctrl_.obj
 0002:00005190       ?ProcessVerifier@NativeDll@<CrtImplementationDetails>@@0IB 0046a190     LIBCMT:_trnsctrl_.obj
 0002:00005198       ??_7type_info@@6B@         0046a198     LIBCMT:typinfo.obj
 0002:0000519c       __FPinit                   0046a19c     LIBCMT:_fpinit_.obj
 0002:000051a0       __FPmtinit                 0046a1a0     LIBCMT:_fpinit_.obj
 0002:000051a4       __FPmtterm                 0046a1a4     LIBCMT:_fpinit_.obj
 0002:00005200       ??_C@_0P@MIGLKIOC@CorExitProcess?$AA@ 0046a200     LIBCMT:crt0dat.obj
 0002:00005210       ??_C@_1BI@BGOHAHKC@?$AAm?$AAs?$AAc?$AAo?$AAr?$AAe?$AAe?$AA?4?$AAd?$AAl?$AAl?$AA?$AA@ 0046a210     LIBCMT:crt0dat.obj
 0002:00005228       ??_C@_0P@GGKDKEEG@runtime?5error?5?$AA@ 0046a228     LIBCMT:crt0msg.obj
 0002:00005238       ??_C@_02PCIJFNDE@?$AN?6?$AA@ 0046a238     LIBCMT:crt0msg.obj
 0002:0000523c       ??_C@_0O@MJNIPGOH@TLOSS?5error?$AN?6?$AA@ 0046a23c     LIBCMT:crt0msg.obj
 0002:0000524c       ??_C@_0N@BONNPDHF@SING?5error?$AN?6?$AA@ 0046a24c     LIBCMT:crt0msg.obj
 0002:0000525c       ??_C@_0P@MBDAJNE@DOMAIN?5error?$AN?6?$AA@ 0046a25c     LIBCMT:crt0msg.obj
 0002:00005270       ??_C@_0JL@DFDOOABL@R6034?$AN?6An?5application?5has?5made?5a@ 0046a270     LIBCMT:crt0msg.obj
 0002:00005310       ??_C@_0PH@EPAFIJ@R6033?$AN?6?9?5Attempt?5to?5use?5MSIL?5cod@ 0046a310     LIBCMT:crt0msg.obj
 0002:00005408       ??_C@_0DD@BKEEABMM@R6032?$AN?6?9?5not?5enough?5space?5for?5lo@ 0046a408     LIBCMT:crt0msg.obj
 0002:00005440       ??_C@_0GD@OFKILIED@R6031?$AN?6?9?5Attempt?5to?5initialize?5t@ 0046a440     LIBCMT:crt0msg.obj
 0002:000054a4       ??_C@_0BP@LPMHJOKI@R6030?$AN?6?9?5CRT?5not?5initialized?$AN?6?$AA@ 0046a4a4     LIBCMT:crt0msg.obj
 0002:000054c4       ??_C@_0CF@KJDAIALP@R6028?$AN?6?9?5unable?5to?5initialize?5he@ 0046a4c4     LIBCMT:crt0msg.obj
 0002:000054ec       ??_C@_0DF@GAKBPDFP@R6027?$AN?6?9?5not?5enough?5space?5for?5lo@ 0046a4ec     LIBCMT:crt0msg.obj
 0002:00005524       ??_C@_0DF@IBLNNAIG@R6026?$AN?6?9?5not?5enough?5space?5for?5st@ 0046a524     LIBCMT:crt0msg.obj
 0002:0000555c       ??_C@_0CG@IOHKGFNJ@R6025?$AN?6?9?5pure?5virtual?5function?5c@ 0046a55c     LIBCMT:crt0msg.obj
 0002:00005584       ??_C@_0DF@JIJJFJDC@R6024?$AN?6?9?5not?5enough?5space?5for?5_o@ 0046a584     LIBCMT:crt0msg.obj
 0002:000055bc       ??_C@_0CJ@EGEJHFME@R6019?$AN?6?9?5unable?5to?5open?5console?5@ 0046a5bc     LIBCMT:crt0msg.obj
 0002:000055e8       ??_C@_0CB@GNHNIELH@R6018?$AN?6?9?5unexpected?5heap?5error?$AN?6@ 0046a5e8     LIBCMT:crt0msg.obj
 0002:0000560c       ??_C@_0CN@FOLDKNG@R6017?$AN?6?9?5unexpected?5multithread?5@ 0046a60c     LIBCMT:crt0msg.obj
 0002:0000563c       ??_C@_0CM@FAHFJNHO@R6016?$AN?6?9?5not?5enough?5space?5for?5th@ 0046a63c     LIBCMT:crt0msg.obj
 0002:00005668       ??_C@_0JG@LBKMGKLD@?$AN?6This?5application?5has?5requested@ 0046a668     LIBCMT:crt0msg.obj
 0002:00005700       ??_C@_0CM@FLCNIPKK@R6009?$AN?6?9?5not?5enough?5space?5for?5en@ 0046a700     LIBCMT:crt0msg.obj
 0002:0000572c       ??_C@_0CK@KMMJOAPP@R6008?$AN?6?9?5not?5enough?5space?5for?5ar@ 0046a72c     LIBCMT:crt0msg.obj
 0002:00005758       ??_C@_0CN@LEKKICBM@R6002?$AN?6?9?5floating?5point?5support?5@ 0046a758     LIBCMT:crt0msg.obj
 0002:00005788       ??_C@_0CF@GOGNBNAK@Microsoft?5Visual?5C?$CL?$CL?5Runtime?5Lib@ 0046a788     LIBCMT:crt0msg.obj
 0002:000057b0       ??_C@_03KHICJKCI@?4?4?4?$AA@ 0046a7b0     LIBCMT:crt0msg.obj
 0002:000057b4       ??_C@_0BH@DNAGHKFM@?$DMprogram?5name?5unknown?$DO?$AA@ 0046a7b4     LIBCMT:crt0msg.obj
 0002:000057cc       ??_C@_0BK@OFGJDLJJ@Runtime?5Error?$CB?6?6Program?3?5?$AA@ 0046a7cc     LIBCMT:crt0msg.obj
 0002:000057e8       ??_C@_0BI@DFKBFLJE@GetProcessWindowStation?$AA@ 0046a7e8     LIBCMT:crtmboxw.obj
 0002:00005800       ??_C@_0BK@DEKFELLI@GetUserObjectInformationW?$AA@ 0046a800     LIBCMT:crtmboxw.obj
 0002:0000581c       ??_C@_0BD@HHGDFDBJ@GetLastActivePopup?$AA@ 0046a81c     LIBCMT:crtmboxw.obj
 0002:00005830       ??_C@_0BA@HNOPNCHB@GetActiveWindow?$AA@ 0046a830     LIBCMT:crtmboxw.obj
 0002:00005840       ??_C@_0M@DLDCCGNP@MessageBoxW?$AA@ 0046a840     LIBCMT:crtmboxw.obj
 0002:0000584c       ??_C@_1BG@GOEBHBDC@?$AAU?$AAS?$AAE?$AAR?$AA3?$AA2?$AA?4?$AAD?$AAL?$AAL?$AA?$AA@ 0046a84c     LIBCMT:crtmboxw.obj
 0002:00005864       ??_C@_1O@CEDCILHN@?$AA?$CI?$AAn?$AAu?$AAl?$AAl?$AA?$CJ?$AA?$AA@ 0046a864     LIBCMT:output.obj
 0002:00005874       ??_C@_06OJHGLDPL@?$CInull?$CJ?$AA@ 0046a874     LIBCMT:output.obj
 0002:00005880       ___lookuptable             0046a880     LIBCMT:output.obj
 0002:000058e0       ??_7exception@std@@6B@     0046a8e0     LIBCMT:stdexcpt.obj
 0002:000058e8       ??_C@_0BC@EOODALEL@Unknown?5exception?$AA@ 0046a8e8     LIBCMT:stdexcpt.obj
 0002:00005900       ??_7bad_cast@std@@6B@      0046a900     LIBCMT:stdexcpt.obj
 0002:0000590c       ??_7bad_typeid@std@@6B@    0046a90c     LIBCMT:stdexcpt.obj
 0002:00005918       ??_7__non_rtti_object@std@@6B@ 0046a918     LIBCMT:stdexcpt.obj
 0002:00005940       __pDestructExceptionObject 0046a940     LIBCMT:frame.obj
 0002:00005948       ??_7bad_exception@std@@6B@ 0046a948     LIBCMT:frame.obj
 0002:00005950       ??_C@_0O@DPKOEFFH@bad?5exception?$AA@ 0046a950     LIBCMT:frame.obj
 0002:00005960       ??_C@_0O@NLDKAIKN@EncodePointer?$AA@ 0046a960     LIBCMT:tidtable.obj
 0002:00005970       ??_C@_1BK@DBDEIDLH@?$AAK?$AAE?$AAR?$AAN?$AAE?$AAL?$AA3?$AA2?$AA?4?$AAD?$AAL?$AAL?$AA?$AA@ 0046a970     LIBCMT:tidtable.obj
 0002:0000598c       ??_C@_0O@KBPMFGHI@DecodePointer?$AA@ 0046a98c     LIBCMT:tidtable.obj
 0002:0000599c       ??_C@_07PEJMOBNF@FlsFree?$AA@ 0046a99c     LIBCMT:tidtable.obj
 0002:000059a4       ??_C@_0M@JCPCPOEF@FlsSetValue?$AA@ 0046a9a4     LIBCMT:tidtable.obj
 0002:000059b0       ??_C@_0M@GDNOONDI@FlsGetValue?$AA@ 0046a9b0     LIBCMT:tidtable.obj
 0002:000059bc       ??_C@_08KNHFBNJ@FlsAlloc?$AA@ 0046a9bc     LIBCMT:tidtable.obj
 0002:000059c8       ??_C@_05KLBDPFGC@e?$CL000?$AA@ 0046a9c8     LIBCMT:cvt.obj
 0002:000059d0       __real@4150017ec0000000    0046a9d0     LIBCMT:_testfdiv_.obj
 0002:000059d8       __real@4147ffff80000000    0046a9d8     LIBCMT:_testfdiv_.obj
 0002:000059e0       ??_C@_0BK@NHEOCAHP@IsProcessorFeaturePresent?$AA@ 0046a9e0     LIBCMT:_testfdiv_.obj
 0002:000059fc       ??_C@_08CPNIBGIE@KERNEL32?$AA@ 0046a9fc     LIBCMT:_testfdiv_.obj
 0002:00005a08       __XcptActTab               0046aa08     LIBCMT:winxfltr.obj
 0002:00005aa0       ??_C@_07LCBHPJJN@LC_TIME?$AA@ 0046aaa0     LIBCMT:setlocal.obj
 0002:00005aa8       ??_C@_0L@DLHIECNL@LC_NUMERIC?$AA@ 0046aaa8     LIBCMT:setlocal.obj
 0002:00005ab4       ??_C@_0M@MIENIKLA@LC_MONETARY?$AA@ 0046aab4     LIBCMT:setlocal.obj
 0002:00005ac0       ??_C@_08EADHIDAD@LC_CTYPE?$AA@ 0046aac0     LIBCMT:setlocal.obj
 0002:00005acc       ??_C@_0L@KFJHEKIK@LC_COLLATE?$AA@ 0046aacc     LIBCMT:setlocal.obj
 0002:00005ad8       ??_C@_06NEFDFEKB@LC_ALL?$AA@ 0046aad8     LIBCMT:setlocal.obj
 0002:00005ae0       ___lc_category             0046aae0     LIBCMT:setlocal.obj
 0002:00005ba8       ??_C@_03EGDHDPFD@_?4?0?$AA@ 0046aba8     LIBCMT:setlocal.obj
 0002:00005bac       ??_C@_01LFCBOECM@?4?$AA@   0046abac     LIBCMT:setlocal.obj
 0002:00005bb0       ??_C@_01IDAFKMJL@_?$AA@    0046abb0     LIBCMT:setlocal.obj
 0002:00005bb4       ??_C@_01ICJEACDI@?$DL?$AA@ 0046abb4     LIBCMT:setlocal.obj
 0002:00005bb8       ??_C@_01NEMOKFLO@?$DN?$AA@ 0046abb8     LIBCMT:setlocal.obj
 0002:00005bbc       ??_C@_01GFHCPBMG@C?$AA@    0046abbc     LIBCMT:setlocal.obj
 0002:00005bc0       ??_C@_02BALPLPBG@?$DN?$DL?$AA@ 0046abc0     LIBCMT:setlocal.obj
 0002:00005bc8       ___lookuptable_s           0046abc8     LIBCMT:outputs.obj
 0002:00005c24       ??_C@_13NOLLCAOD@?$AA?$AA?$AA?$AA@ 0046ac24     LIBCMT:a_map.obj
 0002:000064e8       __DEFAULT_CW_in_mem        0046b4e8     LIBCMT:_common_.obj
 0002:000064ea       __pi_by_2_to_61            0046b4ea     LIBCMT:_common_.obj
 0002:00006590       ??_C@_03IIINPABG@tan?$AA@  0046b590     LIBCMT:_libm_error_.obj
 0002:00006594       ??_C@_03LALBNOCG@cos?$AA@  0046b594     LIBCMT:_libm_error_.obj
 0002:00006598       ??_C@_03BLEJJJBH@sin?$AA@  0046b598     LIBCMT:_libm_error_.obj
 0002:0000659c       ??_C@_04EHEDPDJG@modf?$AA@ 0046b59c     LIBCMT:_libm_error_.obj
 0002:000065a4       ??_C@_05PBJFFIGL@floor?$AA@ 0046b5a4     LIBCMT:_libm_error_.obj
 0002:000065ac       ??_C@_04GFPJNGEK@ceil?$AA@ 0046b5ac     LIBCMT:_libm_error_.obj
 0002:000065b4       ??_C@_04MLLJIGOK@atan?$AA@ 0046b5b4     LIBCMT:_libm_error_.obj
 0002:000065bc       ??_C@_05EOHGHCHD@exp10?$AA@ 0046b5bc     LIBCMT:_libm_error_.obj
 0002:000065c4       ??_C@_04PDIFKINK@acos?$AA@ 0046b5c4     LIBCMT:_libm_error_.obj
 0002:000065cc       ??_C@_04FIHNOPOL@asin?$AA@ 0046b5cc     LIBCMT:_libm_error_.obj
 0002:000065d4       ??_C@_03MGHMBJCF@log?$AA@  0046b5d4     LIBCMT:_libm_error_.obj
 0002:000065d8       ??_C@_05HGHHAHAP@log10?$AA@ 0046b5d8     LIBCMT:_libm_error_.obj
 0002:000065e0       ??_C@_03KHJOGHMM@exp?$AA@  0046b5e0     LIBCMT:_libm_error_.obj
 0002:000065e4       ??_C@_03JGHBODFD@pow?$AA@  0046b5e4     LIBCMT:_libm_error_.obj
 0002:00006e90       ??_C@_0L@KDOEJCKC@_nextafter?$AA@ 0046be90     LIBCMT:_fpexcept_.obj
 0002:00006e9c       ??_C@_05JGDBENOH@_logb?$AA@ 0046be9c     LIBCMT:_fpexcept_.obj
 0002:00006ea4       ??_C@_03ONILCKOB@_yn?$AA@  0046bea4     LIBCMT:_fpexcept_.obj
 0002:00006ea8       ??_C@_03NAKIGLHK@_y1?$AA@  0046bea8     LIBCMT:_fpexcept_.obj
 0002:00006eac       ??_C@_03MJLDFKDL@_y0?$AA@  0046beac     LIBCMT:_fpexcept_.obj
 0002:00006eb0       ??_C@_05GKKHEGJL@frexp?$AA@ 0046beb0     LIBCMT:_fpexcept_.obj
 0002:00006eb8       ??_C@_04KEPJIHGP@fmod?$AA@ 0046beb8     LIBCMT:_fpexcept_.obj
 0002:00006ec0       ??_C@_06MEIMCGCF@_hypot?$AA@ 0046bec0     LIBCMT:_fpexcept_.obj
 0002:00006ec8       ??_C@_05KBKMEMPO@_cabs?$AA@ 0046bec8     LIBCMT:_fpexcept_.obj
 0002:00006ed0       ??_C@_05CEJMAHNP@ldexp?$AA@ 0046bed0     LIBCMT:_fpexcept_.obj
 0002:00006ed8       ??_C@_04ODHECPBC@fabs?$AA@ 0046bed8     LIBCMT:_fpexcept_.obj
 0002:00006ee0       ??_C@_04EIAKFFMI@sqrt?$AA@ 0046bee0     LIBCMT:_fpexcept_.obj
 0002:00006ee8       ??_C@_05KNGEOGJB@atan2?$AA@ 0046bee8     LIBCMT:_fpexcept_.obj
 0002:00006ef0       ??_C@_04FJHINJAO@tanh?$AA@ 0046bef0     LIBCMT:_fpexcept_.obj
 0002:00006ef8       ??_C@_04HPJJNFIM@cosh?$AA@ 0046bef8     LIBCMT:_fpexcept_.obj
 0002:00006f00       ??_C@_04COOMCNPB@sinh?$AA@ 0046bf00     LIBCMT:_fpexcept_.obj
 0002:00006f08       ??_C@_0BC@JEAENNKH@SystemFunction036?$AA@ 0046bf08     LIBCMT:rand_s.obj
 0002:00006f1c       ??_C@_0N@JJPEKNFO@ADVAPI32?4DLL?$AA@ 0046bf1c     LIBCMT:rand_s.obj
 0002:00006f2c       ??_C@_0BK@CIDNPOGP@GetUserObjectInformationA?$AA@ 0046bf2c     LIBCMT:crtmbox.obj
 0002:00006f48       ??_C@_0M@CHKKJDAI@MessageBoxA?$AA@ 0046bf48     LIBCMT:crtmbox.obj
 0002:00006f54       ??_C@_0L@NDEGIDAG@USER32?4DLL?$AA@ 0046bf54     LIBCMT:crtmbox.obj
 0002:00006f68       ??_C@_0BK@CFCOFLF@?5Complete?5Object?5Locator?8?$AA@ 0046bf68     LIBCMT:undname.obj
 0002:00006f84       ??_C@_0BN@MECKDCOJ@?5Class?5Hierarchy?5Descriptor?8?$AA@ 0046bf84     LIBCMT:undname.obj
 0002:00006fa4       ??_C@_0BD@LGICGFMM@?5Base?5Class?5Array?8?$AA@ 0046bfa4     LIBCMT:undname.obj
 0002:00006fb8       ??_C@_0BM@LDKODKLH@?5Base?5Class?5Descriptor?5at?5?$CI?$AA@ 0046bfb8     LIBCMT:undname.obj
 0002:00006fd4       ??_C@_0BC@DAFEJGAK@?5Type?5Descriptor?8?$AA@ 0046bfd4     LIBCMT:undname.obj
 0002:00006fe8       ??_C@_0BM@PMGGMLDN@?$GAlocal?5static?5thread?5guard?8?$AA@ 0046bfe8     LIBCMT:undname.obj
 0002:00007004       ??_C@_0CL@FGIJHLCE@?$GAmanaged?5vector?5copy?5constructor@ 0046c004     LIBCMT:undname.obj
 0002:00007030       ??_C@_0CJ@GJELGAMM@?$GAvector?5vbase?5copy?5constructor?5i@ 0046c030     LIBCMT:undname.obj
 0002:0000705c       ??_C@_0CD@CGAJBKEJ@?$GAvector?5copy?5constructor?5iterato@ 0046c05c     LIBCMT:undname.obj
 0002:00007080       ??_C@_0CB@PDBIFEP@?$GAdynamic?5atexit?5destructor?5for?5?8@ 0046c080     LIBCMT:undname.obj
 0002:000070a4       ??_C@_0BL@CLIPGLGB@?$GAdynamic?5initializer?5for?5?8?$AA@ 0046c0a4     LIBCMT:undname.obj
 0002:000070c0       ??_C@_0CM@FCBBDIGB@?$GAeh?5vector?5vbase?5copy?5constructo@ 0046c0c0     LIBCMT:undname.obj
 0002:000070ec       ??_C@_0CG@HLDDJMAG@?$GAeh?5vector?5copy?5constructor?5iter@ 0046c0ec     LIBCMT:undname.obj
 0002:00007114       ??_C@_0CF@IMGKMJNO@?$GAmanaged?5vector?5destructor?5itera@ 0046c114     LIBCMT:undname.obj
 0002:0000713c       ??_C@_0CG@CFDHKGGD@?$GAmanaged?5vector?5constructor?5iter@ 0046c13c     LIBCMT:undname.obj
 0002:00007164       ??_C@_0BN@CKNJLHMB@?$GAplacement?5delete?$FL?$FN?5closure?8?$AA@ 0046c164     LIBCMT:undname.obj
 0002:00007184       ??_C@_0BL@CNOONJFP@?$GAplacement?5delete?5closure?8?$AA@ 0046c184     LIBCMT:undname.obj
 0002:000071a0       ??_C@_0P@HJKNJFNN@?$GAomni?5callsig?8?$AA@ 0046c1a0     LIBCMT:undname.obj
 0002:000071b0       ??_C@_09LBNFPBCA@?5delete?$FL?$FN?$AA@ 0046c1b0     LIBCMT:undname.obj
 0002:000071bc       ??_C@_06FHBGPFGH@?5new?$FL?$FN?$AA@ 0046c1bc     LIBCMT:undname.obj
 0002:000071c4       ??_C@_0CE@IIHCMGGL@?$GAlocal?5vftable?5constructor?5closu@ 0046c1c4     LIBCMT:undname.obj
 0002:000071e8       ??_C@_0BA@KKLDJDLB@?$GAlocal?5vftable?8?$AA@ 0046c1e8     LIBCMT:undname.obj
 0002:000071f8       ??_C@_05KHLCHHI@?$GARTTI?$AA@ 0046c1f8     LIBCMT:undname.obj
 0002:00007200       ??_C@_03KLGMFNMG@?$GAEH?$AA@ 0046c200     LIBCMT:undname.obj
 0002:00007204       ??_C@_0BA@KBCDOMBN@?$GAudt?5returning?8?$AA@ 0046c204     LIBCMT:undname.obj
 0002:00007214       ??_C@_0BL@LLKPOHJI@?$GAcopy?5constructor?5closure?8?$AA@ 0046c214     LIBCMT:undname.obj
 0002:00007230       ??_C@_0CH@OOJPLCPH@?$GAeh?5vector?5vbase?5constructor?5ite@ 0046c230     LIBCMT:undname.obj
 0002:00007258       ??_C@_0CA@GCEOPDGL@?$GAeh?5vector?5destructor?5iterator?8?$AA@ 0046c258     LIBCMT:undname.obj
 0002:00007278       ??_C@_0CB@JONCMFFK@?$GAeh?5vector?5constructor?5iterator?8@ 0046c278     LIBCMT:undname.obj
 0002:0000729c       ??_C@_0BL@NILFHHPC@?$GAvirtual?5displacement?5map?8?$AA@ 0046c29c     LIBCMT:undname.obj
 0002:000072b8       ??_C@_0CE@IKBNEHA@?$GAvector?5vbase?5constructor?5iterat@ 0046c2b8     LIBCMT:undname.obj
 0002:000072dc       ??_C@_0BN@LFPFMEDL@?$GAvector?5destructor?5iterator?8?$AA@ 0046c2dc     LIBCMT:undname.obj
 0002:000072fc       ??_C@_0BO@PFGOCPJJ@?$GAvector?5constructor?5iterator?8?$AA@ 0046c2fc     LIBCMT:undname.obj
 0002:0000731c       ??_C@_0BN@IMDCHIKM@?$GAscalar?5deleting?5destructor?8?$AA@ 0046c31c     LIBCMT:undname.obj
 0002:0000733c       ??_C@_0BO@OBMKPJIG@?$GAdefault?5constructor?5closure?8?$AA@ 0046c33c     LIBCMT:undname.obj
 0002:0000735c       ??_C@_0BN@DEGPLNFK@?$GAvector?5deleting?5destructor?8?$AA@ 0046c35c     LIBCMT:undname.obj
 0002:0000737c       ??_C@_0BD@JDLKDPAB@?$GAvbase?5destructor?8?$AA@ 0046c37c     LIBCMT:undname.obj
 0002:00007390       ??_C@_08OBABFOLI@?$GAstring?8?$AA@ 0046c390     LIBCMT:undname.obj
 0002:0000739c       ??_C@_0BF@KDPPACIK@?$GAlocal?5static?5guard?8?$AA@ 0046c39c     LIBCMT:undname.obj
 0002:000073b4       ??_C@_08LLFFHHDJ@?$GAtypeof?8?$AA@ 0046c3b4     LIBCMT:undname.obj
 0002:000073c0       ??_C@_07FEEIOKP@?$GAvcall?8?$AA@ 0046c3c0     LIBCMT:undname.obj
 0002:000073c8       ??_C@_09BLBHBJP@?$GAvbtable?8?$AA@ 0046c3c8     LIBCMT:undname.obj
 0002:000073d4       ??_C@_09IFPLHPGF@?$GAvftable?8?$AA@ 0046c3d4     LIBCMT:undname.obj
 0002:000073e0       ??_C@_02MHEGNOJ@?$FO?$DN?$AA@ 0046c3e0     LIBCMT:undname.obj
 0002:000073e4       ??_C@_02DHLNPPGH@?$HM?$DN?$AA@ 0046c3e4     LIBCMT:undname.obj
 0002:000073e8       ??_C@_02FGJGFEAB@?$CG?$DN?$AA@ 0046c3e8     LIBCMT:undname.obj
 0002:000073ec       ??_C@_03CDNPDDLA@?$DM?$DM?$DN?$AA@ 0046c3ec     LIBCMT:undname.obj
 0002:000073f0       ??_C@_03IKFCCPFF@?$DO?$DO?$DN?$AA@ 0046c3f0     LIBCMT:undname.obj
 0002:000073f4       ??_C@_02FENAOKFI@?$CF?$DN?$AA@ 0046c3f4     LIBCMT:undname.obj
 0002:000073f8       ??_C@_02FJEHGPIO@?1?$DN?$AA@ 0046c3f8     LIBCMT:undname.obj
 0002:000073fc       ??_C@_02FKMDLLOA@?9?$DN?$AA@ 0046c3fc     LIBCMT:undname.obj
 0002:00007400       ??_C@_02FOEOMHFC@?$CL?$DN?$AA@ 0046c400     LIBCMT:undname.obj
 0002:00007404       ??_C@_02FPIMKNGF@?$CK?$DN?$AA@ 0046c404     LIBCMT:undname.obj
 0002:00007408       ??_C@_02NONPIBCD@?$HM?$HM?$AA@ 0046c408     LIBCMT:undname.obj
 0002:0000740c       ??_C@_02PPKAJPJL@?$CG?$CG?$AA@ 0046c40c     LIBCMT:undname.obj
 0002:00007410       ??_C@_01DNKMNLPK@?$HM?$AA@ 0046c410     LIBCMT:undname.obj
 0002:00007414       ??_C@_01JKBOJNNK@?$FO?$AA@ 0046c414     LIBCMT:undname.obj
 0002:00007418       ??_C@_01PJKLJHI@?$HO?$AA@  0046c418     LIBCMT:undname.obj
 0002:0000741c       ??_C@_02HCKGKOFO@?$CI?$CJ?$AA@ 0046c41c     LIBCMT:undname.obj
 0002:00007420       ??_C@_01IHBHIGKO@?0?$AA@   0046c420     LIBCMT:undname.obj
 0002:00007424       ??_C@_02EEKDKGMJ@?$DO?$DN?$AA@ 0046c424     LIBCMT:undname.obj
 0002:00007428       ??_C@_02EHCHHCKH@?$DM?$DN?$AA@ 0046c428     LIBCMT:undname.obj
 0002:0000742c       ??_C@_01FGNFDNOH@?$CF?$AA@ 0046c42c     LIBCMT:undname.obj
 0002:00007430       ??_C@_01KMDKNFGN@?1?$AA@   0046c430     LIBCMT:undname.obj
 0002:00007434       ??_C@_03MNHNFDLC@?9?$DO?$CK?$AA@ 0046c434     LIBCMT:undname.obj
 0002:00007438       ??_C@_01HNPIGOCE@?$CG?$AA@ 0046c438     LIBCMT:undname.obj
 0002:0000743c       ??_C@_01MIFGBAGJ@?$CL?$AA@ 0046c43c     LIBCMT:undname.obj
 0002:00007440       ??_C@_01JOAMLHOP@?9?$AA@   0046c440     LIBCMT:undname.obj
 0002:00007444       ??_C@_02BAABKJLB@?9?9?$AA@ 0046c444     LIBCMT:undname.obj
 0002:00007448       ??_C@_02ECNGHCIF@?$CL?$CL?$AA@ 0046c448     LIBCMT:undname.obj
 0002:0000744c       ??_C@_01NBENCBCI@?$CK?$AA@ 0046c44c     LIBCMT:undname.obj
 0002:00007450       ??_C@_02HBOOOICD@?9?$DO?$AA@ 0046c450     LIBCMT:undname.obj
 0002:00007454       ??_C@_08LHJFAFGD@operator?$AA@ 0046c454     LIBCMT:undname.obj
 0002:00007460       ??_C@_02GPECMEKF@?$FL?$FN?$AA@ 0046c460     LIBCMT:undname.obj
 0002:00007464       ??_C@_02FDNJECIE@?$CB?$DN?$AA@ 0046c464     LIBCMT:undname.obj
 0002:00007468       ??_C@_02EGOFBIJA@?$DN?$DN?$AA@ 0046c468     LIBCMT:undname.obj
 0002:0000746c       ??_C@_01DCLJPIOD@?$CB?$AA@ 0046c46c     LIBCMT:undname.obj
 0002:00007470       ??_C@_02FODMEDOG@?$DM?$DM?$AA@ 0046c470     LIBCMT:undname.obj
 0002:00007474       ??_C@_02GPIOPFAK@?$DO?$DO?$AA@ 0046c474     LIBCMT:undname.obj
 0002:00007478       ??_C@_07FPCDHGMM@?5delete?$AA@ 0046c478     LIBCMT:undname.obj
 0002:00007480       ??_C@_04NIHEBCM@?5new?$AA@ 0046c480     LIBCMT:undname.obj
 0002:00007488       ??_C@_0M@GFIIJFMG@__unaligned?$AA@ 0046c488     LIBCMT:undname.obj
 0002:00007494       ??_C@_0L@PILCLIHE@__restrict?$AA@ 0046c494     LIBCMT:undname.obj
 0002:000074a0       ??_C@_07JOMMBBKO@__ptr64?$AA@ 0046c4a0     LIBCMT:undname.obj
 0002:000074a8       ??_C@_09HIJEGCPM@__clrcall?$AA@ 0046c4a8     LIBCMT:undname.obj
 0002:000074b4       ??_C@_0L@JMKHOMEK@__fastcall?$AA@ 0046c4b4     LIBCMT:undname.obj
 0002:000074c0       ??_C@_0L@NPHFGOKO@__thiscall?$AA@ 0046c4c0     LIBCMT:undname.obj
 0002:000074cc       ??_C@_09IFJBGAPI@__stdcall?$AA@ 0046c4cc     LIBCMT:undname.obj
 0002:000074d8       ??_C@_08GHMPAG@__pascal?$AA@ 0046c4d8     LIBCMT:undname.obj
 0002:000074e4       ??_C@_07KOLFKCDI@__cdecl?$AA@ 0046c4e4     LIBCMT:undname.obj
 0002:000074ec       ??_C@_08EHJDFFNH@__based?$CI?$AA@ 0046c4ec     LIBCMT:undname.obj
 0002:00007678       ??_7DNameNode@@6B@         0046c678     LIBCMT:undname.obj
 0002:00007684       ??_7charNode@@6B@          0046c684     LIBCMT:undname.obj
 0002:00007690       ??_7pDNameNode@@6B@        0046c690     LIBCMT:undname.obj
 0002:0000769c       ??_7DNameStatusNode@@6B@   0046c69c     LIBCMT:undname.obj
 0002:000076a8       ??_7pairNode@@6B@          0046c6a8     LIBCMT:undname.obj
 0002:000076b4       ??_7pcharNode@@6B@         0046c6b4     LIBCMT:undname.obj
 0002:000076c0       ??_C@_04OKOHEJBO@?5?$DP?$DP?5?$AA@ 0046c6c0     LIBCMT:undname.obj
 0002:000076c8       ??_C@_06EEGAIFAK@?$HLflat?$HN?$AA@ 0046c6c8     LIBCMT:undname.obj
 0002:000076d0       ??_C@_05JIBOFOHK@?$HLfor?5?$AA@ 0046c6d0     LIBCMT:undname.obj
 0002:000076d8       ??_C@_0BN@IBLMMFAP@?$GAnon?9type?9template?9parameter?$AA@ 0046c6d8     LIBCMT:undname.obj
 0002:000076f8       ??_C@_09EBBEKKIH@unsigned?5?$AA@ 0046c6f8     LIBCMT:undname.obj
 0002:00007704       ??_C@_05CJIMAING@long?5?$AA@ 0046c704     LIBCMT:undname.obj
 0002:0000770c       ??_C@_04LAHKHJMA@int?5?$AA@ 0046c70c     LIBCMT:undname.obj
 0002:00007714       ??_C@_06EHJMALKF@short?5?$AA@ 0046c714     LIBCMT:undname.obj
 0002:0000771c       ??_C@_05CIHEBHNO@char?5?$AA@ 0046c71c     LIBCMT:undname.obj
 0002:00007724       ??_C@_04GKJNKENE@void?$AA@ 0046c724     LIBCMT:undname.obj
 0002:0000772c       ??_C@_0L@EGPHHEKN@?$DMellipsis?$DO?$AA@ 0046c72c     LIBCMT:undname.obj
 0002:00007738       ??_C@_0M@ELJOJFFH@?0?$DMellipsis?$DO?$AA@ 0046c738     LIBCMT:undname.obj
 0002:00007744       ??_C@_04EENFHACM@?0?4?4?4?$AA@ 0046c744     LIBCMT:undname.obj
 0002:0000774c       ??_C@_07HDJPLPEK@?5throw?$CI?$AA@ 0046c74c     LIBCMT:undname.obj
 0002:00007754       ??_C@_02GOGNNPBN@?$CJ?$FL?$AA@ 0046c754     LIBCMT:undname.obj
 0002:00007758       ??_C@_02MDINNEEG@s?5?$AA@  0046c758     LIBCMT:undname.obj
 0002:0000775c       ??_C@_0BE@EODMJLIF@?$GAtemplate?9parameter?$AA@ 0046c75c     LIBCMT:undname.obj
 0002:00007770       ??_C@_04HIBGFPH@NULL?$AA@  0046c770     LIBCMT:undname.obj
 0002:00007778       ??_C@_0O@GKABPPIF@cli?3?3pin_ptr?$DM?$AA@ 0046c778     LIBCMT:undname.obj
 0002:00007788       ??_C@_0M@EALIELKG@cli?3?3array?$DM?$AA@ 0046c788     LIBCMT:undname.obj
 0002:00007794       ??_C@_05BEFAKPML@void?5?$AA@ 0046c794     LIBCMT:undname.obj
 0002:0000779c       ??_C@_02OHHJMEON@?8?8?$AA@ 0046c79c     LIBCMT:undname.obj
 0002:000077a0       ??_C@_0BG@JNJLAMPM@?$GAanonymous?5namespace?8?$AA@ 0046c7a0     LIBCMT:undname.obj
 0002:000077b8       ??_C@_01NLNLIGKH@?$GA?$AA@ 0046c7b8     LIBCMT:undname.obj
 0002:000077bc       ??_C@_0O@KHGCOMHP@generic?9type?9?$AA@ 0046c7bc     LIBCMT:undname.obj
 0002:000077cc       ??_C@_0BE@JAEOCHPE@template?9parameter?9?$AA@ 0046c7cc     LIBCMT:undname.obj
 0002:000077e0       ??_C@_02MOLJINC@?3?3?$AA@  0046c7e0     LIBCMT:undname.obj
 0002:000077e4       ??_C@_0P@GCIFDJCJ@?$GAunknown?5ecsu?8?$AA@ 0046c7e4     LIBCMT:undname.obj
 0002:000077f4       ??_C@_06MOJHIBMG@union?5?$AA@ 0046c7f4     LIBCMT:undname.obj
 0002:000077fc       ??_C@_07DIBCDNGL@struct?5?$AA@ 0046c7fc     LIBCMT:undname.obj
 0002:00007804       ??_C@_06LJBABKPM@class?5?$AA@ 0046c804     LIBCMT:undname.obj
 0002:0000780c       ??_C@_05LJGMCFOG@enum?5?$AA@ 0046c80c     LIBCMT:undname.obj
 0002:00007814       ??_C@_08KOFANOFK@coclass?5?$AA@ 0046c814     LIBCMT:undname.obj
 0002:00007820       ??_C@_0N@DLIEFKNA@cointerface?5?$AA@ 0046c820     LIBCMT:undname.obj
 0002:00007830       ??_C@_02KCKGHPCA@?$CJ?5?$AA@ 0046c830     LIBCMT:undname.obj
 0002:00007834       ??_C@_0M@DHNBOJMP@extern?5?$CCC?$CC?5?$AA@ 0046c834     LIBCMT:undname.obj
 0002:00007840       ??_C@_08KJLFOPNE@?$FLthunk?$FN?3?$AA@ 0046c840     LIBCMT:undname.obj
 0002:0000784c       ??_C@_08GPDDCMKI@public?3?5?$AA@ 0046c84c     LIBCMT:undname.obj
 0002:00007858       ??_C@_0M@GAIFPFIP@protected?3?5?$AA@ 0046c858     LIBCMT:undname.obj
 0002:00007864       ??_C@_09LAPHOOG@private?3?5?$AA@ 0046c864     LIBCMT:undname.obj
 0002:00007870       ??_C@_08NIEOINHE@virtual?5?$AA@ 0046c870     LIBCMT:undname.obj
 0002:0000787c       ??_C@_07PGOEDBHP@static?5?$AA@ 0046c87c     LIBCMT:undname.obj
 0002:00007884       ??_C@_0DA@HGFJFBBE@?$GAtemplate?5static?5data?5member?5des@ 0046c884     LIBCMT:undname.obj
 0002:000078b4       ??_C@_0DB@ILEFOCIJ@?$GAtemplate?5static?5data?5member?5con@ 0046c8b4     LIBCMT:undname.obj
 0002:000078e8       ??_C@_0CB@KJDOOODE@?$GAlocal?5static?5destructor?5helper?8@ 0046c8e8     LIBCMT:undname.obj
 0002:0000790c       ??_C@_0L@HNGCOGAE@?$GAadjustor?$HL?$AA@ 0046c90c     LIBCMT:undname.obj
 0002:00007918       ??_C@_0L@GHPFDFH@?$GAvtordisp?$HL?$AA@ 0046c918     LIBCMT:undname.obj
 0002:00007924       ??_C@_0N@CBHHHENL@?$GAvtordispex?$HL?$AA@ 0046c924     LIBCMT:undname.obj
 0002:00007934       ??_C@_02IGFCGPIL@?$HN?8?$AA@ 0046c934     LIBCMT:undname.obj
 0002:00007938       ??_C@_03OPGICMGF@?$HN?8?5?$AA@ 0046c938     LIBCMT:undname.obj
 0002:0000793c       ??_C@_06LIJLOJAG@const?5?$AA@ 0046c93c     LIBCMT:undname.obj
 0002:00007944       ??_C@_09GAIEOBLP@volatile?5?$AA@ 0046c944     LIBCMT:undname.obj
 0002:00007950       ??_C@_04HEJADOOB@CV?3?5?$AA@ 0046c950     LIBCMT:undname.obj
 0002:00007958       ??_C@_08PABEKFH@volatile?$AA@ 0046c958     LIBCMT:undname.obj
 0002:00007964       ??_C@_09EFNPDFFP@?5volatile?$AA@ 0046c964     LIBCMT:undname.obj
 0002:00007970       ??_C@_05BNCCCJPP@const?$AA@ 0046c970     LIBCMT:undname.obj
 0002:00007978       ??_C@_07EDHNAJHC@signed?5?$AA@ 0046c978     LIBCMT:undname.obj
 0002:00007980       ??_C@_06BNJCAIGJ@double?$AA@ 0046c980     LIBCMT:undname.obj
 0002:00007988       ??_C@_07NFANNNEC@UNKNOWN?$AA@ 0046c988     LIBCMT:undname.obj
 0002:00007990       ??_C@_08GAHOLHEO@__int128?$AA@ 0046c990     LIBCMT:undname.obj
 0002:0000799c       ??_C@_04DDKJGDCM@bool?$AA@ 0046c99c     LIBCMT:undname.obj
 0002:000079a4       ??_C@_07CLGGIAMF@wchar_t?$AA@ 0046c9a4     LIBCMT:undname.obj
 0002:000079ac       ??_C@_07LFCOJCAC@__int64?$AA@ 0046c9ac     LIBCMT:undname.obj
 0002:000079b4       ??_C@_07ICFHOGAF@__int16?$AA@ 0046c9b4     LIBCMT:undname.obj
 0002:000079bc       ??_C@_07OFLPPHGP@__int32?$AA@ 0046c9bc     LIBCMT:undname.obj
 0002:000079c4       ??_C@_06EBGKOKIG@__int8?$AA@ 0046c9c4     LIBCMT:undname.obj
 0002:000079cc       ??_C@_06GCICPBLB@__w64?5?$AA@ 0046c9cc     LIBCMT:undname.obj
 0002:000079d4       ??_C@_05KNFBNCOH@float?$AA@ 0046c9d4     LIBCMT:undname.obj
 0002:000079dc       ??_C@_04GOKPGOLB@long?$AA@ 0046c9dc     LIBCMT:undname.obj
 0002:000079e4       ??_C@_03JBIPMCLC@int?$AA@  0046c9e4     LIBCMT:undname.obj
 0002:000079e8       ??_C@_05BFKKPKCG@short?$AA@ 0046c9e8     LIBCMT:undname.obj
 0002:000079f0       ??_C@_04ENMBGAPA@char?$AA@ 0046c9f0     LIBCMT:undname.obj
 0002:000079f8       ___newctype                0046c9f8     LIBCMT:ctype.obj
 0002:00007cf8       __wctype                   0046ccf8     LIBCMT:ctype.obj
 0002:00007f00       ___newclmap                0046cf00     LIBCMT:ctype.obj
 0002:00008080       ___newcumap                0046d080     LIBCMT:ctype.obj
 0002:00008200       ??_C@_08JCCMCCIL@HH?3mm?3ss?$AA@ 0046d200     LIBCMT:strftime.obj
 0002:0000820c       ??_C@_0BE@CKGJFCPC@dddd?0?5MMMM?5dd?0?5yyyy?$AA@ 0046d20c     LIBCMT:strftime.obj
 0002:00008220       ??_C@_08BPBNCDIB@MM?1dd?1yy?$AA@ 0046d220     LIBCMT:strftime.obj
 0002:0000822c       ??_C@_02CJNFDJBF@PM?$AA@   0046d22c     LIBCMT:strftime.obj
 0002:00008230       ??_C@_02DEDBPAFC@AM?$AA@   0046d230     LIBCMT:strftime.obj
 0002:00008234       ??_C@_08EDHMEBNP@December?$AA@ 0046d234     LIBCMT:strftime.obj
 0002:00008240       ??_C@_08HCHEGEOA@November?$AA@ 0046d240     LIBCMT:strftime.obj
 0002:0000824c       ??_C@_07JJNFCEND@October?$AA@ 0046d24c     LIBCMT:strftime.obj
 0002:00008254       ??_C@_09BHHEALKD@September?$AA@ 0046d254     LIBCMT:strftime.obj
 0002:00008260       ??_C@_06LBBHFDDG@August?$AA@ 0046d260     LIBCMT:strftime.obj
 0002:00008268       ??_C@_04MIEPOIFP@July?$AA@ 0046d268     LIBCMT:strftime.obj
 0002:00008270       ??_C@_04CNLMGBGM@June?$AA@ 0046d270     LIBCMT:strftime.obj
 0002:00008278       ??_C@_05DMJDNLEJ@April?$AA@ 0046d278     LIBCMT:strftime.obj
 0002:00008280       ??_C@_05HPCKOFNC@March?$AA@ 0046d280     LIBCMT:strftime.obj
 0002:00008288       ??_C@_08GNJGEPFN@February?$AA@ 0046d288     LIBCMT:strftime.obj
 0002:00008294       ??_C@_07CGJPFGJA@January?$AA@ 0046d294     LIBCMT:strftime.obj
 0002:0000829c       ??_C@_03MKABNOCG@Dec?$AA@  0046d29c     LIBCMT:strftime.obj
 0002:000082a0       ??_C@_03JPJOFNIA@Nov?$AA@  0046d2a0     LIBCMT:strftime.obj
 0002:000082a4       ??_C@_03BMAOKBAD@Oct?$AA@  0046d2a4     LIBCMT:strftime.obj
 0002:000082a8       ??_C@_03GGCAPAJC@Sep?$AA@  0046d2a8     LIBCMT:strftime.obj
 0002:000082ac       ??_C@_03IFJFEIGA@Aug?$AA@  0046d2ac     LIBCMT:strftime.obj
 0002:000082b0       ??_C@_03LBGABGKK@Jul?$AA@  0046d2b0     LIBCMT:strftime.obj
 0002:000082b4       ??_C@_03IDFGHECI@Jun?$AA@  0046d2b4     LIBCMT:strftime.obj
 0002:000082b8       ??_C@_03CNMDKL@May?$AA@    0046d2b8     LIBCMT:strftime.obj
 0002:000082bc       ??_C@_03LEOLGMJP@Apr?$AA@  0046d2bc     LIBCMT:strftime.obj
 0002:000082c0       ??_C@_03ODNJBKGA@Mar?$AA@  0046d2c0     LIBCMT:strftime.obj
 0002:000082c4       ??_C@_03HJBDCHOM@Feb?$AA@  0046d2c4     LIBCMT:strftime.obj
 0002:000082c8       ??_C@_03JIHJHPIE@Jan?$AA@  0046d2c8     LIBCMT:strftime.obj
 0002:000082cc       ??_C@_08INBOOONO@Saturday?$AA@ 0046d2cc     LIBCMT:strftime.obj
 0002:000082d8       ??_C@_06JECMNKMI@Friday?$AA@ 0046d2d8     LIBCMT:strftime.obj
 0002:000082e0       ??_C@_08HACCIKIA@Thursday?$AA@ 0046d2e0     LIBCMT:strftime.obj
 0002:000082ec       ??_C@_09DLIGFAKA@Wednesday?$AA@ 0046d2ec     LIBCMT:strftime.obj
 0002:000082f8       ??_C@_07BAAGCFCM@Tuesday?$AA@ 0046d2f8     LIBCMT:strftime.obj
 0002:00008300       ??_C@_06JLEDEDGH@Monday?$AA@ 0046d300     LIBCMT:strftime.obj
 0002:00008308       ??_C@_06OOPIFAJ@Sunday?$AA@ 0046d308     LIBCMT:strftime.obj
 0002:00008310       ??_C@_03FEFJNEK@Sat?$AA@   0046d310     LIBCMT:strftime.obj
 0002:00008314       ??_C@_03IDIOELNC@Fri?$AA@  0046d314     LIBCMT:strftime.obj
 0002:00008318       ??_C@_03IOFIKPDN@Thu?$AA@  0046d318     LIBCMT:strftime.obj
 0002:0000831c       ??_C@_03MHOMLAJA@Wed?$AA@  0046d31c     LIBCMT:strftime.obj
 0002:00008320       ??_C@_03NAGEINEP@Tue?$AA@  0046d320     LIBCMT:strftime.obj
 0002:00008324       ??_C@_03PDAGKDH@Mon?$AA@   0046d324     LIBCMT:strftime.obj
 0002:00008328       ??_C@_03KOEHGMDN@Sun?$AA@  0046d328     LIBCMT:strftime.obj
 0002:0000832c       ??_C@_03EBAPMIKO@a?1p?$AA@ 0046d32c     LIBCMT:strftime.obj
 0002:00008330       ??_C@_05JAMEPDIN@am?1pm?$AA@ 0046d330     LIBCMT:strftime.obj
 0002:00008338       ??_C@_0O@FMJNFNKE@united?9states?$AA@ 0046d338     LIBCMT:getqloc.obj
 0002:00008348       ??_C@_0P@NDHFFKCA@united?9kingdom?$AA@ 0046d348     LIBCMT:getqloc.obj
 0002:00008358       ??_C@_0BC@HHDADLGF@trinidad?5?$CG?5tobago?$AA@ 0046d358     LIBCMT:getqloc.obj
 0002:0000836c       ??_C@_0M@IOAEBDAC@south?9korea?$AA@ 0046d36c     LIBCMT:getqloc.obj
 0002:00008378       ??_C@_0N@FIELFKIJ@south?9africa?$AA@ 0046d378     LIBCMT:getqloc.obj
 0002:00008388       ??_C@_0M@OPNDHCMC@south?5korea?$AA@ 0046d388     LIBCMT:getqloc.obj
 0002:00008394       ??_C@_0N@MDEOEPFI@south?5africa?$AA@ 0046d394     LIBCMT:getqloc.obj
 0002:000083a4       ??_C@_06FKAPCJLB@slovak?$AA@ 0046d3a4     LIBCMT:getqloc.obj
 0002:000083ac       ??_C@_0M@EFJANOAL@puerto?9rico?$AA@ 0046d3ac     LIBCMT:getqloc.obj
 0002:000083b8       ??_C@_08PGOJKDAI@pr?9china?$AA@ 0046d3b8     LIBCMT:getqloc.obj
 0002:000083c4       ??_C@_08JHDOMCMI@pr?5china?$AA@ 0046d3c4     LIBCMT:getqloc.obj
 0002:000083d0       ??_C@_02JHCHFBLL@nz?$AA@   0046d3d0     LIBCMT:getqloc.obj
 0002:000083d4       ??_C@_0M@LINHDHKP@new?9zealand?$AA@ 0046d3d4     LIBCMT:getqloc.obj
 0002:000083e0       ??_C@_09IIIPPBDB@hong?9kong?$AA@ 0046d3e0     LIBCMT:getqloc.obj
 0002:000083ec       ??_C@_07HJLCKBG@holland?$AA@ 0046d3ec     LIBCMT:getqloc.obj
 0002:000083f4       ??_C@_0O@LEHGMHAG@great?5britain?$AA@ 0046d3f4     LIBCMT:getqloc.obj
 0002:00008404       ??_C@_07FACOMELA@england?$AA@ 0046d404     LIBCMT:getqloc.obj
 0002:0000840c       ??_C@_05JIHCEICB@czech?$AA@ 0046d40c     LIBCMT:getqloc.obj
 0002:00008414       ??_C@_05BBJOBLGB@china?$AA@ 0046d414     LIBCMT:getqloc.obj
 0002:0000841c       ??_C@_07GPKPHICP@britain?$AA@ 0046d41c     LIBCMT:getqloc.obj
 0002:00008424       ??_C@_07MHIPBHMG@america?$AA@ 0046d424     LIBCMT:getqloc.obj
 0002:0000842c       ??_C@_03KIALPMKC@usa?$AA@  0046d42c     LIBCMT:getqloc.obj
 0002:00008430       ??_C@_02FGJGKGGD@us?$AA@   0046d430     LIBCMT:getqloc.obj
 0002:00008434       ??_C@_02NEINDODK@uk?$AA@   0046d434     LIBCMT:getqloc.obj
 0002:00008438       ??_C@_05JMPCFJFJ@swiss?$AA@ 0046d438     LIBCMT:getqloc.obj
 0002:00008440       ??_C@_0BA@HLOCPIOD@swedish?9finland?$AA@ 0046d440     LIBCMT:getqloc.obj
 0002:00008450       ??_C@_0BC@PKCNIABK@spanish?9venezuela?$AA@ 0046d450     LIBCMT:getqloc.obj
 0002:00008464       ??_C@_0BA@GBHHMIJI@spanish?9uruguay?$AA@ 0046d464     LIBCMT:getqloc.obj
 0002:00008474       ??_C@_0BE@BHDOHPMC@spanish?9puerto?5rico?$AA@ 0046d474     LIBCMT:getqloc.obj
 0002:00008488       ??_C@_0N@KMOIDGGN@spanish?9peru?$AA@ 0046d488     LIBCMT:getqloc.obj
 0002:00008498       ??_C@_0BB@HMHLPGPH@spanish?9paraguay?$AA@ 0046d498     LIBCMT:getqloc.obj
 0002:000084ac       ??_C@_0P@MCPKNGFD@spanish?9panama?$AA@ 0046d4ac     LIBCMT:getqloc.obj
 0002:000084bc       ??_C@_0BC@IHOHGAIL@spanish?9nicaragua?$AA@ 0046d4bc     LIBCMT:getqloc.obj
 0002:000084d0       ??_C@_0P@KLMJDNFJ@spanish?9modern?$AA@ 0046d4d0     LIBCMT:getqloc.obj
 0002:000084e0       ??_C@_0BA@BPAPGBCM@spanish?9mexican?$AA@ 0046d4e0     LIBCMT:getqloc.obj
 0002:000084f0       ??_C@_0BB@PDECHHHE@spanish?9honduras?$AA@ 0046d4f0     LIBCMT:getqloc.obj
 0002:00008504       ??_C@_0BC@KLHKFGDB@spanish?9guatemala?$AA@ 0046d504     LIBCMT:getqloc.obj
 0002:00008518       ??_C@_0BE@MFOOKJAI@spanish?9el?5salvador?$AA@ 0046d518     LIBCMT:getqloc.obj
 0002:0000852c       ??_C@_0BA@FCOKFPFC@spanish?9ecuador?$AA@ 0046d52c     LIBCMT:getqloc.obj
 0002:0000853c       ??_C@_0BL@PLMGIMOO@spanish?9dominican?5republic?$AA@ 0046d53c     LIBCMT:getqloc.obj
 0002:00008558       ??_C@_0BD@HLGDNMHB@spanish?9costa?5rica?$AA@ 0046d558     LIBCMT:getqloc.obj
 0002:0000856c       ??_C@_0BB@PKCBKCPE@spanish?9colombia?$AA@ 0046d56c     LIBCMT:getqloc.obj
 0002:00008580       ??_C@_0O@MCBIJGNE@spanish?9chile?$AA@ 0046d580     LIBCMT:getqloc.obj
 0002:00008590       ??_C@_0BA@BEFEIGJJ@spanish?9bolivia?$AA@ 0046d590     LIBCMT:getqloc.obj
 0002:000085a0       ??_C@_0BC@EMECMPD@spanish?9argentina?$AA@ 0046d5a0     LIBCMT:getqloc.obj
 0002:000085b4       ??_C@_0BF@EALFLENP@portuguese?9brazilian?$AA@ 0046d5b4     LIBCMT:getqloc.obj
 0002:000085cc       ??_C@_0BC@HBLEBLNN@norwegian?9nynorsk?$AA@ 0046d5cc     LIBCMT:getqloc.obj
 0002:000085e0       ??_C@_0BB@HMACDDCK@norwegian?9bokmal?$AA@ 0046d5e0     LIBCMT:getqloc.obj
 0002:000085f4       ??_C@_09BAFFPPHE@norwegian?$AA@ 0046d5f4     LIBCMT:getqloc.obj
 0002:00008600       ??_C@_0O@EAJFJDFG@italian?9swiss?$AA@ 0046d600     LIBCMT:getqloc.obj
 0002:00008610       ??_C@_0O@CNOMPGD@irish?9english?$AA@ 0046d610     LIBCMT:getqloc.obj
 0002:00008620       ??_C@_0N@EDHBGCKG@german?9swiss?$AA@ 0046d620     LIBCMT:getqloc.obj
 0002:00008630       ??_C@_0BC@JACMHNBP@german?9luxembourg?$AA@ 0046d630     LIBCMT:getqloc.obj
 0002:00008644       ??_C@_0BE@HBGMGFEG@german?9lichtenstein?$AA@ 0046d644     LIBCMT:getqloc.obj
 0002:00008658       ??_C@_0BA@HKKBIBKL@german?9austrian?$AA@ 0046d658     LIBCMT:getqloc.obj
 0002:00008668       ??_C@_0N@GCAEPEBK@french?9swiss?$AA@ 0046d668     LIBCMT:getqloc.obj
 0002:00008678       ??_C@_0BC@DJFJJCK@french?9luxembourg?$AA@ 0046d678     LIBCMT:getqloc.obj
 0002:0000868c       ??_C@_0BA@NNCEDFIC@french?9canadian?$AA@ 0046d68c     LIBCMT:getqloc.obj
 0002:0000869c       ??_C@_0P@CMPOCLM@french?9belgian?$AA@ 0046d69c     LIBCMT:getqloc.obj
 0002:000086ac       ??_C@_0M@GHHDJOK@english?9usa?$AA@ 0046d6ac     LIBCMT:getqloc.obj
 0002:000086b8       ??_C@_0L@PLDJKEIL@english?9us?$AA@ 0046d6b8     LIBCMT:getqloc.obj
 0002:000086c4       ??_C@_0L@HJCCDMNC@english?9uk?$AA@ 0046d6c4     LIBCMT:getqloc.obj
 0002:000086d0       ??_C@_0BK@CKLIAGJB@english?9trinidad?5y?5tobago?$AA@ 0046d6d0     LIBCMT:getqloc.obj
 0002:000086ec       ??_C@_0BF@JMJMGNNF@english?9south?5africa?$AA@ 0046d6ec     LIBCMT:getqloc.obj
 0002:00008704       ??_C@_0L@DKIIFDFD@english?9nz?$AA@ 0046d704     LIBCMT:getqloc.obj
 0002:00008710       ??_C@_0BA@ONHGJCLH@english?9jamaica?$AA@ 0046d710     LIBCMT:getqloc.obj
 0002:00008720       ??_C@_0M@HJBGHOPO@english?9ire?$AA@ 0046d720     LIBCMT:getqloc.obj
 0002:0000872c       ??_C@_0BC@LFEKMIFB@english?9caribbean?$AA@ 0046d72c     LIBCMT:getqloc.obj
 0002:00008740       ??_C@_0M@OLDPFKHI@english?9can?$AA@ 0046d740     LIBCMT:getqloc.obj
 0002:0000874c       ??_C@_0P@OMDEHBMP@english?9belize?$AA@ 0046d74c     LIBCMT:getqloc.obj
 0002:0000875c       ??_C@_0M@KFHFPFED@english?9aus?$AA@ 0046d75c     LIBCMT:getqloc.obj
 0002:00008768       ??_C@_0BB@MNMBKDFE@english?9american?$AA@ 0046d768     LIBCMT:getqloc.obj
 0002:0000877c       ??_C@_0O@KIDLNNBA@dutch?9belgian?$AA@ 0046d77c     LIBCMT:getqloc.obj
 0002:0000878c       ??_C@_0BE@JBKABBMH@chinese?9traditional?$AA@ 0046d78c     LIBCMT:getqloc.obj
 0002:000087a0       ??_C@_0BC@MJJMPKCG@chinese?9singapore?$AA@ 0046d7a0     LIBCMT:getqloc.obj
 0002:000087b4       ??_C@_0BD@FDKADDCP@chinese?9simplified?$AA@ 0046d7b4     LIBCMT:getqloc.obj
 0002:000087c8       ??_C@_0BB@DBEFDDME@chinese?9hongkong?$AA@ 0046d7c8     LIBCMT:getqloc.obj
 0002:000087dc       ??_C@_07DHNMFMCI@chinese?$AA@ 0046d7dc     LIBCMT:getqloc.obj
 0002:000087e4       ??_C@_03FNDDCHI@chi?$AA@   0046d7e4     LIBCMT:getqloc.obj
 0002:000087e8       ??_C@_03BMMIADDJ@chh?$AA@  0046d7e8     LIBCMT:getqloc.obj
 0002:000087ec       ??_C@_08OAIPJDGI@canadian?$AA@ 0046d7ec     LIBCMT:getqloc.obj
 0002:000087f8       ??_C@_07HBPMNPNJ@belgian?$AA@ 0046d7f8     LIBCMT:getqloc.obj
 0002:00008800       ??_C@_0L@OEKOPBEL@australian?$AA@ 0046d800     LIBCMT:getqloc.obj
 0002:0000880c       ??_C@_0BB@MEIMBEDG@american?9english?$AA@ 0046d80c     LIBCMT:getqloc.obj
 0002:00008820       ??_C@_0BB@DFMDPDGB@american?5english?$AA@ 0046d820     LIBCMT:getqloc.obj
 0002:00008834       ??_C@_08IJLOKOLL@american?$AA@ 0046d834     LIBCMT:getqloc.obj
 0002:00008840       ___rg_language             0046d840     LIBCMT:getqloc.obj
 0002:00008a48       ___rg_country              0046da48     LIBCMT:getqloc.obj
 0002:00008b00       ___rglangidNotDefault      0046db00     LIBCMT:getqloc.obj
 0002:00008b14       ??_C@_01GBGANLPD@0?$AA@    0046db14     LIBCMT:getqloc.obj
 0002:00008b18       ??_C@_03NFKLAGEF@OCP?$AA@  0046db18     LIBCMT:getqloc.obj
 0002:00008b1c       ??_C@_03DFHEHBHG@ACP?$AA@  0046db1c     LIBCMT:getqloc.obj
 0002:00008b20       ??_C@_0BC@NFIEMBLL@Norwegian?9Nynorsk?$AA@ 0046db20     LIBCMT:getqloc.obj
 0002:00008b34       ??_C@_06IMKFLFPG@1?$CDQNAN?$AA@ 0046db34     LIBCMT:_x10fout_.obj
 0002:00008b3c       ??_C@_05DNEBIAHO@1?$CDINF?$AA@ 0046db3c     LIBCMT:_x10fout_.obj
 0002:00008b44       ??_C@_05PHHOCPM@1?$CDIND?$AA@ 0046db44     LIBCMT:_x10fout_.obj
 0002:00008b4c       ??_C@_06PGGFOGJG@1?$CDSNAN?$AA@ 0046db4c     LIBCMT:_x10fout_.obj
 0002:00008b54       ??_C@_06GDENEHCP@CONIN$?$AA@ 0046db54     LIBCMT:initcon.obj
 0002:00008b5c       ??_C@_07GPDNMNG@CONOUT$?$AA@ 0046db5c     LIBCMT:initcon.obj
 0002:00008b64       ___dnames                  0046db64     LIBCMT:timeset.obj
 0002:00008b7c       ___mnames                  0046db7c     LIBCMT:timeset.obj
 0002:00008ba4       ??_C@_02CLFPBFFP@TZ?$AA@   0046dba4     LIBCMT:tzset.obj
 0002:00008ba8       ?_BADOFF@std@@3JB          0046dba8     libcpmt:ios.obj
 0002:00008bb0       __load_config_used         0046dbb0     LIBCMT:loadcfg.obj
 0002:00008c54       ??_R4NetworkIDGenerator@@6B@ 0046dc54     NetworkIDGenerator.obj
 0002:00008c68       ??_R3NetworkIDGenerator@@8 0046dc68     NetworkIDGenerator.obj
 0002:00008c78       ??_R2NetworkIDGenerator@@8 0046dc78     NetworkIDGenerator.obj
 0002:00008c80       ??_R1A@?0A@EA@NetworkIDGenerator@@8 0046dc80     NetworkIDGenerator.obj
 0002:00008c9c       ??_R4?$BinarySearchTree@UNetworkIDNode@@@DataStructures@@6B@ 0046dc9c     NetworkIDGenerator.obj
 0002:00008cb0       ??_R3?$BinarySearchTree@UNetworkIDNode@@@DataStructures@@8 0046dcb0     NetworkIDGenerator.obj
 0002:00008cc0       ??_R2?$BinarySearchTree@UNetworkIDNode@@@DataStructures@@8 0046dcc0     NetworkIDGenerator.obj
 0002:00008cc8       ??_R1A@?0A@EA@?$BinarySearchTree@UNetworkIDNode@@@DataStructures@@8 0046dcc8     NetworkIDGenerator.obj
 0002:00008ce4       ??_R4?$AVLBalancedBinarySearchTree@UNetworkIDNode@@@DataStructures@@6B@ 0046dce4     NetworkIDGenerator.obj
 0002:00008cf8       ??_R3?$AVLBalancedBinarySearchTree@UNetworkIDNode@@@DataStructures@@8 0046dcf8     NetworkIDGenerator.obj
 0002:00008d08       ??_R2?$AVLBalancedBinarySearchTree@UNetworkIDNode@@@DataStructures@@8 0046dd08     NetworkIDGenerator.obj
 0002:00008d14       ??_R1A@?0A@EA@?$AVLBalancedBinarySearchTree@UNetworkIDNode@@@DataStructures@@8 0046dd14     NetworkIDGenerator.obj
 0002:00008d30       ??_R4RakClientInterface@@6B@ 0046dd30     RakClient.obj
 0002:00008d44       ??_R3RakClientInterface@@8 0046dd44     RakClient.obj
 0002:00008d54       ??_R2RakClientInterface@@8 0046dd54     RakClient.obj
 0002:00008d5c       ??_R1A@?0A@EA@RakClientInterface@@8 0046dd5c     RakClient.obj
 0002:00008d78       ??_R4RakClient@@6BRakPeer@@@ 0046dd78     RakClient.obj
 0002:00008d8c       ??_R3RakClient@@8          0046dd8c     RakClient.obj
 0002:00008d9c       ??_R2RakClient@@8          0046dd9c     RakClient.obj
 0002:00008db0       ??_R1A@?0A@EA@RakClient@@8 0046ddb0     RakClient.obj
 0002:00008dcc       ??_R1A@?0A@EA@RakPeer@@8   0046ddcc     RakClient.obj
 0002:00008de8       ??_R3RakPeer@@8            0046dde8     RakClient.obj
 0002:00008df8       ??_R2RakPeer@@8            0046ddf8     RakClient.obj
 0002:00008e04       ??_R1A@?0A@EA@RakPeerInterface@@8 0046de04     RakClient.obj
 0002:00008e20       ??_R3RakPeerInterface@@8   0046de20     RakClient.obj
 0002:00008e30       ??_R2RakPeerInterface@@8   0046de30     RakClient.obj
 0002:00008e38       ??_R1KGI@?0A@EA@RakClientInterface@@8 0046de38     RakClient.obj
 0002:00008e54       ??_R4RakClient@@6BRakClientInterface@@@ 0046de54     RakClient.obj
 0002:00008e68       ??_R4RakPeerInterface@@6B@ 0046de68     RakPeer.obj
 0002:00008e7c       ??_R4RakPeer@@6B@          0046de7c     RakPeer.obj
 0002:00008e90       ??_R4RakServerInterface@@6B@ 0046de90     rakserver.obj
 0002:00008ea4       ??_R3RakServerInterface@@8 0046dea4     rakserver.obj
 0002:00008eb4       ??_R2RakServerInterface@@8 0046deb4     rakserver.obj
 0002:00008ebc       ??_R1A@?0A@EA@RakServerInterface@@8 0046debc     rakserver.obj
 0002:00008ed8       ??_R4RakServer@@6BRakServerInterface@@@ 0046ded8     rakserver.obj
 0002:00008eec       ??_R3RakServer@@8          0046deec     rakserver.obj
 0002:00008efc       ??_R2RakServer@@8          0046defc     rakserver.obj
 0002:00008f10       ??_R1A@?0A@EA@RakServer@@8 0046df10     rakserver.obj
 0002:00008f2c       ??_R17?0A@EA@RakPeer@@8    0046df2c     rakserver.obj
 0002:00008f48       ??_R17?0A@EA@RakPeerInterface@@8 0046df48     rakserver.obj
 0002:00008f64       ??_R4RakServer@@6BRakPeer@@@ 0046df64     rakserver.obj
 0002:00008f78       ??_R4CSHA1@@6B@            0046df78     SHA1.obj
 0002:00008f8c       ??_R3CSHA1@@8              0046df8c     SHA1.obj
 0002:00008f9c       ??_R2CSHA1@@8              0046df9c     SHA1.obj
 0002:00008fa4       ??_R1A@?0A@EA@CSHA1@@8     0046dfa4     SHA1.obj
 0002:00008fc0       ??_R4TiXmlBase@@6B@        0046dfc0     tinyxml.obj
 0002:00008fd4       ??_R3TiXmlBase@@8          0046dfd4     tinyxml.obj
 0002:00008fe4       ??_R2TiXmlBase@@8          0046dfe4     tinyxml.obj
 0002:00008fec       ??_R1A@?0A@EA@TiXmlBase@@8 0046dfec     tinyxml.obj
 0002:00009008       ??_R4TiXmlAttribute@@6B@   0046e008     tinyxml.obj
 0002:0000901c       ??_R3TiXmlAttribute@@8     0046e01c     tinyxml.obj
 0002:0000902c       ??_R2TiXmlAttribute@@8     0046e02c     tinyxml.obj
 0002:00009038       ??_R1A@?0A@EA@TiXmlAttribute@@8 0046e038     tinyxml.obj
 0002:00009054       ??_R4TiXmlNode@@6B@        0046e054     tinyxml.obj
 0002:00009068       ??_R3TiXmlNode@@8          0046e068     tinyxml.obj
 0002:00009078       ??_R2TiXmlNode@@8          0046e078     tinyxml.obj
 0002:00009084       ??_R1A@?0A@EA@TiXmlNode@@8 0046e084     tinyxml.obj
 0002:000090a0       ??_R4TiXmlDocument@@6B@    0046e0a0     tinyxml.obj
 0002:000090b4       ??_R3TiXmlDocument@@8      0046e0b4     tinyxml.obj
 0002:000090c4       ??_R2TiXmlDocument@@8      0046e0c4     tinyxml.obj
 0002:000090d4       ??_R1A@?0A@EA@TiXmlDocument@@8 0046e0d4     tinyxml.obj
 0002:000090f0       ??_R4TiXmlComment@@6B@     0046e0f0     tinyxml.obj
 0002:00009104       ??_R3TiXmlComment@@8       0046e104     tinyxml.obj
 0002:00009114       ??_R2TiXmlComment@@8       0046e114     tinyxml.obj
 0002:00009124       ??_R1A@?0A@EA@TiXmlComment@@8 0046e124     tinyxml.obj
 0002:00009140       ??_R4TiXmlDeclaration@@6B@ 0046e140     tinyxml.obj
 0002:00009154       ??_R3TiXmlDeclaration@@8   0046e154     tinyxml.obj
 0002:00009164       ??_R2TiXmlDeclaration@@8   0046e164     tinyxml.obj
 0002:00009174       ??_R1A@?0A@EA@TiXmlDeclaration@@8 0046e174     tinyxml.obj
 0002:00009190       ??_R4TiXmlText@@6B@        0046e190     tinyxml.obj
 0002:000091a4       ??_R3TiXmlText@@8          0046e1a4     tinyxml.obj
 0002:000091b4       ??_R2TiXmlText@@8          0046e1b4     tinyxml.obj
 0002:000091c4       ??_R1A@?0A@EA@TiXmlText@@8 0046e1c4     tinyxml.obj
 0002:000091e0       ??_R4TiXmlUnknown@@6B@     0046e1e0     tinyxml.obj
 0002:000091f4       ??_R3TiXmlUnknown@@8       0046e1f4     tinyxml.obj
 0002:00009204       ??_R2TiXmlUnknown@@8       0046e204     tinyxml.obj
 0002:00009214       ??_R1A@?0A@EA@TiXmlUnknown@@8 0046e214     tinyxml.obj
 0002:00009230       ??_R4TiXmlElement@@6B@     0046e230     tinyxml.obj
 0002:00009244       ??_R3TiXmlElement@@8       0046e244     tinyxml.obj
 0002:00009254       ??_R2TiXmlElement@@8       0046e254     tinyxml.obj
 0002:00009264       ??_R1A@?0A@EA@TiXmlElement@@8 0046e264     tinyxml.obj
 0002:00009280       ??_R4bad_alloc@std@@6B@    0046e280     LIBCMT:new.obj
 0002:00009294       ??_R3bad_alloc@std@@8      0046e294     LIBCMT:new.obj
 0002:000092a4       ??_R2bad_alloc@std@@8      0046e2a4     LIBCMT:new.obj
 0002:000092b0       ??_R1A@?0A@EA@bad_alloc@std@@8 0046e2b0     LIBCMT:new.obj
 0002:000092cc       ??_R1A@?0A@EA@exception@std@@8 0046e2cc     LIBCMT:new.obj
 0002:000092e8       ??_R3exception@std@@8      0046e2e8     LIBCMT:new.obj
 0002:000092f8       ??_R2exception@std@@8      0046e2f8     LIBCMT:new.obj
 0002:00009300       ??_R4type_info@@6B@        0046e300     LIBCMT:typinfo.obj
 0002:00009314       ??_R3type_info@@8          0046e314     LIBCMT:typinfo.obj
 0002:00009324       ??_R2type_info@@8          0046e324     LIBCMT:typinfo.obj
 0002:0000932c       ??_R1A@?0A@EA@type_info@@8 0046e32c     LIBCMT:typinfo.obj
 0002:00009348       ??_R4exception@std@@6B@    0046e348     LIBCMT:stdexcpt.obj
 0002:0000935c       ??_R4bad_cast@std@@6B@     0046e35c     LIBCMT:stdexcpt.obj
 0002:00009370       ??_R3bad_cast@std@@8       0046e370     LIBCMT:stdexcpt.obj
 0002:00009380       ??_R2bad_cast@std@@8       0046e380     LIBCMT:stdexcpt.obj
 0002:0000938c       ??_R1A@?0A@EA@bad_cast@std@@8 0046e38c     LIBCMT:stdexcpt.obj
 0002:000093a8       ??_R4bad_typeid@std@@6B@   0046e3a8     LIBCMT:stdexcpt.obj
 0002:000093bc       ??_R3bad_typeid@std@@8     0046e3bc     LIBCMT:stdexcpt.obj
 0002:000093cc       ??_R2bad_typeid@std@@8     0046e3cc     LIBCMT:stdexcpt.obj
 0002:000093d8       ??_R1A@?0A@EA@bad_typeid@std@@8 0046e3d8     LIBCMT:stdexcpt.obj
 0002:000093f4       ??_R4__non_rtti_object@std@@6B@ 0046e3f4     LIBCMT:stdexcpt.obj
 0002:00009408       ??_R3__non_rtti_object@std@@8 0046e408     LIBCMT:stdexcpt.obj
 0002:00009418       ??_R2__non_rtti_object@std@@8 0046e418     LIBCMT:stdexcpt.obj
 0002:00009428       ??_R1A@?0A@EA@__non_rtti_object@std@@8 0046e428     LIBCMT:stdexcpt.obj
 0002:00009444       ??_R4bad_exception@std@@6B@ 0046e444     LIBCMT:frame.obj
 0002:00009458       ??_R3bad_exception@std@@8  0046e458     LIBCMT:frame.obj
 0002:00009468       ??_R2bad_exception@std@@8  0046e468     LIBCMT:frame.obj
 0002:00009474       ??_R1A@?0A@EA@bad_exception@std@@8 0046e474     LIBCMT:frame.obj
 0002:00009490       ___safe_se_handler_table   0046e490     <linker-defined>
 0002:00009724       ___rtc_iaa                 0046e724     LIBCMT:_initsect_.obj
 0002:00009728       ___rtc_izz                 0046e728     LIBCMT:_initsect_.obj
 0002:0000972c       ___rtc_taa                 0046e72c     LIBCMT:_initsect_.obj
 0002:00009730       ___rtc_tzz                 0046e730     LIBCMT:_initsect_.obj
 0002:0000b68c       __TI2?AVbad_alloc@std@@    0047068c     LIBCMT:new.obj
 0002:0000b69c       __CTA2?AVbad_alloc@std@@   0047069c     LIBCMT:new.obj
 0002:0000b6a8       __CT??_R0?AVbad_alloc@std@@@8??0bad_alloc@std@@QAE@ABV01@@Z12 004706a8     LIBCMT:new.obj
 0002:0000b6c4       __CT??_R0?AVexception@std@@@8??0exception@std@@QAE@ABV01@@Z12 004706c4     LIBCMT:new.obj
 0002:0000bc5c       __TI2?AVbad_exception@std@@ 00470c5c     LIBCMT:frame.obj
 0002:0000bc6c       __CTA2?AVbad_exception@std@@ 00470c6c     LIBCMT:frame.obj
 0002:0000bc78       __CT??_R0?AVbad_exception@std@@@8??0bad_exception@std@@QAE@ABV01@@Z12 00470c78     LIBCMT:frame.obj
 0002:0000c2ec       __IMPORT_DESCRIPTOR_WS2_32 004712ec     ws2_32:WS2_32.dll
 0002:0000c300       __IMPORT_DESCRIPTOR_COMCTL32 00471300     comctl32:COMCTL32.dll
 0002:0000c314       __IMPORT_DESCRIPTOR_KERNEL32 00471314     kernel32:KERNEL32.dll
 0002:0000c328       __IMPORT_DESCRIPTOR_USER32 00471328     user32:USER32.dll
 0002:0000c33c       __IMPORT_DESCRIPTOR_GDI32  0047133c     gdi32:GDI32.dll
 0002:0000c350       __IMPORT_DESCRIPTOR_sqlite3 00471350     sqlite3:sqlite3.dll
 0002:0000c364       __NULL_IMPORT_DESCRIPTOR   00471364     ws2_32:WS2_32.dll
 0003:00000078       ??_R0?AVNetworkIDGenerator@@@8 00473078     NetworkIDGenerator.obj
 0003:000000a0       ??_R0?AV?$BinarySearchTree@UNetworkIDNode@@@DataStructures@@@8 004730a0     NetworkIDGenerator.obj
 0003:000000e8       ??_R0?AV?$AVLBalancedBinarySearchTree@UNetworkIDNode@@@DataStructures@@@8 004730e8     NetworkIDGenerator.obj
 0003:00000148       ?IDTree@NetworkIDGenerator@@2V?$AVLBalancedBinarySearchTree@UNetworkIDNode@@@DataStructures@@A 00473148     NetworkIDGenerator.obj
 0003:00000180       ??_R0?AVRakClientInterface@@@8 00473180     RakClient.obj
 0003:000001a4       ??_R0?AVRakClient@@@8      004731a4     RakClient.obj
 0003:000001bc       ??_R0?AVRakPeer@@@8        004731bc     RakClient.obj
 0003:000001d4       ??_R0?AVRakPeerInterface@@@8 004731d4     RakClient.obj
 0003:0000028c       ??_R0?AVRakServerInterface@@@8 0047328c     rakserver.obj
 0003:000002b0       ??_R0?AVRakServer@@@8      004732b0     rakserver.obj
 0003:00000318       ?Logtable@@3PAEA           00473318     rijndael.obj
 0003:00000418       ?Alogtable@@3PAEA          00473418     rijndael.obj
 0003:00000518       ?S@@3PAEA                  00473518     rijndael.obj
 0003:00000618       ?Si@@3PAEA                 00473618     rijndael.obj
 0003:00000718       ?T1@@3PAY03EA              00473718     rijndael.obj
 0003:00000b18       ?T2@@3PAY03EA              00473b18     rijndael.obj
 0003:00000f18       ?T3@@3PAY03EA              00473f18     rijndael.obj
 0003:00001318       ?T4@@3PAY03EA              00474318     rijndael.obj
 0003:00001718       ?T5@@3PAY03EA              00474718     rijndael.obj
 0003:00001b18       ?T6@@3PAY03EA              00474b18     rijndael.obj
 0003:00001f18       ?T7@@3PAY03EA              00474f18     rijndael.obj
 0003:00002318       ?T8@@3PAY03EA              00475318     rijndael.obj
 0003:00002718       ?S5@@3PAEA                 00475718     rijndael.obj
 0003:00002818       ?U1@@3PAY03EA              00475818     rijndael.obj
 0003:00002c18       ?U2@@3PAY03EA              00475c18     rijndael.obj
 0003:00003018       ?U3@@3PAY03EA              00476018     rijndael.obj
 0003:00003418       ?U4@@3PAY03EA              00476418     rijndael.obj
 0003:00003818       ?rcon@@3PAIA               00476818     rijndael.obj
 0003:000038bc       ??_R0?AVCSHA1@@@8          004768bc     SHA1.obj
 0003:00003908       ?englishCharacterFrequencies@@3PAIA 00476908     StringCompressor.obj
 0003:00003d58       ?sampEncrTable@@3PAEA      00476d58     samp_netencr.obj
 0003:00003f8c       ?RPC_ServerJoin@@3HA       00476f8c     SAMPRPC.obj
 0003:00003f90       ?RPC_ServerQuit@@3HA       00476f90     SAMPRPC.obj
 0003:00003f94       ?RPC_InitGame@@3HA         00476f94     SAMPRPC.obj
 0003:00003f98       ?RPC_ClientJoin@@3HA       00476f98     SAMPRPC.obj
 0003:00003f9c       ?RPC_NPCJoin@@3HA          00476f9c     SAMPRPC.obj
 0003:00003fa0       ?RPC_Death@@3HA            00476fa0     SAMPRPC.obj
 0003:00003fa4       ?RPC_RequestClass@@3HA     00476fa4     SAMPRPC.obj
 0003:00003fa8       ?RPC_RequestSpawn@@3HA     00476fa8     SAMPRPC.obj
 0003:00003fac       ?RPC_SetInteriorId@@3HA    00476fac     SAMPRPC.obj
 0003:00003fb0       ?RPC_Spawn@@3HA            00476fb0     SAMPRPC.obj
 0003:00003fb4       ?RPC_Chat@@3HA             00476fb4     SAMPRPC.obj
 0003:00003fb8       ?RPC_EnterVehicle@@3HA     00476fb8     SAMPRPC.obj
 0003:00003fbc       ?RPC_ExitVehicle@@3HA      00476fbc     SAMPRPC.obj
 0003:00003fc0       ?RPC_DamageVehicle@@3HA    00476fc0     SAMPRPC.obj
 0003:00003fc4       ?RPC_MenuSelect@@3HA       00476fc4     SAMPRPC.obj
 0003:00003fc8       ?RPC_MenuQuit@@3HA         00476fc8     SAMPRPC.obj
 0003:00003fcc       ?RPC_ScmEvent@@3HA         00476fcc     SAMPRPC.obj
 0003:00003fd0       ?RPC_AdminMapTeleport@@3HA 00476fd0     SAMPRPC.obj
 0003:00003fd4       ?RPC_WorldPlayerAdd@@3HA   00476fd4     SAMPRPC.obj
 0003:00003fd8       ?RPC_WorldPlayerDeath@@3HA 00476fd8     SAMPRPC.obj
 0003:00003fdc       ?RPC_WorldPlayerRemove@@3HA 00476fdc     SAMPRPC.obj
 0003:00003fe0       ?RPC_WorldVehicleAdd@@3HA  00476fe0     SAMPRPC.obj
 0003:00003fe4       ?RPC_WorldVehicleRemove@@3HA 00476fe4     SAMPRPC.obj
 0003:00003fe8       ?RPC_SetCheckpoint@@3HA    00476fe8     SAMPRPC.obj
 0003:00003fec       ?RPC_DisableCheckpoint@@3HA 00476fec     SAMPRPC.obj
 0003:00003ff0       ?RPC_SetRaceCheckpoint@@3HA 00476ff0     SAMPRPC.obj
 0003:00003ff4       ?RPC_DisableRaceCheckpoint@@3HA 00476ff4     SAMPRPC.obj
 0003:00003ff8       ?RPC_UpdateScoresPingsIPs@@3HA 00476ff8     SAMPRPC.obj
 0003:00003ffc       ?RPC_SvrStats@@3HA         00476ffc     SAMPRPC.obj
 0003:00004000       ?RPC_GameModeRestart@@3HA  00477000     SAMPRPC.obj
 0003:00004004       ?RPC_ConnectionRejected@@3HA 00477004     SAMPRPC.obj
 0003:00004008       ?RPC_ClientMessage@@3HA    00477008     SAMPRPC.obj
 0003:0000400c       ?RPC_WorldTime@@3HA        0047700c     SAMPRPC.obj
 0003:00004010       ?RPC_Pickup@@3HA           00477010     SAMPRPC.obj
 0003:00004014       ?RPC_DestroyPickup@@3HA    00477014     SAMPRPC.obj
 0003:00004018       ?RPC_DestroyWeaponPickup@@3HA 00477018     SAMPRPC.obj
 0003:0000401c       ?RPC_Weather@@3HA          0047701c     SAMPRPC.obj
 0003:00004020       ?RPC_SetTimeEx@@3HA        00477020     SAMPRPC.obj
 0003:00004024       ?RPC_ToggleClock@@3HA      00477024     SAMPRPC.obj
 0003:00004028       ?RPC_ServerCommand@@3HA    00477028     SAMPRPC.obj
 0003:0000402c       ?RPC_PickedUpPickup@@3HA   0047702c     SAMPRPC.obj
 0003:00004030       ?RPC_PickedUpWeapon@@3HA   00477030     SAMPRPC.obj
 0003:00004034       ?RPC_VehicleDestroyed@@3HA 00477034     SAMPRPC.obj
 0003:00004038       ?RPC_DialogResponse@@3HA   00477038     SAMPRPC.obj
 0003:0000403c       ?RPC_PlayAudioStream@@3HA  0047703c     SAMPRPC.obj
 0003:00004040       ?RPC_ClickPlayer@@3HA      00477040     SAMPRPC.obj
 0003:00004044       ?RPC_PlayerUpdate@@3HA     00477044     SAMPRPC.obj
 0003:00004048       ?RPC_ClickTextDraw@@3HA    00477048     SAMPRPC.obj
 0003:0000404c       ?RPC_MapMarker@@3HA        0047704c     SAMPRPC.obj
 0003:00004050       ?RPC_PlayerGiveDamage@@3HA 00477050     SAMPRPC.obj
 0003:00004054       ?RPC_ScrSetSpawnInfo@@3HA  00477054     SAMPRPC.obj
 0003:00004058       ?RPC_ScrSetPlayerTeam@@3HA 00477058     SAMPRPC.obj
 0003:0000405c       ?RPC_ScrSetPlayerSkin@@3HA 0047705c     SAMPRPC.obj
 0003:00004060       ?RPC_ScrSetPlayerName@@3HA 00477060     SAMPRPC.obj
 0003:00004064       ?RPC_ScrSetPlayerPos@@3HA  00477064     SAMPRPC.obj
 0003:00004068       ?RPC_ScrSetPlayerPosFindZ@@3HA 00477068     SAMPRPC.obj
 0003:0000406c       ?RPC_ScrSetPlayerHealth@@3HA 0047706c     SAMPRPC.obj
 0003:00004070       ?RPC_ScrPutPlayerInVehicle@@3HA 00477070     SAMPRPC.obj
 0003:00004074       ?RPC_ScrRemovePlayerFromVehicle@@3HA 00477074     SAMPRPC.obj
 0003:00004078       ?RPC_ScrSetPlayerColor@@3HA 00477078     SAMPRPC.obj
 0003:0000407c       ?RPC_ScrDisplayGameText@@3HA 0047707c     SAMPRPC.obj
 0003:00004080       ?RPC_ScrSetInterior@@3HA   00477080     SAMPRPC.obj
 0003:00004084       ?RPC_ScrSetCameraPos@@3HA  00477084     SAMPRPC.obj
 0003:00004088       ?RPC_ScrSetCameraLookAt@@3HA 00477088     SAMPRPC.obj
 0003:0000408c       ?RPC_ScrSetVehiclePos@@3HA 0047708c     SAMPRPC.obj
 0003:00004090       ?RPC_ScrSetVehicleZAngle@@3HA 00477090     SAMPRPC.obj
 0003:00004094       ?RPC_ScrVehicleParams@@3HA 00477094     SAMPRPC.obj
 0003:00004098       ?RPC_ScrSetCameraBehindPlayer@@3HA 00477098     SAMPRPC.obj
 0003:0000409c       ?RPC_ScrTogglePlayerControllable@@3HA 0047709c     SAMPRPC.obj
 0003:000040a0       ?RPC_ScrPlaySound@@3HA     004770a0     SAMPRPC.obj
 0003:000040a4       ?RPC_ScrSetWorldBounds@@3HA 004770a4     SAMPRPC.obj
 0003:000040a8       ?RPC_ScrHaveSomeMoney@@3HA 004770a8     SAMPRPC.obj
 0003:000040ac       ?RPC_ScrSetPlayerFacingAngle@@3HA 004770ac     SAMPRPC.obj
 0003:000040b0       ?RPC_ScrResetMoney@@3HA    004770b0     SAMPRPC.obj
 0003:000040b4       ?RPC_ScrResetPlayerWeapons@@3HA 004770b4     SAMPRPC.obj
 0003:000040b8       ?RPC_ScrGivePlayerWeapon@@3HA 004770b8     SAMPRPC.obj
 0003:000040bc       ?RPC_ScrRespawnVehicle@@3HA 004770bc     SAMPRPC.obj
 0003:000040c0       ?RPC_ScrLinkVehicle@@3HA   004770c0     SAMPRPC.obj
 0003:000040c4       ?RPC_ScrSetPlayerArmour@@3HA 004770c4     SAMPRPC.obj
 0003:000040c8       ?RPC_ScrDeathMessage@@3HA  004770c8     SAMPRPC.obj
 0003:000040cc       ?RPC_ScrSetMapIcon@@3HA    004770cc     SAMPRPC.obj
 0003:000040d0       ?RPC_ScrDisableMapIcon@@3HA 004770d0     SAMPRPC.obj
 0003:000040d4       ?RPC_ScrSetWeaponAmmo@@3HA 004770d4     SAMPRPC.obj
 0003:000040d8       ?RPC_ScrSetGravity@@3HA    004770d8     SAMPRPC.obj
 0003:000040dc       ?RPC_ScrSetVehicleHealth@@3HA 004770dc     SAMPRPC.obj
 0003:000040e0       ?RPC_ScrAttachTrailerToVehicle@@3HA 004770e0     SAMPRPC.obj
 0003:000040e4       ?RPC_ScrDetachTrailerFromVehicle@@3HA 004770e4     SAMPRPC.obj
 0003:000040e8       ?RPC_ScrCreateObject@@3HA  004770e8     SAMPRPC.obj
 0003:000040ec       ?RPC_ScrSetObjectPos@@3HA  004770ec     SAMPRPC.obj
 0003:000040f0       ?RPC_ScrSetObjectRotation@@3HA 004770f0     SAMPRPC.obj
 0003:000040f4       ?RPC_ScrDestroyObject@@3HA 004770f4     SAMPRPC.obj
 0003:000040f8       ?RPC_ScrCreateExplosion@@3HA 004770f8     SAMPRPC.obj
 0003:000040fc       ?RPC_ScrShowNameTag@@3HA   004770fc     SAMPRPC.obj
 0003:00004100       ?RPC_ScrMoveObject@@3HA    00477100     SAMPRPC.obj
 0003:00004104       ?RPC_ScrStopObject@@3HA    00477104     SAMPRPC.obj
 0003:00004108       ?RPC_ScrNumberPlate@@3HA   00477108     SAMPRPC.obj
 0003:0000410c       ?RPC_ScrTogglePlayerSpectating@@3HA 0047710c     SAMPRPC.obj
 0003:00004110       ?RPC_ScrSetPlayerSpectating@@3HA 00477110     SAMPRPC.obj
 0003:00004114       ?RPC_ScrPlayerSpectatePlayer@@3HA 00477114     SAMPRPC.obj
 0003:00004118       ?RPC_ScrPlayerSpectateVehicle@@3HA 00477118     SAMPRPC.obj
 0003:0000411c       ?RPC_ScrRemoveComponent@@3HA 0047711c     SAMPRPC.obj
 0003:00004120       ?RPC_ScrForceSpawnSelection@@3HA 00477120     SAMPRPC.obj
 0003:00004124       ?RPC_ScrAttachObjectToPlayer@@3HA 00477124     SAMPRPC.obj
 0003:00004128       ?RPC_ScrInitMenu@@3HA      00477128     SAMPRPC.obj
 0003:0000412c       ?RPC_ScrShowMenu@@3HA      0047712c     SAMPRPC.obj
 0003:00004130       ?RPC_ScrHideMenu@@3HA      00477130     SAMPRPC.obj
 0003:00004134       ?RPC_ScrSetPlayerWantedLevel@@3HA 00477134     SAMPRPC.obj
 0003:00004138       ?RPC_ScrShowTextDraw@@3HA  00477138     SAMPRPC.obj
 0003:0000413c       ?RPC_ScrHideTextDraw@@3HA  0047713c     SAMPRPC.obj
 0003:00004140       ?RPC_ScrEditTextDraw@@3HA  00477140     SAMPRPC.obj
 0003:00004144       ?RPC_ScrAddGangZone@@3HA   00477144     SAMPRPC.obj
 0003:00004148       ?RPC_ScrRemoveGangZone@@3HA 00477148     SAMPRPC.obj
 0003:0000414c       ?RPC_ScrFlashGangZone@@3HA 0047714c     SAMPRPC.obj
 0003:00004150       ?RPC_ScrStopFlashGangZone@@3HA 00477150     SAMPRPC.obj
 0003:00004154       ?RPC_ScrApplyAnimation@@3HA 00477154     SAMPRPC.obj
 0003:00004158       ?RPC_ScrClearAnimations@@3HA 00477158     SAMPRPC.obj
 0003:0000415c       ?RPC_ScrSetSpecialAction@@3HA 0047715c     SAMPRPC.obj
 0003:00004160       ?RPC_ScrEnableStuntBonus@@3HA 00477160     SAMPRPC.obj
 0003:00004164       ?RPC_ScrSetFightingStyle@@3HA 00477164     SAMPRPC.obj
 0003:00004168       ?RPC_ScrSetPlayerVelocity@@3HA 00477168     SAMPRPC.obj
 0003:0000416c       ?RPC_ScrSetVehicleVelocity@@3HA 0047716c     SAMPRPC.obj
 0003:00004170       ?RPC_ScrToggleWidescreen@@3HA 00477170     SAMPRPC.obj
 0003:00004174       ?RPC_ScrSetVehicleTireStatus@@3HA 00477174     SAMPRPC.obj
 0003:00004178       ?RPC_ScrSetPlayerDrunkVisuals@@3HA 00477178     SAMPRPC.obj
 0003:0000417c       ?RPC_ScrSetPlayerDrunkHandling@@3HA 0047717c     SAMPRPC.obj
 0003:00004180       ?RPC_ScrDialogBox@@3HA     00477180     SAMPRPC.obj
 0003:000041b8       ?condenseWhiteSpace@TiXmlBase@@0_NA 004771b8     tinyxml.obj
 0003:000041bc       ??_R0?AVTiXmlBase@@@8      004771bc     tinyxml.obj
 0003:000041d4       ??_R0?AVTiXmlAttribute@@@8 004771d4     tinyxml.obj
 0003:000041f4       ??_R0?AVTiXmlNode@@@8      004771f4     tinyxml.obj
 0003:0000420c       ??_R0?AVTiXmlDocument@@@8  0047720c     tinyxml.obj
 0003:00004228       ??_R0?AVTiXmlComment@@@8   00477228     tinyxml.obj
 0003:00004244       ??_R0?AVTiXmlDeclaration@@@8 00477244     tinyxml.obj
 0003:00004264       ??_R0?AVTiXmlText@@@8      00477264     tinyxml.obj
 0003:0000427c       ??_R0?AVTiXmlUnknown@@@8   0047727c     tinyxml.obj
 0003:00004298       ??_R0?AVTiXmlElement@@@8   00477298     tinyxml.obj
 0003:000042b8       ?errorString@TiXmlBase@@1PAPBDA 004772b8     tinyxmlerror.obj
 0003:000042f8       ?entity@TiXmlBase@@0PAUEntity@1@A 004772f8     tinyxmlparser.obj
 0003:00004368       ?vehicle_list@@3PAUvehicle_entry@@A 00477368     common.obj
 0003:00005148       ?iReconnectTime@@3HA       00478148     main.obj
 0003:0000514c       ?normalMode_goto@@3GA      0047814c     main.obj
 0003:000051ec       ?dwTimeReconnect@@3KA      004781ec     netgame.obj
 0003:00005224       ?imitateID@@3GA            00478224     netrpc.obj
 0003:00005290       ?rec_continueAfterFin@@3_NA 00478290     vehplayer.obj
 0003:00005390       ??_R0?AVbad_alloc@std@@@8  00478390     LIBCMT:new.obj
 0003:000053ac       ??_R0?AVexception@std@@@8  004783ac     LIBCMT:new.obj
 0003:000053d4       ??_R0?AVtype_info@@@8      004783d4     LIBCMT:typinfo.obj
 0003:000053ec       __fltused                  004783ec     LIBCMT:_fpinit_.obj
 0003:000053f0       __ldused                   004783f0     LIBCMT:_fpinit_.obj
 0003:00005400       __iob                      00478400     LIBCMT:_file.obj
 0003:000056b0       ___app_type                004786b0     LIBCMT:wincrt0.obj
 0003:000057d8       __amblksiz                 004787d8     LIBCMT:heapinit.obj
 0003:000057dc       __aexit_rtn                004787dc     LIBCMT:crt0dat.obj
 0003:00005a08       ___abort_behavior          00478a08     LIBCMT:abort.obj
 0003:00005a0c       ___security_cookie         00478a0c     LIBCMT:gs_cookie.obj
 0003:00005a10       ___security_cookie_complement 00478a10     LIBCMT:gs_cookie.obj
 0003:00005a14       ___nullstring              00478a14     LIBCMT:output.obj
 0003:00005a18       ___wnullstring             00478a18     LIBCMT:output.obj
 0003:00005a20       ??_R0?AVbad_cast@std@@@8   00478a20     LIBCMT:stdexcpt.obj
 0003:00005a3c       ??_R0?AVbad_typeid@std@@@8 00478a3c     LIBCMT:stdexcpt.obj
 0003:00005a5c       ??_R0?AV__non_rtti_object@std@@@8 00478a5c     LIBCMT:stdexcpt.obj
 0003:00005a84       ??_R0?AVbad_exception@std@@@8 00478a84     LIBCMT:frame.obj
 0003:00005aa4       ___flsindex                00478aa4     LIBCMT:tidtable.obj
 0003:00005aa8       ___getvalueindex           00478aa8     LIBCMT:tidtable.obj
 0003:00005ac0       __cfltcvt_tab              00478ac0     LIBCMT:cmiscdat.obj
 0003:00005ae8       __First_FPE_Indx           00478ae8     LIBCMT:winxfltr.obj
 0003:00005aec       __Num_FPE                  00478aec     LIBCMT:winxfltr.obj
 0003:00005af0       __XcptActTabSize           00478af0     LIBCMT:winxfltr.obj
 0003:00005af4       __XcptActTabCount          00478af4     LIBCMT:winxfltr.obj
 0003:00005af8       __lookuptrailbytes         00478af8     LIBCMT:read.obj
 0003:00005bf8       ___badioinfo               00478bf8     LIBCMT:ioinit.obj
 0003:00005c40       ___initialmbcinfo          00478c40     LIBCMT:mbctype.obj
 0003:00005e60       __mbctype                  00478e60     LIBCMT:mbctype.obj
 0003:00005f68       __mbcasemap                00478f68     LIBCMT:mbctype.obj
 0003:00006068       ___ptmbcinfo               00479068     LIBCMT:mbctype.obj
 0003:00006164       ___globallocalestatus      00479164     LIBCMT:glstatus.obj
 0003:00006168       ___clocalestr              00479168     LIBCMT:nlsdata2.obj
 0003:00006170       ___initiallocinfo          00479170     LIBCMT:nlsdata2.obj
 0003:00006248       ___ptlocinfo               00479248     LIBCMT:nlsdata2.obj
 0003:0000624c       ___lc_clike                0047924c     LIBCMT:nlsdata2.obj
 0003:00006250       ___initiallocalestructinfo 00479250     LIBCMT:nlsdata2.obj
 0003:00006260       __indefinite               00479260     LIBCMT:_87disp_.obj
 0003:0000626a       __piby2                    0047926a     LIBCMT:_87disp_.obj
 0003:000062a0       __d_inf                    004792a0     LIBCMT:_util_.obj
 0003:000062a8       __d_ind                    004792a8     LIBCMT:_util_.obj
 0003:000062b0       __d_max                    004792b0     LIBCMT:_util_.obj
 0003:000062b8       __d_min                    004792b8     LIBCMT:_util_.obj
 0003:000062c0       __d_mzero                  004792c0     LIBCMT:_util_.obj
 0003:000063cc       __NLG_Destination          004793cc     LIBCMT:exsup.obj
 0003:000063e4       __pctype                   004793e4     LIBCMT:ctype.obj
 0003:000063e8       __pwctype                  004793e8     LIBCMT:ctype.obj
 0003:000063f0       ___lc_time_c               004793f0     LIBCMT:strftime.obj
 0003:000064a8       ___lc_time_curr            004794a8     LIBCMT:strftime.obj
 0003:000064ac       ___lconv_static_decimal    004794ac     LIBCMT:lconv.obj
 0003:000064b0       ___lconv_c                 004794b0     LIBCMT:lconv.obj
 0003:000064e0       ___lconv                   004794e0     LIBCMT:lconv.obj
 0003:000064e4       ___mb_cur_max              004794e4     LIBCMT:nlsdata1.obj
 0003:000064e8       ___decimal_point           004794e8     LIBCMT:nlsdata1.obj
 0003:000064ec       ___decimal_point_length    004794ec     LIBCMT:nlsdata1.obj
 0003:00006520       __pow10pos                 00479520     LIBCMT:_constpow_.obj
 0003:00006680       __pow10neg                 00479680     LIBCMT:_constpow_.obj
 0003:000067dc       __matherr_flag             004797dc     LIBCMT:_matherr_.obj
 0003:000067e0       __coninpfh                 004797e0     LIBCMT:initcon.obj
 0003:000067e4       __confh                    004797e4     LIBCMT:initcon.obj
 0003:000067e8       __timezone                 004797e8     LIBCMT:timeset.obj
 0003:000067ec       __daylight                 004797ec     LIBCMT:timeset.obj
 0003:000067f0       __dstbias                  004797f0     LIBCMT:timeset.obj
 0003:00006878       __tzname                   00479878     LIBCMT:timeset.obj
 0003:000068a0       __lpdays                   004798a0     LIBCMT:days.obj
 0003:000068d4       __days                     004798d4     LIBCMT:days.obj
 0003:00006910       ?_Sync@ios_base@std@@0_NA  00479910     libcpmt:ios.obj
 0003:0000693c       ?staticItemID@NetworkIDGenerator@@0GA 0047993c     NetworkIDGenerator.obj
 0003:00006940       ?externalPlayerId@NetworkIDGenerator@@0UPlayerID@@A 00479940     NetworkIDGenerator.obj
 0003:00006948       ?current@?1??Find@?$BinarySearchTree@UNetworkIDNode@@@DataStructures@@IAEAAPAUnode@23@ABUNetworkIDNode@@PAPAU423@@Z@4PAU423@A 00479948     NetworkIDGenerator.obj
 0003:0000694c       ?parent@?1??FindParent@?$BinarySearchTree@UNetworkIDNode@@@DataStructures@@IAEAAPAUnode@23@ABUNetworkIDNode@@@Z@4PAU423@A 0047994c     NetworkIDGenerator.obj
 0003:00006950       ?dummyptr@?1??GetPointerToNode@?$BinarySearchTree@UNetworkIDNode@@@DataStructures@@QAEAAPAUNetworkIDNode@@ABU4@@Z@4PAU4@A 00479950     NetworkIDGenerator.obj
 0003:00006954       ?tempnode@?1??GetPointerToNode@?$BinarySearchTree@UNetworkIDNode@@@DataStructures@@QAEAAPAUNetworkIDNode@@ABU4@@Z@4PAUnode@23@A 00479954     NetworkIDGenerator.obj
 0003:00006958       ?peerToPeerMode@NetworkID@@2_NA 00479958     NetworkTypes.obj
 0003:000074a8       ?ROUNDS@@3HA               0047a4a8     rijndael.obj
 0003:000074b0       ?winsockInfo@SocketLayer@@0UWSAData@@A 0047a4b0     SocketLayer.obj
 0003:00007640       ?socketLayerStarted@SocketLayer@@0_NA 0047a640     SocketLayer.obj
 0003:00007641       ?I@SocketLayer@@0V1@A      0047a641     SocketLayer.obj
 0003:00007644       ?instance@StringCompressor@@0PAV1@A 0047a644     StringCompressor.obj
 0003:00007648       ?referenceCount@StringCompressor@@0HA 0047a648     StringCompressor.obj
 0003:0000764c       ?instance@StringTable@@1PAV1@A 0047a64c     StringTable.obj
 0003:00007650       ?referenceCount@StringTable@@1HA 0047a650     StringTable.obj
 0003:00007658       ?dblSpace@@3HA             0047a658     samp_netencr.obj
 0003:00007660       ?decrBuffer@@3PAEA         0047a660     samp_netencr.obj
 0003:00008660       ?encrBuffer@@3PAEA         0047b660     samp_netencr.obj
 0003:00009660       ?buf@@3PADA                0047c660     samp_netencr.obj
 0003:00029660       ?nullrep_@TiXmlString@@0URep@1@A 0049c660     tinystr.obj
 0003:00029670       ?szInputBuffer@@3PADA      0049c670     console.obj
 0003:00029870       ?iFollowingPassenger@@3HA  0049c870     localplayer.obj
 0003:00029874       ?iFollowingDriver@@3HA     0049c874     localplayer.obj
 0003:00029878       ?dwLastInVehicleDataSentTick@@3KA 0049c878     localplayer.obj
 0003:0002987c       ?dwLastOnFootDataSentTick@@3KA 0049c87c     localplayer.obj
 0003:00029880       ?dwLastUnocDataSentTick@@3KA 0049c880     localplayer.obj
 0003:00029884       ?dwLastPassengerDataSentTick@@3KA 0049c884     localplayer.obj
 0003:00029888       ?dwLastAimDataSentTick@@3KA 0049c888     localplayer.obj
 0003:00029890       ?g_szNickName@@3PADA       0049c890     main.obj
 0003:000298b0       ?playerInfo@@3PAUstPlayerInfo@@A 0049c8b0     main.obj
 0003:00073078       ?vehiclePool@@3PAUstVehiclePool@@A 004e6078     main.obj
 0003:0007ccb8       ?g_myPlayerID@@3GA         004efcb8     main.obj
 0003:0007ccbc       ?pRakClient@@3PAVRakClientInterface@@A 004efcbc     main.obj
 0003:0007ccc0       ?iAreWeConnected@@3HA      004efcc0     main.obj
 0003:0007ccc4       ?iConnectionRequested@@3HA 004efcc4     main.obj
 0003:0007ccc8       ?iSpawned@@3HA             004efcc8     main.obj
 0003:0007cccc       ?iGameInited@@3HA          004efccc     main.obj
 0003:0007ccd0       ?vid@@3HA                  004efcd0     main.obj
 0003:0007ccd4       ?dd@@3HA                   004efcd4     main.obj
 0003:0007ccd8       ?flLog@@3PAU_iobuf@@A      004efcd8     main.obj
 0003:0007ccdc       ?dwAutoRunTick@@3KA        004efcdc     main.obj
 0003:0007ccec       ?inCarUpdateTick@@3KA      004efcec     misc_funcs.obj
 0003:0007ccf0       ?iPassengerNotificationSent@@3HA 004efcf0     netgame.obj
 0003:0007ccf4       ?iDriverNotificationSent@@3HA 004efcf4     netgame.obj
 0003:0007cd00       ?g_szHostName@@3PADA       004efd00     netrpc.obj
 0003:0007ce00       ?iNetModeNormalOnfootSendRate@@3HA 004efe00     netrpc.obj
 0003:0007ce04       ?iNetModeFiringSendRate@@3HA 004efe04     netrpc.obj
 0003:0007ce08       ?iNetModeSendMultiplier@@3HA 004efe08     netrpc.obj
 0003:0007ce0c       ?iNetModeNormalIncarSendRate@@3HA 004efe0c     netrpc.obj
 0003:0007ce10       ?sampDialog@@3UstSAMPDialog@@A 004efe10     netrpc.obj
 0003:0007d220       ?GTAMenu@@3UstGTAMenu@@A   004f0220     netrpc.obj
 0003:0007d2a4       ?iGettingNewName@@3HA      004f02a4     netrpc.obj
 0003:0007d2a8       ?hSAMPDlgFont@@3PAUHFONT__@@A 004f02a8     netrpc.obj
 0003:0007d2ac       ?hDlgThread@@3PAXA         004f02ac     netrpc.obj
 0003:0007d2b0       ?hwndSAMPDlg@@3PAUHWND__@@A 004f02b0     netrpc.obj
 0003:0007d2b8       ?routeVehicleID@@3GA       004f02b8     vehplayer.obj
 0003:0007d2c0       ?rec_angle@@3PAY08MA       004f02c0     vehplayer.obj
 0003:000a12c0       ?rec_pos@@3PAY02MA         005142c0     vehplayer.obj
 0003:000ad2c0       ?rec_playNext@@3MA         005202c0     vehplayer.obj
 0003:000ad2c4       ?rec_state@@3W4eRecordingState@@A 005202c4     vehplayer.obj
 0003:000ad2c8       ?rec_speed@@3PAY02MA       005202c8     vehplayer.obj
 0003:000b92c8       ?rec_spin@@3PAY02MA        0052c2c8     vehplayer.obj
 0003:000c52c8       ?rec_tempTableCpy@@3PADA   005382c8     vehplayer.obj
 0003:000c5308       ?rec_maxNum@@3HA           00538308     vehplayer.obj
 0003:000c530c       ?rec_index@@3HA            0053830c     vehplayer.obj
 0003:000c5310       ?g_hfText@@3PAUHFONT__@@A  00538310     window.obj
 0003:000c5314       ?hwnd@@3PAUHWND__@@A       00538314     window.obj
 0003:000c5318       ?inputhwnd@@3PAUHWND__@@A  00538318     window.obj
 0003:000c531c       ?g_hInst@@3PAUHINSTANCE__@@A 0053831c     window.obj
 0003:000c5320       ?loghwnd@@3PAUHWND__@@A    00538320     window.obj
 0003:000c5324       ?texthwnd@@3PAUHWND__@@A   00538324     window.obj
 0003:000c5328       ?settings@@3UstSettings@@A 00538328     xmlsets.obj
 0003:000e9c88       ?xmlSettings@@3VTiXmlDocument@@A 0055cc88     xmlsets.obj
 0003:000e9ce0       ___fastflag                0055cce0     LIBCMT:_fpinit_.obj
 0003:000e9ce4       __adjust_fdiv              0055cce4     LIBCMT:_fpinit_.obj
 0003:000e9ce8       __cflush                   0055cce8     LIBCMT:_file.obj
 0003:000e9cec       __aenvptr                  0055ccec     LIBCMT:wincrt0.obj
 0003:000e9cf0       __wenvptr                  0055ccf0     LIBCMT:wincrt0.obj
 0003:000e9cf4       ___error_mode              0055ccf4     LIBCMT:wincrt0.obj
 0003:000e9e48       ___sbh_pHeaderDefer        0055ce48     LIBCMT:sbheap.obj
 0003:000e9e4c       __crtheap                  0055ce4c     LIBCMT:heapinit.obj
 0003:000e9e50       __umaskval                 0055ce50     LIBCMT:crt0dat.obj
 0003:000e9e54       ___argc                    0055ce54     LIBCMT:crt0dat.obj
 0003:000e9e58       ___argv                    0055ce58     LIBCMT:crt0dat.obj
 0003:000e9e5c       ___wargv                   0055ce5c     LIBCMT:crt0dat.obj
 0003:000e9e60       __environ                  0055ce60     LIBCMT:crt0dat.obj
 0003:000e9e64       ___initenv                 0055ce64     LIBCMT:crt0dat.obj
 0003:000e9e68       __wenviron                 0055ce68     LIBCMT:crt0dat.obj
 0003:000e9e6c       ___winitenv                0055ce6c     LIBCMT:crt0dat.obj
 0003:000e9e70       __pgmptr                   0055ce70     LIBCMT:crt0dat.obj
 0003:000e9e74       __wpgmptr                  0055ce74     LIBCMT:crt0dat.obj
 0003:000e9e78       __exitflag                 0055ce78     LIBCMT:crt0dat.obj
 0003:000e9e7c       __C_Termination_Done       0055ce7c     LIBCMT:crt0dat.obj
 0003:000e9e80       __C_Exit_Done              0055ce80     LIBCMT:crt0dat.obj
 0003:000ea19c       ?_pnhHeap@@3P6AHI@ZA       0055d19c     LIBCMT:handler.obj
 0003:000ea1a0       __newmode                  0055d1a0     LIBCMT:_newmode.obj
 0003:000ea1a4       ___pInvalidArgHandler      0055d1a4     LIBCMT:invarg.obj
 0003:000ea1d0       __stdbuf                   0055d1d0     LIBCMT:_sftbuf.obj
 0003:000ea1d8       _gpFlsAlloc                0055d1d8     LIBCMT:tidtable.obj
 0003:000ea1dc       _gpFlsGetValue             0055d1dc     LIBCMT:tidtable.obj
 0003:000ea1e0       _gpFlsSetValue             0055d1e0     LIBCMT:tidtable.obj
 0003:000ea1e4       _gpFlsFree                 0055d1e4     LIBCMT:tidtable.obj
 0003:000ea1e8       ?__pInconsistency@@3P6AXXZA 0055d1e8     LIBCMT:hooks.obj
 0003:000ea1fc       ___pPurecall               0055d1fc     LIBCMT:inithelp.obj
 0003:000ea200       __maxwait                  0055d200     LIBCMT:crtheap.obj
 0003:000ea208       ___mbulinfo                0055d208     LIBCMT:mbctype.obj
 0003:000ea214       ___mbcodepage              0055d214     LIBCMT:mbctype.obj
 0003:000ea218       ___ismbcodepage            0055d218     LIBCMT:mbctype.obj
 0003:000ea21c       ___mblcid                  0055d21c     LIBCMT:mbctype.obj
 0003:000ea220       ___locale_changed          0055d220     LIBCMT:setlocal.obj
 0003:000ea224       ___lc_handle               0055d224     LIBCMT:nlsdata2.obj
 0003:000ea23c       ___lc_codepage             0055d23c     LIBCMT:nlsdata2.obj
 0003:000ea240       ___lc_collate_cp           0055d240     LIBCMT:nlsdata2.obj
 0003:000ea248       __commode                  0055d248     LIBCMT:ncommode.obj
 0003:000ea6b8       ?pArgList@UnDecorator@@0PAVReplicator@@A 0055d6b8     LIBCMT:undname.obj
 0003:000ea6bc       ?pZNameList@UnDecorator@@0PAVReplicator@@A 0055d6bc     LIBCMT:undname.obj
 0003:000ea6c0       ?pTemplateArgList@UnDecorator@@0PAVReplicator@@A 0055d6c0     LIBCMT:undname.obj
 0003:000ea6c4       ?gName@UnDecorator@@0PBDB  0055d6c4     LIBCMT:undname.obj
 0003:000ea6c8       ?name@UnDecorator@@0PBDB   0055d6c8     LIBCMT:undname.obj
 0003:000ea6cc       ?outputString@UnDecorator@@0PADA 0055d6cc     LIBCMT:undname.obj
 0003:000ea6d0       ?maxStringLength@UnDecorator@@0HA 0055d6d0     LIBCMT:undname.obj
 0003:000ea6d4       ?disableFlags@UnDecorator@@0KA 0055d6d4     LIBCMT:undname.obj
 0003:000ea6d8       ?m_pGetParameter@UnDecorator@@0P6APADJ@ZA 0055d6d8     LIBCMT:undname.obj
 0003:000ea6dc       ?fExplicitTemplateParams@UnDecorator@@0_NA 0055d6dc     LIBCMT:undname.obj
 0003:000ea6dd       ?fGetTemplateArgumentList@UnDecorator@@0_NA 0055d6dd     LIBCMT:undname.obj
 0003:000ea6e0       ?nodes@?1??make@DNameStatusNode@@SAPAV2@W4DNameStatus@@@Z@4PAV2@A 0055d6e0     LIBCMT:undname.obj
 0003:000ea710       ??_B?1??make@DNameStatusNode@@SAPAV1@W4DNameStatus@@@Z@51 0055d710     LIBCMT:undname.obj
 0003:000ea718       __outputformat             0055d718     LIBCMT:outputformat.obj
 0003:000ea720       ___lconv_static_null       0055d720     LIBCMT:lconv.obj
 0003:000ea7e0       __fmode                    0055d7e0     LIBCMT:txtmode.obj
 0003:000ea850       ?_Fpz@std@@3_JA            0055d850     libcpmt:ios.obj
 0003:000ea858       ?_Index@ios_base@std@@0HA  0055d858     libcpmt:ios.obj
 0003:000ea890       __debugger_hook_dummy      0055d890     <common>
 0003:000ea894       __pmatherr                 0055d894     <common>
 0003:000ea898       ___use_sse2_mathfcns       0055d898     <common>
 0003:000ea89c       ___setlc_active            0055d89c     <common>
 0003:000ea8a0       ___unguarded_readlc_active 0055d8a0     <common>
 0003:000ea8a4       __nhandle                  0055d8a4     <common>
 0003:000ea8c0       ___pioinfo                 0055d8c0     <common>
 0003:000ea9c0       ___sse2_available          0055d9c0     <common>
 0003:000ea9c4       ___env_initialized         0055d9c4     <common>
 0003:000ea9c8       ___onexitend               0055d9c8     <common>
 0003:000ea9cc       ___onexitbegin             0055d9cc     <common>
 0003:000ea9d0       ___mbctype_initialized     0055d9d0     <common>
 0003:000ea9d4       ___dyn_tls_init_callback   0055d9d4     <common>
 0003:000ea9d8       ___active_heap             0055d9d8     <common>
 0003:000ea9dc       ___sbh_initialized         0055d9dc     <common>
 0003:000ea9e0       ___sbh_cntHeaderList       0055d9e0     <common>
 0003:000ea9e4       ___sbh_pHeaderList         0055d9e4     <common>
 0003:000ea9e8       ___sbh_threshold           0055d9e8     <common>
 0003:000ea9ec       ___sbh_pHeaderScan         0055d9ec     <common>
 0003:000ea9f0       ___sbh_sizeHeaderList      0055d9f0     <common>
 0003:000ea9f4       ___sbh_indGroupDefer       0055d9f4     <common>
 0003:000ea9f8       __acmdln                   0055d9f8     <common>
 0003:000ea9fc       ___piob                    0055d9fc     <common>
 0003:000eaa00       __bufin                    0055da00     <common>
 0003:000eba00       __nstream                  0055ea00     <common>

 entry point at        0001:00038235

 Static symbols

 0001:fffff000       __unwindfunclet$??1TiXmlDeclaration@@UAE@XZ$0 00400000 f   tinyxmlparser.obj
 0001:fffff000       __unwindfunclet$??0TiXmlText@@QAE@PBD@Z$0 00400000 f   tinyxmlparser.obj
 0001:fffff000       __unwindfunclet$??1TiXmlAttribute@@UAE@XZ$0 00400000 f   tinyxmlparser.obj
 0001:fffff000       __unwindfunclet$??1TiXmlDocument@@UAE@XZ$0 00400000 f   xmlsets.obj
 0001:fffff008       __unwindfunclet$??1TiXmlAttribute@@UAE@XZ$1 00400008 f   tinyxmlparser.obj
 0001:fffff008       __unwindfunclet$??1TiXmlDeclaration@@UAE@XZ$1 00400008 f   tinyxmlparser.obj
 0001:fffff008       __ehhandler$??0TiXmlText@@QAE@PBD@Z 00400008 f   tinyxmlparser.obj
 0001:fffff008       __ehhandler$??1TiXmlDocument@@UAE@XZ 00400008 f   xmlsets.obj
 0001:fffff013       __unwindfunclet$??1TiXmlDeclaration@@UAE@XZ$2 00400013 f   tinyxmlparser.obj
 0001:fffff013       __ehhandler$??1TiXmlAttribute@@UAE@XZ 00400013 f   tinyxmlparser.obj
 0001:fffff01e       __ehhandler$??1TiXmlDeclaration@@UAE@XZ 0040001e f   tinyxmlparser.obj
 0001:00032b59       _swprintf                  00433b59 f   LIBCMT:wassert.obj
 0001:000339f1       ?CatchGuardHandler@@YA?AW4_EXCEPTION_DISPOSITION@@PAUEHExceptionRecord@@PAUCatchGuardRN@@PAX2@Z 004349f1 f   LIBCMT:_trnsctrl_.obj
 0001:00033afb       ?TranslatorGuardHandler@@YA?AW4_EXCEPTION_DISPOSITION@@PAUEHExceptionRecord@@PAUTranslatorGuardRN@@PAX2@Z 00434afb f   LIBCMT:_trnsctrl_.obj
 0001:00033d1f       ?ArrayUnwindFilter@@YAHPAU_EXCEPTION_POINTERS@@@Z 00434d1f f   LIBCMT:ehvecdtr.obj
 0001:00034449       __onexit_nolock            00435449 f   LIBCMT:onexit.obj
 0001:00034587       _xtoa@16                   00435587 f   LIBCMT:xtoa.obj
 0001:00034636       @x64toa@20                 00435636 f   LIBCMT:xtoa.obj
 0001:00034828       __callthreadstartex        00435828 f   LIBCMT:threadex.obj
 0001:00034869       __threadstartex@4          00435869 f   LIBCMT:threadex.obj
 0001:000357c9       _vscan_fn                  004367c9 f   LIBCMT:sscanf.obj
 0001:0003713c       _flsall                    0043813c f   LIBCMT:fflush.obj
 0001:00038047       _fast_error_exit           00439047 f   LIBCMT:wincrt0.obj
 0001:00038070       _check_managed_app         00439070 f   LIBCMT:wincrt0.obj
 0001:000380b7       ___tmainCRTStartup         004390b7 f   LIBCMT:wincrt0.obj
 0001:00039490       _ValidateLocalCookies      0043a490 f   LIBCMT:chandler4.obj
 0001:000397a8       __initterm                 0043a7a8 f   LIBCMT:crt0dat.obj
 0001:000398e6       _doexit                    0043a8e6 f   LIBCMT:crt0dat.obj
 0001:00039e62       _fastcopy_I                0043ae62 f   LIBCMT:p4_memcpy.obj
 0001:00039fcc       _has_osfxsr_set            0043afcc f   LIBCMT:cpu_disp.obj
 0001:0003a08b       _fastzero_I                0043b08b f   LIBCMT:p4_memset.obj
 0001:0003a90e       _ctrlevent_capture@4       0043b90e f   LIBCMT:winsig.obj
 0001:0003a9a9       _siglookup                 0043b9a9 f   LIBCMT:winsig.obj
 0001:0003af55       _xtow_s@20                 0043bf55 f   LIBCMT:xtows.obj
 0001:0003b0b8       @x64tow_s@24               0043c0b8 f   LIBCMT:xtows.obj
 0001:0003b618       _write_char                0043c618 f   LIBCMT:output.obj
 0001:0003b64b       _write_multi_char          0043c64b f   LIBCMT:output.obj
 0001:0003b671       _write_string              0043c671 f   LIBCMT:output.obj
 0001:0003c778       ?ExFilterRethrow@@YAHPAU_EXCEPTION_POINTERS@@@Z 0043d778 f   LIBCMT:frame.obj
 0001:0003cb6c       ?IsInExceptionSpec@@YAEPAUEHExceptionRecord@@PBU_s_ESTypeList@@@Z 0043db6c f   LIBCMT:frame.obj
 0001:0003cbe7       ?CallUnexpected@@YAXPBU_s_ESTypeList@@@Z 0043dbe7 f   LIBCMT:frame.obj
 0001:0003cc18       __catch$?CallUnexpected@@YAXPBU_s_ESTypeList@@@Z$0 0043dc18 f   LIBCMT:frame.obj
 0001:0003cc30       ?Is_bad_exception_allowed@@YAEPBU_s_ESTypeList@@@Z 0043dc30 f   LIBCMT:frame.obj
 0001:0003cce8       ?CallCatchBlock@@YAPAXPAUEHExceptionRecord@@PAUEHRegistrationNode@@PAU_CONTEXT@@PBU_s_FuncInfo@@PAXHK@Z 0043dce8 f   LIBCMT:frame.obj
 0001:0003d1da       ?CatchIt@@YAXPAUEHExceptionRecord@@PAUEHRegistrationNode@@PAU_CONTEXT@@PAXPBU_s_FuncInfo@@PBU_s_HandlerType@@PBU_s_CatchableType@@PBU_s_TryBlockMapEntry@@H1E@Z 0043e1da f   LIBCMT:frame.obj
 0001:0003d248       ?FindHandlerForForeignException@@YAXPAUEHExceptionRecord@@PAUEHRegistrationNode@@PAU_CONTEXT@@PAXPBU_s_FuncInfo@@HH1@Z 0043e248 f   LIBCMT:frame.obj
 0001:0003d33c       ?FindHandler@@YAXPAUEHExceptionRecord@@PAUEHRegistrationNode@@PAU_CONTEXT@@PAXPBU_s_FuncInfo@@EH1@Z 0043e33c f   LIBCMT:frame.obj
 0001:0003eb4d       __shift                    0043fb4d f   LIBCMT:cvt.obj
 0001:0003eb92       __cftoe2_l                 0043fb92 f   LIBCMT:cvt.obj
 0001:0003f184       __cftof2_l                 00440184 f   LIBCMT:cvt.obj
 0001:0003f71e       _xcptlookup                0044071e f   LIBCMT:winxfltr.obj
 0001:00040b8c       __unwind_handler4          00441b8c f   LIBCMT:exsup4.obj
 0001:000414eb       ___check_float_string      004424eb f   LIBCMT:input.obj
 0001:00041554       __hextodec                 00442554 f   LIBCMT:input.obj
 0001:00041574       __inc                      00442574 f   LIBCMT:input.obj
 0001:0004158a       __un_inc                   0044258a f   LIBCMT:input.obj
 0001:0004159d       __whiteout                 0044259d f   LIBCMT:input.obj
 0001:00042584       ___check_float_string      00443584 f   LIBCMT:inputs.obj
 0001:000425db       __hextodec                 004435db f   LIBCMT:inputs.obj
 0001:000425fb       __inc                      004435fb f   LIBCMT:inputs.obj
 0001:00042611       __un_inc                   00443611 f   LIBCMT:inputs.obj
 0001:00042624       __whiteout                 00443624 f   LIBCMT:inputs.obj
 0001:00043772       ?strtoxl@@YAKPAUlocaleinfo_struct@@PBDPAPBDHH@Z 00444772 f   LIBCMT:strtol.obj
 0001:00043a32       ?strtoxq@@YA_KPAUlocaleinfo_struct@@PBDPAPBDHH@Z 00444a32 f   LIBCMT:strtoq.obj
 0001:00043d5a       ?CPtoLCID@@YAHH@Z          00444d5a f   LIBCMT:mbctype.obj
 0001:00043d89       ?setSBCS@@YAXPAUthreadmbcinfostruct@@@Z 00444d89 f   LIBCMT:mbctype.obj
 0001:00043ded       ?setSBUpLow@@YAXPAUthreadmbcinfostruct@@@Z 00444ded f   LIBCMT:mbctype.obj
 0001:00044024       ?getSystemCP@@YAHH@Z       00445024 f   LIBCMT:mbctype.obj
 0001:000446f8       __copytlocinfo_nolock      004456f8 f   LIBCMT:setlocal.obj
 0001:0004471e       __updatetlocinfoEx_nolock  0044571e f   LIBCMT:setlocal.obj
 0001:0004483c       _sync_legacy_variables_lk  0044583c f   LIBCMT:setlocal.obj
 0001:00044be9       __setlocale_get_all        00445be9 f   LIBCMT:setlocal.obj
 0001:00044f97       __setlocale_set_cat        00445f97 f   LIBCMT:setlocal.obj
 0001:00045299       __setlocale_nolock         00446299 f   LIBCMT:setlocal.obj
 0001:00046611       _write_char                00447611 f   LIBCMT:outputs.obj
 0001:00046644       _write_multi_char          00447644 f   LIBCMT:outputs.obj
 0001:0004666a       _write_string              0044766a f   LIBCMT:outputs.obj
 0001:000473b2       _write_char                004483b2 f   LIBCMT:outputp.obj
 0001:000473e5       _write_multi_char          004483e5 f   LIBCMT:outputp.obj
 0001:0004740b       _write_string              0044840b f   LIBCMT:outputp.obj
 0001:00048763       ?strncnt@@YAHPBDH@Z        00449763 f   LIBCMT:a_map.obj
 0001:00048781       ?__crtLCMapStringA_stat@@YAHPAUlocaleinfo_struct@@KKPBDHPADHHH@Z 00449781 f   LIBCMT:a_map.obj
 0001:0004a61c       __get_fname                0044b61c f   LIBCMT:_fpexcept_.obj
 0001:0004acd5       _parse_cmdline             0044bcd5 f   LIBCMT:stdargv.obj
 0001:0004b55c       _write_char                0044c55c f   LIBCMT:woutput.obj
 0001:0004b58b       _write_multi_char          0044c58b f   LIBCMT:woutput.obj
 0001:0004b5b2       _write_string              0044c5b2 f   LIBCMT:woutput.obj
 0001:0004c19c       _write_char                0044d19c f   LIBCMT:woutputs.obj
 0001:0004c1cb       _write_multi_char          0044d1cb f   LIBCMT:woutputs.obj
 0001:0004c1f2       _write_string              0044d1f2 f   LIBCMT:woutputs.obj
 0001:0004cf3a       _write_char                0044df3a f   LIBCMT:woutputp.obj
 0001:0004cf69       _write_multi_char          0044df69 f   LIBCMT:woutputp.obj
 0001:0004cf90       _write_string              0044df90 f   LIBCMT:woutputp.obj
 0001:0004e8c8       __unwind_handler           0044f8c8 f   LIBCMT:exsup.obj
 0001:0004f630       ?und_strlen@@YAIPBD@Z      00450630 f   LIBCMT:undname.obj
 0001:0004f63e       ?und_memcpy@@YAXPADPBDI@Z  0045063e f   LIBCMT:undname.obj
 0001:0004f654       ?und_strncmp@@YAIPBD0I@Z   00450654 f   LIBCMT:undname.obj
 0001:00053f38       ?__crtGetLocaleInfoW_stat@@YAHPAUlocaleinfo_struct@@KKPA_WHH@Z 00454f38 f   LIBCMT:w_loc.obj
 0001:00053f85       ?__crtGetLocaleInfoA_stat@@YAHPAUlocaleinfo_struct@@KKPADHH@Z 00454f85 f   LIBCMT:a_loc.obj
 0001:000547f4       __tsopen_nolock            004557f4 f   LIBCMT:open.obj
 0001:000558ee       ?__crtGetStringTypeA_stat@@YAHPAUlocaleinfo_struct@@KPBDHPAGHHH@Z 004568ee f   LIBCMT:a_str.obj
 0001:00055b19       __get_lc_time              00456b19 f   LIBCMT:inittime.obj
 0001:00056142       _fix_grouping              00457142 f   LIBCMT:initnum.obj
 0001:00056384       _fix_grouping              00457384 f   LIBCMT:initmon.obj
 0001:000570d9       ?_store_str@@YAXPADPAPADPAI@Z 004580d9 f   LIBCMT:strftime.obj
 0001:000570f9       ?_store_number@@YAXHPAPADPAI@Z 004580f9 f   LIBCMT:strftime.obj
 0001:0005712f       ?_store_num@@YAXHHPAPADPAII@Z 0045812f f   LIBCMT:strftime.obj
 0001:000571aa       ?_expandtime@@YAHPAUlocaleinfo_struct@@DPBUtm@@PAPADPAIPAU__lc_time_data@@I@Z 004581aa f   LIBCMT:strftime.obj
 0001:00057592       ?_store_winword@@YAHPAUlocaleinfo_struct@@HPBUtm@@PAPADPAIPAU__lc_time_data@@@Z 00458592 f   LIBCMT:strftime.obj
 0001:00057c66       _TranslateName             00458c66 f   LIBCMT:getqloc.obj
 0001:00057cc8       _GetLcidFromDefault        00458cc8 f   LIBCMT:getqloc.obj
 0001:00057cdc       _ProcessCodePage           00458cdc f   LIBCMT:getqloc.obj
 0001:00057d80       _TestDefaultCountry        00458d80 f   LIBCMT:getqloc.obj
 0001:00057da4       _LcidFromHexString         00458da4 f   LIBCMT:getqloc.obj
 0001:00057dd8       _GetPrimaryLen             00458dd8 f   LIBCMT:getqloc.obj
 0001:00057df3       _CountryEnumProc@4         00458df3 f   LIBCMT:getqloc.obj
 0001:00057e8b       _TestDefaultLanguage       00458e8b f   LIBCMT:getqloc.obj
 0001:00057eff       _LangCountryEnumProc@4     00458eff f   LIBCMT:getqloc.obj
 0001:000580d1       _LanguageEnumProc@4        004590d1 f   LIBCMT:getqloc.obj
 0001:00058192       _GetLcidFromCountry        00459192 f   LIBCMT:getqloc.obj
 0001:000581be       _GetLcidFromLangCountry    004591be f   LIBCMT:getqloc.obj
 0001:00058225       _GetLcidFromLanguage       00459225 f   LIBCMT:getqloc.obj
 0001:00058452       _cmpResult                 00459452 f   LIBCMT:memcmp.obj
 0001:00058464       _cmpBYTE                   00459464 f   LIBCMT:memcmp.obj
 0001:0005847c       _cmpWORD                   0045947c f   LIBCMT:memcmp.obj
 0001:000584bc       _cmpDWORD                  004594bc f   LIBCMT:memcmp.obj
 0001:00058534       _unaligned_memcmp          00459534 f   LIBCMT:memcmp.obj
 0001:0005ca36       ?x_ismbbtype_l@@YAHPAUlocaleinfo_struct@@IHH@Z 0045da36 f   LIBCMT:ismbbyte.obj
 0001:0005cefe       ?wcstoxl@@YAKPAUlocaleinfo_struct@@PB_WPAPB_WHH@Z 0045defe f   LIBCMT:wcstol.obj
 0001:0005db22       __abstract_cw              0045eb22 f   LIBCMT:_ieee87_.obj
 0001:0005dbc1       __hw_cw                    0045ebc1 f   LIBCMT:_ieee87_.obj
 0001:0005dc4f       __abstract_sw              0045ec4f f   LIBCMT:_ieee87_.obj
 0001:0005dc92       ___abstract_cw_sse2        0045ec92 f   LIBCMT:_ieee87_.obj
 0001:0005dd32       ___hw_cw_sse2              0045ed32 f   LIBCMT:_ieee87_.obj
 0001:0005ddd2       ___abstract_sw_sse2        0045edd2 f   LIBCMT:_ieee87_.obj
 0001:0005de15       ___fpreset_sse2            0045ee15 f   LIBCMT:_ieee87_.obj
 0001:0005deeb       ___statusfp_sse2           0045eeeb f   LIBCMT:_ieee87_.obj
 0001:0005df26       ___clearfp_sse2            0045ef26 f   LIBCMT:_ieee87_.obj
 0001:0005df76       ___control87_sse2          0045ef76 f   LIBCMT:_ieee87_.obj
 0001:0005f3a0       __tzset_nolock             004603a0 f   LIBCMT:tzset.obj
 0001:0005f6e6       _cvtdate                   004606e6 f   LIBCMT:tzset.obj
 0001:0005f8dd       __isindst_nolock           004608dd f   LIBCMT:tzset.obj
 0001:0005fcdd       _xtoa_s@20                 00460cdd f   LIBCMT:xtoas.obj
 0001:0005fe25       @x64toa_s@24               00460e25 f   LIBCMT:xtoas.obj
 0001:0005ff71       ?__crtGetStringTypeW_stat@@YAHPAUlocaleinfo_struct@@KPB_WHPAGHH@Z 00460f71 f   LIBCMT:w_str.obj
 0001:00060418       __getenv_s_helper          00461418 f   LIBCMT:getenv.obj
 0001:000604ad       __dupenv_s_helper          004614ad f   LIBCMT:getenv.obj
 0001:0006098e       ?strncnt@@YAHPBDH@Z        0046198e f   LIBCMT:a_cmp.obj
 0001:000609ac       ?__crtCompareStringA_stat@@YAHPAUlocaleinfo_struct@@KKPBDH1HH@Z 004619ac f   LIBCMT:a_cmp.obj
 0001:00060e81       _findenv                   00461e81 f   LIBCMT:setenv.obj
 0001:00060ed3       _copy_environ              00461ed3 f   LIBCMT:setenv.obj
 0001:00061850       __unwindfunclet$?Compress@DataCompressor@@SAXPAEIPAVBitStream@RakNet@@@Z$0 00462850 f   DataCompressor.obj
 0001:0006185b       __ehhandler$?Compress@DataCompressor@@SAXPAEIPAVBitStream@RakNet@@@Z 0046285b f   DataCompressor.obj
 0001:00061870       __unwindfunclet$?DecompressAndAllocate@DataCompressor@@SAIPAVBitStream@RakNet@@PAPAE@Z$0 00462870 f   DataCompressor.obj
 0001:0006187b       __ehhandler$?DecompressAndAllocate@DataCompressor@@SAIPAVBitStream@RakNet@@PAPAE@Z 0046287b f   DataCompressor.obj
 0001:00061890       __unwindfunclet$?DecodeArray@HuffmanEncodingTree@@QAEXPAEIPAVBitStream@RakNet@@@Z$0 00462890 f   DS_HuffmanEncodingTree.obj
 0001:0006189b       __ehhandler$?DecodeArray@HuffmanEncodingTree@@QAEXPAEIPAVBitStream@RakNet@@@Z 0046289b f   DS_HuffmanEncodingTree.obj
 0001:000618b0       __unwindfunclet$?FreeMemory@HuffmanEncodingTree@@QAEXXZ$0 004628b0 f   DS_HuffmanEncodingTree.obj
 0001:000618b8       __ehhandler$?FreeMemory@HuffmanEncodingTree@@QAEXXZ 004628b8 f   DS_HuffmanEncodingTree.obj
 0001:000618d0       __unwindfunclet$??1?$LinkedList@PAUHuffmanEncodingTreeNode@@@DataStructures@@QAE@XZ$0 004628d0 f   DS_HuffmanEncodingTree.obj
 0001:000618d8       __ehhandler$??1?$LinkedList@PAUHuffmanEncodingTreeNode@@@DataStructures@@QAE@XZ 004628d8 f   DS_HuffmanEncodingTree.obj
 0001:000618f0       __unwindfunclet$?GenerateFromFrequencyTable@HuffmanEncodingTree@@QAEXQAI@Z$0 004628f0 f   DS_HuffmanEncodingTree.obj
 0001:000618fb       __unwindfunclet$?GenerateFromFrequencyTable@HuffmanEncodingTree@@QAEXQAI@Z$1 004628fb f   DS_HuffmanEncodingTree.obj
 0001:00061906       __unwindfunclet$?GenerateFromFrequencyTable@HuffmanEncodingTree@@QAEXQAI@Z$2 00462906 f   DS_HuffmanEncodingTree.obj
 0001:00061911       __ehhandler$?GenerateFromFrequencyTable@HuffmanEncodingTree@@QAEXQAI@Z 00462911 f   DS_HuffmanEncodingTree.obj
 0001:00061920       __unwindfunclet$?Insert@?$List@UColumnDescriptor@Table@DataStructures@@@DataStructures@@QAEXUColumnDescriptor@Table@2@@Z$0 00462920 f   DS_Table.obj
 0001:0006192b       __ehhandler$?Insert@?$List@UColumnDescriptor@Table@DataStructures@@@DataStructures@@QAEXUColumnDescriptor@Table@2@@Z 0046292b f   DS_Table.obj
 0001:00061940       __unwindfunclet$??1?$MemoryPool@U?$Page@IPAURow@Table@DataStructures@@$0BA@@DataStructures@@@DataStructures@@QAE@XZ$0 00462940 f   DS_Table.obj
 0001:0006194b       __ehhandler$??1?$MemoryPool@U?$Page@IPAURow@Table@DataStructures@@$0BA@@DataStructures@@@DataStructures@@QAE@XZ 0046294b f   DS_Table.obj
 0001:00061960       __unwindfunclet$??1?$OrderedList@PAURow@Table@DataStructures@@PAU123@$1?RowSort@@YAHABQAU123@0@Z@DataStructures@@QAE@XZ$0 00462960 f   DS_Table.obj
 0001:00061968       __ehhandler$??1?$OrderedList@PAURow@Table@DataStructures@@PAU123@$1?RowSort@@YAHABQAU123@0@Z@DataStructures@@QAE@XZ 00462968 f   DS_Table.obj
 0001:00061980       __unwindfunclet$?FreePages@?$BPlusTree@IPAURow@Table@DataStructures@@$0BA@@DataStructures@@IAEXXZ$0 00462980 f   DS_Table.obj
 0001:00061988       __ehhandler$?FreePages@?$BPlusTree@IPAURow@Table@DataStructures@@$0BA@@DataStructures@@IAEXXZ 00462988 f   DS_Table.obj
 0001:000619a0       __unwindfunclet$?SortTable@Table@DataStructures@@QAEXPAUSortQuery@12@IPAPAURow@12@@Z$0 004629a0 f   DS_Table.obj
 0001:000619a8       __unwindfunclet$?SortTable@Table@DataStructures@@QAEXPAUSortQuery@12@IPAPAURow@12@@Z$1 004629a8 f   DS_Table.obj
 0001:000619b0       __ehhandler$?SortTable@Table@DataStructures@@QAEXPAUSortQuery@12@IPAPAURow@12@@Z 004629b0 f   DS_Table.obj
 0001:000619c0       __unwindfunclet$?AddRow@Table@DataStructures@@QAEPAURow@12@IAAV?$List@UCell@Table@DataStructures@@@2@@Z$1 004629c0 f   DS_Table.obj
 0001:000619cb       __ehhandler$?AddRow@Table@DataStructures@@QAEPAURow@12@IAAV?$List@UCell@Table@DataStructures@@@2@@Z 004629cb f   DS_Table.obj
 0001:000619e0       __unwindfunclet$?AddRowColumns@Table@DataStructures@@IAEPAURow@12@IPAU312@V?$List@I@2@@Z$0 004629e0 f   DS_Table.obj
 0001:000619e8       __unwindfunclet$?AddRowColumns@Table@DataStructures@@IAEPAURow@12@IPAU312@V?$List@I@2@@Z$2 004629e8 f   DS_Table.obj
 0001:000619f3       __ehhandler$?AddRowColumns@Table@DataStructures@@IAEPAURow@12@IPAU312@V?$List@I@2@@Z 004629f3 f   DS_Table.obj
 0001:00061a00       __unwindfunclet$??1?$BPlusTree@IPAURow@Table@DataStructures@@$0BA@@DataStructures@@QAE@XZ$0 00462a00 f   DS_Table.obj
 0001:00061a08       __ehhandler$??1?$BPlusTree@IPAURow@Table@DataStructures@@$0BA@@DataStructures@@QAE@XZ 00462a08 f   DS_Table.obj
 0001:00061a20       __unwindfunclet$??1Table@DataStructures@@QAE@XZ$0 00462a20 f   DS_Table.obj
 0001:00061a28       __unwindfunclet$??1Table@DataStructures@@QAE@XZ$1 00462a28 f   DS_Table.obj
 0001:00061a33       __ehhandler$??1Table@DataStructures@@QAE@XZ 00462a33 f   DS_Table.obj
 0001:00061a40       __unwindfunclet$?QueryTable@Table@DataStructures@@QAEXPAIIPAUFilterQuery@12@I0IPAV12@@Z$0 00462a40 f   DS_Table.obj
 0001:00061a48       __unwindfunclet$?QueryTable@Table@DataStructures@@QAEXPAIIPAUFilterQuery@12@I0IPAV12@@Z$1 00462a48 f   DS_Table.obj
 0001:00061a50       __ehhandler$?QueryTable@Table@DataStructures@@QAEXPAIIPAUFilterQuery@12@I0IPAV12@@Z 00462a50 f   DS_Table.obj
 0001:00061a60       __unwindfunclet$??0InternalPacketPool@@QAE@XZ$0 00462a60 f   InternalPacketPool.obj
 0001:00061a68       __ehhandler$??0InternalPacketPool@@QAE@XZ 00462a68 f   InternalPacketPool.obj
 0001:00061a80       __unwindfunclet$??1InternalPacketPool@@QAE@XZ$0 00462a80 f   InternalPacketPool.obj
 0001:00061a88       __ehhandler$??1InternalPacketPool@@QAE@XZ 00462a88 f   InternalPacketPool.obj
 0001:00061aa0       __unwindfunclet$??1?$AVLBalancedBinarySearchTree@UNetworkIDNode@@@DataStructures@@UAE@XZ$0 00462aa0 f   NetworkIDGenerator.obj
 0001:00061aa8       __ehhandler$??1?$AVLBalancedBinarySearchTree@UNetworkIDNode@@@DataStructures@@UAE@XZ 00462aa8 f   NetworkIDGenerator.obj
 0001:00061ac0       __unwindfunclet$??1RakClient@@UAE@XZ$0 00462ac0 f   RakClient.obj
 0001:00061ac8       __unwindfunclet$??1RakClient@@UAE@XZ$1 00462ac8 f   RakClient.obj
 0001:00061ad6       __unwindfunclet$??1RakClient@@UAE@XZ$2 00462ad6 f   RakClient.obj
 0001:00061ae4       __ehhandler$??1RakClient@@UAE@XZ 00462ae4 f   RakClient.obj
 0001:00061af0       __unwindfunclet$??0RakClient@@QAE@XZ$0 00462af0 f   RakClient.obj
 0001:00061af8       __unwindfunclet$??0RakClient@@QAE@XZ$1 00462af8 f   RakClient.obj
 0001:00061b06       __unwindfunclet$??0RakClient@@QAE@XZ$2 00462b06 f   RakClient.obj
 0001:00061b14       __ehhandler$??0RakClient@@QAE@XZ 00462b14 f   RakClient.obj
 0001:00061b20       __unwindfunclet$?Receive@RakClient@@UAEPAUPacket@@XZ$0 00462b20 f   RakClient.obj
 0001:00061b2b       __unwindfunclet$?Receive@RakClient@@UAEPAUPacket@@XZ$1 00462b2b f   RakClient.obj
 0001:00061b36       __unwindfunclet$?Receive@RakClient@@UAEPAUPacket@@XZ$2 00462b36 f   RakClient.obj
 0001:00061b41       __ehhandler$?Receive@RakClient@@UAEPAUPacket@@XZ 00462b41 f   RakClient.obj
 0001:00061b50       __unwindfunclet$?GetRakClientInterface@RakNetworkFactory@@SAPAVRakClientInterface@@XZ$0 00462b50 f   RakNetworkFactory.obj
 0001:00061b5b       __ehhandler$?GetRakClientInterface@RakNetworkFactory@@SAPAVRakClientInterface@@XZ 00462b5b f   RakNetworkFactory.obj
 0001:00061b70       __unwindfunclet$?GetRakServerInterface@RakNetworkFactory@@SAPAVRakServerInterface@@XZ$0 00462b70 f   RakNetworkFactory.obj
 0001:00061b7b       __ehhandler$?GetRakServerInterface@RakNetworkFactory@@SAPAVRakServerInterface@@XZ 00462b7b f   RakNetworkFactory.obj
 0001:00061b90       __unwindfunclet$?GetRakPeerInterface@RakNetworkFactory@@SAPAVRakPeerInterface@@XZ$0 00462b90 f   RakNetworkFactory.obj
 0001:00061b9b       __ehhandler$?GetRakPeerInterface@RakNetworkFactory@@SAPAVRakPeerInterface@@XZ 00462b9b f   RakNetworkFactory.obj
 0001:00061bb0       __unwindfunclet$??0RemoteSystemStruct@RakPeer@@QAE@XZ$0 00462bb0 f   RakPeer.obj
 0001:00061bbb       __unwindfunclet$??0RemoteSystemStruct@RakPeer@@QAE@XZ$1 00462bbb f   RakPeer.obj
 0001:00061bc9       __ehhandler$??0RemoteSystemStruct@RakPeer@@QAE@XZ 00462bc9 f   RakPeer.obj
 0001:00061be0       __unwindfunclet$??1RemoteSystemStruct@RakPeer@@QAE@XZ$0 00462be0 f   RakPeer.obj
 0001:00061beb       __unwindfunclet$??1RemoteSystemStruct@RakPeer@@QAE@XZ$1 00462beb f   RakPeer.obj
 0001:00061bf9       __ehhandler$??1RemoteSystemStruct@RakPeer@@QAE@XZ 00462bf9 f   RakPeer.obj
 0001:00061c10       __unwindfunclet$?GenerateCompressionLayer@RakPeer@@UAE_NQAI_N@Z$0 00462c10 f   RakPeer.obj
 0001:00061c1b       __unwindfunclet$?GenerateCompressionLayer@RakPeer@@UAE_NQAI_N@Z$1 00462c1b f   RakPeer.obj
 0001:00061c26       __ehhandler$?GenerateCompressionLayer@RakPeer@@UAE_NQAI_N@Z 00462c26 f   RakPeer.obj
 0001:00061c30       __unwindfunclet$?Ping@RakPeer@@UAEXPBDG_N@Z$0 00462c30 f   RakPeer.obj
 0001:00061c3b       __ehhandler$?Ping@RakPeer@@UAEXPBDG_N@Z 00462c3b f   RakPeer.obj
 0001:00061c50       __unwindfunclet$?AdvertiseSystem@RakPeer@@UAEXPBDG0H@Z$0 00462c50 f   RakPeer.obj
 0001:00061c5b       __ehhandler$?AdvertiseSystem@RakPeer@@UAEXPBDG0H@Z 00462c5b f   RakPeer.obj
 0001:00061c70       __unwindfunclet$?HandleRPCPacket@RakPeer@@IAE_NPBDHUPlayerID@@@Z$0 00462c70 f   RakPeer.obj
 0001:00061c7b       __unwindfunclet$?HandleRPCPacket@RakPeer@@IAE_NPBDHUPlayerID@@@Z$1 00462c7b f   RakPeer.obj
 0001:00061c86       __unwindfunclet$?HandleRPCPacket@RakPeer@@IAE_NPBDHUPlayerID@@@Z$2 00462c86 f   RakPeer.obj
 0001:00061c91       __unwindfunclet$?HandleRPCPacket@RakPeer@@IAE_NPBDHUPlayerID@@@Z$3 00462c91 f   RakPeer.obj
 0001:00061c9c       __ehhandler$?HandleRPCPacket@RakPeer@@IAE_NPBDHUPlayerID@@@Z 00462c9c f   RakPeer.obj
 0001:00061cb0       __unwindfunclet$?SendImmediate@RakPeer@@IAE_NPADHW4PacketPriority@@W4PacketReliability@@DUPlayerID@@_N4_J@Z$0 00462cb0 f   RakPeer.obj
 0001:00061cbb       __ehhandler$?SendImmediate@RakPeer@@IAE_NPADHW4PacketPriority@@W4PacketReliability@@DUPlayerID@@_N4_J@Z 00462cbb f   RakPeer.obj
 0001:00061cd0       __unwindfunclet$??1?$OrderedList@UPlayerID@@UPlayerIDAndIndex@@$1?PlayerIDAndIndexComp@@YAHABU1@ABU2@@Z@DataStructures@@QAE@XZ$0 00462cd0 f   RakPeer.obj
 0001:00061cd8       __ehhandler$??1?$OrderedList@UPlayerID@@UPlayerIDAndIndex@@$1?PlayerIDAndIndexComp@@YAHABU1@ABU2@@Z@DataStructures@@QAE@XZ 00462cd8 f   RakPeer.obj
 0001:00061cf0       __unwindfunclet$??0RakPeer@@QAE@XZ$0 00462cf0 f   RakPeer.obj
 0001:00061cf8       __unwindfunclet$??0RakPeer@@QAE@XZ$1 00462cf8 f   RakPeer.obj
 0001:00061d03       __unwindfunclet$??0RakPeer@@QAE@XZ$2 00462d03 f   RakPeer.obj
 0001:00061d11       __unwindfunclet$??0RakPeer@@QAE@XZ$3 00462d11 f   RakPeer.obj
 0001:00061d1f       __unwindfunclet$??0RakPeer@@QAE@XZ$4 00462d1f f   RakPeer.obj
 0001:00061d37       __unwindfunclet$??0RakPeer@@QAE@XZ$5 00462d37 f   RakPeer.obj
 0001:00061d45       __unwindfunclet$??0RakPeer@@QAE@XZ$6 00462d45 f   RakPeer.obj
 0001:00061d53       __unwindfunclet$??0RakPeer@@QAE@XZ$7 00462d53 f   RakPeer.obj
 0001:00061d61       __unwindfunclet$??0RakPeer@@QAE@XZ$8 00462d61 f   RakPeer.obj
 0001:00061d6f       __unwindfunclet$??0RakPeer@@QAE@XZ$9 00462d6f f   RakPeer.obj
 0001:00061d7d       __unwindfunclet$??0RakPeer@@QAE@XZ$10 00462d7d f   RakPeer.obj
 0001:00061d8b       __unwindfunclet$??0RakPeer@@QAE@XZ$11 00462d8b f   RakPeer.obj
 0001:00061d99       __unwindfunclet$??0RakPeer@@QAE@XZ$12 00462d99 f   RakPeer.obj
 0001:00061da7       __unwindfunclet$??0RakPeer@@QAE@XZ$13 00462da7 f   RakPeer.obj
 0001:00061db5       __unwindfunclet$??0RakPeer@@QAE@XZ$14 00462db5 f   RakPeer.obj
 0001:00061dc3       __ehhandler$??0RakPeer@@QAE@XZ 00462dc3 f   RakPeer.obj
 0001:00061dd0       __unwindfunclet$?RPC@RakPeer@@UAE_NPAHPBDIW4PacketPriority@@W4PacketReliability@@DUPlayerID@@_N5UNetworkID@@PAVBitStream@RakNet@@@Z$0 00462dd0 f   RakPeer.obj
 0001:00061ddb       __ehhandler$?RPC@RakPeer@@UAE_NPAHPBDIW4PacketPriority@@W4PacketReliability@@DUPlayerID@@_N5UNetworkID@@PAVBitStream@RakNet@@@Z 00462ddb f   RakPeer.obj
 0001:00061df0       __unwindfunclet$?OnConnectionRequest@RakPeer@@IAEXPAURemoteSystemStruct@1@PAE_N@Z$0 00462df0 f   RakPeer.obj
 0001:00061dfb       __ehhandler$?OnConnectionRequest@RakPeer@@IAEXPAURemoteSystemStruct@1@PAE_N@Z 00462dfb f   RakPeer.obj
 0001:00061e10       __unwindfunclet$?NotifyAndFlagForDisconnect@RakPeer@@IAEXUPlayerID@@_NE@Z$0 00462e10 f   RakPeer.obj
 0001:00061e1b       __ehhandler$?NotifyAndFlagForDisconnect@RakPeer@@IAEXUPlayerID@@_NE@Z 00462e1b f   RakPeer.obj
 0001:00061e30       __unwindfunclet$?ShiftIncomingTimestamp@RakPeer@@IBEXPAEUPlayerID@@@Z$0 00462e30 f   RakPeer.obj
 0001:00061e3b       __ehhandler$?ShiftIncomingTimestamp@RakPeer@@IBEXPAEUPlayerID@@@Z 00462e3b f   RakPeer.obj
 0001:00061e50       __unwindfunclet$?SecuredConnectionResponse@RakPeer@@IAEXUPlayerID@@@Z$0 00462e50 f   RakPeer.obj
 0001:00061e5b       __ehhandler$?SecuredConnectionResponse@RakPeer@@IAEXUPlayerID@@@Z 00462e5b f   RakPeer.obj
 0001:00061e70       __unwindfunclet$?SendStaticDataInternal@RakPeer@@IAEXUPlayerID@@_N@Z$0 00462e70 f   RakPeer.obj
 0001:00061e7b       __ehhandler$?SendStaticDataInternal@RakPeer@@IAEXUPlayerID@@_N@Z 00462e7b f   RakPeer.obj
 0001:00061e90       __unwindfunclet$?PingInternal@RakPeer@@IAEXUPlayerID@@_N@Z$0 00462e90 f   RakPeer.obj
 0001:00061e9b       __ehhandler$?PingInternal@RakPeer@@IAEXUPlayerID@@_N@Z 00462e9b f   RakPeer.obj
 0001:00061eb0       __unwindfunclet$?ProcessNetworkPacket@@YGXIGPBDHPAVRakPeer@@@Z$0 00462eb0 f   RakPeer.obj
 0001:00061ebb       __unwindfunclet$?ProcessNetworkPacket@@YGXIGPBDHPAVRakPeer@@@Z$1 00462ebb f   RakPeer.obj
 0001:00061ec6       __unwindfunclet$?ProcessNetworkPacket@@YGXIGPBDHPAVRakPeer@@@Z$2 00462ec6 f   RakPeer.obj
 0001:00061ed1       __ehhandler$?ProcessNetworkPacket@@YGXIGPBDHPAVRakPeer@@@Z 00462ed1 f   RakPeer.obj
 0001:00061ee0       __unwindfunclet$??1RakPeer@@UAE@XZ$0 00462ee0 f   RakPeer.obj
 0001:00061ee8       __unwindfunclet$??1RakPeer@@UAE@XZ$1 00462ee8 f   RakPeer.obj
 0001:00061ef3       __unwindfunclet$??1RakPeer@@UAE@XZ$2 00462ef3 f   RakPeer.obj
 0001:00061f01       __unwindfunclet$??1RakPeer@@UAE@XZ$3 00462f01 f   RakPeer.obj
 0001:00061f0f       __unwindfunclet$??1RakPeer@@UAE@XZ$4 00462f0f f   RakPeer.obj
 0001:00061f27       __unwindfunclet$??1RakPeer@@UAE@XZ$5 00462f27 f   RakPeer.obj
 0001:00061f35       __unwindfunclet$??1RakPeer@@UAE@XZ$6 00462f35 f   RakPeer.obj
 0001:00061f43       __unwindfunclet$??1RakPeer@@UAE@XZ$7 00462f43 f   RakPeer.obj
 0001:00061f51       __unwindfunclet$??1RakPeer@@UAE@XZ$8 00462f51 f   RakPeer.obj
 0001:00061f5f       __unwindfunclet$??1RakPeer@@UAE@XZ$9 00462f5f f   RakPeer.obj
 0001:00061f6d       __unwindfunclet$??1RakPeer@@UAE@XZ$10 00462f6d f   RakPeer.obj
 0001:00061f7b       __unwindfunclet$??1RakPeer@@UAE@XZ$11 00462f7b f   RakPeer.obj
 0001:00061f89       __unwindfunclet$??1RakPeer@@UAE@XZ$12 00462f89 f   RakPeer.obj
 0001:00061f97       __unwindfunclet$??1RakPeer@@UAE@XZ$13 00462f97 f   RakPeer.obj
 0001:00061fa5       __unwindfunclet$??1RakPeer@@UAE@XZ$14 00462fa5 f   RakPeer.obj
 0001:00061fb3       __ehhandler$??1RakPeer@@UAE@XZ 00462fb3 f   RakPeer.obj
 0001:00061fc0       __unwindfunclet$?SecuredConnectionConfirmation@RakPeer@@IAEXPAURemoteSystemStruct@1@PAD@Z$0 00462fc0 f   RakPeer.obj
 0001:00061fcb       __ehhandler$?SecuredConnectionConfirmation@RakPeer@@IAEXPAURemoteSystemStruct@1@PAD@Z 00462fcb f   RakPeer.obj
 0001:00061fe0       __unwindfunclet$?RunUpdateCycle@RakPeer@@IAE_NXZ$0 00462fe0 f   RakPeer.obj
 0001:00061feb       __unwindfunclet$?RunUpdateCycle@RakPeer@@IAE_NXZ$1 00462feb f   RakPeer.obj
 0001:00061ff6       __unwindfunclet$?RunUpdateCycle@RakPeer@@IAE_NXZ$2 00462ff6 f   RakPeer.obj
 0001:00062001       __unwindfunclet$?RunUpdateCycle@RakPeer@@IAE_NXZ$3 00463001 f   RakPeer.obj
 0001:0006200c       __unwindfunclet$?RunUpdateCycle@RakPeer@@IAE_NXZ$4 0046300c f   RakPeer.obj
 0001:00062017       __unwindfunclet$?RunUpdateCycle@RakPeer@@IAE_NXZ$5 00463017 f   RakPeer.obj
 0001:00062022       __unwindfunclet$?RunUpdateCycle@RakPeer@@IAE_NXZ$6 00463022 f   RakPeer.obj
 0001:0006202d       __unwindfunclet$?RunUpdateCycle@RakPeer@@IAE_NXZ$7 0046302d f   RakPeer.obj
 0001:00062038       __unwindfunclet$?RunUpdateCycle@RakPeer@@IAE_NXZ$8 00463038 f   RakPeer.obj
 0001:00062043       __ehhandler$?RunUpdateCycle@RakPeer@@IAE_NXZ 00463043 f   RakPeer.obj
 0001:00062050       __unwindfunclet$?Initialize@RakPeer@@UAE_NGGHPBD@Z$0 00463050 f   RakPeer.obj
 0001:0006205e       __ehhandler$?Initialize@RakPeer@@UAE_NGGHPBD@Z 0046305e f   RakPeer.obj
 0001:00062070       __unwindfunclet$??1RakServer@@UAE@XZ$0 00463070 f   rakserver.obj
 0001:00062078       __ehhandler$??1RakServer@@UAE@XZ 00463078 f   rakserver.obj
 0001:00062090       __unwindfunclet$??0RakServer@@QAE@XZ$0 00463090 f   rakserver.obj
 0001:00062098       __ehhandler$??0RakServer@@QAE@XZ 00463098 f   rakserver.obj
 0001:000620b0       __unwindfunclet$?Receive@RakServer@@UAEPAUPacket@@XZ$0 004630b0 f   rakserver.obj
 0001:000620bb       __unwindfunclet$?Receive@RakServer@@UAEPAUPacket@@XZ$1 004630bb f   rakserver.obj
 0001:000620c6       __unwindfunclet$?Receive@RakServer@@UAEPAUPacket@@XZ$2 004630c6 f   rakserver.obj
 0001:000620d1       __unwindfunclet$?Receive@RakServer@@UAEPAUPacket@@XZ$3 004630d1 f   rakserver.obj
 0001:000620dc       __ehhandler$?Receive@RakServer@@UAEPAUPacket@@XZ 004630dc f   rakserver.obj
 0001:000620f0       __unwindfunclet$?ChangeStaticClientData@RakServer@@UAEXUPlayerID@@U2@@Z$0 004630f0 f   rakserver.obj
 0001:000620fb       __ehhandler$?ChangeStaticClientData@RakServer@@UAEXUPlayerID@@U2@@Z 004630fb f   rakserver.obj
 0001:00062110       __unwindfunclet$?GetSHA1@ReliabilityLayer@@AAEXQAEIQAD@Z$0 00463110 f   ReliabilityLayer.obj
 0001:0006211b       __ehhandler$?GetSHA1@ReliabilityLayer@@AAEXQAEIQAD@Z 0046311b f   ReliabilityLayer.obj
 0001:00062130       __unwindfunclet$??1?$LinkedList@PAUInternalPacket@@@DataStructures@@QAE@XZ$0 00463130 f   ReliabilityLayer.obj
 0001:00062138       __ehhandler$??1?$LinkedList@PAUInternalPacket@@@DataStructures@@QAE@XZ 00463138 f   ReliabilityLayer.obj
 0001:00062150       __unwindfunclet$??1?$MemoryPool@U?$Page@GPAUInternalPacket@@$0CA@@DataStructures@@@DataStructures@@QAE@XZ$0 00463150 f   ReliabilityLayer.obj
 0001:0006215b       __ehhandler$??1?$MemoryPool@U?$Page@GPAUInternalPacket@@$0CA@@DataStructures@@@DataStructures@@QAE@XZ 0046315b f   ReliabilityLayer.obj
 0001:00062170       __unwindfunclet$?Insert@?$List@U?$RangeNode@G@DataStructures@@@DataStructures@@QAEXU?$RangeNode@G@2@@Z$0 00463170 f   ReliabilityLayer.obj
 0001:0006217b       __ehhandler$?Insert@?$List@U?$RangeNode@G@DataStructures@@@DataStructures@@QAEXU?$RangeNode@G@2@@Z 0046317b f   ReliabilityLayer.obj
 0001:00062190       __unwindfunclet$?Insert@?$List@U?$RangeNode@G@DataStructures@@@DataStructures@@QAEXU?$RangeNode@G@2@I@Z$0 00463190 f   ReliabilityLayer.obj
 0001:0006219b       __ehhandler$?Insert@?$List@U?$RangeNode@G@DataStructures@@@DataStructures@@QAEXU?$RangeNode@G@2@I@Z 0046319b f   ReliabilityLayer.obj
 0001:000621b0       __unwindfunclet$??_G?$LinkedList@PAUInternalPacket@@@DataStructures@@QAEPAXI@Z$0 004631b0 f   ReliabilityLayer.obj
 0001:000621b8       __ehhandler$??_G?$LinkedList@PAUInternalPacket@@@DataStructures@@QAEPAXI@Z 004631b8 f   ReliabilityLayer.obj
 0001:000621d0       __unwindfunclet$??1?$OrderedList@IPAUInternalPacket@@$1?SplitPacketIndexComp@@YAHABIABQAU1@@Z@DataStructures@@QAE@XZ$0 004631d0 f   ReliabilityLayer.obj
 0001:000621d8       __ehhandler$??1?$OrderedList@IPAUInternalPacket@@$1?SplitPacketIndexComp@@YAHABIABQAU1@@Z@DataStructures@@QAE@XZ 004631d8 f   ReliabilityLayer.obj
 0001:000621f0       __unwindfunclet$?Serialize@?$RangeList@G@DataStructures@@QAEIPAVBitStream@RakNet@@H_N@Z$0 004631f0 f   ReliabilityLayer.obj
 0001:000621fb       __ehhandler$?Serialize@?$RangeList@G@DataStructures@@QAEIPAVBitStream@RakNet@@H_N@Z 004631fb f   ReliabilityLayer.obj
 0001:00062210       __unwindfunclet$??1?$OrderedList@GPAUSplitPacketChannel@@$1?SplitPacketChannelComp@@YAHABGABQAU1@@Z@DataStructures@@QAE@XZ$0 00463210 f   ReliabilityLayer.obj
 0001:00062218       __ehhandler$??1?$OrderedList@GPAUSplitPacketChannel@@$1?SplitPacketChannelComp@@YAHABGABQAU1@@Z@DataStructures@@QAE@XZ 00463218 f   ReliabilityLayer.obj
 0001:00062230       __unwindfunclet$?FreePages@?$BPlusTree@GPAUInternalPacket@@$0CA@@DataStructures@@IAEXXZ$0 00463230 f   ReliabilityLayer.obj
 0001:00062238       __ehhandler$?FreePages@?$BPlusTree@GPAUInternalPacket@@$0CA@@DataStructures@@IAEXXZ 00463238 f   ReliabilityLayer.obj
 0001:00062250       __unwindfunclet$??1?$OrderedList@GU?$RangeNode@G@DataStructures@@$1??$RangeNodeComp@G@2@YAHABGABU12@@Z@DataStructures@@QAE@XZ$0 00463250 f   ReliabilityLayer.obj
 0001:00062258       __ehhandler$??1?$OrderedList@GU?$RangeNode@G@DataStructures@@$1??$RangeNodeComp@G@2@YAHABGABU12@@Z@DataStructures@@QAE@XZ 00463258 f   ReliabilityLayer.obj
 0001:00062270       __unwindfunclet$??1?$RangeList@G@DataStructures@@QAE@XZ$0 00463270 f   ReliabilityLayer.obj
 0001:00062278       __ehhandler$??1?$RangeList@G@DataStructures@@QAE@XZ 00463278 f   ReliabilityLayer.obj
 0001:00062290       __unwindfunclet$??1?$BPlusTree@GPAUInternalPacket@@$0CA@@DataStructures@@QAE@XZ$0 00463290 f   ReliabilityLayer.obj
 0001:00062298       __ehhandler$??1?$BPlusTree@GPAUInternalPacket@@$0CA@@DataStructures@@QAE@XZ 00463298 f   ReliabilityLayer.obj
 0001:000622b0       __unwindfunclet$??0ReliabilityLayer@@QAE@XZ$0 004632b0 f   ReliabilityLayer.obj
 0001:000622b8       __unwindfunclet$??0ReliabilityLayer@@QAE@XZ$1 004632b8 f   ReliabilityLayer.obj
 0001:000622c3       __unwindfunclet$??0ReliabilityLayer@@QAE@XZ$2 004632c3 f   ReliabilityLayer.obj
 0001:000622ce       __unwindfunclet$??0ReliabilityLayer@@QAE@XZ$3 004632ce f   ReliabilityLayer.obj
 0001:000622d9       __unwindfunclet$??0ReliabilityLayer@@QAE@XZ$4 004632d9 f   ReliabilityLayer.obj
 0001:000622e4       __unwindfunclet$??0ReliabilityLayer@@QAE@XZ$5 004632e4 f   ReliabilityLayer.obj
 0001:000622fa       __unwindfunclet$??0ReliabilityLayer@@QAE@XZ$6 004632fa f   ReliabilityLayer.obj
 0001:00062308       __unwindfunclet$??0ReliabilityLayer@@QAE@XZ$7 00463308 f   ReliabilityLayer.obj
 0001:00062316       __unwindfunclet$??0ReliabilityLayer@@QAE@XZ$8 00463316 f   ReliabilityLayer.obj
 0001:00062324       __unwindfunclet$??0ReliabilityLayer@@QAE@XZ$9 00463324 f   ReliabilityLayer.obj
 0001:00062332       __unwindfunclet$??0ReliabilityLayer@@QAE@XZ$10 00463332 f   ReliabilityLayer.obj
 0001:00062340       __unwindfunclet$??0ReliabilityLayer@@QAE@XZ$11 00463340 f   ReliabilityLayer.obj
 0001:0006234e       __ehhandler$??0ReliabilityLayer@@QAE@XZ 0046334e f   ReliabilityLayer.obj
 0001:00062360       __unwindfunclet$?FreeThreadSafeMemory@ReliabilityLayer@@AAEXXZ$1 00463360 f   ReliabilityLayer.obj
 0001:00062368       __ehhandler$?FreeThreadSafeMemory@ReliabilityLayer@@AAEXXZ 00463368 f   ReliabilityLayer.obj
 0001:00062380       __unwindfunclet$?HandleSocketReceiveFromConnectedPlayer@ReliabilityLayer@@QAE_NPBDHUPlayerID@@AAV?$List@PAVPluginInterface@@@DataStructures@@H@Z$7 00463380 f   ReliabilityLayer.obj
 0001:0006238b       __unwindfunclet$?HandleSocketReceiveFromConnectedPlayer@ReliabilityLayer@@QAE_NPBDHUPlayerID@@AAV?$List@PAVPluginInterface@@@DataStructures@@H@Z$8 0046338b f   ReliabilityLayer.obj
 0001:00062396       __ehhandler$?HandleSocketReceiveFromConnectedPlayer@ReliabilityLayer@@QAE_NPBDHUPlayerID@@AAV?$List@PAVPluginInterface@@@DataStructures@@H@Z 00463396 f   ReliabilityLayer.obj
 0001:000623a0       __unwindfunclet$??1ReliabilityLayer@@QAE@XZ$0 004633a0 f   ReliabilityLayer.obj
 0001:000623a8       __unwindfunclet$??1ReliabilityLayer@@QAE@XZ$1 004633a8 f   ReliabilityLayer.obj
 0001:000623b3       __unwindfunclet$??1ReliabilityLayer@@QAE@XZ$2 004633b3 f   ReliabilityLayer.obj
 0001:000623be       __unwindfunclet$??1ReliabilityLayer@@QAE@XZ$3 004633be f   ReliabilityLayer.obj
 0001:000623c9       __unwindfunclet$??1ReliabilityLayer@@QAE@XZ$4 004633c9 f   ReliabilityLayer.obj
 0001:000623d4       __unwindfunclet$??1ReliabilityLayer@@QAE@XZ$5 004633d4 f   ReliabilityLayer.obj
 0001:000623ea       __unwindfunclet$??1ReliabilityLayer@@QAE@XZ$6 004633ea f   ReliabilityLayer.obj
 0001:000623f8       __unwindfunclet$??1ReliabilityLayer@@QAE@XZ$7 004633f8 f   ReliabilityLayer.obj
 0001:00062406       __unwindfunclet$??1ReliabilityLayer@@QAE@XZ$8 00463406 f   ReliabilityLayer.obj
 0001:00062414       __unwindfunclet$??1ReliabilityLayer@@QAE@XZ$9 00463414 f   ReliabilityLayer.obj
 0001:00062422       __unwindfunclet$??1ReliabilityLayer@@QAE@XZ$10 00463422 f   ReliabilityLayer.obj
 0001:00062430       __unwindfunclet$??1ReliabilityLayer@@QAE@XZ$11 00463430 f   ReliabilityLayer.obj
 0001:0006243e       __ehhandler$??1ReliabilityLayer@@QAE@XZ 0046343e f   ReliabilityLayer.obj
 0001:00062450       __unwindfunclet$??1RPCMap@@QAE@XZ$0 00463450 f   RPCMap.obj
 0001:00062458       __ehhandler$??1RPCMap@@QAE@XZ 00463458 f   RPCMap.obj
 0001:00062470       __unwindfunclet$??1?$OrderedList@HUMapNode@?$Map@HPAVHuffmanEncodingTree@@$1??$defaultMapKeyComparison@H@DataStructures@@YAHABH0@Z@DataStructures@@$1?NodeComparisonFunc@23@SAHABHABU123@@Z@DataStructures@@QAE@XZ$0 00463470 f   StringCompressor.obj
 0001:00062478       __ehhandler$??1?$OrderedList@HUMapNode@?$Map@HPAVHuffmanEncodingTree@@$1??$defaultMapKeyComparison@H@DataStructures@@YAHABH0@Z@DataStructures@@$1?NodeComparisonFunc@23@SAHABHABU123@@Z@DataStructures@@QAE@XZ 00463478 f   StringCompressor.obj
 0001:00062490       __unwindfunclet$?EncodeString@StringCompressor@@QAEXPBDHPAVBitStream@RakNet@@H@Z$0 00463490 f   StringCompressor.obj
 0001:0006249b       __ehhandler$?EncodeString@StringCompressor@@QAEXPBDHPAVBitStream@RakNet@@H@Z 0046349b f   StringCompressor.obj
 0001:000624b0       __unwindfunclet$??1?$Map@HPAVHuffmanEncodingTree@@$1??$defaultMapKeyComparison@H@DataStructures@@YAHABH0@Z@DataStructures@@QAE@XZ$0 004634b0 f   StringCompressor.obj
 0001:000624b8       __ehhandler$??1?$Map@HPAVHuffmanEncodingTree@@$1??$defaultMapKeyComparison@H@DataStructures@@YAHABH0@Z@DataStructures@@QAE@XZ 004634b8 f   StringCompressor.obj
 0001:000624d0       __unwindfunclet$??0StringCompressor@@AAE@XZ$0 004634d0 f   StringCompressor.obj
 0001:000624d8       __unwindfunclet$??0StringCompressor@@AAE@XZ$1 004634d8 f   StringCompressor.obj
 0001:000624e3       __ehhandler$??0StringCompressor@@AAE@XZ 004634e3 f   StringCompressor.obj
 0001:000624f0       __unwindfunclet$?GenerateTreeFromStrings@StringCompressor@@QAEXPAEIH@Z$0 004634f0 f   StringCompressor.obj
 0001:000624fe       __ehhandler$?GenerateTreeFromStrings@StringCompressor@@QAEXPAEIH@Z 004634fe f   StringCompressor.obj
 0001:00062510       __unwindfunclet$??1StringCompressor@@QAE@XZ$0 00463510 f   StringCompressor.obj
 0001:00062518       __ehhandler$??1StringCompressor@@QAE@XZ 00463518 f   StringCompressor.obj
 0001:00062530       __unwindfunclet$?AddReference@StringCompressor@@SAXXZ$0 00463530 f   StringCompressor.obj
 0001:0006253b       __ehhandler$?AddReference@StringCompressor@@SAXXZ 0046353b f   StringCompressor.obj
 0001:00062550       __unwindfunclet$??1?$OrderedList@PADUStrAndBool@@$1?StrAndBoolComp@@YAHABQADABU1@@Z@DataStructures@@QAE@XZ$0 00463550 f   StringTable.obj
 0001:00062558       __ehhandler$??1?$OrderedList@PADUStrAndBool@@$1?StrAndBoolComp@@YAHABQADABU1@@Z@DataStructures@@QAE@XZ 00463558 f   StringTable.obj
 0001:00062570       __unwindfunclet$??1StringTable@@QAE@XZ$0 00463570 f   StringTable.obj
 0001:00062578       __ehhandler$??1StringTable@@QAE@XZ 00463578 f   StringTable.obj
 0001:00062590       __unwindfunclet$??0SystemAddressList@@QAE@UPlayerID@@@Z$0 00463590 f   SystemAddressList.obj
 0001:00062598       __ehhandler$??0SystemAddressList@@QAE@UPlayerID@@@Z 00463598 f   SystemAddressList.obj
 0001:000625b0       __unwindfunclet$?Save@SystemAddressList@@QAE_NPBD@Z$0 004635b0 f   SystemAddressList.obj
 0001:000625bb       __ehhandler$?Save@SystemAddressList@@QAE_NPBD@Z 004635bb f   SystemAddressList.obj
 0001:000625d0       __unwindfunclet$?Load@SystemAddressList@@QAE_NPBD@Z$0 004635d0 f   SystemAddressList.obj
 0001:000625db       __ehhandler$?Load@SystemAddressList@@QAE_NPBD@Z 004635db f   SystemAddressList.obj
 0001:000625f0       __unwindfunclet$?DeserializeTable@TableSerializer@@SA_NPAEIPAVTable@DataStructures@@@Z$0 004635f0 f   TableSerializer.obj
 0001:000625fb       __ehhandler$?DeserializeTable@TableSerializer@@SA_NPAEIPAVTable@DataStructures@@@Z 004635fb f   TableSerializer.obj
 0001:00062610       __unwindfunclet$?reserve@TiXmlString@@QAEXI@Z$0 00463610 f   tinystr.obj
 0001:00062618       __ehhandler$?reserve@TiXmlString@@QAEXI@Z 00463618 f   tinystr.obj
 0001:00062630       __unwindfunclet$?assign@TiXmlString@@QAEAAV1@PBDI@Z$0 00463630 f   tinystr.obj
 0001:00062638       __ehhandler$?assign@TiXmlString@@QAEAAV1@PBDI@Z 00463638 f   tinystr.obj
 0001:00062650       __unwindfunclet$??H@YA?AVTiXmlString@@ABV0@0@Z$0 00463650 f   tinystr.obj
 0001:00062669       __ehhandler$??H@YA?AVTiXmlString@@ABV0@0@Z 00463669 f   tinystr.obj
 0001:00062680       __unwindfunclet$??H@YA?AVTiXmlString@@ABV0@PBD@Z$0 00463680 f   tinystr.obj
 0001:00062699       __ehhandler$??H@YA?AVTiXmlString@@ABV0@PBD@Z 00463699 f   tinystr.obj
 0001:000626b0       __unwindfunclet$??H@YA?AVTiXmlString@@PBDABV0@@Z$0 004636b0 f   tinystr.obj
 0001:000626c9       __ehhandler$??H@YA?AVTiXmlString@@PBDABV0@@Z 004636c9 f   tinystr.obj
 0001:000626e0       __unwindfunclet$??1TiXmlAttribute@@UAE@XZ$0 004636e0 f   tinyxml.obj
 0001:000626e8       __unwindfunclet$??1TiXmlAttribute@@UAE@XZ$1 004636e8 f   tinyxml.obj
 0001:000626f3       __ehhandler$??1TiXmlAttribute@@UAE@XZ 004636f3 f   tinyxml.obj
 0001:00062700       __unwindfunclet$??1TiXmlNode@@UAE@XZ$0 00463700 f   tinyxml.obj
 0001:00062708       __unwindfunclet$??1TiXmlNode@@UAE@XZ$1 00463708 f   tinyxml.obj
 0001:00062713       __ehhandler$??1TiXmlNode@@UAE@XZ 00463713 f   tinyxml.obj
 0001:00062720       __unwindfunclet$??0TiXmlDocument@@QAE@XZ$0 00463720 f   tinyxml.obj
 0001:00062728       __unwindfunclet$??0TiXmlDocument@@QAE@XZ$1 00463728 f   tinyxml.obj
 0001:00062733       __ehhandler$??0TiXmlDocument@@QAE@XZ 00463733 f   tinyxml.obj
 0001:00062740       __unwindfunclet$??0TiXmlDocument@@QAE@PBD@Z$0 00463740 f   tinyxml.obj
 0001:00062748       __unwindfunclet$??0TiXmlDocument@@QAE@PBD@Z$1 00463748 f   tinyxml.obj
 0001:00062753       __ehhandler$??0TiXmlDocument@@QAE@PBD@Z 00463753 f   tinyxml.obj
 0001:00062760       __unwindfunclet$?Clone@TiXmlDocument@@MBEPAVTiXmlNode@@XZ$0 00463760 f   tinyxml.obj
 0001:0006276b       __ehhandler$?Clone@TiXmlDocument@@MBEPAVTiXmlNode@@XZ 0046376b f   tinyxml.obj
 0001:00062780       __unwindfunclet$?Print@TiXmlAttribute@@QBEXPAU_iobuf@@HPAVTiXmlString@@@Z$0 00463780 f   tinyxml.obj
 0001:00062788       __unwindfunclet$?Print@TiXmlAttribute@@QBEXPAU_iobuf@@HPAVTiXmlString@@@Z$1 00463788 f   tinyxml.obj
 0001:00062790       __ehhandler$?Print@TiXmlAttribute@@QBEXPAU_iobuf@@HPAVTiXmlString@@@Z 00463790 f   tinyxml.obj
 0001:000627a0       __unwindfunclet$??0TiXmlComment@@QAE@ABV0@@Z$0 004637a0 f   tinyxml.obj
 0001:000627a8       __ehhandler$??0TiXmlComment@@QAE@ABV0@@Z 004637a8 f   tinyxml.obj
 0001:000627c0       __unwindfunclet$?Print@TiXmlText@@UBEXPAU_iobuf@@H@Z$0 004637c0 f   tinyxml.obj
 0001:000627c8       __ehhandler$?Print@TiXmlText@@UBEXPAU_iobuf@@H@Z 004637c8 f   tinyxml.obj
 0001:000627e0       __unwindfunclet$??0TiXmlDeclaration@@QAE@PBD00@Z$0 004637e0 f   tinyxml.obj
 0001:000627e8       __unwindfunclet$??0TiXmlDeclaration@@QAE@PBD00@Z$1 004637e8 f   tinyxml.obj
 0001:000627f3       __unwindfunclet$??0TiXmlDeclaration@@QAE@PBD00@Z$2 004637f3 f   tinyxml.obj
 0001:000627fe       __unwindfunclet$??0TiXmlDeclaration@@QAE@PBD00@Z$3 004637fe f   tinyxml.obj
 0001:00062809       __ehhandler$??0TiXmlDeclaration@@QAE@PBD00@Z 00463809 f   tinyxml.obj
 0001:00062820       __unwindfunclet$?Visit@TiXmlPrinter@@UAE_NABVTiXmlText@@@Z$0 00463820 f   tinyxml.obj
 0001:00062828       __unwindfunclet$?Visit@TiXmlPrinter@@UAE_NABVTiXmlText@@@Z$1 00463828 f   tinyxml.obj
 0001:00062830       __ehhandler$?Visit@TiXmlPrinter@@UAE_NABVTiXmlText@@@Z 00463830 f   tinyxml.obj
 0001:00062840       __unwindfunclet$??0TiXmlText@@QAE@PBD@Z$0 00463840 f   tinyxml.obj
 0001:00062848       __ehhandler$??0TiXmlText@@QAE@PBD@Z 00463848 f   tinyxml.obj
 0001:00062860       __unwindfunclet$??1TiXmlDeclaration@@UAE@XZ$0 00463860 f   tinyxml.obj
 0001:00062868       __unwindfunclet$??1TiXmlDeclaration@@UAE@XZ$1 00463868 f   tinyxml.obj
 0001:00062873       __unwindfunclet$??1TiXmlDeclaration@@UAE@XZ$2 00463873 f   tinyxml.obj
 0001:0006287e       __ehhandler$??1TiXmlDeclaration@@UAE@XZ 0046387e f   tinyxml.obj
 0001:00062890       __unwindfunclet$??1TiXmlDocument@@UAE@XZ$0 00463890 f   tinyxml.obj
 0001:00062898       __ehhandler$??1TiXmlDocument@@UAE@XZ 00463898 f   tinyxml.obj
 0001:000628b0       __unwindfunclet$??0TiXmlElement@@QAE@PBD@Z$0 004638b0 f   tinyxml.obj
 0001:000628b8       __unwindfunclet$??0TiXmlElement@@QAE@PBD@Z$1 004638b8 f   tinyxml.obj
 0001:000628c3       __ehhandler$??0TiXmlElement@@QAE@PBD@Z 004638c3 f   tinyxml.obj
 0001:000628d0       __unwindfunclet$??1TiXmlElement@@UAE@XZ$0 004638d0 f   tinyxml.obj
 0001:000628d8       __unwindfunclet$??1TiXmlElement@@UAE@XZ$1 004638d8 f   tinyxml.obj
 0001:000628e3       __ehhandler$??1TiXmlElement@@UAE@XZ 004638e3 f   tinyxml.obj
 0001:000628f0       __unwindfunclet$?Clone@TiXmlElement@@UBEPAVTiXmlNode@@XZ$0 004638f0 f   tinyxml.obj
 0001:000628fb       __ehhandler$?Clone@TiXmlElement@@UBEPAVTiXmlNode@@XZ 004638fb f   tinyxml.obj
 0001:00062910       __unwindfunclet$??0TiXmlDocument@@QAE@ABV0@@Z$0 00463910 f   tinyxml.obj
 0001:00062918       __unwindfunclet$??0TiXmlDocument@@QAE@ABV0@@Z$1 00463918 f   tinyxml.obj
 0001:00062923       __ehhandler$??0TiXmlDocument@@QAE@ABV0@@Z 00463923 f   tinyxml.obj
 0001:00062930       __unwindfunclet$?LoadFile@TiXmlDocument@@QAE_NPBDW4TiXmlEncoding@@@Z$0 00463930 f   tinyxml.obj
 0001:00062938       __ehhandler$?LoadFile@TiXmlDocument@@QAE_NPBDW4TiXmlEncoding@@@Z 00463938 f   tinyxml.obj
 0001:00062950       __unwindfunclet$?Clone@TiXmlText@@MBEPAVTiXmlNode@@XZ$0 00463950 f   tinyxml.obj
 0001:0006295b       __ehhandler$?Clone@TiXmlText@@MBEPAVTiXmlNode@@XZ 0046395b f   tinyxml.obj
 0001:00062970       __unwindfunclet$??0TiXmlDeclaration@@QAE@ABV0@@Z$0 00463970 f   tinyxml.obj
 0001:00062978       __unwindfunclet$??0TiXmlDeclaration@@QAE@ABV0@@Z$1 00463978 f   tinyxml.obj
 0001:00062983       __unwindfunclet$??0TiXmlDeclaration@@QAE@ABV0@@Z$2 00463983 f   tinyxml.obj
 0001:0006298e       __unwindfunclet$??0TiXmlDeclaration@@QAE@ABV0@@Z$3 0046398e f   tinyxml.obj
 0001:00062999       __ehhandler$??0TiXmlDeclaration@@QAE@ABV0@@Z 00463999 f   tinyxml.obj
 0001:000629b0       __unwindfunclet$??0TiXmlElement@@QAE@ABV0@@Z$0 004639b0 f   tinyxml.obj
 0001:000629b8       __unwindfunclet$??0TiXmlElement@@QAE@ABV0@@Z$1 004639b8 f   tinyxml.obj
 0001:000629c3       __ehhandler$??0TiXmlElement@@QAE@ABV0@@Z 004639c3 f   tinyxml.obj
 0001:000629d0       __unwindfunclet$?GetEntity@TiXmlBase@@KAPBDPBDPADPAHW4TiXmlEncoding@@@Z$0 004639d0 f   tinyxmlparser.obj
 0001:000629d8       __ehhandler$?GetEntity@TiXmlBase@@KAPBDPBDPADPAHW4TiXmlEncoding@@@Z 004639d8 f   tinyxmlparser.obj
 0001:000629f0       __unwindfunclet$?Identify@TiXmlNode@@IAEPAV1@PBDW4TiXmlEncoding@@@Z$0 004639f0 f   tinyxmlparser.obj
 0001:000629fb       __unwindfunclet$?Identify@TiXmlNode@@IAEPAV1@PBDW4TiXmlEncoding@@@Z$1 004639fb f   tinyxmlparser.obj
 0001:00062a06       __unwindfunclet$?Identify@TiXmlNode@@IAEPAV1@PBDW4TiXmlEncoding@@@Z$2 00463a06 f   tinyxmlparser.obj
 0001:00062a11       __unwindfunclet$?Identify@TiXmlNode@@IAEPAV1@PBDW4TiXmlEncoding@@@Z$3 00463a11 f   tinyxmlparser.obj
 0001:00062a1c       __unwindfunclet$?Identify@TiXmlNode@@IAEPAV1@PBDW4TiXmlEncoding@@@Z$5 00463a1c f   tinyxmlparser.obj
 0001:00062a27       __unwindfunclet$?Identify@TiXmlNode@@IAEPAV1@PBDW4TiXmlEncoding@@@Z$4 00463a27 f   tinyxmlparser.obj
 0001:00062a32       __ehhandler$?Identify@TiXmlNode@@IAEPAV1@PBDW4TiXmlEncoding@@@Z 00463a32 f   tinyxmlparser.obj
 0001:00062a40       __unwindfunclet$?ReadValue@TiXmlElement@@IAEPBDPBDPAVTiXmlParsingData@@W4TiXmlEncoding@@@Z$0 00463a40 f   tinyxmlparser.obj
 0001:00062a4b       __ehhandler$?ReadValue@TiXmlElement@@IAEPBDPBDPAVTiXmlParsingData@@W4TiXmlEncoding@@@Z 00463a4b f   tinyxmlparser.obj
 0001:00062a60       __unwindfunclet$?Parse@TiXmlElement@@UAEPBDPBDPAVTiXmlParsingData@@W4TiXmlEncoding@@@Z$0 00463a60 f   tinyxmlparser.obj
 0001:00062a68       __ehhandler$?Parse@TiXmlElement@@UAEPBDPBDPAVTiXmlParsingData@@W4TiXmlEncoding@@@Z 00463a68 f   tinyxmlparser.obj
 0001:00062a80       __unwindfunclet$?Parse@TiXmlText@@UAEPBDPBDPAVTiXmlParsingData@@W4TiXmlEncoding@@@Z$0 00463a80 f   tinyxmlparser.obj
 0001:00062a88       __ehhandler$?Parse@TiXmlText@@UAEPBDPBDPAVTiXmlParsingData@@W4TiXmlEncoding@@@Z 00463a88 f   tinyxmlparser.obj
 0001:00062aa0       __unwindfunclet$?Parse@TiXmlDeclaration@@UAEPBDPBDPAVTiXmlParsingData@@W4TiXmlEncoding@@@Z$0 00463aa0 f   tinyxmlparser.obj
 0001:00062aa8       __unwindfunclet$?Parse@TiXmlDeclaration@@UAEPBDPBDPAVTiXmlParsingData@@W4TiXmlEncoding@@@Z$1 00463aa8 f   tinyxmlparser.obj
 0001:00062ab0       __unwindfunclet$?Parse@TiXmlDeclaration@@UAEPBDPBDPAVTiXmlParsingData@@W4TiXmlEncoding@@@Z$2 00463ab0 f   tinyxmlparser.obj
 0001:00062ab8       __ehhandler$?Parse@TiXmlDeclaration@@UAEPBDPBDPAVTiXmlParsingData@@W4TiXmlEncoding@@@Z 00463ab8 f   tinyxmlparser.obj
 0001:00062ad0       __unwindfunclet$?RunCommand@@YAHPADH@Z$1 00463ad0 f   cmds.obj
 0001:00062adb       __unwindfunclet$?RunCommand@@YAHPADH@Z$0 00463adb f   cmds.obj
 0001:00062ae6       __ehhandler$?RunCommand@@YAHPADH@Z 00463ae6 f   cmds.obj
 0001:00062af0       __unwindfunclet$?SendInCarFullSyncData@@YAXPAU_INCAR_SYNC_DATA@@HG@Z$0 00463af0 f   localplayer.obj
 0001:00062afb       __ehhandler$?SendInCarFullSyncData@@YAXPAU_INCAR_SYNC_DATA@@HG@Z 00463afb f   localplayer.obj
 0001:00062b10       __unwindfunclet$?SendPassengerFullSyncData@@YAXG@Z$0 00463b10 f   localplayer.obj
 0001:00062b1b       __ehhandler$?SendPassengerFullSyncData@@YAXG@Z 00463b1b f   localplayer.obj
 0001:00062b30       __unwindfunclet$?SendAimSyncData@@YAXPAU_AIM_SYNC_DATA@@KHG@Z$0 00463b30 f   localplayer.obj
 0001:00062b3b       __ehhandler$?SendAimSyncData@@YAXPAU_AIM_SYNC_DATA@@KHG@Z 00463b3b f   localplayer.obj
 0001:00062b50       __unwindfunclet$?SendUnoccupiedSyncData@@YAXPAU_UNOCCUPIED_SYNC_DATA@@@Z$0 00463b50 f   localplayer.obj
 0001:00062b5b       __ehhandler$?SendUnoccupiedSyncData@@YAXPAU_UNOCCUPIED_SYNC_DATA@@@Z 00463b5b f   localplayer.obj
 0001:00062b70       __unwindfunclet$?SendSpectatorData@@YAXPAU_SPECTATOR_SYNC_DATA@@@Z$0 00463b70 f   localplayer.obj
 0001:00062b7b       __ehhandler$?SendSpectatorData@@YAXPAU_SPECTATOR_SYNC_DATA@@@Z 00463b7b f   localplayer.obj
 0001:00062b90       __unwindfunclet$?SendEnterVehicleNotification@@YAXGH@Z$0 00463b90 f   localplayer.obj
 0001:00062b9b       __ehhandler$?SendEnterVehicleNotification@@YAXGH@Z 00463b9b f   localplayer.obj
 0001:00062bb0       __unwindfunclet$?SendExitVehicleNotification@@YAXG@Z$0 00463bb0 f   localplayer.obj
 0001:00062bbb       __ehhandler$?SendExitVehicleNotification@@YAXG@Z 00463bbb f   localplayer.obj
 0001:00062bd0       __unwindfunclet$?SendWastedNotification@@YAXEG@Z$0 00463bd0 f   localplayer.obj
 0001:00062bdb       __ehhandler$?SendWastedNotification@@YAXEG@Z 00463bdb f   localplayer.obj
 0001:00062bf0       __unwindfunclet$?NotifyVehicleDeath@@YAXG@Z$0 00463bf0 f   localplayer.obj
 0001:00062bfb       __ehhandler$?NotifyVehicleDeath@@YAXG@Z 00463bfb f   localplayer.obj
 0001:00062c10       __unwindfunclet$?SendDamageVehicle@@YAXGKKEE@Z$0 00463c10 f   localplayer.obj
 0001:00062c1b       __ehhandler$?SendDamageVehicle@@YAXGKKEE@Z 00463c1b f   localplayer.obj
 0001:00062c30       __unwindfunclet$?SendOnFootFullSyncData@@YAXPAU_ONFOOT_SYNC_DATA@@HG@Z$0 00463c30 f   localplayer.obj
 0001:00062c3b       __ehhandler$?SendOnFootFullSyncData@@YAXPAU_ONFOOT_SYNC_DATA@@HG@Z 00463c3b f   localplayer.obj
 0001:00062c50       __unwindfunclet$?sampSpawn@@YAXXZ$0 00463c50 f   misc_funcs.obj
 0001:00062c5b       __unwindfunclet$?sampSpawn@@YAXXZ$1 00463c5b f   misc_funcs.obj
 0001:00062c66       __ehhandler$?sampSpawn@@YAXXZ 00463c66 f   misc_funcs.obj
 0001:00062c70       __unwindfunclet$?sampRequestClass@@YAXH@Z$0 00463c70 f   misc_funcs.obj
 0001:00062c7b       __ehhandler$?sampRequestClass@@YAXH@Z 00463c7b f   misc_funcs.obj
 0001:00062c90       __unwindfunclet$?sampSmth@@YAXXZ$0 00463c90 f   misc_funcs.obj
 0001:00062c9b       __ehhandler$?sampSmth@@YAXXZ 00463c9b f   misc_funcs.obj
 0001:00062cb0       __unwindfunclet$?sampFakeNpc@@YAXXZ$0 00463cb0 f   misc_funcs.obj
 0001:00062cbb       __ehhandler$?sampFakeNpc@@YAXXZ 00463cbb f   misc_funcs.obj
 0001:00062cd0       __unwindfunclet$?sendServerCommand@@YAXPAD@Z$0 00463cd0 f   misc_funcs.obj
 0001:00062cdb       __ehhandler$?sendServerCommand@@YAXPAD@Z 00463cdb f   misc_funcs.obj
 0001:00062cf0       __unwindfunclet$?sendChat@@YAXPAD@Z$0 00463cf0 f   misc_funcs.obj
 0001:00062cfb       __ehhandler$?sendChat@@YAXPAD@Z 00463cfb f   misc_funcs.obj
 0001:00062d10       __unwindfunclet$?SendScmEvent@@YAXHKKK@Z$0 00463d10 f   misc_funcs.obj
 0001:00062d1b       __ehhandler$?SendScmEvent@@YAXHKKK@Z 00463d1b f   misc_funcs.obj
 0001:00062d30       __unwindfunclet$?sendDialogResponse@@YAXGEGPAD@Z$0 00463d30 f   misc_funcs.obj
 0001:00062d3b       __ehhandler$?sendDialogResponse@@YAXGEGPAD@Z 00463d3b f   misc_funcs.obj
 0001:00062d50       __unwindfunclet$?sampReg@@YAXXZ$0 00463d50 f   misc_funcs.obj
 0001:00062d5b       __ehhandler$?sampReg@@YAXXZ 00463d5b f   misc_funcs.obj
 0001:00062d70       __unwindfunclet$?UpdatePlayerScoresAndPings@@YAXHH@Z$0 00463d70 f   netgame.obj
 0001:00062d7b       __unwindfunclet$?UpdatePlayerScoresAndPings@@YAXHH@Z$1 00463d7b f   netgame.obj
 0001:00062d86       __ehhandler$?UpdatePlayerScoresAndPings@@YAXHH@Z 00463d86 f   netgame.obj
 0001:00062d90       __unwindfunclet$?Packet_ConnectionSucceeded@@YAXPAUPacket@@@Z$0 00463d90 f   netgame.obj
 0001:00062d9b       __unwindfunclet$?Packet_ConnectionSucceeded@@YAXPAUPacket@@@Z$1 00463d9b f   netgame.obj
 0001:00062da6       __ehhandler$?Packet_ConnectionSucceeded@@YAXPAUPacket@@@Z 00463da6 f   netgame.obj
 0001:00062db0       __unwindfunclet$?Packet_UnoccupiedSync@@YAXPAUPacket@@@Z$0 00463db0 f   netgame.obj
 0001:00062dbb       __ehhandler$?Packet_UnoccupiedSync@@YAXPAUPacket@@@Z 00463dbb f   netgame.obj
 0001:00062dd0       __unwindfunclet$?Packet_AimSync@@YAXPAUPacket@@@Z$0 00463dd0 f   netgame.obj
 0001:00062ddb       __ehhandler$?Packet_AimSync@@YAXPAUPacket@@@Z 00463ddb f   netgame.obj
 0001:00062df0       __unwindfunclet$?Packet_PassengerSync@@YAXPAUPacket@@@Z$0 00463df0 f   netgame.obj
 0001:00062dfb       __ehhandler$?Packet_PassengerSync@@YAXPAUPacket@@@Z 00463dfb f   netgame.obj
 0001:00062e10       __unwindfunclet$?Packet_TrailerSync@@YAXPAUPacket@@@Z$0 00463e10 f   netgame.obj
 0001:00062e1b       __ehhandler$?Packet_TrailerSync@@YAXPAUPacket@@@Z 00463e1b f   netgame.obj
 0001:00062e30       __unwindfunclet$?Packet_MarkersSync@@YAXPAUPacket@@@Z$0 00463e30 f   netgame.obj
 0001:00062e3b       __ehhandler$?Packet_MarkersSync@@YAXPAUPacket@@@Z 00463e3b f   netgame.obj
 0001:00062e50       __unwindfunclet$?Packet_PlayerSync@@YAXPAUPacket@@@Z$0 00463e50 f   netgame.obj
 0001:00062e5b       __ehhandler$?Packet_PlayerSync@@YAXPAUPacket@@@Z 00463e5b f   netgame.obj
 0001:00062e70       __unwindfunclet$?Packet_VehicleSync@@YAXPAUPacket@@@Z$0 00463e70 f   netgame.obj
 0001:00062e7b       __ehhandler$?Packet_VehicleSync@@YAXPAUPacket@@@Z 00463e7b f   netgame.obj
 0001:00062e90       __unwindfunclet$?WorldVehicleAdd@@YAXPAURPCParameters@@@Z$0 00463e90 f   netrpc.obj
 0001:00062e9b       __ehhandler$?WorldVehicleAdd@@YAXPAURPCParameters@@@Z 00463e9b f   netrpc.obj
 0001:00062eb0       __unwindfunclet$?ServerJoin@@YAXPAURPCParameters@@@Z$0 00463eb0 f   netrpc.obj
 0001:00062ebb       __ehhandler$?ServerJoin@@YAXPAURPCParameters@@@Z 00463ebb f   netrpc.obj
 0001:00062ed0       __unwindfunclet$?ServerQuit@@YAXPAURPCParameters@@@Z$0 00463ed0 f   netrpc.obj
 0001:00062edb       __ehhandler$?ServerQuit@@YAXPAURPCParameters@@@Z 00463edb f   netrpc.obj
 0001:00062ef0       __unwindfunclet$?InitGame@@YAXPAURPCParameters@@@Z$0 00463ef0 f   netrpc.obj
 0001:00062efb       __ehhandler$?InitGame@@YAXPAURPCParameters@@@Z 00463efb f   netrpc.obj
 0001:00062f10       __unwindfunclet$?WorldPlayerAdd@@YAXPAURPCParameters@@@Z$0 00463f10 f   netrpc.obj
 0001:00062f1b       __ehhandler$?WorldPlayerAdd@@YAXPAURPCParameters@@@Z 00463f1b f   netrpc.obj
 0001:00062f30       __unwindfunclet$?WorldPlayerDeath@@YAXPAURPCParameters@@@Z$0 00463f30 f   netrpc.obj
 0001:00062f3b       __ehhandler$?WorldPlayerDeath@@YAXPAURPCParameters@@@Z 00463f3b f   netrpc.obj
 0001:00062f50       __unwindfunclet$?WorldPlayerRemove@@YAXPAURPCParameters@@@Z$0 00463f50 f   netrpc.obj
 0001:00062f5b       __ehhandler$?WorldPlayerRemove@@YAXPAURPCParameters@@@Z 00463f5b f   netrpc.obj
 0001:00062f70       __unwindfunclet$?WorldVehicleRemove@@YAXPAURPCParameters@@@Z$0 00463f70 f   netrpc.obj
 0001:00062f7b       __ehhandler$?WorldVehicleRemove@@YAXPAURPCParameters@@@Z 00463f7b f   netrpc.obj
 0001:00062f90       __unwindfunclet$?ConnectionRejected@@YAXPAURPCParameters@@@Z$0 00463f90 f   netrpc.obj
 0001:00062f9b       __ehhandler$?ConnectionRejected@@YAXPAURPCParameters@@@Z 00463f9b f   netrpc.obj
 0001:00062fb0       __unwindfunclet$?ClientMessage@@YAXPAURPCParameters@@@Z$0 00463fb0 f   netrpc.obj
 0001:00062fbb       __ehhandler$?ClientMessage@@YAXPAURPCParameters@@@Z 00463fbb f   netrpc.obj
 0001:00062fd0       __unwindfunclet$?Chat@@YAXPAURPCParameters@@@Z$0 00463fd0 f   netrpc.obj
 0001:00062fdb       __ehhandler$?Chat@@YAXPAURPCParameters@@@Z 00463fdb f   netrpc.obj
 0001:00062ff0       __unwindfunclet$?UpdateScoresPingsIPs@@YAXPAURPCParameters@@@Z$0 00463ff0 f   netrpc.obj
 0001:00062ffb       __ehhandler$?UpdateScoresPingsIPs@@YAXPAURPCParameters@@@Z 00463ffb f   netrpc.obj
 0001:00063010       __unwindfunclet$?ScrInitMenu@@YAXPAURPCParameters@@@Z$0 00464010 f   netrpc.obj
 0001:0006301b       __ehhandler$?ScrInitMenu@@YAXPAURPCParameters@@@Z 0046401b f   netrpc.obj
 0001:00063030       __unwindfunclet$?ScrDialogBox@@YAXPAURPCParameters@@@Z$0 00464030 f   netrpc.obj
 0001:0006303b       __ehhandler$?ScrDialogBox@@YAXPAURPCParameters@@@Z 0046403b f   netrpc.obj
 0001:00063050       __unwindfunclet$?ScrGameText@@YAXPAURPCParameters@@@Z$0 00464050 f   netrpc.obj
 0001:0006305b       __ehhandler$?ScrGameText@@YAXPAURPCParameters@@@Z 0046405b f   netrpc.obj
 0001:00063070       __unwindfunclet$?ScrPlayAudioStream@@YAXPAURPCParameters@@@Z$0 00464070 f   netrpc.obj
 0001:0006307b       __ehhandler$?ScrPlayAudioStream@@YAXPAURPCParameters@@@Z 0046407b f   netrpc.obj
 0001:00063085       __ehhandler$?CallUnexpected@@YAXPBU_s_ESTypeList@@@Z 00464085 f   LIBCMT:frame.obj
 0001:000630a0       ??__E?IDTree@NetworkIDGenerator@@2V?$AVLBalancedBinarySearchTree@UNetworkIDNode@@@DataStructures@@A@@YAXXZ 004640a0 f   NetworkIDGenerator.obj
 0001:000630b0       ??__E?externalPlayerId@NetworkIDGenerator@@0UPlayerID@@A@@YAXXZ 004640b0 f   NetworkIDGenerator.obj
 0001:000630d0       ??__E?I@SocketLayer@@0V1@A@@YAXXZ 004640d0 f   SocketLayer.obj
 0001:00063100       ??__EdwLastOnFootDataSentTick@@YAXXZ 00464100 f   localplayer.obj
 0001:00063110       ??__EdwLastInVehicleDataSentTick@@YAXXZ 00464110 f   localplayer.obj
 0001:00063120       ??__EdwLastPassengerDataSentTick@@YAXXZ 00464120 f   localplayer.obj
 0001:00063130       ??__EdwLastAimDataSentTick@@YAXXZ 00464130 f   localplayer.obj
 0001:00063140       ??__EdwLastUnocDataSentTick@@YAXXZ 00464140 f   localplayer.obj
 0001:00063150       ??__EdwAutoRunTick@@YAXXZ  00464150 f   main.obj
 0001:00063160       ??__EinCarUpdateTick@@YAXXZ 00464160 f   misc_funcs.obj
 0001:00063170       ??__ExmlSettings@@YAXXZ    00464170 f   xmlsets.obj
 0001:00063186       ??__Einitlocks@std@@YAXXZ  00464186 f   libcpmt:xlock.obj
 0001:000631a0       ??__F?IDTree@NetworkIDGenerator@@2V?$AVLBalancedBinarySearchTree@UNetworkIDNode@@@DataStructures@@A@@YAXXZ 004641a0 f   NetworkIDGenerator.obj
 0001:000631b0       ??__F?I@SocketLayer@@0V1@A@@YAXXZ 004641b0 f   SocketLayer.obj
 0001:000631d0       ??__FxmlSettings@@YAXXZ    004641d0 f   xmlsets.obj
 0001:000631da       ??__Fnomem@?5???2@YAPAXI@Z@YAXXZ 004641da f   LIBCMT:new.obj
 0001:000631ee       ??__Finitlocks@std@@YAXXZ  004641ee f   libcpmt:xlock.obj
